Archive member included to satisfy reference by file (symbol)

..\..\..\Libraries\libs\libplatform.a(audio.o)
                              Output\obj\Libraries\bsp\bsp_sys.o (adpll_init)
..\..\..\Libraries\libs\libplatform.a(cm.o)
                              Output\obj\Libraries\bsp\bsp_param.o (cm_sync)
..\..\..\Libraries\libs\libplatform.a(os_flash.o)
                              ..\..\..\Libraries\libs\libplatform.a(cm.o) (os_spiflash_read)
..\..\..\Libraries\libs\libplatform.a(xcfg.o)
                              Output\obj\Libraries\bsp\bsp_sys.o (xcfg_init)
..\..\..\Libraries\libs\libplatform.a(device.o)
                              Output\obj\Libraries\bsp\bsp_sys.o (dev_init)
..\..\..\Libraries\libs\libplatform.a(main.o)
                              Output\obj\Libraries\bsp\bsp_bt.o (delay_5ms)
..\..\..\Libraries\libs\libplatform.a(interrupt.o)
                              Output\obj\Libraries\bsp\bsp_fot.o (tick_get)
..\..\..\Libraries\libs\libplatform.a(startup.o)
                              ..\..\..\Libraries\libs\libplatform.a(interrupt.o) (user_timer_isr_en)
..\..\..\Libraries\libs\libplatform.a(sys_hook.o)
                              ..\..\..\Libraries\libs\libplatform.a(startup.o) (sys_hook_init)
..\..\..\Libraries\libs\libplatform.a(reset.o)
                              (_start)
..\..\..\Libraries\libs\libplatform.a(spiflash.o)
                              ..\..\..\Libraries\libs\libplatform.a(os_flash.o) (spiflash_program)
..\..\..\Libraries\libs\libplatform.a(debug.o)
                              ..\..\..\Libraries\libs\libplatform.a(main.o) (debug_set)
..\..\..\Libraries\libs\libplatform.a(fot_update.o)
                              ..\..\..\Libraries\libs\libplatform.a(xcfg.o) (get_spiloader_offset)
..\..\..\Libraries\libs\libplatform.a(lock.o)
                              ..\..\..\Libraries\libs\libplatform.a(main.o) (lock_init)
..\..\..\Libraries\libs\libplatform.a(patch.o)
                              ..\..\..\Libraries\libs\libplatform.a(main.o) (patch_init)
..\..\..\Libraries\libs\libplatform.a(power.o)
                              Output\obj\Libraries\bsp\bsp_sys.o (pmu_init)
..\..\..\Libraries\libs\libplatform.a(rc.o)
                              ..\..\..\Libraries\libs\libplatform.a(main.o) (rc_compile)
..\..\..\Libraries\libs\libplatform.a(s_sys.o)
                              ..\..\..\Libraries\libs\libplatform.a(main.o) (s_bcnt)
..\..\..\Libraries\libs\libplatform.a(sys.o)
                              ..\..\..\Libraries\libs\libplatform.a(main.o) (sys_get_rc2m_clkhz)
..\..\..\Libraries\libs\libplatform.a(sys_clk.o)
                              Output\obj\Libraries\BT\ble\ble.o (get_cur_sysclk)
..\..\..\Libraries\libs\libplatform.a(voltage_trim.o)
                              ..\..\..\Libraries\libs\libplatform.a(main.o) (voltage_trim_value_init)
..\..\..\Libraries\libs\libplatform.a(weak_symbol.o)
                              ..\..\..\Libraries\libs\libplatform.a(main.o) (update_complete)
..\..\..\Libraries\libs\libplatform.a(huart.o)
                              ..\..\..\Libraries\libs\libplatform.a(interrupt.o) (huart_isr)
..\..\..\Libraries\libs\libplatform.a(usb.o)
                              ..\..\..\Libraries\libs\libplatform.a(startup.o) (thread_usb_entry)
..\..\..\Libraries\libs\libplatform.a(bt.o)
                              ..\..\..\Libraries\libs\libplatform.a(reset.o) (bthw_txrx_isr)
..\..\..\Libraries\libs\libdrivers.a(usb_device_hid.o)
                              Output\obj\Libraries\bsp\bsp_sys.o (ude_tmr_isr)
..\..\..\Libraries\libs\libdrivers.a(usb_device_printer.o)
                              ..\..\..\Libraries\libs\libplatform.a(usb.o) (ude_bulk_tx_process)
..\..\..\Libraries\libs\libdrivers.a(usb_device_run_loop.o)
                              ..\..\..\Libraries\libs\libdrivers.a(usb_device_hid.o) (ude_cfgval_get)
..\..\..\Libraries\libs\libdrivers.a(usb_host_manage.o)
                              ..\..\..\Libraries\libs\libplatform.a(device.o) (usb_host_init)
..\..\..\Libraries\libs\libdrivers.a(usb_host_storage.o)
                              ..\..\..\Libraries\libs\libdrivers.a(usb_host_manage.o) (uhs_start)
..\..\..\Libraries\libs\libdrivers.a(usb_comm.o)
                              ..\..\..\Libraries\libs\libdrivers.a(usb_host_storage.o) (usb_interrupt_disable)
..\..\..\Libraries\libs\libdrivers.a(usb_detect.o)
                              ..\..\..\Libraries\libs\libdrivers.a(usb_host_manage.o) (usbchk_switch_otg_device)
..\..\..\Libraries\libs\libdrivers.a(usb_device_desc.o)
                              ..\..\..\Libraries\libs\libdrivers.a(usb_device_run_loop.o) (usb_get_hid_config_descriptor)
..\..\..\Libraries\libs\libdrivers.a(usb_device_enum.o)
                              ..\..\..\Libraries\libs\libdrivers.a(usb_device_run_loop.o) (ude_run_loop_execute)
..\..\..\Libraries\libs\libdrivers.a(usb_device_ep.o)
                              ..\..\..\Libraries\libs\libdrivers.a(usb_device_hid.o) (usb_set_cur_ep)
..\..\..\Libraries\libs\libdrivers.a(usb_host_enum.o)
                              ..\..\..\Libraries\libs\libdrivers.a(usb_host_manage.o) (uhe_start)
..\..\..\Libraries\libs\libdrivers.a(weak_symbol.o)
                              ..\..\..\Libraries\libs\libdrivers.a(usb_host_enum.o) (iphone_power_set)
..\..\..\Libraries\libs\libdrivers.a(usb_device_audio.o)
                              ..\..\..\Libraries\libs\libdrivers.a(usb_device_enum.o) (uda_get_spk_mute)
..\..\..\Libraries\libs\libbtstack_master.a(nanos.o)
                              ..\..\..\Libraries\libs\libplatform.a(startup.o) (nanos_var_init)
..\..\..\Libraries\libs\libbtstack_master.a(patch.o)
                              ..\..\..\Libraries\libs\libplatform.a(patch.o) (bb_patch_init)
..\..\..\Libraries\libs\libbtstack_master.a(platform.o)
                              ..\..\..\Libraries\libs\libplatform.a(interrupt.o) (timer_sync_init)
..\..\..\Libraries\libs\libbtstack_master.a(bt_sco.o)
                              ..\..\..\Libraries\libs\libplatform.a(interrupt.o) (bt_codec_isr)
..\..\..\Libraries\libs\libbtstack_master.a(bt_acl.o)
                              ..\..\..\Libraries\libs\libbtstack_master.a(patch.o) (bt_acl_env)
..\..\..\Libraries\libs\libbtstack_master.a(ble_con.o)
                              ..\..\..\Libraries\libs\libbtstack_master.a(patch.o) (ble_con_evt_prio_check)
..\..\..\Libraries\libs\libbtstack_master.a(bb_utils.o)
                              ..\..\..\Libraries\libs\libbtstack_master.a(ble_con.o) (bb_sca2ppm)
..\..\..\Libraries\libs\libbtstack_master.a(bb_int.o)
                              ..\..\..\Libraries\libs\libplatform.a(bt.o) (bb_hal_isr)
..\..\..\Libraries\libs\libbtstack_master.a(bb.o)
                              ..\..\..\Libraries\libs\libbtstack_master.a(nanos.o) (bb_get_heap_info)
..\..\..\Libraries\libs\libbtstack_master.a(platform.o)
                              ..\..\..\Libraries\libs\libbtstack_master.a(bb.o) (dummy_void)
..\..\..\Libraries\libs\libbtstack_master.a(extern_tws.o)
                              ..\..\..\Libraries\libs\libbtstack_master.a(bb_int.o) (cfg_bt_tws_limit_pair_time)
..\..\..\Libraries\libs\libbtstack_master.a(extern_bt.o)
                              ..\..\..\Libraries\libs\libbtstack_master.a(bb_int.o) (cfg_bt_sniff_clk_sel)
..\..\..\Libraries\libs\libbtstack_master.a(extern.o)
                              ..\..\..\Libraries\libs\libplatform.a(reset.o) (ext_aubuf_isr)
..\..\..\Libraries\libs\libbtstack_master.a(spp.o)
                              Output\obj\Libraries\bsp\bsp_fot.o (bt_spp_tx)
..\..\..\Libraries\libs\libbtstack_master.a(sdp_util.o)
                              ..\..\..\Libraries\libs\libbtstack_master.a(spp.o) (mfi_search_uuid128)
..\..\..\Libraries\libs\libbtstack_master.a(sdp_tbl.o)
                              Output\obj\Libraries\BT\spp\profile.o (sdp_spp_service_record)
..\..\..\Libraries\libs\libbtstack_master.a(sdp_server.o)
                              Output\obj\Libraries\BT\spp\profile.o (sdp_add_service)
..\..\..\Libraries\libs\libbtstack_master.a(sdp_client.o)
                              ..\..\..\Libraries\libs\libbtstack_master.a(sdp_server.o) (sdp_client_init)
..\..\..\Libraries\libs\libbtstack_master.a(rfcomm.o)
                              ..\..\..\Libraries\libs\libbtstack_master.a(spp.o) (rfcomm_can_send_packet_now)
..\..\..\Libraries\libs\libbtstack_master.a(btstack_link_key_db.o)
                              Output\obj\Libraries\BT\spp\bt.o (link_info_page_size)
..\..\..\Libraries\libs\libbtstack_master.a(btstack_util.o)
                              ..\..\..\Libraries\libs\libbtstack_master.a(rfcomm.o) (bd_addr_cmp)
..\..\..\Libraries\libs\libbtstack_master.a(btstack_txpkt.o)
                              Output\obj\Libraries\BT\ble\ab_link\app.o (txpkt_init)
..\..\..\Libraries\libs\libbtstack_master.a(btstack_run_loop.o)
                              ..\..\..\Libraries\libs\libbtstack_master.a(rfcomm.o) (btstack_run_loop_set_timer_handler)
..\..\..\Libraries\libs\libbtstack_master.a(btstack_memory.o)
                              ..\..\..\Libraries\libs\libbtstack_master.a(rfcomm.o) (btstack_memory_rfcomm_multiplexer_get)
..\..\..\Libraries\libs\libbtstack_master.a(btstack_linked_list.o)
                              ..\..\..\Libraries\libs\libbtstack_master.a(rfcomm.o) (btstack_linked_list_empty)
..\..\..\Libraries\libs\libbtstack_master.a(btstack_link_ctrl.o)
                              ..\..\..\Libraries\libs\libbtstack_master.a(spp.o) (provide_link_ctrl_context_for_bd_addr)
..\..\..\Libraries\libs\libbtstack_master.a(sm.o)
                              Output\obj\Examples\BLE_Host\Source\ble_init.o (gap_random_address_set_mode)
..\..\..\Libraries\libs\libbtstack_master.a(le_device_db_memory.o)
                              ..\..\..\Libraries\libs\libbtstack_master.a(sm.o) (le_device_db_set_local_bd_addr)
..\..\..\Libraries\libs\libbtstack_master.a(gatt_server.o)
                              Output\obj\Libraries\BT\ble\ab_link\app.o (ble_init_att_for_handle)
..\..\..\Libraries\libs\libbtstack_master.a(gatt_profile.o)
                              Output\obj\Libraries\BT\ble\ab_link\app.o (ble_gatts_service_add)
..\..\..\Libraries\libs\libbtstack_master.a(gatt_client.o)
                              Output\obj\Examples\BLE_Host\Source\ble_client.o (att_client_register_handler)
..\..\..\Libraries\libs\libbtstack_master.a(att_server.o)
                              Output\obj\Examples\BLE_Host\Source\ble_init.o (att_server_init)
..\..\..\Libraries\libs\libbtstack_master.a(att_dispatch.o)
                              ..\..\..\Libraries\libs\libbtstack_master.a(gatt_client.o) (att_dispatch_register_client)
..\..\..\Libraries\libs\libbtstack_master.a(att_db.o)
                              ..\..\..\Libraries\libs\libbtstack_master.a(gatt_server.o) (att_uuid_for_handle)
..\..\..\Libraries\libs\libbtstack_master.a(ad_parser.o)
                              ..\..\..\Libraries\libs\libbtstack_master.a(gatt_server.o) (ad_param)
..\..\..\Libraries\libs\libbtstack_master.a(btstack_main.o)
                              Output\obj\Examples\BLE_Host\Source\ble_init.o (le_sm_init)
..\..\..\Libraries\libs\libbtstack_master.a(btstack_hal.o)
                              ..\..\..\Libraries\libs\libbtstack_master.a(btstack_run_loop.o) (hal_tick_init)
..\..\..\Libraries\libs\libbtstack_master.a(btstack_api.o)
                              ..\..\..\Libraries\libs\libplatform.a(startup.o) (btstack_var_init)
..\..\..\Libraries\libs\libbtstack_master.a(bt_api.o)
                              Output\obj\Libraries\bsp\bsp_bt.o (bt_setup)
..\..\..\Libraries\libs\libbtstack_master.a(ble_api.o)
                              Output\obj\Libraries\BT\ble\ab_link\app.o (ble_get_status)
..\..\..\Libraries\libs\libbtstack_master.a(bb_sche.o)
                              ..\..\..\Libraries\libs\libbtstack_master.a(ble_con.o) (bb_sche_frag_ble_dur_set)
..\..\..\Libraries\libs\libbtstack_master.a(patch_asm.o)
                              ..\..\..\Libraries\libs\libbtstack_master.a(patch.o) (bb_v1_patch0)
..\..\..\Libraries\libs\libbtstack_master.a(bb_dbg.o)
                              ..\..\..\Libraries\libs\libbtstack_master.a(bb.o) (bb_dbg_init)
..\..\..\Libraries\libs\libbtstack_master.a(bb_clk.o)
                              ..\..\..\Libraries\libs\libbtstack_master.a(bb.o) (bb_clk_init)
..\..\..\Libraries\libs\libbtstack_master.a(aes.o)
                              ..\..\..\Libraries\libs\libbtstack_master.a(bb.o) (aes_init)
..\..\..\Libraries\libs\libbtstack_master.a(vs_proc.o)
                              ..\..\..\Libraries\libs\libbtstack_master.a(btstack_api.o) (bt_fcc_test_ctrl)
..\..\..\Libraries\libs\libbtstack_master.a(vs_fcc.o)
                              ..\..\..\Libraries\libs\libbtstack_master.a(vs_proc.o) (vs_fcc_test_cmd_do)
..\..\..\Libraries\libs\libbtstack_master.a(vs.o)
                              ..\..\..\Libraries\libs\libbtstack_master.a(bb.o) (vs_init)
..\..\..\Libraries\libs\libbtstack_master.a(rf_smart.o)
                              ..\..\..\Libraries\libs\libbtstack_master.a(vs_fcc.o) (rfphy_pll_afc)
..\..\..\Libraries\libs\libbtstack_master.a(rf.o)
                              ..\..\..\Libraries\libs\libbtstack_master.a(bt_acl.o) (rf_txpwr_get_dbm)
..\..\..\Libraries\libs\libbtstack_master.a(bt_hook.o)
                              ..\..\..\Libraries\libs\libbtstack_master.a(bb.o) (bt_isr_hook)
..\..\..\Libraries\libs\libbtstack_master.a(ble_hook.o)
                              ..\..\..\Libraries\libs\libbtstack_master.a(bb.o) (ble_isr_hook)
..\..\..\Libraries\libs\libbtstack_master.a(hct_tl.o)
                              ..\..\..\Libraries\libs\libbtstack_master.a(bb_int.o) (hct_queue_is_empty)
..\..\..\Libraries\libs\libbtstack_master.a(hct_msg.o)
                              ..\..\..\Libraries\libs\libbtstack_master.a(hct_tl.o) (hci_look_for_cmd_desc)
..\..\..\Libraries\libs\libbtstack_master.a(hct_fc.o)
                              ..\..\..\Libraries\libs\libbtstack_master.a(hct_tl.o) (hci_fc_acl_packet_sent)
..\..\..\Libraries\libs\libbtstack_master.a(hct.o)
                              ..\..\..\Libraries\libs\libbtstack_master.a(vs_proc.o) (hci_send_2_host)
..\..\..\Libraries\libs\libbtstack_master.a(tws_sco.o)
                              ..\..\..\Libraries\libs\libbtstack_master.a(bt_hook.o) (bt_sco_get_index)
..\..\..\Libraries\libs\libbtstack_master.a(tws_acl.o)
                              ..\..\..\Libraries\libs\libbtstack_master.a(patch_asm.o) (tws_switch_acl_is_pause)
..\..\..\Libraries\libs\libbtstack_master.a(lm.o)
                              ..\..\..\Libraries\libs\libbtstack_master.a(btstack_main.o) (lm_set_scan_int)
..\..\..\Libraries\libs\libbtstack_master.a(bt_hal.o)
                              ..\..\..\Libraries\libs\libbtstack_master.a(bt_hook.o) (bt_channel_assess)
..\..\..\Libraries\libs\libbtstack_master.a(bt21.o)
                              ..\..\..\Libraries\libs\libbtstack_master.a(bb.o) (bt_buf_acl_rx_free)
..\..\..\Libraries\libs\libbtstack_master.a(bc.o)
                              ..\..\..\Libraries\libs\libbtstack_master.a(bt21.o) (bc_init)
..\..\..\Libraries\libs\libbtstack_master.a(ble_hal.o)
                              ..\..\..\Libraries\libs\libbtstack_master.a(ble_con.o) (ble_channel_assess)
..\..\..\Libraries\libs\libbtstack_master.a(ble_adv.o)
                              ..\..\..\Libraries\libs\libbtstack_master.a(ble_hal.o) (ble_adv_init)
..\..\..\Libraries\libs\libbtstack_master.a(ble.o)
                              ..\..\..\Libraries\libs\libbtstack_master.a(bb.o) (ble_var_init)
..\..\..\Libraries\libs\libbtstack_master.a(l2cap_test.o)
                              ..\..\..\Libraries\libs\libbtstack_master.a(btstack_main.o) (l2cap_vd_acl_init)
..\..\..\Libraries\libs\libbtstack_master.a(l2cap.o)
                              ..\..\..\Libraries\libs\libbtstack_master.a(btstack_main.o) (l2cap_init)
..\..\..\Libraries\libs\libbtstack_master.a(hci_sco.o)
                              ..\..\..\Libraries\libs\libbtstack_master.a(btstack_api.o) (sco_init_var)
..\..\..\Libraries\libs\libbtstack_master.a(hci_dump.o)
                              ..\..\..\Libraries\libs\libbtstack_master.a(btstack_api.o) (hci_dump_open)
..\..\..\Libraries\libs\libbtstack_master.a(hci_cmd.o)
                              ..\..\..\Libraries\libs\libbtstack_master.a(sm.o) (hci_le_long_term_key_negative_reply)
..\..\..\Libraries\libs\libbtstack_master.a(hci.o)
                              ..\..\..\Libraries\libs\libbtstack_master.a(l2cap.o) (gap_get_connection_parameter_range)
..\..\..\Libraries\libs\libbtstack_master.a(hid_usage.o)
                              ..\..\..\Libraries\libs\libbtstack_master.a(bt_api.o) (hid_report_set)
..\..\..\Libraries\libs\libbtstack_master.a(hid_device.o)
                              ..\..\..\Libraries\libs\libbtstack_master.a(bt_api.o) (bt_hid_is_connected)
..\..\..\Libraries\libs\libbtstack_master.a(hfp_hf.o)
                              ..\..\..\Libraries\libs\libbtstack_master.a(btstack_api.o) (hfp_hf_get_siri_status)
..\..\..\Libraries\libs\libbtstack_master.a(hfp.o)
                              ..\..\..\Libraries\libs\libbtstack_master.a(btstack_main.o) (hfp_var_init)
..\..\..\Libraries\libs\libbtstack_master.a(avdtp.o)
                              ..\..\..\Libraries\libs\libbtstack_master.a(bt_hook.o) (a2dp_get_play_index)
..\..\..\Libraries\libs\libbtstack_master.a(a2dp.o)
                              ..\..\..\Libraries\libs\libbtstack_master.a(btstack_api.o) (a2dp_is_playing)
..\..\..\Libraries\libs\libbtstack_master.a(btstack_memory_pool.o)
                              ..\..\..\Libraries\libs\libbtstack_master.a(btstack_memory.o) (btstack_memory_pool_get)
..\..\..\Libraries\libs\libbtstack_master.a(btstack_adv0.o)
                              ..\..\..\Libraries\libs\libbtstack_master.a(btstack_api.o) (btstack_adv0_ctrl)
..\..\..\Libraries\libs\libbtstack_master.a(hci_transport_hcic.o)
                              ..\..\..\Libraries\libs\libbtstack_master.a(hci.o) (hcic_rx_flush)
..\..\..\Libraries\libs\libbtstack_master.a(btstack_chipset_inner.o)
                              ..\..\..\Libraries\libs\libbtstack_master.a(btstack_api.o) (btstack_chipset_inner_instance)
..\..\..\Libraries\libs\libbtstack_master.a(lm_hook.o)
                              ..\..\..\Libraries\libs\libbtstack_master.a(lm.o) (lm_init_hook)
..\..\..\Libraries\libs\libbtstack_master.a(lm_sp.o)
                              ..\..\..\Libraries\libs\libbtstack_master.a(lm.o) (lm_oob_f1)
..\..\..\Libraries\libs\libbtstack_master.a(lm_proc.o)
                              ..\..\..\Libraries\libs\libbtstack_master.a(lm.o) (lm_msg_env)
..\..\..\Libraries\libs\libbtstack_master.a(lm_key.o)
                              ..\..\..\Libraries\libs\libbtstack_master.a(lm.o) (lm_e22)
..\..\..\Libraries\libs\libbtstack_master.a(lc.o)
                              ..\..\..\Libraries\libs\libbtstack_master.a(bt21.o) (lc_init)
..\..\..\Libraries\libs\libbtstack_master.a(mgr.o)
                              ..\..\..\Libraries\libs\libbtstack_master.a(ble.o) (mgr_init)
..\..\..\Libraries\libs\libbtstack_master.a(ll.o)
                              ..\..\..\Libraries\libs\libbtstack_master.a(ble.o) (ll_init)
..\..\..\Libraries\libs\libbtstack_master.a(ble_test.o)
                              ..\..\..\Libraries\libs\libbtstack_master.a(ble_hal.o) (ble_test_init)
..\..\..\Libraries\libs\libbtstack_master.a(ble_scan.o)
                              ..\..\..\Libraries\libs\libbtstack_master.a(ble.o) (ble_get_scan_var)
..\..\..\Libraries\libs\libbtstack_master.a(ble_per_adv.o)
                              ..\..\..\Libraries\libs\libbtstack_master.a(ble.o) (ble_get_per_adv_var)
..\..\..\Libraries\libs\libbtstack_master.a(ble_init.o)
                              ..\..\..\Libraries\libs\libbtstack_master.a(ble_hal.o) (ble_init_init)
..\..\..\Libraries\libs\libbtstack_master.a(ble_buf.o)
                              ..\..\..\Libraries\libs\libbtstack_master.a(ble.o) (ble_buf_init)
..\..\..\Libraries\libs\libbtstack_master.a(ble_adv0.o)
                              ..\..\..\Libraries\libs\libbtstack_master.a(ble.o) (ble_adv0_init)
..\..\..\Libraries\libs\libbtstack_master.a(extern_hfhs.o)
                              ..\..\..\Libraries\libs\libbtstack_master.a(hfp.o) (hfp_notice_network_time)
..\..\..\Libraries\libs\libbtstack_master.a(extern_ble.o)
                              ..\..\..\Libraries\libs\libbtstack_master.a(btstack_adv0.o) (ble_adv0_get_adv_data_cb)
..\..\..\Libraries\libs\libbtstack_master.a(l2cap_signaling.o)
                              ..\..\..\Libraries\libs\libbtstack_master.a(l2cap.o) (l2cap_next_sig_id)
..\..\..\Libraries\libs\libbtstack_master.a(lc_hook.o)
                              ..\..\..\Libraries\libs\libbtstack_master.a(lm_proc.o) (lc_auto_sniff_step_set)
..\..\..\Libraries\libs\libbtstack_master.a(lm_sco.o)
                              ..\..\..\Libraries\libs\libbtstack_master.a(lc.o) (lm_init_sync)
..\..\..\Libraries\libs\libbtstack_master.a(lc_util.o)
                              ..\..\..\Libraries\libs\libbtstack_master.a(lc.o) (lc_compute_pkt_types)
..\..\..\Libraries\libs\libbtstack_master.a(lc_sniff.o)
                              ..\..\..\Libraries\libs\libbtstack_master.a(lc.o) (lc_sniff_init)
..\..\..\Libraries\libs\libbtstack_master.a(lc_sco.o)
                              ..\..\..\Libraries\libs\libbtstack_master.a(lc.o) (lc_sco_init)
..\..\..\Libraries\libs\libbtstack_master.a(lc_proc.o)
                              ..\..\..\Libraries\libs\libbtstack_master.a(lc.o) (lc_msg_env)
..\..\..\Libraries\libs\libbtstack_master.a(lc_lmppdu.o)
                              ..\..\..\Libraries\libs\libbtstack_master.a(lc_proc.o) (lmp_estab_allowed)
..\..\..\Libraries\libs\libbtstack_master.a(mgr_proc.o)
                              ..\..\..\Libraries\libs\libbtstack_master.a(mgr.o) (mgr_msg_env)
..\..\..\Libraries\libs\libbtstack_master.a(mgr_init.o)
                              ..\..\..\Libraries\libs\libbtstack_master.a(mgr_proc.o) (ble_init_end_ind_func)
..\..\..\Libraries\libs\libbtstack_master.a(mgr_hci.o)
                              ..\..\..\Libraries\libs\libbtstack_master.a(mgr_proc.o) (hci_command_mgr_func)
..\..\..\Libraries\libs\libbtstack_master.a(ll_scan.o)
                              ..\..\..\Libraries\libs\libbtstack_master.a(mgr_hci.o) (hci_le_set_scan_param_cmd_func)
..\..\..\Libraries\libs\libbtstack_master.a(ll_adv.o)
                              ..\..\..\Libraries\libs\libbtstack_master.a(mgr_hci.o) (hci_le_rd_adv_ch_tx_pw_cmd_func)
..\..\..\Libraries\libs\libbtstack_master.a(ll_proc.o)
                              ..\..\..\Libraries\libs\libbtstack_master.a(ll.o) (ll_msg_env)
..\..\..\Libraries\libs\libbtstack_master.a(ll_ping.o)
                              ..\..\..\Libraries\libs\libbtstack_master.a(ll_proc.o) (hci_rd_auth_payl_to_cmd_func)
..\..\..\Libraries\libs\libbtstack_master.a(ll_phy_upd.o)
                              ..\..\..\Libraries\libs\libbtstack_master.a(ll_proc.o) (hci_le_rd_phy_cmd_func)
..\..\..\Libraries\libs\libbtstack_master.a(ll_past.o)
                              ..\..\..\Libraries\libs\libbtstack_master.a(ll_proc.o) (hci_le_per_adv_set_info_transf_cmd_func)
..\..\..\Libraries\libs\libbtstack_master.a(ll_length.o)
                              ..\..\..\Libraries\libs\libbtstack_master.a(ll_proc.o) (hci_le_set_data_len_cmd_func)
..\..\..\Libraries\libs\libbtstack_master.a(ll_feature.o)
                              ..\..\..\Libraries\libs\libbtstack_master.a(ll_proc.o) (hci_le_rd_rem_feats_cmd_func)
..\..\..\Libraries\libs\libbtstack_master.a(ll_encrypt.o)
                              ..\..\..\Libraries\libs\libbtstack_master.a(ll_proc.o) (hci_le_en_enc_cmd_func)
..\..\..\Libraries\libs\libbtstack_master.a(ll_disconnect.o)
                              ..\..\..\Libraries\libs\libbtstack_master.a(ll_proc.o) (ble_disc_ind_func)
..\..\..\Libraries\libs\libbtstack_master.a(ll_con_upd.o)
                              ..\..\..\Libraries\libs\libbtstack_master.a(ll_proc.o) (hci_le_con_upd_cmd_func)
..\..\..\Libraries\libs\libbtstack_master.a(ll_cntl.o)
                              ..\..\..\Libraries\libs\libbtstack_master.a(ll.o) (ll_cntl_tx_check)
..\..\..\Libraries\libs\libbtstack_master.a(ll_clk_acc.o)
                              ..\..\..\Libraries\libs\libbtstack_master.a(ll_cntl.o) (ll_clk_acc_req_func)
..\..\..\Libraries\libs\libbtstack_master.a(ll_chmap_upd.o)
                              ..\..\..\Libraries\libs\libbtstack_master.a(ll_cntl.o) (ll_channel_map_ind_func)
..\..\..\Libraries\libs\libbtstack_master.a(aes_rpa.o)
                              ..\..\..\Libraries\libs\libbtstack_master.a(ll_adv.o) (aes_rpa_gen)
..\..\..\Libraries\libs\libbtstack_master.a(scan_hook.o)
                              ..\..\..\Libraries\libs\libbtstack_master.a(ll_scan.o) (ble_scan_end_ind_hook)
..\..\..\Libraries\libs\libbtstack_master.a(adv_hook.o)
                              ..\..\..\Libraries\libs\libbtstack_master.a(ll_adv.o) (ble_adv_end_ind_hook)
..\..\..\Libraries\libs\libbtstack_master.a(ll_version.o)
                              ..\..\..\Libraries\libs\libbtstack_master.a(ll_proc.o) (ll_op_ver_exch_ind_func)
..\..\..\Libraries\libs\libbtstack_master.a(ll_pwr.o)
                              ..\..\..\Libraries\libs\libbtstack_master.a(ll_proc.o) (hci_rd_tx_pwr_lvl_cmd_func)

Allocating common symbols
Common symbol       size              file

RECEIVE_BUF         0x200             Output\obj\Examples\BLE_Host\Source\hsuart_transfer.o
fot_var             0x22              Output\obj\Libraries\bsp\bsp_fot.o
f_bt                0x7               Output\obj\Libraries\bsp\bsp_bt.o
TRANSMIT_BUF        0x400             Output\obj\Examples\BLE_Host\Source\hsuart_transfer.o
BtTxBuferCount      0x2               Output\obj\Examples\BLE_Host\Source\hsuart_transfer.o
RECEIVE_Len         0x2               Output\obj\Examples\BLE_Host\Source\hsuart_transfer.o
ticks_50ms          0x4               Output\obj\Libraries\bsp\bsp_sys.o
xcfg_cb             0xae              Output\obj\Libraries\bsp\bsp_sys.o

Discarded input sections

 .text          0x0000000000000000        0x0 Output\obj\Libraries\bsp\bsp_bt.o
 .data          0x0000000000000000        0x0 Output\obj\Libraries\bsp\bsp_bt.o
 .bss           0x0000000000000000        0x0 Output\obj\Libraries\bsp\bsp_bt.o
 .text.bsp_spp_disinit
                0x0000000000000000       0xda Output\obj\Libraries\bsp\bsp_bt.o
 .text.bsp_bt_close
                0x0000000000000000        0x2 Output\obj\Libraries\bsp\bsp_bt.o
 .text.tws_user_key_process
                0x0000000000000000        0x2 Output\obj\Libraries\bsp\bsp_bt.o
 .text.tws_warning_process
                0x0000000000000000        0x2 Output\obj\Libraries\bsp\bsp_bt.o
 .text.bsp_bt_vol_change
                0x0000000000000000        0x2 Output\obj\Libraries\bsp\bsp_bt.o
 .text.bsp_bt_get_hfp_vol
                0x0000000000000000        0x4 Output\obj\Libraries\bsp\bsp_bt.o
 .text.bsp_bt_call_volume_msg
                0x0000000000000000        0x2 Output\obj\Libraries\bsp\bsp_bt.o
 .text          0x0000000000000000        0x0 Output\obj\Libraries\bsp\bsp_cm.o
 .data          0x0000000000000000        0x0 Output\obj\Libraries\bsp\bsp_cm.o
 .bss           0x0000000000000000        0x0 Output\obj\Libraries\bsp\bsp_cm.o
 .text          0x0000000000000000        0x0 Output\obj\Libraries\bsp\bsp_fot.o
 .data          0x0000000000000000        0x0 Output\obj\Libraries\bsp\bsp_fot.o
 .bss           0x0000000000000000        0x0 Output\obj\Libraries\bsp\bsp_fot.o
 .text          0x0000000000000000        0x0 Output\obj\Libraries\bsp\bsp_param.o
 .data          0x0000000000000000        0x0 Output\obj\Libraries\bsp\bsp_param.o
 .bss           0x0000000000000000        0x0 Output\obj\Libraries\bsp\bsp_param.o
 .text          0x0000000000000000        0x0 Output\obj\Libraries\bsp\bsp_sys.o
 .data          0x0000000000000000        0x0 Output\obj\Libraries\bsp\bsp_sys.o
 .bss           0x0000000000000000        0x0 Output\obj\Libraries\bsp\bsp_sys.o
 .text.bsp_get_bat_level
                0x0000000000000000        0x6 Output\obj\Libraries\bsp\bsp_sys.o
 .rodata        0x0000000000000000       0x20 Output\obj\Libraries\bsp\bsp_sys.o
 .text          0x0000000000000000        0x0 Output\obj\Libraries\BT\ble\ab_link\app.o
 .data          0x0000000000000000        0x0 Output\obj\Libraries\BT\ble\ab_link\app.o
 .bss           0x0000000000000000        0x0 Output\obj\Libraries\BT\ble\ab_link\app.o
 .text.gatt_callback_fota
                0x0000000000000000       0x2c Output\obj\Libraries\BT\ble\ab_link\app.o
 .text.gatt_callback_app
                0x0000000000000000       0x1a Output\obj\Libraries\BT\ble\ab_link\app.o
 .text.ble_get_scan_data
                0x0000000000000000       0x68 Output\obj\Libraries\BT\ble\ab_link\app.o
 .text.ble_get_adv_data
                0x0000000000000000       0x6a Output\obj\Libraries\BT\ble\ab_link\app.o
 .text.ble_send_packet1
                0x0000000000000000       0x28 Output\obj\Libraries\BT\ble\ab_link\app.o
 .text.ble_send_packet2
                0x0000000000000000       0x28 Output\obj\Libraries\BT\ble\ab_link\app.o
 .text.ble_read_value
                0x0000000000000000       0x24 Output\obj\Libraries\BT\ble\ab_link\app.o
 .text.bsp_ble_process
                0x0000000000000000        0x2 Output\obj\Libraries\BT\ble\ab_link\app.o
 .text.ble_app_gatts_service_init
                0x0000000000000000      0x1a6 Output\obj\Libraries\BT\ble\ab_link\app.o
 .text.ble_app_init
                0x0000000000000000        0x8 Output\obj\Libraries\BT\ble\ab_link\app.o
 .text.ble_disconnect_event_process
                0x0000000000000000        0xa Output\obj\Libraries\BT\ble\ab_link\app.o
 .text.ble_slave_process
                0x0000000000000000       0x84 Output\obj\Libraries\BT\ble\ab_link\app.o
 .rodata        0x0000000000000000       0xbc Output\obj\Libraries\BT\ble\ab_link\app.o
 .sdata         0x0000000000000000        0xe Output\obj\Libraries\BT\ble\ab_link\app.o
 .text          0x0000000000000000        0x0 Output\obj\Libraries\BT\ble\adv0.o
 .data          0x0000000000000000        0x0 Output\obj\Libraries\BT\ble\adv0.o
 .bss           0x0000000000000000        0x0 Output\obj\Libraries\BT\ble\adv0.o
 .text          0x0000000000000000        0x0 Output\obj\Libraries\BT\ble\ble.o
 .data          0x0000000000000000        0x0 Output\obj\Libraries\BT\ble\ble.o
 .bss           0x0000000000000000        0x0 Output\obj\Libraries\BT\ble\ble.o
 .text.ble_exit_transmit
                0x0000000000000000       0x32 Output\obj\Libraries\BT\ble\ble.o
 .text.ble_get_bat_level
                0x0000000000000000        0x8 Output\obj\Libraries\BT\ble\ble.o
 .text.ble_init_att
                0x0000000000000000        0x8 Output\obj\Libraries\BT\ble\ble.o
 .text          0x0000000000000000        0x0 Output\obj\Libraries\BT\spp\bt.o
 .data          0x0000000000000000        0x0 Output\obj\Libraries\BT\spp\bt.o
 .bss           0x0000000000000000        0x0 Output\obj\Libraries\BT\spp\bt.o
 .text.bt_clr_master_addr
                0x0000000000000000        0x2 Output\obj\Libraries\BT\spp\bt.o
 .text.bt_save_master_addr
                0x0000000000000000        0x2 Output\obj\Libraries\BT\spp\bt.o
 .text.bt_get_master_addr
                0x0000000000000000        0x4 Output\obj\Libraries\BT\spp\bt.o
 .text.bt_clr_all_link_info
                0x0000000000000000        0x8 Output\obj\Libraries\BT\spp\bt.o
 .text.bt_tws_clr_link_info
                0x0000000000000000        0x2 Output\obj\Libraries\BT\spp\bt.o
 .text.bt_get_rand_seed
                0x0000000000000000        0xa Output\obj\Libraries\BT\spp\bt.o
 .rodata        0x0000000000000000        0xa Output\obj\Libraries\BT\spp\bt.o
 .text          0x0000000000000000        0x0 Output\obj\Libraries\BT\spp\hid.o
 .data          0x0000000000000000        0x0 Output\obj\Libraries\BT\spp\hid.o
 .bss           0x0000000000000000        0x0 Output\obj\Libraries\BT\spp\hid.o
 .text.bsp_bt_hid_photo
                0x0000000000000000        0x4 Output\obj\Libraries\BT\spp\hid.o
 .text.bsp_bt_hid_vol_change
                0x0000000000000000        0x4 Output\obj\Libraries\BT\spp\hid.o
 .text.bsp_bt_hid_screen_left
                0x0000000000000000       0x32 Output\obj\Libraries\BT\spp\hid.o
 .text.bsp_bt_hid_screen_right
                0x0000000000000000       0x32 Output\obj\Libraries\BT\spp\hid.o
 .comment       0x0000000000000000       0x12 Output\obj\Libraries\BT\spp\hid.o
 .text          0x0000000000000000        0x0 Output\obj\Libraries\BT\spp\profile.o
 .bss           0x0000000000000000        0x0 Output\obj\Libraries\BT\spp\profile.o
 .text          0x0000000000000000        0x0 Output\obj\Libraries\BT\spp\spp.o
 .data          0x0000000000000000        0x0 Output\obj\Libraries\BT\spp\spp.o
 .bss           0x0000000000000000        0x0 Output\obj\Libraries\BT\spp\spp.o
 .text.bsp_spp_process
                0x0000000000000000        0x2 Output\obj\Libraries\BT\spp\spp.o
 .text          0x0000000000000000        0x0 Output\obj\Libraries\Device\Source\gw3323_clk.o
 .data          0x0000000000000000        0x0 Output\obj\Libraries\Device\Source\gw3323_clk.o
 .bss           0x0000000000000000        0x0 Output\obj\Libraries\Device\Source\gw3323_clk.o
 .text.clock_gate1_cmd
                0x0000000000000000       0x16 Output\obj\Libraries\Device\Source\gw3323_clk.o
 .text.clock_gate2_cmd
                0x0000000000000000       0x16 Output\obj\Libraries\Device\Source\gw3323_clk.o
 .text          0x0000000000000000        0x0 Output\obj\Libraries\Device\Source\gw3323_gpio.o
 .data          0x0000000000000000        0x0 Output\obj\Libraries\Device\Source\gw3323_gpio.o
 .bss           0x0000000000000000        0x0 Output\obj\Libraries\Device\Source\gw3323_gpio.o
 .text.gpio_pic_config_reset
                0x0000000000000000        0xa Output\obj\Libraries\Device\Source\gw3323_gpio.o
 .text.gpio_pic_config
                0x0000000000000000       0x88 Output\obj\Libraries\Device\Source\gw3323_gpio.o
 .com_text.isr  0x0000000000000000       0x28 Output\obj\Libraries\Device\Source\gw3323_gpio.o
 .text          0x0000000000000000        0x0 Output\obj\Libraries\Device\Source\gw3323_hsuart.o
 .data          0x0000000000000000        0x0 Output\obj\Libraries\Device\Source\gw3323_hsuart.o
 .bss           0x0000000000000000        0x0 Output\obj\Libraries\Device\Source\gw3323_hsuart.o
 .text.hsuart_rx_idle_config
                0x0000000000000000        0x6 Output\obj\Libraries\Device\Source\gw3323_hsuart.o
 .text          0x0000000000000000        0x0 Output\obj\Libraries\Device\Source\gw3323_spi.o
 .data          0x0000000000000000        0x0 Output\obj\Libraries\Device\Source\gw3323_spi.o
 .bss           0x0000000000000000        0x0 Output\obj\Libraries\Device\Source\gw3323_spi.o
 .text.spi_init
                0x0000000000000000       0x28 Output\obj\Libraries\Device\Source\gw3323_spi.o
 .text.spi_cmd  0x0000000000000000       0x10 Output\obj\Libraries\Device\Source\gw3323_spi.o
 .text.spi_dir_sel
                0x0000000000000000       0x16 Output\obj\Libraries\Device\Source\gw3323_spi.o
 .text.spi_it_cmd
                0x0000000000000000       0x12 Output\obj\Libraries\Device\Source\gw3323_spi.o
 .text.spi_lfsr_cmd
                0x0000000000000000       0x12 Output\obj\Libraries\Device\Source\gw3323_spi.o
 .text.spi_multi_bit_bus_cmd
                0x0000000000000000       0x12 Output\obj\Libraries\Device\Source\gw3323_spi.o
 .text.spi_hold_rx_cmd
                0x0000000000000000       0x12 Output\obj\Libraries\Device\Source\gw3323_spi.o
 .text.spi_hold_tx_cmd
                0x0000000000000000       0x12 Output\obj\Libraries\Device\Source\gw3323_spi.o
 .text.spi_soft_hold_cmd
                0x0000000000000000       0x12 Output\obj\Libraries\Device\Source\gw3323_spi.o
 .text.spi_get_flag
                0x0000000000000000        0xa Output\obj\Libraries\Device\Source\gw3323_spi.o
 .text.spi_clear_flag
                0x0000000000000000        0x8 Output\obj\Libraries\Device\Source\gw3323_spi.o
 .text.spi_set_dma_cnt
                0x0000000000000000        0x4 Output\obj\Libraries\Device\Source\gw3323_spi.o
 .text.spi_set_dma_addr
                0x0000000000000000        0x4 Output\obj\Libraries\Device\Source\gw3323_spi.o
 .text.spi_receive_data
                0x0000000000000000        0x8 Output\obj\Libraries\Device\Source\gw3323_spi.o
 .text.spi_send_data
                0x0000000000000000        0x4 Output\obj\Libraries\Device\Source\gw3323_spi.o
 .comment       0x0000000000000000       0x12 Output\obj\Libraries\Device\Source\gw3323_spi.o
 .text          0x0000000000000000        0x0 Output\obj\Libraries\libs\strong_symbol.o
 .data          0x0000000000000000        0x0 Output\obj\Libraries\libs\strong_symbol.o
 .bss           0x0000000000000000        0x0 Output\obj\Libraries\libs\strong_symbol.o
 .text.aac_dec_init
                0x0000000000000000        0x2 Output\obj\Libraries\libs\strong_symbol.o
 .text.aac_decode_init
                0x0000000000000000        0x2 Output\obj\Libraries\libs\strong_symbol.o
 .text.aac_dec_frame
                0x0000000000000000        0x4 Output\obj\Libraries\libs\strong_symbol.o
 .text.aac_nor_dec_frame
                0x0000000000000000        0x4 Output\obj\Libraries\libs\strong_symbol.o
 .text.aac_tws_dec_frame
                0x0000000000000000        0x4 Output\obj\Libraries\libs\strong_symbol.o
 .text.aac_cache_free_do
                0x0000000000000000        0x2 Output\obj\Libraries\libs\strong_symbol.o
 .text.aac_cache_read_do
                0x0000000000000000        0x4 Output\obj\Libraries\libs\strong_symbol.o
 .text.tws_pack_aac
                0x0000000000000000        0x4 Output\obj\Libraries\libs\strong_symbol.o
 .com_text.aac.obuf
                0x0000000000000000        0x2 Output\obj\Libraries\libs\strong_symbol.o
 .aacdec.text   0x0000000000000000        0x2 Output\obj\Libraries\libs\strong_symbol.o
 .text.btstack_tws_init
                0x0000000000000000        0x2 Output\obj\Libraries\libs\strong_symbol.o
 .text.a2dp_play_init
                0x0000000000000000        0x2 Output\obj\Libraries\libs\strong_symbol.o
 .bcom_text.sbc.play
                0x0000000000000000       0x28 Output\obj\Libraries\libs\strong_symbol.o
 .bcom_text.sbc_cache
                0x0000000000000000        0xc Output\obj\Libraries\libs\strong_symbol.o
 .sbcdec.code   0x0000000000000000        0x6 Output\obj\Libraries\libs\strong_symbol.o
 .com_text.bb.tws
                0x0000000000000000        0x2 Output\obj\Libraries\libs\strong_symbol.o
 .bcom_text.bb.btisr
                0x0000000000000000       0x12 Output\obj\Libraries\libs\strong_symbol.o
 .text.bt_tws_set_spr
                0x0000000000000000        0x4 Output\obj\Libraries\libs\strong_symbol.o
 .com_text.sbc.play
                0x0000000000000000        0x2 Output\obj\Libraries\libs\strong_symbol.o
 .bcom_text.sbc.send
                0x0000000000000000        0x2 Output\obj\Libraries\libs\strong_symbol.o
 .bcom_text.lc.tws
                0x0000000000000000        0x4 Output\obj\Libraries\libs\strong_symbol.o
 .bcom_text.a2dp.lost
                0x0000000000000000        0x4 Output\obj\Libraries\libs\strong_symbol.o
 .bcom_text.sbc
                0x0000000000000000        0x2 Output\obj\Libraries\libs\strong_symbol.o
 .bcom_text.bb.tws_switch
                0x0000000000000000        0x4 Output\obj\Libraries\libs\strong_symbol.o
 .bcom_text.bb.bttx
                0x0000000000000000        0x6 Output\obj\Libraries\libs\strong_symbol.o
 .text.tws_set_snoop_ticks
                0x0000000000000000        0x4 Output\obj\Libraries\libs\strong_symbol.o
 .text.ble_test_start
                0x0000000000000000        0x4 Output\obj\Libraries\libs\strong_symbol.o
 .text.ble_test_stop
                0x0000000000000000        0x4 Output\obj\Libraries\libs\strong_symbol.o
 .text.huart_init
                0x0000000000000000        0x2 Output\obj\Libraries\libs\strong_symbol.o
 .com_text.bt_rec
                0x0000000000000000        0x2 Output\obj\Libraries\libs\strong_symbol.o
 .text.bt_sco_fill_remote_buf
                0x0000000000000000        0x2 Output\obj\Libraries\libs\strong_symbol.o
 .text.btstack_pbap
                0x0000000000000000        0x2 Output\obj\Libraries\libs\strong_symbol.o
 .text.bsp_charge_ctrl_process
                0x0000000000000000        0x2 Output\obj\Libraries\libs\strong_symbol.o
 .text.usb_dev_isr
                0x0000000000000000        0x2 Output\obj\Libraries\libs\strong_symbol.o
 .text.ude_isoc_tx_process
                0x0000000000000000        0x2 Output\obj\Libraries\libs\strong_symbol.o
 .text.ude_isoc_rx_process
                0x0000000000000000        0x2 Output\obj\Libraries\libs\strong_symbol.o
 .text.lock_code_usbdev
                0x0000000000000000        0x2 Output\obj\Libraries\libs\strong_symbol.o
 .text.unlock_code_usbdev
                0x0000000000000000        0x2 Output\obj\Libraries\libs\strong_symbol.o
 .text.dac_get_max_anl_vol
                0x0000000000000000        0x4 Output\obj\Libraries\libs\strong_symbol.o
 .com_text.dac  0x0000000000000000        0x2 Output\obj\Libraries\libs\strong_symbol.o
 .text.bsp.dac  0x0000000000000000        0x2 Output\obj\Libraries\libs\strong_symbol.o
 .text          0x0000000000000000        0x0 Output\obj\Examples\BLE_Host\Source\ble_client.o
 .data          0x0000000000000000        0x0 Output\obj\Examples\BLE_Host\Source\ble_client.o
 .text.ble_client_user_process
                0x0000000000000000       0x92 Output\obj\Examples\BLE_Host\Source\ble_client.o
 .text          0x0000000000000000        0x0 Output\obj\Examples\BLE_Host\Source\ble_init.o
 .data          0x0000000000000000        0x0 Output\obj\Examples\BLE_Host\Source\ble_init.o
 .bss           0x0000000000000000        0x0 Output\obj\Examples\BLE_Host\Source\ble_init.o
 .text          0x0000000000000000        0x0 Output\obj\Examples\BLE_Host\Source\gpio_input_key.o
 .data          0x0000000000000000        0x0 Output\obj\Examples\BLE_Host\Source\gpio_input_key.o
 .bss           0x0000000000000000        0x0 Output\obj\Examples\BLE_Host\Source\gpio_input_key.o
 .text.gpio_input_init
                0x0000000000000000       0x34 Output\obj\Examples\BLE_Host\Source\gpio_input_key.o
 .comment       0x0000000000000000       0x12 Output\obj\Examples\BLE_Host\Source\gpio_input_key.o
 .text          0x0000000000000000        0x0 Output\obj\Examples\BLE_Host\Source\hsuart_transfer.o
 .data          0x0000000000000000        0x0 Output\obj\Examples\BLE_Host\Source\hsuart_transfer.o
 .bss           0x0000000000000000        0x0 Output\obj\Examples\BLE_Host\Source\hsuart_transfer.o
 .text.huart_SendByte
                0x0000000000000000       0x42 Output\obj\Examples\BLE_Host\Source\hsuart_transfer.o
 .text.huart_SendArray
                0x0000000000000000       0x38 Output\obj\Examples\BLE_Host\Source\hsuart_transfer.o
 .text.huart_SendString
                0x0000000000000000       0x2e Output\obj\Examples\BLE_Host\Source\hsuart_transfer.o
 .text.huart_Pow
                0x0000000000000000       0x14 Output\obj\Examples\BLE_Host\Source\hsuart_transfer.o
 .text.huart_SendNumber
                0x0000000000000000       0x42 Output\obj\Examples\BLE_Host\Source\hsuart_transfer.o
 .text          0x0000000000000000        0x0 Output\obj\Examples\BLE_Host\Project\config.o
 .data          0x0000000000000000        0x0 Output\obj\Examples\BLE_Host\Project\config.o
 .bss           0x0000000000000000        0x0 Output\obj\Examples\BLE_Host\Project\config.o
 .text          0x0000000000000000        0x0 Output\obj\Examples\BLE_Host\Project\main.o
 .data          0x0000000000000000        0x0 Output\obj\Examples\BLE_Host\Project\main.o
 .bss           0x0000000000000000        0x0 Output\obj\Examples\BLE_Host\Project\main.o
 .text          0x0000000000000000        0x0 ..\..\..\Libraries\libs\libplatform.a(audio.o)
 .data          0x0000000000000000        0x0 ..\..\..\Libraries\libs\libplatform.a(audio.o)
 .bss           0x0000000000000000        0x0 ..\..\..\Libraries\libs\libplatform.a(audio.o)
 .com_text.dac  0x0000000000000000       0x66 ..\..\..\Libraries\libs\libplatform.a(audio.o)
 .text.spires   0x0000000000000000       0x40 ..\..\..\Libraries\libs\libplatform.a(audio.o)
 .text          0x0000000000000000        0x0 ..\..\..\Libraries\libs\libplatform.a(cm.o)
 .data          0x0000000000000000        0x0 ..\..\..\Libraries\libs\libplatform.a(cm.o)
 .text.cm_move_allpages
                0x0000000000000000      0x140 ..\..\..\Libraries\libs\libplatform.a(cm.o)
 .text.cm_get_startaddr
                0x0000000000000000        0xa ..\..\..\Libraries\libs\libplatform.a(cm.o)
 .text.cm_get_area
                0x0000000000000000       0x14 ..\..\..\Libraries\libs\libplatform.a(cm.o)
 .text.cm_release_all
                0x0000000000000000       0x90 ..\..\..\Libraries\libs\libplatform.a(cm.o)
 .text.cm_read8
                0x0000000000000000       0x28 ..\..\..\Libraries\libs\libplatform.a(cm.o)
 .text.cm_read16
                0x0000000000000000       0x28 ..\..\..\Libraries\libs\libplatform.a(cm.o)
 .text.cm_read32
                0x0000000000000000       0x24 ..\..\..\Libraries\libs\libplatform.a(cm.o)
 .text.cm_write8
                0x0000000000000000       0x28 ..\..\..\Libraries\libs\libplatform.a(cm.o)
 .text.cm_write16
                0x0000000000000000       0x28 ..\..\..\Libraries\libs\libplatform.a(cm.o)
 .text.cm_write32
                0x0000000000000000       0x24 ..\..\..\Libraries\libs\libplatform.a(cm.o)
 .text.cm_clear
                0x0000000000000000       0x60 ..\..\..\Libraries\libs\libplatform.a(cm.o)
 .text          0x0000000000000000        0x0 ..\..\..\Libraries\libs\libplatform.a(os_flash.o)
 .data          0x0000000000000000        0x0 ..\..\..\Libraries\libs\libplatform.a(os_flash.o)
 .bss           0x0000000000000000        0x0 ..\..\..\Libraries\libs\libplatform.a(os_flash.o)
 .text          0x0000000000000000        0x0 ..\..\..\Libraries\libs\libplatform.a(xcfg.o)
 .data          0x0000000000000000        0x0 ..\..\..\Libraries\libs\libplatform.a(xcfg.o)
 .bss           0x0000000000000000        0x0 ..\..\..\Libraries\libs\libplatform.a(xcfg.o)
 .text          0x0000000000000000        0x0 ..\..\..\Libraries\libs\libplatform.a(device.o)
 .data          0x0000000000000000        0x0 ..\..\..\Libraries\libs\libplatform.a(device.o)
 .bss           0x0000000000000000        0x0 ..\..\..\Libraries\libs\libplatform.a(device.o)
 .text.sd_disable
                0x0000000000000000       0x18 ..\..\..\Libraries\libs\libplatform.a(device.o)
 .text.sd_disable_user
                0x0000000000000000       0x46 ..\..\..\Libraries\libs\libplatform.a(device.o)
 .text.sd_enable_user
                0x0000000000000000       0x2c ..\..\..\Libraries\libs\libplatform.a(device.o)
 .com_text.device
                0x0000000000000000       0x10 ..\..\..\Libraries\libs\libplatform.a(device.o)
 .com_text.device.udisk
                0x0000000000000000        0xe ..\..\..\Libraries\libs\libplatform.a(device.o)
 .com_text.device.filter
                0x0000000000000000       0xe0 ..\..\..\Libraries\libs\libplatform.a(device.o)
 .text.device   0x0000000000000000       0x40 ..\..\..\Libraries\libs\libplatform.a(device.o)
 .text.dev_is_invalid
                0x0000000000000000        0xe ..\..\..\Libraries\libs\libplatform.a(device.o)
 .com_text.sd.api
                0x0000000000000000       0x3c ..\..\..\Libraries\libs\libplatform.a(device.o)
 .text.fs_lock  0x0000000000000000       0x14 ..\..\..\Libraries\libs\libplatform.a(device.o)
 .text.fs_unlock
                0x0000000000000000       0x12 ..\..\..\Libraries\libs\libplatform.a(device.o)
 .sbss          0x0000000000000000        0x4 ..\..\..\Libraries\libs\libplatform.a(device.o)
 .text          0x0000000000000000        0x0 ..\..\..\Libraries\libs\libplatform.a(main.o)
 .data          0x0000000000000000        0x0 ..\..\..\Libraries\libs\libplatform.a(main.o)
 .com_text.exception.do
                0x0000000000000000       0x5a ..\..\..\Libraries\libs\libplatform.a(main.o)
 .com_text.ledseg
                0x0000000000000000       0x40 ..\..\..\Libraries\libs\libplatform.a(main.o)
 .text.uart0_mapping_sel
                0x0000000000000000       0x18 ..\..\..\Libraries\libs\libplatform.a(main.o)
 .text.compiler
                0x0000000000000000       0x20 ..\..\..\Libraries\libs\libplatform.a(main.o)
 .com_text.ledseg.table
                0x0000000000000000        0xc ..\..\..\Libraries\libs\libplatform.a(main.o)
 .text          0x0000000000000000        0x0 ..\..\..\Libraries\libs\libplatform.a(interrupt.o)
 .data          0x0000000000000000        0x0 ..\..\..\Libraries\libs\libplatform.a(interrupt.o)
 .bss           0x0000000000000000        0x0 ..\..\..\Libraries\libs\libplatform.a(interrupt.o)
 .text.timer1_irq_init
                0x0000000000000000       0x38 ..\..\..\Libraries\libs\libplatform.a(interrupt.o)
 .com_text.tws.isr
                0x0000000000000000       0x22 ..\..\..\Libraries\libs\libplatform.a(interrupt.o)
 .text.huart_irq_init
                0x0000000000000000       0x3a ..\..\..\Libraries\libs\libplatform.a(interrupt.o)
 .rodata.str1.4
                0x0000000000000000       0x19 ..\..\..\Libraries\libs\libplatform.a(interrupt.o)
 .text.watch_point_set
                0x0000000000000000       0x48 ..\..\..\Libraries\libs\libplatform.a(interrupt.o)
 .text.wdt_init
                0x0000000000000000       0x3a ..\..\..\Libraries\libs\libplatform.a(interrupt.o)
 .text          0x0000000000000000        0x0 ..\..\..\Libraries\libs\libplatform.a(startup.o)
 .data          0x0000000000000000        0x0 ..\..\..\Libraries\libs\libplatform.a(startup.o)
 .com_text.sndp.api
                0x0000000000000000       0x26 ..\..\..\Libraries\libs\libplatform.a(startup.o)
 .text          0x0000000000000000        0x0 ..\..\..\Libraries\libs\libplatform.a(sys_hook.o)
 .data          0x0000000000000000        0x0 ..\..\..\Libraries\libs\libplatform.a(sys_hook.o)
 .bss           0x0000000000000000        0x0 ..\..\..\Libraries\libs\libplatform.a(sys_hook.o)
 .text          0x0000000000000000        0x0 ..\..\..\Libraries\libs\libplatform.a(reset.o)
 .data          0x0000000000000000        0x0 ..\..\..\Libraries\libs\libplatform.a(reset.o)
 .bss           0x0000000000000000        0x0 ..\..\..\Libraries\libs\libplatform.a(reset.o)
 .text          0x0000000000000000        0x0 ..\..\..\Libraries\libs\libplatform.a(spiflash.o)
 .data          0x0000000000000000        0x0 ..\..\..\Libraries\libs\libplatform.a(spiflash.o)
 .bss           0x0000000000000000        0x0 ..\..\..\Libraries\libs\libplatform.a(spiflash.o)
 .text          0x0000000000000000        0x0 ..\..\..\Libraries\libs\libplatform.a(debug.o)
 .data          0x0000000000000000        0x0 ..\..\..\Libraries\libs\libplatform.a(debug.o)
 .bss           0x0000000000000000        0x0 ..\..\..\Libraries\libs\libplatform.a(debug.o)
 .text.debug_dump_info_nanos_schedule
                0x0000000000000000        0x2 ..\..\..\Libraries\libs\libplatform.a(debug.o)
 .text.debug_dump_info_nanos_timer
                0x0000000000000000        0x2 ..\..\..\Libraries\libs\libplatform.a(debug.o)
 .text          0x0000000000000000        0x0 ..\..\..\Libraries\libs\libplatform.a(fot_update.o)
 .data          0x0000000000000000        0x0 ..\..\..\Libraries\libs\libplatform.a(fot_update.o)
 .text.param_fot_head_info_write
                0x0000000000000000        0x2 ..\..\..\Libraries\libs\libplatform.a(fot_update.o)
 .text.param_fot_head_info_read
                0x0000000000000000        0x2 ..\..\..\Libraries\libs\libplatform.a(fot_update.o)
 .text.param_fot_addr_write
                0x0000000000000000        0x2 ..\..\..\Libraries\libs\libplatform.a(fot_update.o)
 .text.param_fot_addr_read
                0x0000000000000000        0x2 ..\..\..\Libraries\libs\libplatform.a(fot_update.o)
 .text.is_fot_update_en
                0x0000000000000000        0x4 ..\..\..\Libraries\libs\libplatform.a(fot_update.o)
 .text.fot_head_crc_get
                0x0000000000000000       0x9c ..\..\..\Libraries\libs\libplatform.a(fot_update.o)
 .text.fot_get_info
                0x0000000000000000       0x50 ..\..\..\Libraries\libs\libplatform.a(fot_update.o)
 .text          0x0000000000000000        0x0 ..\..\..\Libraries\libs\libplatform.a(lock.o)
 .data          0x0000000000000000        0x0 ..\..\..\Libraries\libs\libplatform.a(lock.o)
 .text.unlock_whcode
                0x0000000000000000       0x3c ..\..\..\Libraries\libs\libplatform.a(lock.o)
 .text.lock_whcode
                0x0000000000000000       0x58 ..\..\..\Libraries\libs\libplatform.a(lock.o)
 .text.unlock_dcode
                0x0000000000000000       0x54 ..\..\..\Libraries\libs\libplatform.a(lock.o)
 .text.lock_dcode
                0x0000000000000000       0x58 ..\..\..\Libraries\libs\libplatform.a(lock.o)
 .text.lock_code_bt_sleep
                0x0000000000000000       0x54 ..\..\..\Libraries\libs\libplatform.a(lock.o)
 .text.unlock_code_bt_sleep
                0x0000000000000000       0x38 ..\..\..\Libraries\libs\libplatform.a(lock.o)
 .text.lock_code_pwrsave
                0x0000000000000000       0x3c ..\..\..\Libraries\libs\libplatform.a(lock.o)
 .text.unlock_code_pwrsave
                0x0000000000000000       0x38 ..\..\..\Libraries\libs\libplatform.a(lock.o)
 .text.lock_code_charge
                0x0000000000000000       0x3c ..\..\..\Libraries\libs\libplatform.a(lock.o)
 .text.unlock_code_charge
                0x0000000000000000        0x8 ..\..\..\Libraries\libs\libplatform.a(lock.o)
 .text.unlock_code_bt_voice
                0x0000000000000000       0x38 ..\..\..\Libraries\libs\libplatform.a(lock.o)
 .text.lock_code_usbdev
                0x0000000000000000       0x54 ..\..\..\Libraries\libs\libplatform.a(lock.o)
 .text.unlock_code_usbdev
                0x0000000000000000       0x38 ..\..\..\Libraries\libs\libplatform.a(lock.o)
 .text.load_code_btdec
                0x0000000000000000       0x54 ..\..\..\Libraries\libs\libplatform.a(lock.o)
 .text.unlock_code_btdec
                0x0000000000000000       0x38 ..\..\..\Libraries\libs\libplatform.a(lock.o)
 .text.load_code_bt_voice
                0x0000000000000000       0x5c ..\..\..\Libraries\libs\libplatform.a(lock.o)
 .text.lock_ram_mp3enc
                0x0000000000000000       0x4c ..\..\..\Libraries\libs\libplatform.a(lock.o)
 .text.unlock_ram_mp3enc
                0x0000000000000000       0x38 ..\..\..\Libraries\libs\libplatform.a(lock.o)
 .text.lock_code_sniff
                0x0000000000000000       0x4c ..\..\..\Libraries\libs\libplatform.a(lock.o)
 .text.unlock_code_sniff
                0x0000000000000000       0x38 ..\..\..\Libraries\libs\libplatform.a(lock.o)
 .text.unlock_code_huart
                0x0000000000000000        0x8 ..\..\..\Libraries\libs\libplatform.a(lock.o)
 .text.lock_code_huart
                0x0000000000000000       0x54 ..\..\..\Libraries\libs\libplatform.a(lock.o)
 .text.lock_code_bb_test
                0x0000000000000000       0x54 ..\..\..\Libraries\libs\libplatform.a(lock.o)
 .text.unlock_code_bb_test
                0x0000000000000000       0x38 ..\..\..\Libraries\libs\libplatform.a(lock.o)
 .text.unlock_code_fota
                0x0000000000000000       0x38 ..\..\..\Libraries\libs\libplatform.a(lock.o)
 .text          0x0000000000000000        0x0 ..\..\..\Libraries\libs\libplatform.a(patch.o)
 .data          0x0000000000000000        0x0 ..\..\..\Libraries\libs\libplatform.a(patch.o)
 .bss           0x0000000000000000        0x0 ..\..\..\Libraries\libs\libplatform.a(patch.o)
 .text          0x0000000000000000        0x0 ..\..\..\Libraries\libs\libplatform.a(power.o)
 .data          0x0000000000000000        0x0 ..\..\..\Libraries\libs\libplatform.a(power.o)
 .bss           0x0000000000000000        0x0 ..\..\..\Libraries\libs\libplatform.a(power.o)
 .com_text.voltage.trim
                0x0000000000000000        0xa ..\..\..\Libraries\libs\libplatform.a(power.o)
 .text          0x0000000000000000        0x0 ..\..\..\Libraries\libs\libplatform.a(rc.o)
 .data          0x0000000000000000        0x0 ..\..\..\Libraries\libs\libplatform.a(rc.o)
 .bss           0x0000000000000000        0x0 ..\..\..\Libraries\libs\libplatform.a(rc.o)
 .text.compiler
                0x0000000000000000        0x2 ..\..\..\Libraries\libs\libplatform.a(rc.o)
 .text          0x0000000000000000        0x0 ..\..\..\Libraries\libs\libplatform.a(s_sys.o)
 .data          0x0000000000000000        0x0 ..\..\..\Libraries\libs\libplatform.a(s_sys.o)
 .bss           0x0000000000000000        0x0 ..\..\..\Libraries\libs\libplatform.a(s_sys.o)
 .text          0x0000000000000000        0x0 ..\..\..\Libraries\libs\libplatform.a(sys.o)
 .data          0x0000000000000000        0x0 ..\..\..\Libraries\libs\libplatform.a(sys.o)
 .bss           0x0000000000000000        0x0 ..\..\..\Libraries\libs\libplatform.a(sys.o)
 .text.dbg_clk_out
                0x0000000000000000       0x44 ..\..\..\Libraries\libs\libplatform.a(sys.o)
 .text.sys_clk_output
                0x0000000000000000      0x136 ..\..\..\Libraries\libs\libplatform.a(sys.o)
 .text.__divdi3
                0x0000000000000000       0x5c ..\..\..\Libraries\libs\libplatform.a(sys.o)
 .text.__umoddi3
                0x0000000000000000       0x30 ..\..\..\Libraries\libs\libplatform.a(sys.o)
 .text.get_random
                0x0000000000000000       0x26 ..\..\..\Libraries\libs\libplatform.a(sys.o)
 .text.random_init
                0x0000000000000000        0xa ..\..\..\Libraries\libs\libplatform.a(sys.o)
 .text.convert_uni2gbk
                0x0000000000000000       0x8a ..\..\..\Libraries\libs\libplatform.a(sys.o)
 .text.lrc      0x0000000000000000       0x58 ..\..\..\Libraries\libs\libplatform.a(sys.o)
 .text.utf8_convert_to_unicode
                0x0000000000000000       0x72 ..\..\..\Libraries\libs\libplatform.a(sys.o)
 .com_text.sys  0x0000000000000000       0x1e ..\..\..\Libraries\libs\libplatform.a(sys.o)
 .text.sw_reset_source_get
                0x0000000000000000       0x2a ..\..\..\Libraries\libs\libplatform.a(sys.o)
 .sleep_text.sleep
                0x0000000000000000      0x128 ..\..\..\Libraries\libs\libplatform.a(sys.o)
 .text.sys.power
                0x0000000000000000       0x96 ..\..\..\Libraries\libs\libplatform.a(sys.o)
 .text          0x0000000000000000        0x0 ..\..\..\Libraries\libs\libplatform.a(sys_clk.o)
 .data          0x0000000000000000        0x0 ..\..\..\Libraries\libs\libplatform.a(sys_clk.o)
 .bss           0x0000000000000000        0x0 ..\..\..\Libraries\libs\libplatform.a(sys_clk.o)
 .com_text.sys  0x0000000000000000        0x4 ..\..\..\Libraries\libs\libplatform.a(sys_clk.o)
 .text.sys_clk.aec
                0x0000000000000000      0x200 ..\..\..\Libraries\libs\libplatform.a(sys_clk.o)
 .text.set_uart0_baud
                0x0000000000000000       0x38 ..\..\..\Libraries\libs\libplatform.a(sys_clk.o)
 .text.set_uart1_baud
                0x0000000000000000       0x38 ..\..\..\Libraries\libs\libplatform.a(sys_clk.o)
 .text.set_uart1_baud_rc2m_clk
                0x0000000000000000       0x24 ..\..\..\Libraries\libs\libplatform.a(sys_clk.o)
 .text.sys_clk_get
                0x0000000000000000        0xa ..\..\..\Libraries\libs\libplatform.a(sys_clk.o)
 .text.sys_clk_req
                0x0000000000000000       0x5e ..\..\..\Libraries\libs\libplatform.a(sys_clk.o)
 .text.sys_clk_free
                0x0000000000000000       0x5c ..\..\..\Libraries\libs\libplatform.a(sys_clk.o)
 .text.sys_clk_free_all
                0x0000000000000000       0x50 ..\..\..\Libraries\libs\libplatform.a(sys_clk.o)
 .text          0x0000000000000000        0x0 ..\..\..\Libraries\libs\libplatform.a(voltage_trim.o)
 .data          0x0000000000000000        0x0 ..\..\..\Libraries\libs\libplatform.a(voltage_trim.o)
 .text          0x0000000000000000        0x0 ..\..\..\Libraries\libs\libplatform.a(weak_symbol.o)
 .data          0x0000000000000000        0x0 ..\..\..\Libraries\libs\libplatform.a(weak_symbol.o)
 .bss           0x0000000000000000        0x0 ..\..\..\Libraries\libs\libplatform.a(weak_symbol.o)
 .text.music_eq_get_bass_tbl
                0x0000000000000000        0x4 ..\..\..\Libraries\libs\libplatform.a(weak_symbol.o)
 .text.music_eq_get_treble_tbl
                0x0000000000000000        0x4 ..\..\..\Libraries\libs\libplatform.a(weak_symbol.o)
 .text.mic_eq_get_bass_tbl
                0x0000000000000000        0x4 ..\..\..\Libraries\libs\libplatform.a(weak_symbol.o)
 .text.mic_eq_get_treble_tbl
                0x0000000000000000        0x4 ..\..\..\Libraries\libs\libplatform.a(weak_symbol.o)
 .text.music_eq_get_tbl
                0x0000000000000000        0x4 ..\..\..\Libraries\libs\libplatform.a(weak_symbol.o)
 .text.bass_treble_get_coef_tbl
                0x0000000000000000        0x4 ..\..\..\Libraries\libs\libplatform.a(weak_symbol.o)
 .text.stream   0x0000000000000000        0x8 ..\..\..\Libraries\libs\libplatform.a(weak_symbol.o)
 .com_text.rec  0x0000000000000000        0x2 ..\..\..\Libraries\libs\libplatform.a(weak_symbol.o)
 .text.update   0x0000000000000000        0x4 ..\..\..\Libraries\libs\libplatform.a(weak_symbol.o)
 .text.qtest    0x0000000000000000       0x1a ..\..\..\Libraries\libs\libplatform.a(weak_symbol.o)
 .text.dacr_is_output
                0x0000000000000000        0x4 ..\..\..\Libraries\libs\libplatform.a(weak_symbol.o)
 .text.sd_is_online
                0x0000000000000000        0x4 ..\..\..\Libraries\libs\libplatform.a(weak_symbol.o)
 .sbss          0x0000000000000000        0x1 ..\..\..\Libraries\libs\libplatform.a(weak_symbol.o)
 .text          0x0000000000000000        0x0 ..\..\..\Libraries\libs\libplatform.a(huart.o)
 .data          0x0000000000000000        0x0 ..\..\..\Libraries\libs\libplatform.a(huart.o)
 .bss           0x0000000000000000        0x0 ..\..\..\Libraries\libs\libplatform.a(huart.o)
 .com_huart.text
                0x0000000000000000      0x1b2 ..\..\..\Libraries\libs\libplatform.a(huart.o)
 .text.huart_tx_done
                0x0000000000000000        0x2 ..\..\..\Libraries\libs\libplatform.a(huart.o)
 .text.lock_code_huart
                0x0000000000000000        0x2 ..\..\..\Libraries\libs\libplatform.a(huart.o)
 .text.huart_irq_init
                0x0000000000000000        0x2 ..\..\..\Libraries\libs\libplatform.a(huart.o)
 .text.huart.huart_init_do
                0x0000000000000000      0x194 ..\..\..\Libraries\libs\libplatform.a(huart.o)
 .text.huart.huart_exit
                0x0000000000000000       0x12 ..\..\..\Libraries\libs\libplatform.a(huart.o)
 .text.huart.huart_setbaudrate
                0x0000000000000000       0x36 ..\..\..\Libraries\libs\libplatform.a(huart.o)
 .com_text.huart.huart_getchar
                0x0000000000000000       0x2e ..\..\..\Libraries\libs\libplatform.a(huart.o)
 .com_huart.rodata
                0x0000000000000000       0x58 ..\..\..\Libraries\libs\libplatform.a(huart.o)
 .sbss          0x0000000000000000        0xc ..\..\..\Libraries\libs\libplatform.a(huart.o)
 .comment       0x0000000000000000       0x13 ..\..\..\Libraries\libs\libplatform.a(huart.o)
 .riscv.attributes
                0x0000000000000000       0x32 ..\..\..\Libraries\libs\libplatform.a(huart.o)
 .text          0x0000000000000000        0x0 ..\..\..\Libraries\libs\libplatform.a(usb.o)
 .data          0x0000000000000000        0x0 ..\..\..\Libraries\libs\libplatform.a(usb.o)
 .bss           0x0000000000000000        0x0 ..\..\..\Libraries\libs\libplatform.a(usb.o)
 .text          0x0000000000000000        0x0 ..\..\..\Libraries\libs\libplatform.a(bt.o)
 .data          0x0000000000000000        0x0 ..\..\..\Libraries\libs\libplatform.a(bt.o)
 .bss           0x0000000000000000        0x0 ..\..\..\Libraries\libs\libplatform.a(bt.o)
 .com_text.isr.txrx
                0x0000000000000000        0x2 ..\..\..\Libraries\libs\libplatform.a(bt.o)
 .text.update   0x0000000000000000        0x4 ..\..\..\Libraries\libs\libplatform.a(bt.o)
 .bt_voice.plc  0x0000000000000000       0x48 ..\..\..\Libraries\libs\libplatform.a(bt.o)
 .rodata.str1.4
                0x0000000000000000        0xd ..\..\..\Libraries\libs\libplatform.a(bt.o)
 .com_text.btstack.uart
                0x0000000000000000       0x26 ..\..\..\Libraries\libs\libplatform.a(bt.o)
 .text          0x0000000000000000        0x0 ..\..\..\Libraries\libs\libdrivers.a(usb_device_hid.o)
 .data          0x0000000000000000        0x0 ..\..\..\Libraries\libs\libdrivers.a(usb_device_hid.o)
 .bss           0x0000000000000000        0x0 ..\..\..\Libraries\libs\libdrivers.a(usb_device_hid.o)
 .com_text.bulkep
                0x0000000000000000       0x80 ..\..\..\Libraries\libs\libdrivers.a(usb_device_hid.o)
 .text.usb_hid_ep_config
                0x0000000000000000        0xa ..\..\..\Libraries\libs\libdrivers.a(usb_device_hid.o)
 .text.usb_user_ep_config
                0x0000000000000000       0x2e ..\..\..\Libraries\libs\libdrivers.a(usb_device_hid.o)
 .text          0x0000000000000000        0x0 ..\..\..\Libraries\libs\libdrivers.a(usb_device_printer.o)
 .data          0x0000000000000000        0x0 ..\..\..\Libraries\libs\libdrivers.a(usb_device_printer.o)
 .bss           0x0000000000000000        0x0 ..\..\..\Libraries\libs\libdrivers.a(usb_device_printer.o)
 .com_text.bulkep
                0x0000000000000000       0xaa ..\..\..\Libraries\libs\libdrivers.a(usb_device_printer.o)
 .text.usb_printer_ep_config
                0x0000000000000000       0x12 ..\..\..\Libraries\libs\libdrivers.a(usb_device_printer.o)
 .text.udp_init
                0x0000000000000000       0xa2 ..\..\..\Libraries\libs\libdrivers.a(usb_device_printer.o)
 .sdata         0x0000000000000000        0x2 ..\..\..\Libraries\libs\libdrivers.a(usb_device_printer.o)
 .text          0x0000000000000000        0x0 ..\..\..\Libraries\libs\libdrivers.a(usb_device_run_loop.o)
 .data          0x0000000000000000        0x0 ..\..\..\Libraries\libs\libdrivers.a(usb_device_run_loop.o)
 .bss           0x0000000000000000        0x0 ..\..\..\Libraries\libs\libdrivers.a(usb_device_run_loop.o)
 .text.usb_device_exit
                0x0000000000000000       0x32 ..\..\..\Libraries\libs\libdrivers.a(usb_device_run_loop.o)
 .usbdev.com    0x0000000000000000       0xa8 ..\..\..\Libraries\libs\libdrivers.a(usb_device_run_loop.o)
 .text.usb_device_init
                0x0000000000000000       0xac ..\..\..\Libraries\libs\libdrivers.a(usb_device_run_loop.o)
 .text.usb_device_enter
                0x0000000000000000       0x74 ..\..\..\Libraries\libs\libdrivers.a(usb_device_run_loop.o)
 .com_text.usb.device
                0x0000000000000000       0x62 ..\..\..\Libraries\libs\libdrivers.a(usb_device_run_loop.o)
 .com_text.irq  0x0000000000000000       0x10 ..\..\..\Libraries\libs\libdrivers.a(usb_device_run_loop.o)
 .usb_buf.device.desc.buf
                0x0000000000000000      0x400 ..\..\..\Libraries\libs\libdrivers.a(usb_device_run_loop.o)
 .usb_buf.isoc  0x0000000000000000      0x140 ..\..\..\Libraries\libs\libdrivers.a(usb_device_run_loop.o)
 .usb_buf.printer
                0x0000000000000000       0x80 ..\..\..\Libraries\libs\libdrivers.a(usb_device_run_loop.o)
 .text          0x0000000000000000        0x0 ..\..\..\Libraries\libs\libdrivers.a(usb_host_manage.o)
 .data          0x0000000000000000        0x0 ..\..\..\Libraries\libs\libdrivers.a(usb_host_manage.o)
 .bss           0x0000000000000000        0x0 ..\..\..\Libraries\libs\libdrivers.a(usb_host_manage.o)
 .text.usb_host_var_init
                0x0000000000000000       0x3c ..\..\..\Libraries\libs\libdrivers.a(usb_host_manage.o)
 .text.uhs_is_iphone
                0x0000000000000000       0x12 ..\..\..\Libraries\libs\libdrivers.a(usb_host_manage.o)
 .text.usb.host.init
                0x0000000000000000       0x96 ..\..\..\Libraries\libs\libdrivers.a(usb_host_manage.o)
 .com_text.irq  0x0000000000000000       0x12 ..\..\..\Libraries\libs\libdrivers.a(usb_host_manage.o)
 .text.udisk_suspend
                0x0000000000000000       0x32 ..\..\..\Libraries\libs\libdrivers.a(usb_host_manage.o)
 .text.udisk_resume
                0x0000000000000000       0x4c ..\..\..\Libraries\libs\libdrivers.a(usb_host_manage.o)
 .com_text.usb.host
                0x0000000000000000       0x82 ..\..\..\Libraries\libs\libdrivers.a(usb_host_manage.o)
 .text.udisk_read
                0x0000000000000000       0x7c ..\..\..\Libraries\libs\libdrivers.a(usb_host_manage.o)
 .text.uhs_set_nluns
                0x0000000000000000        0xa ..\..\..\Libraries\libs\libdrivers.a(usb_host_manage.o)
 .text.udisk_write
                0x0000000000000000       0x54 ..\..\..\Libraries\libs\libdrivers.a(usb_host_manage.o)
 .buf.usb       0x0000000000000000       0x74 ..\..\..\Libraries\libs\libdrivers.a(usb_host_manage.o)
 .comment       0x0000000000000000       0x13 ..\..\..\Libraries\libs\libdrivers.a(usb_host_manage.o)
 .riscv.attributes
                0x0000000000000000       0x32 ..\..\..\Libraries\libs\libdrivers.a(usb_host_manage.o)
 .text          0x0000000000000000        0x0 ..\..\..\Libraries\libs\libdrivers.a(usb_host_storage.o)
 .data          0x0000000000000000        0x0 ..\..\..\Libraries\libs\libdrivers.a(usb_host_storage.o)
 .bss           0x0000000000000000        0x0 ..\..\..\Libraries\libs\libdrivers.a(usb_host_storage.o)
 .text.do_transfer
                0x0000000000000000       0xae ..\..\..\Libraries\libs\libdrivers.a(usb_host_storage.o)
 .text.do_receive
                0x0000000000000000       0xf6 ..\..\..\Libraries\libs\libdrivers.a(usb_host_storage.o)
 .text.do_request
                0x0000000000000000      0x20a ..\..\..\Libraries\libs\libdrivers.a(usb_host_storage.o)
 .text.do_scsi_request
                0x0000000000000000       0xf8 ..\..\..\Libraries\libs\libdrivers.a(usb_host_storage.o)
 .text.uhs_start
                0x0000000000000000      0x18c ..\..\..\Libraries\libs\libdrivers.a(usb_host_storage.o)
 .text.uhs_read
                0x0000000000000000       0x64 ..\..\..\Libraries\libs\libdrivers.a(usb_host_storage.o)
 .text.uhs_write
                0x0000000000000000       0x64 ..\..\..\Libraries\libs\libdrivers.a(usb_host_storage.o)
 .text.uhs_init
                0x0000000000000000       0x26 ..\..\..\Libraries\libs\libdrivers.a(usb_host_storage.o)
 .rodata        0x0000000000000000       0x57 ..\..\..\Libraries\libs\libdrivers.a(usb_host_storage.o)
 .comment       0x0000000000000000       0x13 ..\..\..\Libraries\libs\libdrivers.a(usb_host_storage.o)
 .riscv.attributes
                0x0000000000000000       0x32 ..\..\..\Libraries\libs\libdrivers.a(usb_host_storage.o)
 .text          0x0000000000000000        0x0 ..\..\..\Libraries\libs\libdrivers.a(usb_comm.o)
 .data          0x0000000000000000        0x0 ..\..\..\Libraries\libs\libdrivers.a(usb_comm.o)
 .bss           0x0000000000000000        0x0 ..\..\..\Libraries\libs\libdrivers.a(usb_comm.o)
 .text.usb_init
                0x0000000000000000       0x80 ..\..\..\Libraries\libs\libdrivers.a(usb_comm.o)
 .text.usb_host_enter
                0x0000000000000000       0x56 ..\..\..\Libraries\libs\libdrivers.a(usb_comm.o)
 .usbdev.com    0x0000000000000000       0x20 ..\..\..\Libraries\libs\libdrivers.a(usb_comm.o)
 .com_text.irq  0x0000000000000000       0x2a ..\..\..\Libraries\libs\libdrivers.a(usb_comm.o)
 .buf.usb.ctrl  0x0000000000000000       0x40 ..\..\..\Libraries\libs\libdrivers.a(usb_comm.o)
 .text          0x0000000000000000        0x0 ..\..\..\Libraries\libs\libdrivers.a(usb_detect.o)
 .data          0x0000000000000000        0x0 ..\..\..\Libraries\libs\libdrivers.a(usb_detect.o)
 .bss           0x0000000000000000        0x0 ..\..\..\Libraries\libs\libdrivers.a(usb_detect.o)
 .com_text.usb.dectect
                0x0000000000000000      0x108 ..\..\..\Libraries\libs\libdrivers.a(usb_detect.o)
 .buf.usbchk.cb
                0x0000000000000000        0x2 ..\..\..\Libraries\libs\libdrivers.a(usb_detect.o)
 .comment       0x0000000000000000       0x13 ..\..\..\Libraries\libs\libdrivers.a(usb_detect.o)
 .riscv.attributes
                0x0000000000000000       0x32 ..\..\..\Libraries\libs\libdrivers.a(usb_detect.o)
 .text          0x0000000000000000        0x0 ..\..\..\Libraries\libs\libdrivers.a(usb_device_desc.o)
 .data          0x0000000000000000        0x0 ..\..\..\Libraries\libs\libdrivers.a(usb_device_desc.o)
 .bss           0x0000000000000000        0x0 ..\..\..\Libraries\libs\libdrivers.a(usb_device_desc.o)
 .text.usb_get_device_descriptor
                0x0000000000000000        0x8 ..\..\..\Libraries\libs\libdrivers.a(usb_device_desc.o)
 .text.usb_get_config_descriptor
                0x0000000000000000        0x8 ..\..\..\Libraries\libs\libdrivers.a(usb_device_desc.o)
 .text.usb_get_lang_id_str_descriptor
                0x0000000000000000        0x8 ..\..\..\Libraries\libs\libdrivers.a(usb_device_desc.o)
 .text.usb_get_manufacturer_str_descriptor
                0x0000000000000000        0x8 ..\..\..\Libraries\libs\libdrivers.a(usb_device_desc.o)
 .text.usb_get_product_str_descriptor
                0x0000000000000000        0x8 ..\..\..\Libraries\libs\libdrivers.a(usb_device_desc.o)
 .text.usb_get_serial_str_descriptor
                0x0000000000000000        0x8 ..\..\..\Libraries\libs\libdrivers.a(usb_device_desc.o)
 .text.usb_get_hid_config_descriptor
                0x0000000000000000        0x8 ..\..\..\Libraries\libs\libdrivers.a(usb_device_desc.o)
 .text.usb_get_hid_report_descriptor
                0x0000000000000000        0x8 ..\..\..\Libraries\libs\libdrivers.a(usb_device_desc.o)
 .comment       0x0000000000000000       0x13 ..\..\..\Libraries\libs\libdrivers.a(usb_device_desc.o)
 .riscv.attributes
                0x0000000000000000       0x32 ..\..\..\Libraries\libs\libdrivers.a(usb_device_desc.o)
 .text          0x0000000000000000        0x0 ..\..\..\Libraries\libs\libdrivers.a(usb_device_enum.o)
 .data          0x0000000000000000        0x0 ..\..\..\Libraries\libs\libdrivers.a(usb_device_enum.o)
 .bss           0x0000000000000000        0xa ..\..\..\Libraries\libs\libdrivers.a(usb_device_enum.o)
 .usbdev.com    0x0000000000000000      0x9c2 ..\..\..\Libraries\libs\libdrivers.a(usb_device_enum.o)
 .text.usb_ep0_out_data_callback
                0x0000000000000000        0x4 ..\..\..\Libraries\libs\libdrivers.a(usb_device_enum.o)
 .text.usb_itf_in_req
                0x0000000000000000        0x4 ..\..\..\Libraries\libs\libdrivers.a(usb_device_enum.o)
 .comment       0x0000000000000000       0x13 ..\..\..\Libraries\libs\libdrivers.a(usb_device_enum.o)
 .riscv.attributes
                0x0000000000000000       0x32 ..\..\..\Libraries\libs\libdrivers.a(usb_device_enum.o)
 .text          0x0000000000000000        0x0 ..\..\..\Libraries\libs\libdrivers.a(usb_device_ep.o)
 .data          0x0000000000000000        0x0 ..\..\..\Libraries\libs\libdrivers.a(usb_device_ep.o)
 .text          0x0000000000000000        0x0 ..\..\..\Libraries\libs\libdrivers.a(usb_host_enum.o)
 .data          0x0000000000000000        0x0 ..\..\..\Libraries\libs\libdrivers.a(usb_host_enum.o)
 .bss           0x0000000000000000        0x0 ..\..\..\Libraries\libs\libdrivers.a(usb_host_enum.o)
 .text.wait_transfering
                0x0000000000000000       0x3c ..\..\..\Libraries\libs\libdrivers.a(usb_host_enum.o)
 .text.do_receive
                0x0000000000000000       0x90 ..\..\..\Libraries\libs\libdrivers.a(usb_host_enum.o)
 .text.do_skip_rxdata
                0x0000000000000000       0x4c ..\..\..\Libraries\libs\libdrivers.a(usb_host_enum.o)
 .text.do_request.isra.0
                0x0000000000000000      0x298 ..\..\..\Libraries\libs\libdrivers.a(usb_host_enum.o)
 .text.uhe_reset
                0x0000000000000000       0x34 ..\..\..\Libraries\libs\libdrivers.a(usb_host_enum.o)
 .rodata.str1.4
                0x0000000000000000        0xb ..\..\..\Libraries\libs\libdrivers.a(usb_host_enum.o)
 .text.uhe_start
                0x0000000000000000      0x22c ..\..\..\Libraries\libs\libdrivers.a(usb_host_enum.o)
 .text.uhe_clear_feature
                0x0000000000000000       0x44 ..\..\..\Libraries\libs\libdrivers.a(usb_host_enum.o)
 .text.uhe_init
                0x0000000000000000       0x24 ..\..\..\Libraries\libs\libdrivers.a(usb_host_enum.o)
 .rodata        0x0000000000000000       0x40 ..\..\..\Libraries\libs\libdrivers.a(usb_host_enum.o)
 .rodata.uhe    0x0000000000000000       0x40 ..\..\..\Libraries\libs\libdrivers.a(usb_host_enum.o)
 .comment       0x0000000000000000       0x13 ..\..\..\Libraries\libs\libdrivers.a(usb_host_enum.o)
 .riscv.attributes
                0x0000000000000000       0x32 ..\..\..\Libraries\libs\libdrivers.a(usb_host_enum.o)
 .text          0x0000000000000000        0x0 ..\..\..\Libraries\libs\libdrivers.a(weak_symbol.o)
 .data          0x0000000000000000        0x0 ..\..\..\Libraries\libs\libdrivers.a(weak_symbol.o)
 .bss           0x0000000000000000        0x0 ..\..\..\Libraries\libs\libdrivers.a(weak_symbol.o)
 .text.iphone_power_set
                0x0000000000000000       0x12 ..\..\..\Libraries\libs\libdrivers.a(weak_symbol.o)
 .comment       0x0000000000000000       0x13 ..\..\..\Libraries\libs\libdrivers.a(weak_symbol.o)
 .riscv.attributes
                0x0000000000000000       0x32 ..\..\..\Libraries\libs\libdrivers.a(weak_symbol.o)
 .text          0x0000000000000000        0x0 ..\..\..\Libraries\libs\libdrivers.a(usb_device_audio.o)
 .data          0x0000000000000000        0x0 ..\..\..\Libraries\libs\libdrivers.a(usb_device_audio.o)
 .bss           0x0000000000000000        0x0 ..\..\..\Libraries\libs\libdrivers.a(usb_device_audio.o)
 .usbdev.com    0x0000000000000000      0x36a ..\..\..\Libraries\libs\libdrivers.a(usb_device_audio.o)
 .ude.aubuf     0x0000000000000000      0x8d4 ..\..\..\Libraries\libs\libdrivers.a(usb_device_audio.o)
 .usbdev.com.table
                0x0000000000000000        0x3 ..\..\..\Libraries\libs\libdrivers.a(usb_device_audio.o)
 .comment       0x0000000000000000       0x13 ..\..\..\Libraries\libs\libdrivers.a(usb_device_audio.o)
 .riscv.attributes
                0x0000000000000000       0x32 ..\..\..\Libraries\libs\libdrivers.a(usb_device_audio.o)
 .data          0x0000000000000000        0x0 ..\..\..\Libraries\libs\libbtstack_master.a(nanos.o)
 .bss           0x0000000000000000        0x0 ..\..\..\Libraries\libs\libbtstack_master.a(nanos.o)
 .com_text.md.nanos
                0x0000000000000000       0x3c ..\..\..\Libraries\libs\libbtstack_master.a(nanos.o)
 .data          0x0000000000000000        0x0 ..\..\..\Libraries\libs\libbtstack_master.a(patch.o)
 .bss           0x0000000000000000        0x0 ..\..\..\Libraries\libs\libbtstack_master.a(patch.o)
 .data          0x0000000000000000        0x0 ..\..\..\Libraries\libs\libbtstack_master.a(platform.o)
 .bss           0x0000000000000000        0x0 ..\..\..\Libraries\libs\libbtstack_master.a(platform.o)
 .com_text.bb.isr.timer
                0x0000000000000000        0x2 ..\..\..\Libraries\libs\libbtstack_master.a(platform.o)
 .data          0x0000000000000000        0x0 ..\..\..\Libraries\libs\libbtstack_master.a(bt_sco.o)
 .bss           0x0000000000000000        0x0 ..\..\..\Libraries\libs\libbtstack_master.a(bt_sco.o)
 .bt_voice.bb.cvsd
                0x0000000000000000        0x2 ..\..\..\Libraries\libs\libbtstack_master.a(bt_sco.o)
 .bt_voice.plc  0x0000000000000000        0x2 ..\..\..\Libraries\libs\libbtstack_master.a(bt_sco.o)
 .data          0x0000000000000000        0x0 ..\..\..\Libraries\libs\libbtstack_master.a(bt_acl.o)
 .bss           0x0000000000000000        0x0 ..\..\..\Libraries\libs\libbtstack_master.a(bt_acl.o)
 .data          0x0000000000000000        0x0 ..\..\..\Libraries\libs\libbtstack_master.a(ble_con.o)
 .bss           0x0000000000000000        0x0 ..\..\..\Libraries\libs\libbtstack_master.a(ble_con.o)
 .data          0x0000000000000000        0x0 ..\..\..\Libraries\libs\libbtstack_master.a(bb_utils.o)
 .bss           0x0000000000000000        0x0 ..\..\..\Libraries\libs\libbtstack_master.a(bb_utils.o)
 .srodata       0x0000000000000000        0x5 ..\..\..\Libraries\libs\libbtstack_master.a(bb_utils.o)
 .data          0x0000000000000000        0x0 ..\..\..\Libraries\libs\libbtstack_master.a(bb_int.o)
 .bss           0x0000000000000000        0x0 ..\..\..\Libraries\libs\libbtstack_master.a(bb_int.o)
 .com_text.bb.isr.timer
                0x0000000000000000       0x48 ..\..\..\Libraries\libs\libbtstack_master.a(bb_int.o)
 .text.bb.timer.init
                0x0000000000000000       0x76 ..\..\..\Libraries\libs\libbtstack_master.a(bb_int.o)
 .text.bb.timer.kill
                0x0000000000000000       0x22 ..\..\..\Libraries\libs\libbtstack_master.a(bb_int.o)
 .com_text.bb.timer.get
                0x0000000000000000       0x24 ..\..\..\Libraries\libs\libbtstack_master.a(bb_int.o)
 .sleep_text.bb
                0x0000000000000000      0x232 ..\..\..\Libraries\libs\libbtstack_master.a(bb_int.o)
 .com_text.bb.sleep
                0x0000000000000000       0x4c ..\..\..\Libraries\libs\libbtstack_master.a(bb_int.o)
 .data          0x0000000000000000        0x0 ..\..\..\Libraries\libs\libbtstack_master.a(bb.o)
 .text.update   0x0000000000000000       0x1a ..\..\..\Libraries\libs\libbtstack_master.a(bb.o)
 .data          0x0000000000000000        0x0 ..\..\..\Libraries\libs\libbtstack_master.a(platform.o)
 .bss           0x0000000000000000        0x0 ..\..\..\Libraries\libs\libbtstack_master.a(platform.o)
 .com_text.cpu.sfr
                0x0000000000000000       0x3c ..\..\..\Libraries\libs\libbtstack_master.a(platform.o)
 .com_text.sco  0x0000000000000000        0x8 ..\..\..\Libraries\libs\libbtstack_master.a(platform.o)
 .data          0x0000000000000000        0x0 ..\..\..\Libraries\libs\libbtstack_master.a(extern_tws.o)
 .bss           0x0000000000000000        0x0 ..\..\..\Libraries\libs\libbtstack_master.a(extern_tws.o)
 .sdata         0x0000000000000000        0x7 ..\..\..\Libraries\libs\libbtstack_master.a(extern_tws.o)
 .data          0x0000000000000000        0x0 ..\..\..\Libraries\libs\libbtstack_master.a(extern_bt.o)
 .bss           0x0000000000000000        0x0 ..\..\..\Libraries\libs\libbtstack_master.a(extern_bt.o)
 .com_text.bt_rec
                0x0000000000000000        0x2 ..\..\..\Libraries\libs\libbtstack_master.a(extern_bt.o)
 .com_text.aec  0x0000000000000000        0x4 ..\..\..\Libraries\libs\libbtstack_master.a(extern_bt.o)
 .bt_voice.sco  0x0000000000000000        0x2 ..\..\..\Libraries\libs\libbtstack_master.a(extern_bt.o)
 .bt_voice.bb.cvsd
                0x0000000000000000        0x2 ..\..\..\Libraries\libs\libbtstack_master.a(extern_bt.o)
 .text          0x0000000000000000       0x28 ..\..\..\Libraries\libs\libbtstack_master.a(extern.o)
 .data          0x0000000000000000        0x0 ..\..\..\Libraries\libs\libbtstack_master.a(extern.o)
 .bss           0x0000000000000000        0x0 ..\..\..\Libraries\libs\libbtstack_master.a(extern.o)
 .text.huart    0x0000000000000000        0x2 ..\..\..\Libraries\libs\libbtstack_master.a(extern.o)
 .com_text.huart
                0x0000000000000000        0xe ..\..\..\Libraries\libs\libbtstack_master.a(extern.o)
 .com_text.ticks
                0x0000000000000000        0x4 ..\..\..\Libraries\libs\libbtstack_master.a(extern.o)
 .sbss          0x0000000000000000        0x1 ..\..\..\Libraries\libs\libbtstack_master.a(extern.o)
 .data          0x0000000000000000        0x0 ..\..\..\Libraries\libs\libbtstack_master.a(spp.o)
 .bss           0x0000000000000000        0x0 ..\..\..\Libraries\libs\libbtstack_master.a(spp.o)
 .sbss          0x0000000000000000        0x1 ..\..\..\Libraries\libs\libbtstack_master.a(spp.o)
 .text          0x0000000000000000        0x0 ..\..\..\Libraries\libs\libbtstack_master.a(sdp_util.o)
 .data          0x0000000000000000        0x0 ..\..\..\Libraries\libs\libbtstack_master.a(sdp_util.o)
 .bss           0x0000000000000000        0x0 ..\..\..\Libraries\libs\libbtstack_master.a(sdp_util.o)
 .text          0x0000000000000000        0x0 ..\..\..\Libraries\libs\libbtstack_master.a(sdp_tbl.o)
 .data          0x0000000000000000        0x0 ..\..\..\Libraries\libs\libbtstack_master.a(sdp_tbl.o)
 .bss           0x0000000000000000        0x0 ..\..\..\Libraries\libs\libbtstack_master.a(sdp_tbl.o)
 .rodata.sdp.tbl.avctp_controller
                0x0000000000000000       0x44 ..\..\..\Libraries\libs\libbtstack_master.a(sdp_tbl.o)
 .rodata.sdp.tbl.avctp_target2
                0x0000000000000000       0x41 ..\..\..\Libraries\libs\libbtstack_master.a(sdp_tbl.o)
 .rodata.sdp.tbl.avdtp
                0x0000000000000000       0x41 ..\..\..\Libraries\libs\libbtstack_master.a(sdp_tbl.o)
 .rodata.sdp.tbl.hfp
                0x0000000000000000       0x50 ..\..\..\Libraries\libs\libbtstack_master.a(sdp_tbl.o)
 .rodata.sdp.tbl.hid_consumer
                0x0000000000000000       0xd2 ..\..\..\Libraries\libs\libbtstack_master.a(sdp_tbl.o)
 .rodata.sdp.tbl.hid_did
                0x0000000000000000       0x40 ..\..\..\Libraries\libs\libbtstack_master.a(sdp_tbl.o)
 .rodata.sdp.tbl.hid_keyboard
                0x0000000000000000      0x115 ..\..\..\Libraries\libs\libbtstack_master.a(sdp_tbl.o)
 .rodata.sdp.tbl.hid_tscreen
                0x0000000000000000      0x110 ..\..\..\Libraries\libs\libbtstack_master.a(sdp_tbl.o)
 .rodata.sdp.tbl.hid_tscreen_ext
                0x0000000000000000      0x119 ..\..\..\Libraries\libs\libbtstack_master.a(sdp_tbl.o)
 .rodata.sdp.tbl.spp_dueros
                0x0000000000000000       0x51 ..\..\..\Libraries\libs\libbtstack_master.a(sdp_tbl.o)
 .data          0x0000000000000000        0x0 ..\..\..\Libraries\libs\libbtstack_master.a(sdp_server.o)
 .bss           0x0000000000000000        0x0 ..\..\..\Libraries\libs\libbtstack_master.a(sdp_server.o)
 .text.stack.sdp.server_rmv
                0x0000000000000000       0x2c ..\..\..\Libraries\libs\libbtstack_master.a(sdp_server.o)
 .data          0x0000000000000000        0x0 ..\..\..\Libraries\libs\libbtstack_master.a(sdp_client.o)
 .bss           0x0000000000000000        0x0 ..\..\..\Libraries\libs\libbtstack_master.a(sdp_client.o)
 .data          0x0000000000000000        0x0 ..\..\..\Libraries\libs\libbtstack_master.a(rfcomm.o)
 .bss           0x0000000000000000        0x0 ..\..\..\Libraries\libs\libbtstack_master.a(rfcomm.o)
 .text          0x0000000000000000        0x0 ..\..\..\Libraries\libs\libbtstack_master.a(btstack_link_key_db.o)
 .sbss          0x0000000000000000        0x1 ..\..\..\Libraries\libs\libbtstack_master.a(btstack_link_key_db.o)
 .data          0x0000000000000000        0x0 ..\..\..\Libraries\libs\libbtstack_master.a(btstack_util.o)
 .bss           0x0000000000000000        0x0 ..\..\..\Libraries\libs\libbtstack_master.a(btstack_util.o)
 .data          0x0000000000000000        0x0 ..\..\..\Libraries\libs\libbtstack_master.a(btstack_txpkt.o)
 .bss           0x0000000000000000        0x0 ..\..\..\Libraries\libs\libbtstack_master.a(btstack_txpkt.o)
 .text          0x0000000000000000        0x0 ..\..\..\Libraries\libs\libbtstack_master.a(btstack_run_loop.o)
 .bss           0x0000000000000000        0x0 ..\..\..\Libraries\libs\libbtstack_master.a(btstack_run_loop.o)
 .data          0x0000000000000000        0x0 ..\..\..\Libraries\libs\libbtstack_master.a(btstack_memory.o)
 .text          0x0000000000000000       0x54 ..\..\..\Libraries\libs\libbtstack_master.a(btstack_linked_list.o)
 .data          0x0000000000000000        0x0 ..\..\..\Libraries\libs\libbtstack_master.a(btstack_linked_list.o)
 .bss           0x0000000000000000        0x0 ..\..\..\Libraries\libs\libbtstack_master.a(btstack_linked_list.o)
 .com_text.fifo.search
                0x0000000000000000       0x28 ..\..\..\Libraries\libs\libbtstack_master.a(btstack_linked_list.o)
 .com_text.fifo.add
                0x0000000000000000       0x5e ..\..\..\Libraries\libs\libbtstack_master.a(btstack_linked_list.o)
 .btdec.a2dp.list
                0x0000000000000000      0x1be ..\..\..\Libraries\libs\libbtstack_master.a(btstack_linked_list.o)
 .data          0x0000000000000000        0x0 ..\..\..\Libraries\libs\libbtstack_master.a(btstack_link_ctrl.o)
 .bss           0x0000000000000000        0x0 ..\..\..\Libraries\libs\libbtstack_master.a(btstack_link_ctrl.o)
 .sbss          0x0000000000000000        0x1 ..\..\..\Libraries\libs\libbtstack_master.a(btstack_link_ctrl.o)
 .data          0x0000000000000000        0x0 ..\..\..\Libraries\libs\libbtstack_master.a(sm.o)
 .data          0x0000000000000000        0x0 ..\..\..\Libraries\libs\libbtstack_master.a(le_device_db_memory.o)
 .bss           0x0000000000000000        0x0 ..\..\..\Libraries\libs\libbtstack_master.a(le_device_db_memory.o)
 .data          0x0000000000000000        0x0 ..\..\..\Libraries\libs\libbtstack_master.a(gatt_server.o)
 .bss           0x0000000000000000        0x0 ..\..\..\Libraries\libs\libbtstack_master.a(gatt_server.o)
 .com_text.ble_frame1
                0x0000000000000000       0x2a ..\..\..\Libraries\libs\libbtstack_master.a(gatt_server.o)
 .text.ble.notify_handle
                0x0000000000000000       0x54 ..\..\..\Libraries\libs\libbtstack_master.a(gatt_server.o)
 .sbss          0x0000000000000000        0x1 ..\..\..\Libraries\libs\libbtstack_master.a(gatt_server.o)
 .data          0x0000000000000000        0x0 ..\..\..\Libraries\libs\libbtstack_master.a(gatt_profile.o)
 .bss           0x0000000000000000        0x0 ..\..\..\Libraries\libs\libbtstack_master.a(gatt_profile.o)
 .data          0x0000000000000000        0x0 ..\..\..\Libraries\libs\libbtstack_master.a(gatt_client.o)
 .bss           0x0000000000000000        0x0 ..\..\..\Libraries\libs\libbtstack_master.a(gatt_client.o)
 .data          0x0000000000000000        0x0 ..\..\..\Libraries\libs\libbtstack_master.a(att_server.o)
 .bss           0x0000000000000000        0x0 ..\..\..\Libraries\libs\libbtstack_master.a(att_server.o)
 .data          0x0000000000000000        0x0 ..\..\..\Libraries\libs\libbtstack_master.a(att_dispatch.o)
 .bss           0x0000000000000000        0x0 ..\..\..\Libraries\libs\libbtstack_master.a(att_dispatch.o)
 .data          0x0000000000000000        0x0 ..\..\..\Libraries\libs\libbtstack_master.a(att_db.o)
 .bss           0x0000000000000000        0x0 ..\..\..\Libraries\libs\libbtstack_master.a(att_db.o)
 .text          0x0000000000000000      0x1ea ..\..\..\Libraries\libs\libbtstack_master.a(ad_parser.o)
 .data          0x0000000000000000        0x0 ..\..\..\Libraries\libs\libbtstack_master.a(ad_parser.o)
 .bss           0x0000000000000000        0x0 ..\..\..\Libraries\libs\libbtstack_master.a(ad_parser.o)
 .data          0x0000000000000000        0x0 ..\..\..\Libraries\libs\libbtstack_master.a(btstack_main.o)
 .bss           0x0000000000000000        0x0 ..\..\..\Libraries\libs\libbtstack_master.a(btstack_main.o)
 .data          0x0000000000000000        0x0 ..\..\..\Libraries\libs\libbtstack_master.a(btstack_hal.o)
 .bss           0x0000000000000000        0x0 ..\..\..\Libraries\libs\libbtstack_master.a(btstack_hal.o)
 .com_text.stack.uart_isr
                0x0000000000000000       0x7e ..\..\..\Libraries\libs\libbtstack_master.a(btstack_hal.o)
 .text.stack.hal
                0x0000000000000000       0xa2 ..\..\..\Libraries\libs\libbtstack_master.a(btstack_hal.o)
 .com_text.stack.util
                0x0000000000000000       0x12 ..\..\..\Libraries\libs\libbtstack_master.a(btstack_hal.o)
 .sbss          0x0000000000000000        0x9 ..\..\..\Libraries\libs\libbtstack_master.a(btstack_hal.o)
 .data          0x0000000000000000        0x0 ..\..\..\Libraries\libs\libbtstack_master.a(btstack_api.o)
 .com_text.bb.sleep
                0x0000000000000000       0x34 ..\..\..\Libraries\libs\libbtstack_master.a(btstack_api.o)
 .sleep_text.sleep
                0x0000000000000000        0x8 ..\..\..\Libraries\libs\libbtstack_master.a(btstack_api.o)
 .com_text.sco  0x0000000000000000       0x44 ..\..\..\Libraries\libs\libbtstack_master.a(btstack_api.o)
 .data          0x0000000000000000        0x0 ..\..\..\Libraries\libs\libbtstack_master.a(bt_api.o)
 .bss           0x0000000000000000        0x0 ..\..\..\Libraries\libs\libbtstack_master.a(bt_api.o)
 .text.stack.sleep
                0x0000000000000000       0xc0 ..\..\..\Libraries\libs\libbtstack_master.a(bt_api.o)
 .text.stack.api.hid_con
                0x0000000000000000       0x3a ..\..\..\Libraries\libs\libbtstack_master.a(bt_api.o)
 .text.stack.api.hid_disc
                0x0000000000000000       0x34 ..\..\..\Libraries\libs\libbtstack_master.a(bt_api.o)
 .text.stack.api.hid_send
                0x0000000000000000       0xa6 ..\..\..\Libraries\libs\libbtstack_master.a(bt_api.o)
 .com_text.timer
                0x0000000000000000       0x1a ..\..\..\Libraries\libs\libbtstack_master.a(bt_api.o)
 .sbss          0x0000000000000000        0x1 ..\..\..\Libraries\libs\libbtstack_master.a(bt_api.o)
 .data          0x0000000000000000        0x0 ..\..\..\Libraries\libs\libbtstack_master.a(ble_api.o)
 .bss           0x0000000000000000        0x0 ..\..\..\Libraries\libs\libbtstack_master.a(ble_api.o)
 .sbss          0x0000000000000000        0x1 ..\..\..\Libraries\libs\libbtstack_master.a(ble_api.o)
 .data          0x0000000000000000        0x0 ..\..\..\Libraries\libs\libbtstack_master.a(bb_sche.o)
 .text          0x0000000000000000        0x0 ..\..\..\Libraries\libs\libbtstack_master.a(patch_asm.o)
 .data          0x0000000000000000        0x0 ..\..\..\Libraries\libs\libbtstack_master.a(patch_asm.o)
 .bss           0x0000000000000000        0x0 ..\..\..\Libraries\libs\libbtstack_master.a(patch_asm.o)
 .data          0x0000000000000000        0x0 ..\..\..\Libraries\libs\libbtstack_master.a(bb_dbg.o)
 .bss           0x0000000000000000        0x0 ..\..\..\Libraries\libs\libbtstack_master.a(bb_dbg.o)
 .com_text.bb.putc
                0x0000000000000000       0x60 ..\..\..\Libraries\libs\libbtstack_master.a(bb_dbg.o)
 .data          0x0000000000000000        0x0 ..\..\..\Libraries\libs\libbtstack_master.a(bb_clk.o)
 .bss           0x0000000000000000        0x0 ..\..\..\Libraries\libs\libbtstack_master.a(bb_clk.o)
 .text          0x0000000000000000        0x0 ..\..\..\Libraries\libs\libbtstack_master.a(aes.o)
 .data          0x0000000000000000        0x0 ..\..\..\Libraries\libs\libbtstack_master.a(aes.o)
 .data          0x0000000000000000        0x0 ..\..\..\Libraries\libs\libbtstack_master.a(vs_proc.o)
 .bss           0x0000000000000000        0x0 ..\..\..\Libraries\libs\libbtstack_master.a(vs_proc.o)
 .data          0x0000000000000000        0x0 ..\..\..\Libraries\libs\libbtstack_master.a(vs_fcc.o)
 .bss           0x0000000000000000        0x0 ..\..\..\Libraries\libs\libbtstack_master.a(vs_fcc.o)
 .text.bb.vs.fcc_ble.do
                0x0000000000000000       0x7a ..\..\..\Libraries\libs\libbtstack_master.a(vs_fcc.o)
 .data          0x0000000000000000        0x0 ..\..\..\Libraries\libs\libbtstack_master.a(vs.o)
 .bss           0x0000000000000000        0x0 ..\..\..\Libraries\libs\libbtstack_master.a(vs.o)
 .data          0x0000000000000000        0x0 ..\..\..\Libraries\libs\libbtstack_master.a(rf_smart.o)
 .bss           0x0000000000000000        0x0 ..\..\..\Libraries\libs\libbtstack_master.a(rf_smart.o)
 .text.update   0x0000000000000000       0x44 ..\..\..\Libraries\libs\libbtstack_master.a(rf_smart.o)
 .data          0x0000000000000000        0x0 ..\..\..\Libraries\libs\libbtstack_master.a(rf.o)
 .bss           0x0000000000000000        0x0 ..\..\..\Libraries\libs\libbtstack_master.a(rf.o)
 .sleep_text.bb
                0x0000000000000000       0x30 ..\..\..\Libraries\libs\libbtstack_master.a(rf.o)
 .data          0x0000000000000000        0x0 ..\..\..\Libraries\libs\libbtstack_master.a(bt_hook.o)
 .bss           0x0000000000000000        0x0 ..\..\..\Libraries\libs\libbtstack_master.a(bt_hook.o)
 .com_text.bt21.test.fcc
                0x0000000000000000       0xa0 ..\..\..\Libraries\libs\libbtstack_master.a(bt_hook.o)
 .data          0x0000000000000000        0x0 ..\..\..\Libraries\libs\libbtstack_master.a(ble_hook.o)
 .bss           0x0000000000000000        0x0 ..\..\..\Libraries\libs\libbtstack_master.a(ble_hook.o)
 .data          0x0000000000000000        0x0 ..\..\..\Libraries\libs\libbtstack_master.a(hct_tl.o)
 .com_text.bb.sleep
                0x0000000000000000       0x34 ..\..\..\Libraries\libs\libbtstack_master.a(hct_tl.o)
 .data          0x0000000000000000        0x0 ..\..\..\Libraries\libs\libbtstack_master.a(hct_msg.o)
 .bss           0x0000000000000000        0x0 ..\..\..\Libraries\libs\libbtstack_master.a(hct_msg.o)
 .data          0x0000000000000000        0x0 ..\..\..\Libraries\libs\libbtstack_master.a(hct_fc.o)
 .bss           0x0000000000000000        0x0 ..\..\..\Libraries\libs\libbtstack_master.a(hct_fc.o)
 .data          0x0000000000000000        0x0 ..\..\..\Libraries\libs\libbtstack_master.a(hct.o)
 .bss           0x0000000000000000        0x0 ..\..\..\Libraries\libs\libbtstack_master.a(hct.o)
 .text          0x0000000000000000        0x0 ..\..\..\Libraries\libs\libbtstack_master.a(tws_sco.o)
 .data          0x0000000000000000        0x0 ..\..\..\Libraries\libs\libbtstack_master.a(tws_sco.o)
 .bss           0x0000000000000000        0x0 ..\..\..\Libraries\libs\libbtstack_master.a(tws_sco.o)
 .text          0x0000000000000000        0x0 ..\..\..\Libraries\libs\libbtstack_master.a(tws_acl.o)
 .data          0x0000000000000000        0x0 ..\..\..\Libraries\libs\libbtstack_master.a(tws_acl.o)
 .bss           0x0000000000000000        0x0 ..\..\..\Libraries\libs\libbtstack_master.a(tws_acl.o)
 .data          0x0000000000000000        0x0 ..\..\..\Libraries\libs\libbtstack_master.a(lm.o)
 .bss           0x0000000000000000        0x0 ..\..\..\Libraries\libs\libbtstack_master.a(lm.o)
 .data          0x0000000000000000        0x0 ..\..\..\Libraries\libs\libbtstack_master.a(bt_hal.o)
 .bss           0x0000000000000000        0x0 ..\..\..\Libraries\libs\libbtstack_master.a(bt_hal.o)
 .com_rodata.bb.tbl
                0x0000000000000000       0x2a ..\..\..\Libraries\libs\libbtstack_master.a(bt_hal.o)
 .data          0x0000000000000000        0x0 ..\..\..\Libraries\libs\libbtstack_master.a(bt21.o)
 .bss           0x0000000000000000        0x0 ..\..\..\Libraries\libs\libbtstack_master.a(bt21.o)
 .com_text.bb.sleep
                0x0000000000000000       0x4e ..\..\..\Libraries\libs\libbtstack_master.a(bt21.o)
 .data          0x0000000000000000        0x0 ..\..\..\Libraries\libs\libbtstack_master.a(bc.o)
 .data          0x0000000000000000        0x0 ..\..\..\Libraries\libs\libbtstack_master.a(ble_hal.o)
 .bss           0x0000000000000000        0x0 ..\..\..\Libraries\libs\libbtstack_master.a(ble_hal.o)
 .data          0x0000000000000000        0x0 ..\..\..\Libraries\libs\libbtstack_master.a(ble_adv.o)
 .bss           0x0000000000000000        0x0 ..\..\..\Libraries\libs\libbtstack_master.a(ble_adv.o)
 .data          0x0000000000000000        0x0 ..\..\..\Libraries\libs\libbtstack_master.a(ble.o)
 .bss           0x0000000000000000        0x0 ..\..\..\Libraries\libs\libbtstack_master.a(ble.o)
 .data          0x0000000000000000        0x0 ..\..\..\Libraries\libs\libbtstack_master.a(l2cap_test.o)
 .data          0x0000000000000000        0x0 ..\..\..\Libraries\libs\libbtstack_master.a(l2cap.o)
 .bss           0x0000000000000000        0x0 ..\..\..\Libraries\libs\libbtstack_master.a(l2cap.o)
 .sbss          0x0000000000000000        0x1 ..\..\..\Libraries\libs\libbtstack_master.a(l2cap.o)
 .text          0x0000000000000000        0x4 ..\..\..\Libraries\libs\libbtstack_master.a(hci_sco.o)
 .data          0x0000000000000000        0x0 ..\..\..\Libraries\libs\libbtstack_master.a(hci_sco.o)
 .bss           0x0000000000000000        0x0 ..\..\..\Libraries\libs\libbtstack_master.a(hci_sco.o)
 .sbss          0x0000000000000000        0x1 ..\..\..\Libraries\libs\libbtstack_master.a(hci_sco.o)
 .text          0x0000000000000000       0x18 ..\..\..\Libraries\libs\libbtstack_master.a(hci_dump.o)
 .data          0x0000000000000000        0xc ..\..\..\Libraries\libs\libbtstack_master.a(hci_dump.o)
 .bss           0x0000000000000000        0x0 ..\..\..\Libraries\libs\libbtstack_master.a(hci_dump.o)
 .rodata.str1.4
                0x0000000000000000       0x12 ..\..\..\Libraries\libs\libbtstack_master.a(hci_dump.o)
 .text.stack.util
                0x0000000000000000       0x82 ..\..\..\Libraries\libs\libbtstack_master.a(hci_dump.o)
 .text          0x0000000000000000        0x0 ..\..\..\Libraries\libs\libbtstack_master.a(hci_cmd.o)
 .data          0x0000000000000000        0x0 ..\..\..\Libraries\libs\libbtstack_master.a(hci_cmd.o)
 .bss           0x0000000000000000        0x0 ..\..\..\Libraries\libs\libbtstack_master.a(hci_cmd.o)
 .data          0x0000000000000000        0x0 ..\..\..\Libraries\libs\libbtstack_master.a(hci.o)
 .bss           0x0000000000000000        0x0 ..\..\..\Libraries\libs\libbtstack_master.a(hci.o)
 .com_text.timer
                0x0000000000000000        0xe ..\..\..\Libraries\libs\libbtstack_master.a(hci.o)
 .com_text.sco  0x0000000000000000        0xe ..\..\..\Libraries\libs\libbtstack_master.a(hci.o)
 .rodata.stack.hci_init
                0x0000000000000000       0x11 ..\..\..\Libraries\libs\libbtstack_master.a(hci.o)
 .data          0x0000000000000000        0x0 ..\..\..\Libraries\libs\libbtstack_master.a(hid_usage.o)
 .bss           0x0000000000000000        0x0 ..\..\..\Libraries\libs\libbtstack_master.a(hid_usage.o)
 .text.stack.api.hid_touch
                0x0000000000000000        0xa ..\..\..\Libraries\libs\libbtstack_master.a(hid_usage.o)
 .srodata       0x0000000000000000        0xe ..\..\..\Libraries\libs\libbtstack_master.a(hid_usage.o)
 .data          0x0000000000000000        0x0 ..\..\..\Libraries\libs\libbtstack_master.a(hid_device.o)
 .bss           0x0000000000000000        0x0 ..\..\..\Libraries\libs\libbtstack_master.a(hid_device.o)
 .sbss          0x0000000000000000        0x1 ..\..\..\Libraries\libs\libbtstack_master.a(hid_device.o)
 .data          0x0000000000000000        0x0 ..\..\..\Libraries\libs\libbtstack_master.a(hfp_hf.o)
 .bss           0x0000000000000000        0x0 ..\..\..\Libraries\libs\libbtstack_master.a(hfp_hf.o)
 .data          0x0000000000000000        0x0 ..\..\..\Libraries\libs\libbtstack_master.a(hfp.o)
 .bss           0x0000000000000000        0x0 ..\..\..\Libraries\libs\libbtstack_master.a(hfp.o)
 .sbss          0x0000000000000000        0x1 ..\..\..\Libraries\libs\libbtstack_master.a(hfp.o)
 .text          0x0000000000000000        0x0 ..\..\..\Libraries\libs\libbtstack_master.a(avdtp.o)
 .data          0x0000000000000000        0x0 ..\..\..\Libraries\libs\libbtstack_master.a(avdtp.o)
 .bss           0x0000000000000000        0x0 ..\..\..\Libraries\libs\libbtstack_master.a(avdtp.o)
 .com_text.acl.pend
                0x0000000000000000        0x4 ..\..\..\Libraries\libs\libbtstack_master.a(avdtp.o)
 .sbss          0x0000000000000000        0x1 ..\..\..\Libraries\libs\libbtstack_master.a(avdtp.o)
 .data          0x0000000000000000        0x0 ..\..\..\Libraries\libs\libbtstack_master.a(a2dp.o)
 .bss           0x0000000000000000        0x0 ..\..\..\Libraries\libs\libbtstack_master.a(a2dp.o)
 .sbss          0x0000000000000000        0x1 ..\..\..\Libraries\libs\libbtstack_master.a(a2dp.o)
 .text          0x0000000000000000        0x0 ..\..\..\Libraries\libs\libbtstack_master.a(btstack_memory_pool.o)
 .data          0x0000000000000000        0x0 ..\..\..\Libraries\libs\libbtstack_master.a(btstack_memory_pool.o)
 .bss           0x0000000000000000        0x0 ..\..\..\Libraries\libs\libbtstack_master.a(btstack_memory_pool.o)
 .data          0x0000000000000000        0x0 ..\..\..\Libraries\libs\libbtstack_master.a(btstack_adv0.o)
 .bss           0x0000000000000000        0x0 ..\..\..\Libraries\libs\libbtstack_master.a(btstack_adv0.o)
 .sbss          0x0000000000000000        0x1 ..\..\..\Libraries\libs\libbtstack_master.a(btstack_adv0.o)
 .data          0x0000000000000000        0x0 ..\..\..\Libraries\libs\libbtstack_master.a(hci_transport_hcic.o)
 .bss           0x0000000000000000        0x0 ..\..\..\Libraries\libs\libbtstack_master.a(hci_transport_hcic.o)
 .data          0x0000000000000000        0x0 ..\..\..\Libraries\libs\libbtstack_master.a(btstack_chipset_inner.o)
 .bss           0x0000000000000000        0x0 ..\..\..\Libraries\libs\libbtstack_master.a(btstack_chipset_inner.o)
 .data          0x0000000000000000        0x0 ..\..\..\Libraries\libs\libbtstack_master.a(lm_hook.o)
 .bss           0x0000000000000000        0x0 ..\..\..\Libraries\libs\libbtstack_master.a(lm_hook.o)
 .data          0x0000000000000000        0x0 ..\..\..\Libraries\libs\libbtstack_master.a(lm_sp.o)
 .text.lm.sha256
                0x0000000000000000      0x13a ..\..\..\Libraries\libs\libbtstack_master.a(lm_sp.o)
 .data          0x0000000000000000        0x0 ..\..\..\Libraries\libs\libbtstack_master.a(lm_proc.o)
 .bss           0x0000000000000000        0x0 ..\..\..\Libraries\libs\libbtstack_master.a(lm_proc.o)
 .text.bb.lm.inq.start
                0x0000000000000000      0x104 ..\..\..\Libraries\libs\libbtstack_master.a(lm_proc.o)
 .text.bb.lm.inq.stop
                0x0000000000000000       0x32 ..\..\..\Libraries\libs\libbtstack_master.a(lm_proc.o)
 .text.bb.lm.inq.res
                0x0000000000000000      0x222 ..\..\..\Libraries\libs\libbtstack_master.a(lm_proc.o)
 .data          0x0000000000000000        0x0 ..\..\..\Libraries\libs\libbtstack_master.a(lm_key.o)
 .bss           0x0000000000000000        0x0 ..\..\..\Libraries\libs\libbtstack_master.a(lm_key.o)
 .data          0x0000000000000000        0x0 ..\..\..\Libraries\libs\libbtstack_master.a(lc.o)
 .bss           0x0000000000000000        0x0 ..\..\..\Libraries\libs\libbtstack_master.a(lc.o)
 .com_text.lc   0x0000000000000000       0x9c ..\..\..\Libraries\libs\libbtstack_master.a(lc.o)
 .data          0x0000000000000000        0x0 ..\..\..\Libraries\libs\libbtstack_master.a(mgr.o)
 .bss           0x0000000000000000        0x0 ..\..\..\Libraries\libs\libbtstack_master.a(mgr.o)
 .text          0x0000000000000000        0x0 ..\..\..\Libraries\libs\libbtstack_master.a(ll.o)
 .data          0x0000000000000000        0x0 ..\..\..\Libraries\libs\libbtstack_master.a(ll.o)
 .bss           0x0000000000000000        0x0 ..\..\..\Libraries\libs\libbtstack_master.a(ll.o)
 .data          0x0000000000000000        0x0 ..\..\..\Libraries\libs\libbtstack_master.a(ble_test.o)
 .bss           0x0000000000000000        0x0 ..\..\..\Libraries\libs\libbtstack_master.a(ble_test.o)
 .com_text.ble.isr.test
                0x0000000000000000      0x17a ..\..\..\Libraries\libs\libbtstack_master.a(ble_test.o)
 .com_text.ble.isr.test.ind
                0x0000000000000000       0x5a ..\..\..\Libraries\libs\libbtstack_master.a(ble_test.o)
 .text.bb.ble.test.start
                0x0000000000000000      0x4b0 ..\..\..\Libraries\libs\libbtstack_master.a(ble_test.o)
 .text.bb.ble.test.stop
                0x0000000000000000      0x200 ..\..\..\Libraries\libs\libbtstack_master.a(ble_test.o)
 .srodata       0x0000000000000000        0x7 ..\..\..\Libraries\libs\libbtstack_master.a(ble_test.o)
 .data          0x0000000000000000        0x0 ..\..\..\Libraries\libs\libbtstack_master.a(ble_scan.o)
 .bss           0x0000000000000000        0x0 ..\..\..\Libraries\libs\libbtstack_master.a(ble_scan.o)
 .com_rodata.bb.tbl
                0x0000000000000000       0x10 ..\..\..\Libraries\libs\libbtstack_master.a(ble_scan.o)
 .data          0x0000000000000000        0x0 ..\..\..\Libraries\libs\libbtstack_master.a(ble_per_adv.o)
 .bss           0x0000000000000000        0x0 ..\..\..\Libraries\libs\libbtstack_master.a(ble_per_adv.o)
 .data          0x0000000000000000        0x0 ..\..\..\Libraries\libs\libbtstack_master.a(ble_init.o)
 .bss           0x0000000000000000        0x0 ..\..\..\Libraries\libs\libbtstack_master.a(ble_init.o)
 .data          0x0000000000000000        0x0 ..\..\..\Libraries\libs\libbtstack_master.a(ble_buf.o)
 .text          0x0000000000000000        0x0 ..\..\..\Libraries\libs\libbtstack_master.a(ble_adv0.o)
 .data          0x0000000000000000        0x0 ..\..\..\Libraries\libs\libbtstack_master.a(ble_adv0.o)
 .bss           0x0000000000000000        0x0 ..\..\..\Libraries\libs\libbtstack_master.a(ble_adv0.o)
 .data          0x0000000000000000        0x0 ..\..\..\Libraries\libs\libbtstack_master.a(extern_hfhs.o)
 .bss           0x0000000000000000        0x0 ..\..\..\Libraries\libs\libbtstack_master.a(extern_hfhs.o)
 .sbss          0x0000000000000000        0x1 ..\..\..\Libraries\libs\libbtstack_master.a(extern_hfhs.o)
 .srodata       0x0000000000000000        0x1 ..\..\..\Libraries\libs\libbtstack_master.a(extern_hfhs.o)
 .data          0x0000000000000000        0x0 ..\..\..\Libraries\libs\libbtstack_master.a(extern_ble.o)
 .bss           0x0000000000000000        0x0 ..\..\..\Libraries\libs\libbtstack_master.a(extern_ble.o)
 .sbss          0x0000000000000000        0x1 ..\..\..\Libraries\libs\libbtstack_master.a(extern_ble.o)
 .srodata       0x0000000000000000        0x2 ..\..\..\Libraries\libs\libbtstack_master.a(extern_ble.o)
 .text          0x0000000000000000       0x38 ..\..\..\Libraries\libs\libbtstack_master.a(l2cap_signaling.o)
 .data          0x0000000000000000        0x0 ..\..\..\Libraries\libs\libbtstack_master.a(l2cap_signaling.o)
 .bss           0x0000000000000000        0x0 ..\..\..\Libraries\libs\libbtstack_master.a(l2cap_signaling.o)
 .data          0x0000000000000000        0x0 ..\..\..\Libraries\libs\libbtstack_master.a(lc_hook.o)
 .bss           0x0000000000000000        0x0 ..\..\..\Libraries\libs\libbtstack_master.a(lc_hook.o)
 .data          0x0000000000000000        0x0 ..\..\..\Libraries\libs\libbtstack_master.a(lm_sco.o)
 .bss           0x0000000000000000        0x0 ..\..\..\Libraries\libs\libbtstack_master.a(lm_sco.o)
 .data          0x0000000000000000        0x0 ..\..\..\Libraries\libs\libbtstack_master.a(lc_util.o)
 .bss           0x0000000000000000        0x0 ..\..\..\Libraries\libs\libbtstack_master.a(lc_util.o)
 .data          0x0000000000000000        0x0 ..\..\..\Libraries\libs\libbtstack_master.a(lc_sniff.o)
 .bss           0x0000000000000000        0x0 ..\..\..\Libraries\libs\libbtstack_master.a(lc_sniff.o)
 .data          0x0000000000000000        0x0 ..\..\..\Libraries\libs\libbtstack_master.a(lc_sco.o)
 .bss           0x0000000000000000        0x0 ..\..\..\Libraries\libs\libbtstack_master.a(lc_sco.o)
 .data          0x0000000000000000        0x0 ..\..\..\Libraries\libs\libbtstack_master.a(lc_proc.o)
 .bss           0x0000000000000000        0x0 ..\..\..\Libraries\libs\libbtstack_master.a(lc_proc.o)
 .data          0x0000000000000000        0x0 ..\..\..\Libraries\libs\libbtstack_master.a(lc_lmppdu.o)
 .bss           0x0000000000000000        0x0 ..\..\..\Libraries\libs\libbtstack_master.a(lc_lmppdu.o)
 .data          0x0000000000000000        0x0 ..\..\..\Libraries\libs\libbtstack_master.a(mgr_proc.o)
 .bss           0x0000000000000000        0x0 ..\..\..\Libraries\libs\libbtstack_master.a(mgr_proc.o)
 .data          0x0000000000000000        0x0 ..\..\..\Libraries\libs\libbtstack_master.a(mgr_init.o)
 .bss           0x0000000000000000        0x0 ..\..\..\Libraries\libs\libbtstack_master.a(mgr_init.o)
 .data          0x0000000000000000        0x0 ..\..\..\Libraries\libs\libbtstack_master.a(mgr_hci.o)
 .bss           0x0000000000000000        0x0 ..\..\..\Libraries\libs\libbtstack_master.a(mgr_hci.o)
 .data          0x0000000000000000        0x0 ..\..\..\Libraries\libs\libbtstack_master.a(ll_scan.o)
 .bss           0x0000000000000000        0x0 ..\..\..\Libraries\libs\libbtstack_master.a(ll_scan.o)
 .data          0x0000000000000000        0x0 ..\..\..\Libraries\libs\libbtstack_master.a(ll_adv.o)
 .bss           0x0000000000000000        0x0 ..\..\..\Libraries\libs\libbtstack_master.a(ll_adv.o)
 .data          0x0000000000000000        0x0 ..\..\..\Libraries\libs\libbtstack_master.a(ll_proc.o)
 .data          0x0000000000000000        0x0 ..\..\..\Libraries\libs\libbtstack_master.a(ll_ping.o)
 .bss           0x0000000000000000        0x0 ..\..\..\Libraries\libs\libbtstack_master.a(ll_ping.o)
 .data          0x0000000000000000        0x0 ..\..\..\Libraries\libs\libbtstack_master.a(ll_phy_upd.o)
 .bss           0x0000000000000000        0x0 ..\..\..\Libraries\libs\libbtstack_master.a(ll_phy_upd.o)
 .data          0x0000000000000000        0x0 ..\..\..\Libraries\libs\libbtstack_master.a(ll_past.o)
 .bss           0x0000000000000000        0x0 ..\..\..\Libraries\libs\libbtstack_master.a(ll_past.o)
 .data          0x0000000000000000        0x0 ..\..\..\Libraries\libs\libbtstack_master.a(ll_length.o)
 .bss           0x0000000000000000        0x0 ..\..\..\Libraries\libs\libbtstack_master.a(ll_length.o)
 .data          0x0000000000000000        0x0 ..\..\..\Libraries\libs\libbtstack_master.a(ll_feature.o)
 .bss           0x0000000000000000        0x0 ..\..\..\Libraries\libs\libbtstack_master.a(ll_feature.o)
 .data          0x0000000000000000        0x0 ..\..\..\Libraries\libs\libbtstack_master.a(ll_encrypt.o)
 .bss           0x0000000000000000        0x0 ..\..\..\Libraries\libs\libbtstack_master.a(ll_encrypt.o)
 .data          0x0000000000000000        0x0 ..\..\..\Libraries\libs\libbtstack_master.a(ll_disconnect.o)
 .bss           0x0000000000000000        0x0 ..\..\..\Libraries\libs\libbtstack_master.a(ll_disconnect.o)
 .data          0x0000000000000000        0x0 ..\..\..\Libraries\libs\libbtstack_master.a(ll_con_upd.o)
 .bss           0x0000000000000000        0x0 ..\..\..\Libraries\libs\libbtstack_master.a(ll_con_upd.o)
 .data          0x0000000000000000        0x0 ..\..\..\Libraries\libs\libbtstack_master.a(ll_cntl.o)
 .bss           0x0000000000000000        0x0 ..\..\..\Libraries\libs\libbtstack_master.a(ll_cntl.o)
 .data          0x0000000000000000        0x0 ..\..\..\Libraries\libs\libbtstack_master.a(ll_clk_acc.o)
 .bss           0x0000000000000000        0x0 ..\..\..\Libraries\libs\libbtstack_master.a(ll_clk_acc.o)
 .data          0x0000000000000000        0x0 ..\..\..\Libraries\libs\libbtstack_master.a(ll_chmap_upd.o)
 .bss           0x0000000000000000        0x0 ..\..\..\Libraries\libs\libbtstack_master.a(ll_chmap_upd.o)
 .data          0x0000000000000000        0x0 ..\..\..\Libraries\libs\libbtstack_master.a(aes_rpa.o)
 .bss           0x0000000000000000        0x0 ..\..\..\Libraries\libs\libbtstack_master.a(aes_rpa.o)
 .data          0x0000000000000000        0x0 ..\..\..\Libraries\libs\libbtstack_master.a(scan_hook.o)
 .bss           0x0000000000000000        0x0 ..\..\..\Libraries\libs\libbtstack_master.a(scan_hook.o)
 .data          0x0000000000000000        0x0 ..\..\..\Libraries\libs\libbtstack_master.a(adv_hook.o)
 .bss           0x0000000000000000        0x0 ..\..\..\Libraries\libs\libbtstack_master.a(adv_hook.o)
 .data          0x0000000000000000        0x0 ..\..\..\Libraries\libs\libbtstack_master.a(ll_version.o)
 .bss           0x0000000000000000        0x0 ..\..\..\Libraries\libs\libbtstack_master.a(ll_version.o)
 .data          0x0000000000000000        0x0 ..\..\..\Libraries\libs\libbtstack_master.a(ll_pwr.o)
 .bss           0x0000000000000000        0x0 ..\..\..\Libraries\libs\libbtstack_master.a(ll_pwr.o)

Memory Configuration

Name             Origin             Length             Attributes
init             0x0000000010000000 0x0000000000000200
flash            0x0000000010000200 0x0000000000064000 xr
comm             0x0000000000017000 0x0000000000009000 xr
stack            0x0000000000010800 0x0000000000000400
heap             0x0000000000010c00 0x0000000000003000
data             0x0000000000013c00 0x0000000000003400
bram             0x0000000000020000 0x000000000000c000
cram             0x000000000002c000 0x0000000000014000
aram             0x0000000000050000 0x0000000000004000
dram             0x0000000000058000 0x0000000000004500
eram             0x0000000000054000 0x0000000000000a00
rram             0x0000000000055800 0x0000000000000260
*default*        0x0000000000000000 0xffffffffffffffff

Linker script and memory map

LOAD Output\obj\Libraries\bsp\bsp_bt.o
LOAD Output\obj\Libraries\bsp\bsp_cm.o
LOAD Output\obj\Libraries\bsp\bsp_fot.o
LOAD Output\obj\Libraries\bsp\bsp_param.o
LOAD Output\obj\Libraries\bsp\bsp_sys.o
LOAD Output\obj\Libraries\BT\ble\ab_link\app.o
LOAD Output\obj\Libraries\BT\ble\adv0.o
LOAD Output\obj\Libraries\BT\ble\ble.o
LOAD Output\obj\Libraries\BT\spp\bt.o
LOAD Output\obj\Libraries\BT\spp\hid.o
LOAD Output\obj\Libraries\BT\spp\profile.o
LOAD Output\obj\Libraries\BT\spp\spp.o
LOAD Output\obj\Libraries\Device\Source\gw3323_clk.o
LOAD Output\obj\Libraries\Device\Source\gw3323_gpio.o
LOAD Output\obj\Libraries\Device\Source\gw3323_hsuart.o
LOAD Output\obj\Libraries\Device\Source\gw3323_spi.o
LOAD Output\obj\Libraries\libs\strong_symbol.o
LOAD Output\obj\Examples\BLE_Host\Source\ble_client.o
LOAD Output\obj\Examples\BLE_Host\Source\ble_init.o
LOAD Output\obj\Examples\BLE_Host\Source\gpio_input_key.o
LOAD Output\obj\Examples\BLE_Host\Source\hsuart_transfer.o
LOAD Output\obj\Examples\BLE_Host\Project\config.o
LOAD Output\obj\Examples\BLE_Host\Project\main.o
                0x0000000000064000                __max_flash_size = 0x64000
                0x0000000010000000                __base = 0x10000000
                0x0000000000010600                __cache_stack_vma = 0x10600
                0x0000000000000200                __cache_stack_size = 0x200
                0x0000000000010800                __stack_vma = 0x10800
                0x0000000000000400                __stack_ram_size = 0x400
                0x0000000000010c00                __heap_vma = 0x10c00
                0x0000000000003000                __heap_ram_size = 0x3000
                0x0000000000013c00                __data_vma = 0x13c00
                0x0000000000003400                __data_ram_size = 0x3400
                0x0000000000017000                __comm_vma = 0x17000
                0x0000000000009000                __comm_ram_size = 0x9000
                0x0000000000020000                __bram_vma = 0x20000
                0x000000000000c000                __bram_ram_size = 0xc000
                0x000000000002c000                __cram_vma = 0x2c000
                0x0000000000014000                __cram_ram_size = 0x14000
                0x0000000000050000                __aram_vma = 0x50000
                0x0000000000054000                __eram_vma = 0x54000
                0x0000000000058000                __dram_vma = 0x58000
                0x0000000000055800                __rram_vma = 0x55800

.init           0x0000000010000000       0x4e
 *(.reset)
 .reset         0x0000000010000000       0x4e ..\..\..\Libraries\libs\libplatform.a(reset.o)
                0x0000000010000000                _start

.comm           0x0000000000017000     0x3800 load address 0x0000000010000200
 *(.vector)
 .vector        0x0000000000017000      0x1a2 ..\..\..\Libraries\libs\libplatform.a(reset.o)
                0x00000000000170a0                _exception_isr
                0x00000000000170a2                nop_isr
 *(.plt)
 .plt           0x00000000000171a2       0x10 ..\..\..\Libraries\libs\libplatform.a(main.o)
 *(.com_text*)
 .com_text.fot  0x00000000000171b2       0x4e Output\obj\Libraries\bsp\bsp_fot.o
                0x00000000000171b2                fot_app_connect_auth
                0x00000000000171f4                bsp_fot_is_connect
 .com_text.const
                0x0000000000017200        0x7 Output\obj\Libraries\bsp\bsp_fot.o
 *fill*         0x0000000000017207        0x1 
 .com_text.timer
                0x0000000000017208       0x98 Output\obj\Libraries\bsp\bsp_sys.o
                0x0000000000017208                usr_tmr1ms_isr
                0x000000000001720a                usr_tmr5ms_thread
                0x0000000000017288                timer1_isr
 .com_text.sys  0x00000000000172a0        0x4 Output\obj\Libraries\bsp\bsp_sys.o
                0x00000000000172a0                spiflash_speed_up_en
 .com_text.gpio
                0x00000000000172a4       0x36 Output\obj\Libraries\Device\Source\gw3323_gpio.o
                0x00000000000172a4                gpio_set_bits
                0x00000000000172a8                gpio_reset_bits
                0x00000000000172ac                gpio_writebit
                0x00000000000172b6                gpio_write_data
                0x00000000000172c0                gpio_toggle_bits
                0x00000000000172c8                gpio_read_data
                0x00000000000172d0                gpio_read_bit
 .com_text.hsuart
                0x00000000000172da       0xb6 Output\obj\Libraries\Device\Source\gw3323_hsuart.o
                0x00000000000172da                hsuart_cmd
                0x0000000000017310                hsuart_send_data
                0x000000000001731a                hsuart_receive_data
                0x0000000000017324                hsuart_get_flag
                0x0000000000017330                hsuart_clear_flag
                0x000000000001733c                hsuart_dma_start
                0x0000000000017378                hsuart_dma_stop
 .com_text.stack.uart_isr
                0x0000000000017390        0x4 Output\obj\Libraries\libs\strong_symbol.o
                0x0000000000017390                bt_uart_isr
 .com_text.isr  0x0000000000017394       0x6a Output\obj\Examples\BLE_Host\Source\hsuart_transfer.o
                0x0000000000017394                hsuart_isr
 .com_text.spiflash
                0x00000000000173fe      0x13e ..\..\..\Libraries\libs\libplatform.a(os_flash.o)
                0x00000000000173fe                os_spiflash_read
                0x0000000000017438                os_spiflash_program
                0x00000000000174be                os_spiflash_erase
 .com_text.sd.isr
                0x000000000001753c       0x20 ..\..\..\Libraries\libs\libplatform.a(device.o)
                0x000000000001753c                sdctl_isr
 .com_text.exception.hook
                0x000000000001755c       0x3a ..\..\..\Libraries\libs\libplatform.a(main.o)
                0x000000000001755c                sys_error_hook
 .com_text.exception
                0x0000000000017596       0x5e ..\..\..\Libraries\libs\libplatform.a(main.o)
                0x0000000000017596                exception_isr
 .com_text.delay
                0x00000000000175f4       0x4e ..\..\..\Libraries\libs\libplatform.a(main.o)
                0x00000000000175f4                delay_5ms
                0x000000000001760e                delay_ms
                0x0000000000017626                delay_us
 .com_text.irq  0x0000000000017642      0x178 ..\..\..\Libraries\libs\libplatform.a(interrupt.o)
                0x0000000000017642                bthw_isr
                0x000000000001765c                aubuf_isr
                0x00000000000176d8                timer0_isr
                0x0000000000017742                register_isr
                0x000000000001777c                tick_get
                0x0000000000017784                watch_point_isr
                0x00000000000177a8                tick_check_expire
 .com_text.timer
                0x00000000000177ba        0xe ..\..\..\Libraries\libs\libplatform.a(startup.o)
 .com_text.irq  0x00000000000177c8       0x5a ..\..\..\Libraries\libs\libplatform.a(reset.o)
                0x00000000000177c8                cpu_irq_comm
                0x000000000001781a                btmdm_isr
 .com_text.util.isr
                0x0000000000017822        0x6 ..\..\..\Libraries\libs\libplatform.a(reset.o)
                0x0000000000017822                kick_soft_isr
 .com_text.spiflash
                0x0000000000017828      0x154 ..\..\..\Libraries\libs\libplatform.a(spiflash.o)
                0x00000000000178ba                spiflash_program
                0x0000000000017904                spiflash_erase
                0x0000000000017930                spiflash_get_id
 .com_text.debug
                0x000000000001797c      0x1aa ..\..\..\Libraries\libs\libplatform.a(debug.o)
                0x0000000000017a4e                debug_dump_err_cache_irq
 .com_text.sys  0x0000000000017b26       0x68 ..\..\..\Libraries\libs\libplatform.a(s_sys.o)
                0x0000000000017b26                s_ff1
                0x0000000000017b2c                s_fl1
                0x0000000000017b32                s_log2
                0x0000000000017b3a                s_clb
                0x0000000000017b40                s_bcnt
                0x0000000000017b46                s_ror
                0x0000000000017b4c                s_swapw
                0x0000000000017b52                s_bitrvti
                0x0000000000017b58                s_clip16
                0x0000000000017b5e                s_abs
                0x0000000000017b64                mul_r
                0x0000000000017b70                dummy_func
                0x0000000000017b72                __ashrdi3
                0x0000000000017b80                __ashldi3
 .com_text.thread.driver
                0x0000000000017b8e       0x56 ..\..\..\Libraries\libs\libplatform.a(usb.o)
                0x0000000000017b8e                os_mq_usb_post
                0x0000000000017bb4                thread_user_kick
                0x0000000000017be2                thread_user_func_do
 *fill*         0x0000000000017be4        0x0 
 .com_text.thread.usb
                0x0000000000017be4       0xaa ..\..\..\Libraries\libs\libplatform.a(usb.o)
                0x0000000000017be4                thread_usb_entry
 .com_text.bthw
                0x0000000000017c8e       0x22 ..\..\..\Libraries\libs\libplatform.a(bt.o)
                0x0000000000017c8e                btstack_status_lock
                0x0000000000017ca0                btstack_status_unlock
 .com_text.stack.thread
                0x0000000000017cb0       0x32 ..\..\..\Libraries\libs\libplatform.a(bt.o)
                0x0000000000017cb0                thread_btstack_pend
                0x0000000000017cd2                thread_btstack_post
 .com_text.stack.run_loop
                0x0000000000017ce2       0x48 ..\..\..\Libraries\libs\libplatform.a(bt.o)
                0x0000000000017ce2                thread_btstack_entry
 .com_text.bb.bthw
                0x0000000000017d2a       0x3c ..\..\..\Libraries\libs\libplatform.a(bt.o)
                0x0000000000017d2a                thread_bthw_entry
 .com_text.usbdev
                0x0000000000017d66       0x20 ..\..\..\Libraries\libs\libdrivers.a(usb_device_hid.o)
                0x0000000000017d66                ude_tmr_isr
 *fill*         0x0000000000017d86        0x2 
 .com_text.epsize.table
                0x0000000000017d88        0x4 ..\..\..\Libraries\libs\libdrivers.a(usb_comm.o)
                0x0000000000017d88                epsize_tbl
 .com_text.bb.nanos
                0x0000000000017d8c       0x16 ..\..\..\Libraries\libs\libbtstack_master.a(nanos.o)
                0x0000000000017d8c                nanos_event_set
 .com_text.bb.patch
                0x0000000000017da2       0x9a ..\..\..\Libraries\libs\libbtstack_master.a(patch.o)
                0x0000000000017da2                bb_v1_patch0_do
                0x0000000000017db0                bt_acl_cal_offset_fix
 .com_text.bb.ll.tx
                0x0000000000017e3c        0x2 ..\..\..\Libraries\libs\libbtstack_master.a(platform.o)
                0x0000000000017e3c                bb_ll_tx_cb
 .com_text.bb.ll.rx
                0x0000000000017e3e        0x2 ..\..\..\Libraries\libs\libbtstack_master.a(platform.o)
                0x0000000000017e3e                bb_ll_rx_cb
 .com_text.bb.lmp.rx
                0x0000000000017e40        0x2 ..\..\..\Libraries\libs\libbtstack_master.a(platform.o)
                0x0000000000017e40                bb_lmp_tx_cb
 .com_text.bb.lmp.tx
                0x0000000000017e42        0x2 ..\..\..\Libraries\libs\libbtstack_master.a(platform.o)
                0x0000000000017e42                bb_lmp_rx_cb
 .com_text.timer
                0x0000000000017e44        0x6 ..\..\..\Libraries\libs\libbtstack_master.a(platform.o)
                0x0000000000017e44                timer_get_tick
                0x0000000000017e48                timer_sync
 .com_text.bb.sco
                0x0000000000017e4a       0x1e ..\..\..\Libraries\libs\libbtstack_master.a(bt_sco.o)
                0x0000000000017e4a                bt_sco_is_transp
                0x0000000000017e5a                bt_codec_isr
                0x0000000000017e5c                lc_sco_codec_pkt
 .com_text.bt21.isr
                0x0000000000017e68      0x212 ..\..\..\Libraries\libs\libbtstack_master.a(bt_acl.o)
                0x0000000000017eea                bt_acl_lmp_tx_isr
                0x0000000000017f52                bt_acl_data_tx_isr
                0x0000000000017f88                bt_sco_audio_isr
                0x000000000001803a                bt_acl_get_clkoff
 .com_text.ble.isr.con
                0x000000000001807a       0x82 ..\..\..\Libraries\libs\libbtstack_master.a(ble_con.o)
                0x000000000001807a                ble_con_rx_end
                0x00000000000180cc                ble_con_evt_prio_check
 .com_text.bb.utils
                0x00000000000180fc        0xa ..\..\..\Libraries\libs\libbtstack_master.a(bb_utils.o)
                0x00000000000180fc                bb_slot_to_duration
 .com_text.bb.isr
                0x0000000000018106      0x19c ..\..\..\Libraries\libs\libbtstack_master.a(bb_int.o)
                0x000000000001813a                bb_lpcycles_2_hus
                0x000000000001817c                bb_isr
                0x0000000000018290                bb_hal_isr
 .com_text.bb.btisr
                0x00000000000182a2       0x2e ..\..\..\Libraries\libs\libbtstack_master.a(bb.o)
                0x00000000000182a2                bb_acl_rx0_parse
                0x00000000000182a6                bb_free_acl_buf
                0x00000000000182b2                bb_alloc_acl_buf
 .com_text.bb.isr
                0x00000000000182d0       0x32 ..\..\..\Libraries\libs\libbtstack_master.a(bb.o)
                0x00000000000182d0                bb_notice_status
 .com_text.dummy
                0x0000000000018302        0x6 ..\..\..\Libraries\libs\libbtstack_master.a(platform.o)
                0x0000000000018302                dummy_void
                0x0000000000018304                dummy_false
 .com_text.aubuf.isr
                0x0000000000018308        0x2 ..\..\..\Libraries\libs\libbtstack_master.a(extern.o)
                0x0000000000018308                ext_aubuf_isr
 .com_text.pp.send_pkt
                0x000000000001830a       0x58 ..\..\..\Libraries\libs\libbtstack_master.a(spp.o)
                0x000000000001830a                spp_send_packet
 .com_text.spp.tx
                0x0000000000018362       0xd4 ..\..\..\Libraries\libs\libbtstack_master.a(spp.o)
                0x0000000000018362                spp_is_connect
                0x0000000000018376                spp_default_connected
                0x000000000001838c                spp_custom1_connected
                0x00000000000183a2                spp_custom2_connected
                0x00000000000183b8                bt_spp_tx
                0x00000000000183e2                bt_spp_custom1_tx
                0x000000000001840c                bt_spp_custom2_tx
 .com_text.spp.send_kick
                0x0000000000018436        0xe ..\..\..\Libraries\libs\libbtstack_master.a(spp.o)
                0x0000000000018436                spp_send_kick
 .com_text.spp.send_req
                0x0000000000018444       0x12 ..\..\..\Libraries\libs\libbtstack_master.a(spp.o)
                0x0000000000018444                btstack_spp_send_req
 .com_text.spp.event_send
                0x0000000000018456       0x32 ..\..\..\Libraries\libs\libbtstack_master.a(spp.o)
                0x0000000000018456                spp_event_send
 .com_text.spp.rx_set_new_credit
                0x0000000000018488       0x7e ..\..\..\Libraries\libs\libbtstack_master.a(spp.o)
                0x0000000000018488                spp_set_rx_new_credit
                0x0000000000018496                spp_notify_rx_buffer_len
                0x00000000000184ec                btstack_spp_rx_set_new_credit
 .com_text.txpkt.send
                0x0000000000018506      0x15e ..\..\..\Libraries\libs\libbtstack_master.a(btstack_txpkt.o)
                0x0000000000018506                txpkt_send
                0x00000000000185e4                txpkt_event_send
 .com_text.stack.run_loop
                0x0000000000018664       0xe2 ..\..\..\Libraries\libs\libbtstack_master.a(btstack_run_loop.o)
                0x0000000000018664                btstack_cmp_abs_tick
                0x000000000001866a                btstack_runtime_check
                0x00000000000186b0                btstack_run_loop_execute_once
 .com_text.stack.thread
                0x0000000000018746        0xe ..\..\..\Libraries\libs\libbtstack_master.a(btstack_run_loop.o)
                0x0000000000018746                btstack_run_loop_embedded_trigger
 .com_text.stack.ticks
                0x0000000000018754       0x34 ..\..\..\Libraries\libs\libbtstack_master.a(btstack_run_loop.o)
 .com_text.stack.linked_list
                0x0000000000018788       0x50 ..\..\..\Libraries\libs\libbtstack_master.a(btstack_linked_list.o)
                0x0000000000018788                btstack_linked_list_empty
                0x0000000000018790                btstack_linked_list_iterator_init
                0x000000000001879c                btstack_linked_list_iterator_has_next
                0x00000000000187ba                btstack_linked_list_iterator_next
 .com_text.ble.send_pkt
                0x00000000000187d8       0xd6 ..\..\..\Libraries\libs\libbtstack_master.a(gatt_server.o)
                0x00000000000187d8                ble_send_notify_packet
                0x000000000001886a                att_event_server_send
 .com_text.stack.ble.mtu
                0x00000000000188ae       0x10 ..\..\..\Libraries\libs\libbtstack_master.a(gatt_server.o)
                0x00000000000188ae                ble_get_gatt_mtu
 .com_text.ble.send_kick
                0x00000000000188be        0xe ..\..\..\Libraries\libs\libbtstack_master.a(gatt_server.o)
                0x00000000000188be                ble_send_kick
 .com_text.stack.ticks
                0x00000000000188cc        0xa ..\..\..\Libraries\libs\libbtstack_master.a(btstack_hal.o)
                0x00000000000188ce                sys_tick_handler
 .com_text.isr  0x00000000000188d6       0x1a ..\..\..\Libraries\libs\libbtstack_master.a(btstack_hal.o)
                0x00000000000188d6                bt_timer_isr
 .com_text.stack.api
                0x00000000000188f0      0x13a ..\..\..\Libraries\libs\libbtstack_master.a(btstack_api.o)
                0x00000000000188f0                bt_is_testmode
                0x00000000000188fe                bt_is_l2cap_disconnected
                0x0000000000018918                bt_is_disconnecting
                0x0000000000018932                btstack_status_update
                0x0000000000018940                btstack_set_play_status
                0x000000000001896c                btstack_get_play_status
                0x000000000001897c                bt_get_status
                0x00000000000189c4                bt_get_disp_status
                0x00000000000189c6                bt_is_calling
                0x00000000000189dc                bt_get_l2cap_status
                0x0000000000018a08                bt_tws_get_status
 .com_text.stack.run_loop
                0x0000000000018a2a        0x2 ..\..\..\Libraries\libs\libbtstack_master.a(btstack_api.o)
                0x0000000000018a2a                btstack_msg
 .com_text.stack.ble.api0
                0x0000000000018a2c       0x10 ..\..\..\Libraries\libs\libbtstack_master.a(ble_api.o)
                0x0000000000018a2c                ble_get_status
 .com_text.stack.ble.api1
                0x0000000000018a3c       0x16 ..\..\..\Libraries\libs\libbtstack_master.a(ble_api.o)
                0x0000000000018a3c                ble_is_connect
 .com_text.bb.frag
                0x0000000000018a52       0x3a ..\..\..\Libraries\libs\libbtstack_master.a(bb_sche.o)
 .com_text.bb.prog
                0x0000000000018a8c      0x1f0 ..\..\..\Libraries\libs\libbtstack_master.a(bb_sche.o)
 .com_text.bb.patch
                0x0000000000018c7c       0x52 ..\..\..\Libraries\libs\libbtstack_master.a(patch_asm.o)
                0x0000000000018c7c                bb_v1_patch0
                0x0000000000018c88                bb_v1_patch6
                0x0000000000018c90                bb_v1_patch7
                0x0000000000018caa                bb_v1_patch8
 .com_text.bb.isr
                0x0000000000018cce       0x1a ..\..\..\Libraries\libs\libbtstack_master.a(aes.o)
                0x0000000000018cce                ble_ecpy_aes_res_cb
 .com_text.bb.isr
                0x0000000000018ce8       0x50 ..\..\..\Libraries\libs\libbtstack_master.a(rf.o)
                0x0000000000018ce8                rf_rssi_calc_dbm
                0x0000000000018cf2                rf_txpwr_get_lv
                0x0000000000018d26                rf_txpwr_get_dbm
                0x0000000000018d36                rf_agc_enable
 .com_text.isr.txrx
                0x0000000000018d38       0x76 ..\..\..\Libraries\libs\libbtstack_master.a(rf.o)
                0x0000000000018d38                bb_rf_ext_ctl_cb
                0x0000000000018d3a                bthw_txrx_isr
 *fill*         0x0000000000018dae        0x2 
 .com_text.bt21.isr
                0x0000000000018db0      0x5c8 ..\..\..\Libraries\libs\libbtstack_master.a(bt_hook.o)
                0x0000000000018db0                bt_page_init_func
                0x0000000000018db8                bt_acl_rx_header
                0x0000000000018fb0                bt_acl_test_rx_end
                0x0000000000018fb4                bt_acl_rx_end
                0x000000000001901c                bt_acl_sniff_cacl_win_size
                0x0000000000019074                bt_isr_hook
 .com_text.ble.isr
                0x0000000000019378       0x7c ..\..\..\Libraries\libs\libbtstack_master.a(ble_hook.o)
                0x0000000000019378                ble_isr_hook
 .com_text.bb.hct
                0x00000000000193f4       0x18 ..\..\..\Libraries\libs\libbtstack_master.a(hct_fc.o)
                0x00000000000193f4                hci_fc_acl_packet_sent
 .com_text.bt21.sco
                0x000000000001940c       0x1e ..\..\..\Libraries\libs\libbtstack_master.a(tws_sco.o)
                0x000000000001940c                bt_sco_get_index
 .com_text.bb.tws.sw.chk
                0x000000000001942a        0x4 ..\..\..\Libraries\libs\libbtstack_master.a(tws_acl.o)
                0x000000000001942a                tws_switch_acl_is_pause
 .com_text.bt21.isr
                0x000000000001942e       0x3c ..\..\..\Libraries\libs\libbtstack_master.a(bt_hal.o)
                0x000000000001942e                bt_channel_assess
 .com_text.bt21.isr
                0x000000000001946a       0x52 ..\..\..\Libraries\libs\libbtstack_master.a(bt21.o)
                0x000000000001946a                bt_buf_acl_rx_free
                0x0000000000019478                bt21_isr
 .com_text.ble.isr
                0x00000000000194bc      0x102 ..\..\..\Libraries\libs\libbtstack_master.a(ble_hal.o)
 .com_text.ble.isr.con
                0x00000000000195be       0x3c ..\..\..\Libraries\libs\libbtstack_master.a(ble_hal.o)
                0x00000000000195be                ble_channel_assess
 .com_text.ble.isr.adv
                0x00000000000195fa       0x52 ..\..\..\Libraries\libs\libbtstack_master.a(ble_adv.o)
                0x00000000000195fa                ble_adv_duration_update
 .com_text.bb.isr
                0x000000000001964c       0x18 ..\..\..\Libraries\libs\libbtstack_master.a(ble.o)
                0x000000000001964c                ble_isr
 .com_text.l2cap_test.con
                0x0000000000019664       0x4c ..\..\..\Libraries\libs\libbtstack_master.a(l2cap_test.o)
                0x0000000000019664                l2cap_vd_acl_check
 .com_text.stack.handler.l2cap
                0x00000000000196b0       0x38 ..\..\..\Libraries\libs\libbtstack_master.a(l2cap.o)
                0x00000000000196b0                l2cap_get_channel_for_local_cid
                0x00000000000196c8                l2cap_get_channel_for_remote_cid
 .com_text.sco  0x00000000000196e8        0x4 ..\..\..\Libraries\libs\libbtstack_master.a(hci_sco.o)
                0x00000000000196e8                sco_init_var
                0x00000000000196ea                sco_buffer_reset
 .com_text.stack.hci
                0x00000000000196ec       0x5a ..\..\..\Libraries\libs\libbtstack_master.a(hci.o)
                0x00000000000196ec                hci_connection_for_handle
                0x0000000000019714                hci_can_send_command_packet_now
 .com_text.stack.hci_recv
                0x0000000000019746        0xe ..\..\..\Libraries\libs\libbtstack_master.a(hci.o)
                0x0000000000019746                hci_host_recv_packet
 .com_text.bb.btisr
                0x0000000000019754        0x8 ..\..\..\Libraries\libs\libbtstack_master.a(avdtp.o)
                0x0000000000019754                a2dp_get_play_index
                0x0000000000019758                avdtp_rx_media_parse
 .com_text.stack.hcic
                0x000000000001975c       0x10 ..\..\..\Libraries\libs\libbtstack_master.a(hci_transport_hcic.o)
                0x000000000001975c                hcic_can_send_packet_now
 .com_text.ble.isr.test.clr
                0x000000000001976c       0x22 ..\..\..\Libraries\libs\libbtstack_master.a(ble_test.o)
 .com_text.ble.init
                0x000000000001978e      0xba2 ..\..\..\Libraries\libs\libbtstack_master.a(ble_init.o)
 *(.com_text.stack.handler)
 *(.com_rodata*)
 *fill*         0x000000000001a330        0x0 
 .com_rodata.exception
                0x000000000001a330       0x29 ..\..\..\Libraries\libs\libplatform.a(main.o)
 *fill*         0x000000000001a359        0x3 
 .com_rodata.irq
                0x000000000001a35c       0x1b ..\..\..\Libraries\libs\libplatform.a(interrupt.o)
                0x000000000001a35c                watch_point_str
 *fill*         0x000000000001a377        0x1 
 .com_rodata.miss
                0x000000000001a378       0x29 ..\..\..\Libraries\libs\libplatform.a(debug.o)
 *fill*         0x000000000001a3a1        0x3 
 .com_rodata.bb.sco
                0x000000000001a3a4       0x3c ..\..\..\Libraries\libs\libbtstack_master.a(bt_sco.o)
                0x000000000001a3a4                tbl_msbc_mute
 .com_rodata.bb.tbl
                0x000000000001a3e0       0x32 ..\..\..\Libraries\libs\libbtstack_master.a(bt_acl.o)
 *fill*         0x000000000001a412        0x2 
 .com_rodata.bb.tbl
                0x000000000001a414       0x10 ..\..\..\Libraries\libs\libbtstack_master.a(ble_con.o)
                0x000000000001a414                byte_tx_time
                0x000000000001a41c                fixed_tx_time
 .com_rodata.bb.tbl
                0x000000000001a424       0x44 ..\..\..\Libraries\libs\libbtstack_master.a(bb_utils.o)
                0x000000000001a424                one_bits
                0x000000000001a434                bb_rate_to_byte_dur_us
                0x000000000001a43c                bb_rate_to_phy_mask
                0x000000000001a440                bb_phy_value_to_mask
                0x000000000001a444                bb_phy_mask_to_value
                0x000000000001a44c                bb_phy_to_rate
                0x000000000001a450                bb_rate_to_phy
                0x000000000001a458                bb_sca2ppm
 .com_rodata.bb.tws
                0x000000000001a468        0xd ..\..\..\Libraries\libs\libbtstack_master.a(bb_int.o)
                0x000000000001a468                str_bb_err
 *fill*         0x000000000001a475        0x3 
 .com_rodata.bb.tbl
                0x000000000001a478       0x3c ..\..\..\Libraries\libs\libbtstack_master.a(bb.o)
                0x000000000001a478                bb_priority
 .com_rodata.bb.tbl
                0x000000000001a4b4        0xc ..\..\..\Libraries\libs\libbtstack_master.a(vs_proc.o)
                0x000000000001a4b4                vs_msg_env
 .com_rodata.bb.tbl
                0x000000000001a4c0        0x8 ..\..\..\Libraries\libs\libbtstack_master.a(rf.o)
 .com_rodata.bb.tbl
                0x000000000001a4c8        0xb ..\..\..\Libraries\libs\libbtstack_master.a(bt_hook.o)
 *fill*         0x000000000001a4d3        0x1 
 .com_rodata.bb.tbl
                0x000000000001a4d4       0x12 ..\..\..\Libraries\libs\libbtstack_master.a(bt21.o)
 *fill*         0x000000000001a4e6        0x2 
 .com_rodata.btstakc.hci
                0x000000000001a4e8        0x8 ..\..\..\Libraries\libs\libbtstack_master.a(hci_cmd.o)
                0x000000000001a4e8                hci_num_of_packet_complete
 .com_rodata.hci.trans
                0x000000000001a4f0       0x20 ..\..\..\Libraries\libs\libbtstack_master.a(hci_transport_hcic.o)
 .com_rodata.bb.tbl
                0x000000000001a510        0xc ..\..\..\Libraries\libs\libbtstack_master.a(lm_proc.o)
                0x000000000001a510                lm_msg_env
 .com_rodata.bb.tbl
                0x000000000001a51c        0x8 ..\..\..\Libraries\libs\libbtstack_master.a(ble_init.o)
                0x000000000001a51c                ble_init_max_aux_dur_tab
 .com_rodata.bb.tbl
                0x000000000001a524       0x18 ..\..\..\Libraries\libs\libbtstack_master.a(ble_buf.o)
 .com_rodata.bb.tbl
                0x000000000001a53c        0xc ..\..\..\Libraries\libs\libbtstack_master.a(lc_proc.o)
                0x000000000001a53c                lc_msg_env
 .com_rodata.bb.tbl
                0x000000000001a548        0xc ..\..\..\Libraries\libs\libbtstack_master.a(mgr_proc.o)
                0x000000000001a548                mgr_msg_env
 .com_rodata.bb.tbl
                0x000000000001a554        0xc ..\..\..\Libraries\libs\libbtstack_master.a(ll_proc.o)
                0x000000000001a554                ll_msg_env
 *debug.o(.rodata*)
 .rodata.str1.4
                0x000000000001a560       0xd0 ..\..\..\Libraries\libs\libplatform.a(debug.o)
                                         0xce (size before relaxing)
 *(.data*)
 .data          0x000000000001a630        0xc Output\obj\Libraries\BT\spp\profile.o
                0x000000000001a630                spp_sdp_record_item
 .data          0x000000000001a63c       0x18 ..\..\..\Libraries\libs\libbtstack_master.a(btstack_link_key_db.o)
 .data          0x000000000001a654       0x31 ..\..\..\Libraries\libs\libbtstack_master.a(btstack_run_loop.o)
                0x000000000001a654                data_source_debug_info
 *(.sdata*)
 *fill*         0x000000000001a685        0x1 
 .sdata         0x000000000001a686        0x2 Output\obj\Libraries\bsp\bsp_fot.o
                0x000000000001a686                dev_version
 .sdata         0x000000000001a688        0x1 Output\obj\Libraries\BT\ble\adv0.o
                0x000000000001a688                cfg_ble_adv0_en
 .sdata         0x000000000001a689        0x2 Output\obj\Libraries\BT\ble\ble.o
                0x000000000001a689                cfg_ble_mtu_request_en
                0x000000000001a68a                cfg_ble_security_en
 *fill*         0x000000000001a68b        0x1 
 .sdata         0x000000000001a68c       0x10 Output\obj\Libraries\BT\spp\bt.o
                0x000000000001a68c                bt_local_addr
                0x000000000001a692                cfg_bt_link_info_items
                0x000000000001a694                cfg_bt_sup_to_connect_times
                0x000000000001a696                cfg_bt_pwrup_connect_times
                0x000000000001a697                cfg_bt_connect_times
                0x000000000001a698                cfg_bt_support_profile
                0x000000000001a69a                cfg_bt_dual_mode
                0x000000000001a69b                cfg_bt_max_acl_link
 .sdata         0x000000000001a69c        0x1 Output\obj\Libraries\libs\strong_symbol.o
                0x000000000001a69c                cfg_bt_sniff_mode_dis
 *fill*         0x000000000001a69d        0x3 
 .sdata         0x000000000001a6a0        0x8 Output\obj\Examples\BLE_Host\Source\ble_client.o
                0x000000000001a6a6                target_write_uuid16
 .sdata         0x000000000001a6a8        0x4 ..\..\..\Libraries\libs\libdrivers.a(usb_device_hid.o)
                0x000000000001a6a8                user_ep_type
                0x000000000001a6a9                user_ep_dir
                0x000000000001a6aa                user_ep_idx
                0x000000000001a6ab                hid_in_ep
 .sdata         0x000000000001a6ac       0x11 ..\..\..\Libraries\libs\libbtstack_master.a(extern_bt.o)
                0x000000000001a6ac                cfg_bt_music_low_latency
                0x000000000001a6ae                cfg_bt_music_normal_latency
                0x000000000001a6b0                cfg_bt_ble_adv
                0x000000000001a6bc                cfg_bt_sniff_clk_sel
 *fill*         0x000000000001a6bd        0x3 
 .sdata         0x000000000001a6c0        0x4 ..\..\..\Libraries\libs\libbtstack_master.a(sdp_server.o)
 .sdata         0x000000000001a6c4        0x3 ..\..\..\Libraries\libs\libbtstack_master.a(sm.o)
 *fill*         0x000000000001a6c7        0x1 
 .sdata         0x000000000001a6c8        0x4 ..\..\..\Libraries\libs\libbtstack_master.a(att_server.o)
 .sdata         0x000000000001a6cc        0xc ..\..\..\Libraries\libs\libbtstack_master.a(btstack_hal.o)
 .sdata         0x000000000001a6d8        0x1 ..\..\..\Libraries\libs\libbtstack_master.a(btstack_adv0.o)
 *fill*         0x000000000001a6d9        0x3 
 .sdata         0x000000000001a6dc        0x5 ..\..\..\Libraries\libs\libbtstack_master.a(ble_adv0.o)
 .sdata         0x000000000001a6e1        0x1 ..\..\..\Libraries\libs\libbtstack_master.a(extern_hfhs.o)
                0x000000000001a6e1                cfg_bt_hfp_feature
 .sdata         0x000000000001a6e2        0x3 ..\..\..\Libraries\libs\libbtstack_master.a(l2cap_signaling.o)
 *(.load_text)
 *fill*         0x000000000001a6e5        0x1 
 .load_text     0x000000000001a6e6       0x10 ..\..\..\Libraries\libs\libplatform.a(main.o)
 *(.load_rodata)
                0x000000000001a800                . = ALIGN (0x200)
 *fill*         0x000000000001a6f6      0x10a 

.flash          0x0000000010003a00    0x44e00
                0x0000000010003a00                __code_start_sniff = .
 *(.sniff*)
                0x0000000010003a00                . = ALIGN (0x200)
                0x0000000010003a00                __code_end_sniff = .
                0x0000000010003a00                __code_start_usbdev = .
 *(.usbdev*)
 .usbdev.com    0x0000000010003a00      0x1b2 ..\..\..\Libraries\libs\libdrivers.a(usb_device_hid.o)
                0x0000000010003a00                usb_user_ep_tx_handler
                0x0000000010003a02                usb_user_ep_rx_handler
                0x0000000010003a04                ude_hid_setvalid
                0x0000000010003a18                ude_hid_send
                0x0000000010003a72                usb_user_ep_rx_ack
                0x0000000010003a96                usb_user_ep_tx_process
                0x0000000010003ab2                usb_user_ep_rx_process
                0x0000000010003ae0                usb_int_ep_reset
                0x0000000010003af6                udh_init
                0x0000000010003b52                udu_init
 .usbdev.com    0x0000000010003bb2       0x7c ..\..\..\Libraries\libs\libdrivers.a(usb_device_printer.o)
                0x0000000010003bb2                usb_bulk_reset
                0x0000000010003bc8                ude_rx_ack
                0x0000000010003be0                bulk_tx_handler
                0x0000000010003be2                bulk_rx_handler
                0x0000000010003be4                ude_bulk_tx_process
                0x0000000010003c00                ude_bulk_rx_process
 .usbdev.com    0x0000000010003c2e      0x36c ..\..\..\Libraries\libs\libdrivers.a(usb_device_ep.o)
                0x0000000010003c2e                usb_set_cur_ep
                0x0000000010003c44                usb_ep_init
                0x0000000010003cd0                usb_ep_halt
                0x0000000010003d1c                usb_ep_clear
                0x0000000010003d5c                usb_ep_transfer
                0x0000000010003eea                usb_ep_reset
                0x0000000010003f5e                usb_ep_start_transfer
                0x0000000010003f78                usb_ep_do_transfer
                0x0000000010004000                . = ALIGN (0x200)
 *fill*         0x0000000010003f9a       0x66 
                0x0000000010004000                __code_end_usbdev = .
                0x0000000010004000                __code_start_sleep = .
 *(.saradc_text*)
 *(.sleep_text*)
 .sleep_text.sleep.rc
                0x0000000010004000       0xc2 ..\..\..\Libraries\libs\libplatform.a(rc.o)
                0x0000000010004000                rc_sleep_trim_init
                0x0000000010004002                rc_sleep_trim_clear
                0x0000000010004004                rc_sleep_get_freqcnt
                0x0000000010004072                rc_sleep_reset_sta
                0x0000000010004074                rc_sleep_get_trim_freqcnt
 .sleep_text.rf
                0x00000000100040c2      0x21a ..\..\..\Libraries\libs\libbtstack_master.a(rf_smart.o)
                0x00000000100041a2                rfphy_deep_sleep
                0x000000001000424a                rfphy_idle
                0x0000000010004400                . = ALIGN (0x200)
 *fill*         0x00000000100042dc      0x124 
                0x0000000010004400                __code_end_sleep = .
                0x0000000010004400                __code_start_charge = .
 *(.charge_text*)
 *(.text.bsp.charge)
 *(.text.bsp.tkey)
 *(.text.vhouse)
                0x0000000010004400                . = ALIGN (0x200)
                0x0000000010004400                __code_end_charge = .
                0x0000000010004400                __code_start_pwrsave = .
 *(.text.pwroff*)
                0x0000000010004400                . = ALIGN (0x200)
                0x0000000010004400                __code_end_pwrsave = .
                0x0000000010004400                __code_start_bb_test = .
 *(.bb_test*)
 *(.bb_test_rodata*)
                0x0000000010004400                . = ALIGN (0x200)
                0x0000000010004400                __code_end_bb_test = .
                0x0000000010004400                __code_start_update = .
 *(.text.update*)
 .text.update_sd0baud
                0x0000000010004400       0x3c ..\..\..\Libraries\libs\libplatform.a(sys_clk.o)
                0x0000000010004400                update_sd0baud
 .text.update_complete
                0x000000001000443c        0x2 ..\..\..\Libraries\libs\libplatform.a(weak_symbol.o)
                0x000000001000443c                update_complete
                0x0000000010004600                . = ALIGN (0x200)
 *fill*         0x000000001000443e      0x1c2 
                0x0000000010004600                __code_end_update = .
                0x0000000010004600                __code_start_huart = .
 *(.com_huart*)
                0x0000000010004600                . = ALIGN (0x200)
                0x0000000010004600                __code_end_huart = .
                0x0000000010004600                __code_start_fota = .
 *(.text.fot.cache*)
 .text.fot.cache
                0x0000000010004600      0x744 Output\obj\Libraries\bsp\bsp_fot.o
                0x000000001000466a                fot_recv_proc
                0x0000000010004b5c                bsp_fot_process
                0x0000000010004c44                bsp_usb_fot_process
 *fill*         0x0000000010004d44        0x0 
 .text.fot.cache
                0x0000000010004d44      0x204 ..\..\..\Libraries\libs\libplatform.a(fot_update.o)
                0x0000000010004d44                fot_pkt_process_do
                0x0000000010004eae                fot_write
                0x0000000010005000                . = ALIGN (0x200)
 *fill*         0x0000000010004f48       0xb8 
                0x0000000010005000                __code_end_fota = .
                0x0000000010005000                __code_start_bts = .
 *(.text.stk.tws.txreq*)
 *(.text.stk.l2cap.txreq*)
 .text.stk.l2cap.txreq
                0x0000000010005000      0x110 ..\..\..\Libraries\libs\libbtstack_master.a(l2cap.o)
                0x00000000100050d4                l2cap_request_can_send_now_event
                0x00000000100050ee                l2cap_request_can_send_fix_channel_now_event
 *fill*         0x0000000010005110        0x0 
 .text.stk.l2cap.txreq.rodata
                0x0000000010005110        0xa ..\..\..\Libraries\libs\libbtstack_master.a(l2cap.o)
                0x0000000010005200                . = ALIGN (0x200)
 *fill*         0x000000001000511a       0xe6 
 *(.text.stk.tws.send*)
                0x0000000010005200                . = ALIGN (0x200)
 *(.text.stk.tws.recv*)
                0x0000000010005200                . = ALIGN (0x200)
 *(.text.stk.hci.tx*)
                0x0000000010005200                . = ALIGN (0x200)
 *(.text.bts.hci.rx*)
                0x0000000010005200                . = ALIGN (0x200)
 *(.text.stk.bt.acl.tx*)
 .text.stk.bt.acl.tx.done
                0x0000000010005200       0x76 ..\..\..\Libraries\libs\libbtstack_master.a(lc_proc.o)
                0x0000000010005400                . = ALIGN (0x200)
 *fill*         0x0000000010005276      0x18a 
                0x0000000010005400                __code_end_bts = .
 *(.irq_init.aligned)
                0x0000000010005400                . = ALIGN (0x200)
 *(.text.ble.chmap*)
 .text.ble.chmap
                0x0000000010005400       0x50 ..\..\..\Libraries\libs\libbtstack_master.a(ble_con.o)
                0x0000000010005400                ble_con_ch_map_update
                0x0000000010005600                . = ALIGN (0x200)
 *fill*         0x0000000010005450      0x1b0 
 *(.text*)
 .text.bsp_bt_init
                0x0000000010005600       0xac Output\obj\Libraries\bsp\bsp_bt.o
                0x0000000010005600                bsp_bt_init
 .text.bt_emit_notice
                0x00000000100056ac       0x40 Output\obj\Libraries\bsp\bsp_bt.o
                0x00000000100056ac                bt_emit_notice
 .text.cm_loadparam
                0x00000000100056ec       0x12 Output\obj\Libraries\bsp\bsp_cm.o
                0x00000000100056ec                cm_loadparam
 .text.cm_factory
                0x00000000100056fe       0x20 Output\obj\Libraries\bsp\bsp_cm.o
                0x00000000100056fe                cm_factory
 .text.fot.update
                0x000000001000571e       0x6c Output\obj\Libraries\bsp\bsp_fot.o
                0x000000001000571e                is_fot_start
                0x000000001000572a                fot_update_pause
                0x0000000010005744                bsp_fot_init
                0x000000001000576c                fot_update_continue
 .text.fot_ble_disconnect_callback
                0x000000001000578a       0x32 Output\obj\Libraries\bsp\bsp_fot.o
                0x000000001000578a                fot_ble_disconnect_callback
 .text.fot_ble_connect_callback
                0x00000000100057bc        0xc Output\obj\Libraries\bsp\bsp_fot.o
                0x00000000100057bc                fot_ble_connect_callback
 .text.fot_spp_connect_callback
                0x00000000100057c8        0xc Output\obj\Libraries\bsp\bsp_fot.o
                0x00000000100057c8                fot_spp_connect_callback
 .text.fot_spp_disconnect_callback
                0x00000000100057d4       0x32 Output\obj\Libraries\bsp\bsp_fot.o
                0x00000000100057d4                fot_spp_disconnect_callback
 .text.bsp.param
                0x0000000010005806       0xee Output\obj\Libraries\bsp\bsp_param.o
                0x0000000010005806                param_init
                0x0000000010005824                bsp_param_write
                0x0000000010005828                bsp_param_read
                0x000000001000582c                bsp_param_sync
                0x0000000010005830                param_sync
                0x0000000010005834                param_get_xosc_addr
                0x0000000010005838                param_fot_addr_write
                0x000000001000584e                param_fot_addr_read
                0x0000000010005858                param_fot_remote_ver_write
                0x000000001000586e                param_fot_remote_ver_read
                0x0000000010005878                param_fot_head_info_write
                0x000000001000588e                param_fot_head_info_read
                0x0000000010005898                param_fot_hash_write
                0x00000000100058ae                param_fot_hash_read
                0x00000000100058b8                param_qcheck_code_write
                0x00000000100058ce                param_qcheck_code_read
                0x00000000100058d8                param_sys_vol_write
                0x00000000100058e6                param_sys_vol_read
 .text.bsp.sys.init
                0x00000000100058f4      0x232 Output\obj\Libraries\bsp\bsp_sys.o
                0x000000001000596c                rtc_init
                0x00000000100059de                bsp_update_init
                0x0000000010005a24                bsp_sys_init
 .text.uart0_mapping_sel
                0x0000000010005b26       0x90 Output\obj\Libraries\bsp\bsp_sys.o
                0x0000000010005b26                uart0_mapping_sel
 .text.bsp_get_xosc_xcfg
                0x0000000010005bb6       0x20 Output\obj\Libraries\bsp\bsp_sys.o
                0x0000000010005bb6                bsp_get_xosc_xcfg
 .text.ble_txpkt_init
                0x0000000010005bd6       0x30 Output\obj\Libraries\BT\ble\ab_link\app.o
                0x0000000010005bd6                ble_txpkt_init
 .text.ble_service_change_indicate
                0x0000000010005c06       0x2a Output\obj\Libraries\BT\ble\ab_link\app.o
                0x0000000010005c06                ble_service_change_indicate
 .text.ble_fot_send_packet
                0x0000000010005c30       0x1a Output\obj\Libraries\BT\ble\ab_link\app.o
                0x0000000010005c30                ble_fot_send_packet
 .text.ble_client_cfg_callback
                0x0000000010005c4a       0x3a Output\obj\Libraries\BT\ble\ab_link\app.o
                0x0000000010005c4a                ble_client_cfg_callback
 .text.ble_get_local_bd_addr
                0x0000000010005c84       0x28 Output\obj\Libraries\BT\ble\ble.o
                0x0000000010005c84                ble_get_local_bd_addr
 .text.ble_enter_transmit
                0x0000000010005cac       0x24 Output\obj\Libraries\BT\ble\ble.o
                0x0000000010005cac                ble_enter_transmit
 .text.ble_disconnect_callback
                0x0000000010005cd0       0x18 Output\obj\Libraries\BT\ble\ble.o
                0x0000000010005cd0                ble_disconnect_callback
 .text.ble_connect_callback
                0x0000000010005ce8       0x18 Output\obj\Libraries\BT\ble\ble.o
                0x0000000010005ce8                ble_connect_callback
 .text.bt_get_class_of_device
                0x0000000010005d00       0x18 Output\obj\Libraries\BT\spp\bt.o
                0x0000000010005d00                bt_get_class_of_device
 .text.bt_get_pin_code
                0x0000000010005d18        0xa Output\obj\Libraries\BT\spp\bt.o
                0x0000000010005d18                bt_get_pin_code
 .text.bt_get_local_name
                0x0000000010005d22        0x8 Output\obj\Libraries\BT\spp\bt.o
                0x0000000010005d22                bt_get_local_name
 .text.bt_get_local_bd_addr
                0x0000000010005d2a       0x14 Output\obj\Libraries\BT\spp\bt.o
                0x0000000010005d2a                bt_get_local_bd_addr
 .text.bt_get_link_info
                0x0000000010005d3e       0x24 Output\obj\Libraries\BT\spp\bt.o
                0x0000000010005d3e                bt_get_link_info
 .text.bt_put_link_info
                0x0000000010005d62       0x24 Output\obj\Libraries\BT\spp\bt.o
                0x0000000010005d62                bt_put_link_info
 .text.bt_get_ext_link_info
                0x0000000010005d86        0x8 Output\obj\Libraries\BT\spp\bt.o
                0x0000000010005d86                bt_get_ext_link_info
 .text.bt_put_ext_link_info
                0x0000000010005d8e        0x8 Output\obj\Libraries\BT\spp\bt.o
                0x0000000010005d8e                bt_put_ext_link_info
 .text.bt_sync_link_info
                0x0000000010005d96        0x4 Output\obj\Libraries\BT\spp\bt.o
                0x0000000010005d96                bt_sync_link_info
 .text.bt_init_lib
                0x0000000010005d9a       0x24 Output\obj\Libraries\BT\spp\profile.o
                0x0000000010005d9a                bt_init_lib
 .text.spp_txpkt_init
                0x0000000010005dbe       0x30 Output\obj\Libraries\BT\spp\spp.o
                0x0000000010005dbe                spp_txpkt_init
 .text.spp_rxpkt_init
                0x0000000010005dee        0x8 Output\obj\Libraries\BT\spp\spp.o
                0x0000000010005dee                spp_rxpkt_init
 .text.get_spp_mtu_size
                0x0000000010005df6        0x6 Output\obj\Libraries\BT\spp\spp.o
                0x0000000010005df6                get_spp_mtu_size
 .text.spp_connect_callback
                0x0000000010005dfc       0x18 Output\obj\Libraries\BT\spp\spp.o
                0x0000000010005dfc                spp_connect_callback
 .text.spp_disconnect_callback
                0x0000000010005e14       0x18 Output\obj\Libraries\BT\spp\spp.o
                0x0000000010005e14                spp_disconnect_callback
 .text.spp_rx_callback
                0x0000000010005e2c       0x86 Output\obj\Libraries\BT\spp\spp.o
                0x0000000010005e2c                spp_rx_callback
 .text.clock_gate0_cmd
                0x0000000010005eb2       0x16 Output\obj\Libraries\Device\Source\gw3323_clk.o
                0x0000000010005eb2                clock_gate0_cmd
 .text.gpio_init
                0x0000000010005ec8       0xf6 Output\obj\Libraries\Device\Source\gw3323_gpio.o
                0x0000000010005ec8                gpio_init
 .text.gpio_func_mapping
                0x0000000010005fbe       0x5a Output\obj\Libraries\Device\Source\gw3323_gpio.o
                0x0000000010005fbe                gpio_func_mapping
 .text.hsuart_init
                0x0000000010006018       0x44 Output\obj\Libraries\Device\Source\gw3323_hsuart.o
                0x0000000010006018                hsuart_init
 .text.hsuart_pic_config
                0x000000001000605c       0x3a Output\obj\Libraries\Device\Source\gw3323_hsuart.o
                0x000000001000605c                hsuart_pic_config
 .text.hsuart_dma_config
                0x0000000010006096       0x24 Output\obj\Libraries\Device\Source\gw3323_hsuart.o
                0x0000000010006096                hsuart_dma_config
 .text.vs_ble_test
                0x00000000100060ba        0x4 Output\obj\Libraries\libs\strong_symbol.o
                0x00000000100060ba                vs_ble_test
 .text.vs_fcc_test_cmd
                0x00000000100060be        0x4 Output\obj\Libraries\libs\strong_symbol.o
                0x00000000100060be                vs_fcc_test_cmd
 .text.is_fot_update_en
                0x00000000100060c2        0x4 Output\obj\Libraries\libs\strong_symbol.o
                0x00000000100060c2                is_fot_update_en
 .text.usb_init
                0x00000000100060c6        0x2 Output\obj\Libraries\libs\strong_symbol.o
                0x00000000100060c6                usb_init
 .text.usb_isr  0x00000000100060c8        0x2 Output\obj\Libraries\libs\strong_symbol.o
                0x00000000100060c8                usb_isr
 .text.ude_ep_reset
                0x00000000100060ca        0x2 Output\obj\Libraries\libs\strong_symbol.o
                0x00000000100060ca                ude_ep_reset
 .text.ude_control_flow
                0x00000000100060cc        0x2 Output\obj\Libraries\libs\strong_symbol.o
                0x00000000100060cc                ude_control_flow
 .text.ble_att_read_callback
                0x00000000100060ce       0x2a Output\obj\Examples\BLE_Host\Source\ble_client.o
 .text.ble_clent_event_packet_handle
                0x00000000100060f8      0x39c Output\obj\Examples\BLE_Host\Source\ble_client.o
                0x00000000100060f8                ble_clent_event_packet_handle
 .text.ble_client_notify_callback
                0x0000000010006494       0x3c Output\obj\Examples\BLE_Host\Source\ble_client.o
 .text.ble_client_init
                0x00000000100064d0       0x32 Output\obj\Examples\BLE_Host\Source\ble_client.o
                0x00000000100064d0                ble_client_init
 .text.hsuart_transfer_example
                0x0000000010006502       0x4c Output\obj\Examples\BLE_Host\Source\ble_client.o
                0x0000000010006502                hsuart_transfer_example
 .text.btstack_ble_init_callback
                0x000000001000654e       0x42 Output\obj\Examples\BLE_Host\Source\ble_init.o
                0x000000001000654e                btstack_ble_init_callback
 .text.ble_init_register
                0x0000000010006590        0xc Output\obj\Examples\BLE_Host\Source\ble_init.o
                0x0000000010006590                ble_init_register
 .text.my_hsuart_init
                0x000000001000659c       0xc8 Output\obj\Examples\BLE_Host\Source\hsuart_transfer.o
                0x000000001000659c                my_hsuart_init
 .text.getcfg_vddbt_sel
                0x0000000010006664       0x18 Output\obj\Examples\BLE_Host\Project\config.o
                0x0000000010006664                getcfg_vddbt_sel
 .text.getcfg_vddio_sel
                0x000000001000667c        0xc Output\obj\Examples\BLE_Host\Project\config.o
                0x000000001000667c                getcfg_vddio_sel
 .text.getcfg_vddbt_capless_en
                0x0000000010006688        0xa Output\obj\Examples\BLE_Host\Project\config.o
                0x0000000010006688                getcfg_vddbt_capless_en
 .text.startup.main
                0x0000000010006692       0x32 Output\obj\Examples\BLE_Host\Project\main.o
                0x0000000010006692                main
 .text.pll_vco_band_trimming
                0x00000000100066c4       0x9a ..\..\..\Libraries\libs\libplatform.a(audio.o)
 *fill*         0x000000001000675e       0xa2 
 .text.adpll_divider_update_do
                0x0000000010006800       0xfa ..\..\..\Libraries\libs\libplatform.a(audio.o)
                0x0000000010006800                adpll_divider_update_do
 .text.adpll_divider_update
                0x00000000100068fa       0x68 ..\..\..\Libraries\libs\libplatform.a(audio.o)
                0x00000000100068fa                adpll_divider_update
 .text.adpll_init
                0x0000000010006962      0x106 ..\..\..\Libraries\libs\libplatform.a(audio.o)
                0x0000000010006962                adpll_init
 .text.cm_loadpage
                0x0000000010006a68       0xb4 ..\..\..\Libraries\libs\libplatform.a(cm.o)
 .text.cm_next_freepage
                0x0000000010006b1c       0x54 ..\..\..\Libraries\libs\libplatform.a(cm.o)
 .text.cm_movepage
                0x0000000010006b70       0x60 ..\..\..\Libraries\libs\libplatform.a(cm.o)
 .text.cm_release
                0x0000000010006bd0      0x112 ..\..\..\Libraries\libs\libplatform.a(cm.o)
 .text.cm_savepage
                0x0000000010006ce2       0xc8 ..\..\..\Libraries\libs\libplatform.a(cm.o)
 .text.cm_check_loadpage
                0x0000000010006daa       0xb0 ..\..\..\Libraries\libs\libplatform.a(cm.o)
 .text.cm_sync  0x0000000010006e5a       0x3e ..\..\..\Libraries\libs\libplatform.a(cm.o)
                0x0000000010006e5a                cm_sync
 .text.cm_read  0x0000000010006e98       0x44 ..\..\..\Libraries\libs\libplatform.a(cm.o)
                0x0000000010006e98                cm_read
 .text.cm_write
                0x0000000010006edc       0x5e ..\..\..\Libraries\libs\libplatform.a(cm.o)
                0x0000000010006edc                cm_write
 .text.cm_init  0x0000000010006f3a      0x1e8 ..\..\..\Libraries\libs\libplatform.a(cm.o)
                0x0000000010006f3a                cm_init
 .text.xcfg_init
                0x0000000010007122       0x66 ..\..\..\Libraries\libs\libplatform.a(xcfg.o)
                0x0000000010007122                xcfg_init
 .text.usb_disable
                0x0000000010007188       0x22 ..\..\..\Libraries\libs\libplatform.a(device.o)
                0x0000000010007188                usb_disable
 .text.device.init
                0x00000000100071aa       0xb2 ..\..\..\Libraries\libs\libplatform.a(device.o)
                0x00000000100071aa                dev_init
                0x0000000010007204                dev_delay_times
                0x0000000010007216                dev_delay_online_times
                0x0000000010007224                dev_delay_offline_times
                0x0000000010007232                dev_clr_sta
 .text.platform_main
                0x000000001000725c      0x212 ..\..\..\Libraries\libs\libplatform.a(main.o)
                0x000000001000725c                platform_main
 .text.main_startup
                0x000000001000746e       0x3e ..\..\..\Libraries\libs\libplatform.a(main.o)
                0x000000001000746e                main_startup
 .text.sys_irq_init.part.0
                0x00000000100074ac       0x50 ..\..\..\Libraries\libs\libplatform.a(interrupt.o)
 .text.sys_irq_init
                0x00000000100074fc       0x48 ..\..\..\Libraries\libs\libplatform.a(interrupt.o)
                0x00000000100074fc                sys_irq_init
 .text.timer0_init
                0x0000000010007544       0x64 ..\..\..\Libraries\libs\libplatform.a(interrupt.o)
                0x0000000010007544                timer0_init
 .text.soft_irq_init
                0x00000000100075a8       0x3c ..\..\..\Libraries\libs\libplatform.a(interrupt.o)
                0x00000000100075a8                soft_irq_init
 .text.bthw_irq_init
                0x00000000100075e4       0x38 ..\..\..\Libraries\libs\libplatform.a(interrupt.o)
                0x00000000100075e4                bthw_irq_init
 .text.sd0_irq_init
                0x000000001000761c       0x32 ..\..\..\Libraries\libs\libplatform.a(interrupt.o)
                0x000000001000761c                sd0_irq_init
 .text.usb_irq_init
                0x000000001000764e       0x26 ..\..\..\Libraries\libs\libplatform.a(interrupt.o)
                0x000000001000764e                usb_irq_init
 .text.aubuf_irq_init
                0x0000000010007674       0x32 ..\..\..\Libraries\libs\libplatform.a(interrupt.o)
                0x0000000010007674                aubuf_irq_init
 .text.thread_main_entry
                0x00000000100076a6      0x17a ..\..\..\Libraries\libs\libplatform.a(startup.o)
 .text.bt_set_timer_enable
                0x0000000010007820        0xa ..\..\..\Libraries\libs\libplatform.a(startup.o)
                0x0000000010007820                bt_set_timer_enable
 .text.sys_set_tmr_enable
                0x000000001000782a        0xe ..\..\..\Libraries\libs\libplatform.a(startup.o)
                0x000000001000782a                sys_set_tmr_enable
 .text.thread_idle_create
                0x0000000010007838       0x30 ..\..\..\Libraries\libs\libplatform.a(startup.o)
                0x0000000010007838                thread_idle_create
 .text.startup.init
                0x0000000010007868      0x116 ..\..\..\Libraries\libs\libplatform.a(startup.o)
                0x0000000010007868                platform_init
                0x000000001000786a                sys_startup
 .text.sys_hook_init
                0x000000001000797e        0x2 ..\..\..\Libraries\libs\libplatform.a(sys_hook.o)
                0x000000001000797e                sys_hook_init
 .text.debug_set
                0x0000000010007980       0x1a ..\..\..\Libraries\libs\libplatform.a(debug.o)
                0x0000000010007980                debug_set
 .text.fot.update
                0x000000001000799a      0x88e ..\..\..\Libraries\libs\libplatform.a(fot_update.o)
                0x0000000010007b96                get_keep_mac
                0x0000000010007bda                calc_mac
                0x0000000010007c14                mac_init
                0x0000000010007ce2                set_macbuf
                0x0000000010007d36                clear_macbuf
                0x0000000010007d7e                fot_head_info_analize
                0x0000000010007d92                fot_set_keep
                0x0000000010007e0a                fot_clear_keep
                0x0000000010007e3a                fot_down_first4k
                0x0000000010008106                fot_tws_done_try
                0x0000000010008108                fot_tws_done
                0x0000000010008146                fot_tws_done_sync_err_deal
                0x000000001000816c                fot_head_info_save
                0x0000000010008178                fot_breakpoint_info_read
                0x00000000100081fa                fot_get_err
                0x0000000010008204                is_fot_update_success
                0x0000000010008214                fot_get_curaddr
 .text.fot.init
                0x0000000010008228       0xa2 ..\..\..\Libraries\libs\libplatform.a(fot_update.o)
 .text.is_fot_tws_support
                0x00000000100082ca        0x4 ..\..\..\Libraries\libs\libplatform.a(fot_update.o)
                0x00000000100082ca                is_fot_tws_support
 .text.get_spiloader_offset
                0x00000000100082ce        0xc ..\..\..\Libraries\libs\libplatform.a(fot_update.o)
                0x00000000100082ce                get_spiloader_offset
 .text.fot_checksum_cal
                0x00000000100082da       0xde ..\..\..\Libraries\libs\libplatform.a(fot_update.o)
                0x00000000100082da                fot_checksum_cal
 .text.fot_down_first4k_checksum_cal
                0x00000000100083b8       0x98 ..\..\..\Libraries\libs\libplatform.a(fot_update.o)
                0x00000000100083b8                fot_down_first4k_checksum_cal
 .text.fot_init
                0x0000000010008450       0x2e ..\..\..\Libraries\libs\libplatform.a(fot_update.o)
                0x0000000010008450                fot_init
 .text.fot_set_base_offset
                0x000000001000847e       0x28 ..\..\..\Libraries\libs\libplatform.a(fot_update.o)
                0x000000001000847e                fot_set_base_offset
 .text.lock_init
                0x00000000100084a6       0x10 ..\..\..\Libraries\libs\libplatform.a(lock.o)
                0x00000000100084a6                lock_init
 .text.lock_code_bt_comm
                0x00000000100084b6        0x2 ..\..\..\Libraries\libs\libplatform.a(lock.o)
                0x00000000100084b6                lock_code_bt_comm
 .text.unlock_code_bt_comm
                0x00000000100084b8        0x2 ..\..\..\Libraries\libs\libplatform.a(lock.o)
                0x00000000100084b8                unlock_code_bt_comm
 .text.load_code_fota
                0x00000000100084ba       0x42 ..\..\..\Libraries\libs\libplatform.a(lock.o)
                0x00000000100084ba                load_code_fota
 .text.patch_init
                0x00000000100084fc       0x1e ..\..\..\Libraries\libs\libplatform.a(patch.o)
                0x00000000100084fc                patch_init
 .text.set_buck_mode
                0x000000001000851a       0x46 ..\..\..\Libraries\libs\libplatform.a(power.o)
                0x000000001000851a                set_buck_mode
 .text.vddio_voltage_configure
                0x0000000010008560       0x54 ..\..\..\Libraries\libs\libplatform.a(power.o)
                0x0000000010008560                vddio_voltage_configure
 .text.vddbt_voltage_configure
                0x00000000100085b4       0x4e ..\..\..\Libraries\libs\libplatform.a(power.o)
                0x00000000100085b4                vddbt_voltage_configure
 .text.pmu_voltage_configure
                0x0000000010008602       0x64 ..\..\..\Libraries\libs\libplatform.a(power.o)
                0x0000000010008602                pmu_voltage_configure
 .text.pmu_init
                0x0000000010008666      0x15e ..\..\..\Libraries\libs\libplatform.a(power.o)
                0x0000000010008666                pmu_init
 .text.udivmoddi4
                0x00000000100087c4       0x96 ..\..\..\Libraries\libs\libplatform.a(sys.o)
 .text.sys_get_rc2m_clkhz
                0x000000001000885a      0x178 ..\..\..\Libraries\libs\libplatform.a(sys.o)
                0x000000001000885a                sys_get_rc2m_clkhz
 .text.sys_get_rand_key_init
                0x00000000100089d2       0x76 ..\..\..\Libraries\libs\libplatform.a(sys.o)
                0x00000000100089d2                sys_get_rand_key_init
 .text.sys_get_rand_key
                0x0000000010008a48       0x5a ..\..\..\Libraries\libs\libplatform.a(sys.o)
                0x0000000010008a48                sys_get_rand_key
 .text.bsp.param
                0x0000000010008aa2       0x66 ..\..\..\Libraries\libs\libplatform.a(sys.o)
                0x0000000010008aa2                param_bt_xosc_read
                0x0000000010008ad6                bt_save_xosc_cap
 .text.xosc_init
                0x0000000010008b08       0xa2 ..\..\..\Libraries\libs\libplatform.a(sys.o)
                0x0000000010008b08                xosc_init
 .text.bt_restore_xosc_cap
                0x0000000010008baa        0x4 ..\..\..\Libraries\libs\libplatform.a(sys.o)
                0x0000000010008baa                bt_restore_xosc_cap
 .text.bt_get_xosc_cap
                0x0000000010008bae       0x18 ..\..\..\Libraries\libs\libplatform.a(sys.o)
                0x0000000010008bae                bt_get_xosc_cap
 .text.bt_set_xosc_cap
                0x0000000010008bc6       0x26 ..\..\..\Libraries\libs\libplatform.a(sys.o)
                0x0000000010008bc6                bt_set_xosc_cap
 .text.bt_adj_xosc_cap
                0x0000000010008bec       0x8a ..\..\..\Libraries\libs\libplatform.a(sys.o)
                0x0000000010008bec                bt_adj_xosc_cap
 .text.__udivdi3
                0x0000000010008c76        0x6 ..\..\..\Libraries\libs\libplatform.a(sys.o)
                0x0000000010008c76                __udivdi3
 .text.sys_clk_cacl_curr
                0x0000000010008c7c       0x24 ..\..\..\Libraries\libs\libplatform.a(sys_clk.o)
 *fill*         0x0000000010008ca0        0x0 
 .text.sys_clk  0x0000000010008ca0      0x1f8 ..\..\..\Libraries\libs\libplatform.a(sys_clk.o)
                0x0000000010008ca0                get_clksel_val
                0x0000000010008cb2                get_cur_sysclk
                0x0000000010008cba                set_audec_clkdiv
                0x0000000010008cd8                set_sbcec_clkdiv
                0x0000000010008cda                sysclk_update_baud
                0x0000000010008d12                update_uart1baud_in_sysclk_set
                0x0000000010008d36                sys_clk_set_do
 *fill*         0x0000000010008e98      0x168 
 .text.set_sys_clk_do
                0x0000000010009000      0x1f0 ..\..\..\Libraries\libs\libplatform.a(sys_clk.o)
                0x0000000010009000                set_sys_clk_do
 .text.set_peripherals_clkdiv
                0x00000000100091f0      0x11c ..\..\..\Libraries\libs\libplatform.a(sys_clk.o)
                0x00000000100091f0                set_peripherals_clkdiv
 .text.get_sysclk_nhz
                0x000000001000930c       0x7e ..\..\..\Libraries\libs\libplatform.a(sys_clk.o)
                0x000000001000930c                get_sysclk_nhz
 .text.set_sys_clk
                0x000000001000938a       0x34 ..\..\..\Libraries\libs\libplatform.a(sys_clk.o)
                0x000000001000938a                set_sys_clk
 *fill*         0x00000000100093be        0x2 
 .text.sys_clk.table
                0x00000000100093c0        0xa ..\..\..\Libraries\libs\libplatform.a(sys_clk.o)
                0x00000000100093c0                sysclk_sel_tbl
 .text.voltage.trim
                0x00000000100093ca      0x188 ..\..\..\Libraries\libs\libplatform.a(voltage_trim.o)
                0x00000000100093ca                bt_get_ft_trim_value
                0x0000000010009400                dac_get_ft_trim_value
                0x000000001000941e                voltage_trim_value_init
 .text.stack.api
                0x0000000010009552       0x2a ..\..\..\Libraries\libs\libplatform.a(bt.o)
                0x0000000010009552                bt_send_msg_do
 .text          0x000000001000957c       0x70 ..\..\..\Libraries\libs\libbtstack_master.a(nanos.o)
                0x000000001000957c                nanos_init
                0x00000000100095b0                nanos_var_init
 .text          0x00000000100095ec       0x68 ..\..\..\Libraries\libs\libbtstack_master.a(patch.o)
                0x00000000100095ec                bb_patch_init
 .text          0x0000000010009654        0x2 ..\..\..\Libraries\libs\libbtstack_master.a(platform.o)
                0x0000000010009654                timer_sync_init
 .text          0x0000000010009656       0x1c ..\..\..\Libraries\libs\libbtstack_master.a(bt_sco.o)
                0x0000000010009656                lc_sco_pkt_init
                0x0000000010009658                lc_sco_codec_init
                0x000000001000965c                lc_sco_codec_exit
                0x0000000010009660                lc_sco_codec_setup
                0x0000000010009670                lc_sco_codec_kill
 *fill*         0x0000000010009672      0x18e 
 .text          0x0000000010009800     0x216e ..\..\..\Libraries\libs\libbtstack_master.a(bt_acl.o)
                0x00000000100099d2                bt_acl_init
                0x0000000010009a0e                bt_acl_reset
                0x0000000010009a78                bt_acl_start
                0x0000000010009d1e                bt_acl_init_param
                0x0000000010009e00                bt_acl_stop
                0x0000000010009ec0                bt_acl_flow_off
                0x0000000010009f00                bt_acl_flow_on
                0x0000000010009f80                bt_acl_flush_to_get
                0x0000000010009fc0                bt_acl_flush_to_set
                0x000000001000a000                bt_acl_poll_int_get
                0x000000001000a040                bt_acl_poll_int_set
                0x000000001000a100                bt_acl_sniff_trans
                0x000000001000a200                bt_acl_sniff
                0x000000001000a300                bt_acl_unsniff
                0x000000001000a3b2                bt_acl_tx_enc
                0x000000001000a3d4                bt_acl_rx_enc
                0x000000001000a3fa                bt_acl_bcst_rx_enc
                0x000000001000a424                bt_acl_enc_key_set
                0x000000001000a500                bt_acl_master_clock_get
                0x000000001000a580                bt_acl_clock_offset_get
                0x000000001000a600                bt_acl_rsw_slot_offset_get
                0x000000001000a680                bt_acl_rsw_slot_offset_set
                0x000000001000a700                bt_acl_sup_to_get
                0x000000001000a740                bt_acl_sup_to_set
                0x000000001000a780                bt_acl_tim_acc_set
                0x000000001000a800                bt_acl_edr_set
                0x000000001000a900                bt_acl_tx_pkt_types_set
                0x000000001000aa00                bt_acl_dm1_pkt_type_dis
                0x000000001000aa80                bt_acl_curr_txpwr_get
                0x000000001000ac00                bt_acl_afh_set
                0x000000001000ae00                bt_acl_afh_new
                0x000000001000af00                bt_acl_afh_cfm
                0x000000001000af80                bt_acl_rx_max_slot_get
                0x000000001000afc0                bt_acl_rx_max_slot_set
                0x000000001000b000                bt_acl_test_mode_set
                0x000000001000b0c0                bt_acl_rssi_thr_get
                0x000000001000b0f0                bt_sco_start
                0x000000001000b500                bt_sco_stop
                0x000000001000b580                bt_acl_sniff_clock_set
                0x000000001000b600                bt_acl_sniff_clock_diff
                0x000000001000b700                bt_acl_resche
 *fill*         0x000000001000b96e       0x92 
 .text          0x000000001000ba00      0xca6 ..\..\..\Libraries\libs\libbtstack_master.a(ble_con.o)
                0x000000001000ba00                ble_con_evt_time_update_fix
                0x000000001000bb00                ble_con_start_do
                0x000000001000bb28                ble_con_start
                0x000000001000c000                ble_con_stop
                0x000000001000c080                ble_con_param_update
                0x000000001000c100                ble_con_phys_update
                0x000000001000c180                ble_con_tx_len_update_for_intv
                0x000000001000c200                ble_con_tx_len_update_for_rate
                0x000000001000c280                ble_con_event_counter_get
                0x000000001000c2b0                ble_con_tx_enc
                0x000000001000c2fc                ble_con_rx_enc
                0x000000001000c348                ble_con_enc_key_load
                0x000000001000c400                ble_con_current_tx_power_get
                0x000000001000c480                ble_con_rssi_get
                0x000000001000c4b0                ble_con_offset_get
                0x000000001000c4ec                ble_con_pref_slave_latency_set
                0x000000001000c52c                ble_con_pref_slave_evt_dur_set
                0x000000001000c580                ble_con_peer_sca_set
                0x000000001000c5aa                ble_con_duration_min_set
 *fill*         0x000000001000c6a6       0x5a 
 .text.bb.ble.con.flow
                0x000000001000c700       0xfa ..\..\..\Libraries\libs\libbtstack_master.a(ble_con.o)
                0x000000001000c700                ble_con_data_flow_set
 *fill*         0x000000001000c7fa        0x6 
 .text.bb.ble.con.data_len
                0x000000001000c800       0xfa ..\..\..\Libraries\libs\libbtstack_master.a(ble_con.o)
                0x000000001000c800                ble_con_data_len_update
 .text.le.con   0x000000001000c8fa       0x8c ..\..\..\Libraries\libs\libbtstack_master.a(ble_con.o)
                0x000000001000c8fa                ble_get_con_var
                0x000000001000c904                ble_con_init
 *fill*         0x000000001000c986        0x2 
 .text          0x000000001000c988      0x5d2 ..\..\..\Libraries\libs\libbtstack_master.a(bb_utils.o)
                0x000000001000c9d4                bb_bytes_to_string
                0x000000001000ca12                bb_nb_good_channels
                0x000000001000ca46                bb_util_pack
                0x000000001000ccc8                bb_util_unpack
 .text          0x000000001000cf5a      0x1ba ..\..\..\Libraries\libs\libbtstack_master.a(bb_int.o)
                0x000000001000cf5a                bb_time_set
                0x000000001000cf78                bb_sleep_init
                0x000000001000cfd0                bb_driver_init
 *fill*         0x000000001000d114       0xec 
 .text.bb.aes   0x000000001000d200      0x1f6 ..\..\..\Libraries\libs\libbtstack_master.a(bb_int.o)
                0x000000001000d200                bb_aes_encrypt
 .text          0x000000001000d3f6      0x2b6 ..\..\..\Libraries\libs\libbtstack_master.a(bb.o)
                0x000000001000d3f6                bb_rand_init
                0x000000001000d400                bb_get_heap_info
                0x000000001000d414                bb_var_init
                0x000000001000d41c                bb_reset
                0x000000001000d4ac                bb_init
                0x000000001000d62e                bb_off
                0x000000001000d680                bb_run_loop
 .text          0x000000001000d6ac       0x1a ..\..\..\Libraries\libs\libbtstack_master.a(platform.o)
                0x000000001000d6ac                lm_inq_start_do
                0x000000001000d6b0                lm_inq_stop_do
                0x000000001000d6b4                lm_inq_res_ind_do
                0x000000001000d6b6                bt_pf_init
                0x000000001000d6b8                bt_pf_exit
                0x000000001000d6ba                bt_pf_post
                0x000000001000d6bc                bt_pf_get_info
                0x000000001000d6be                bt_is_ota_enable
 .text          0x000000001000d6c6       0x50 ..\..\..\Libraries\libs\libbtstack_master.a(extern_tws.o)
                0x000000001000d6c6                bt_tws_get_force_role
                0x000000001000d6ca                tws_get_spp_eq_info
                0x000000001000d6ce                tws_set_spp_eq_info
                0x000000001000d6d0                bt_get_right_ear_sta
                0x000000001000d6d4                bt_get_left_ear_sta
                0x000000001000d6d8                bt_change_nr_sta
                0x000000001000d6dc                bt_get_loc_nr_sta
                0x000000001000d6e0                bt_get_auto_anwer_sta
                0x000000001000d6e4                bt_set_menu_ctrl_sta
                0x000000001000d6e6                tws_get_new_bt_name
                0x000000001000d6ea                bt_get_serial_number
                0x000000001000d6ee                bt_get_ch_serial_number
                0x000000001000d6f2                bt_inear_test
                0x000000001000d70e                bt_get_model_number
                0x000000001000d712                bt_get_fw_version
 .text          0x000000001000d716       0x9a ..\..\..\Libraries\libs\libbtstack_master.a(extern_bt.o)
                0x000000001000d716                bt_rf_get_inq_param
                0x000000001000d71a                bt_rf_get_param
                0x000000001000d71e                bt_rf_get_sco_param
                0x000000001000d722                bt_rf_get_fcc_param
                0x000000001000d73a                bt_get_new_local_name
                0x000000001000d73e                bt_set_new_local_name
                0x000000001000d74e                bt_is_always_reconn
                0x000000001000d752                bt_get_conn_fail_delay
                0x000000001000d758                bt_get_connect_addr
                0x000000001000d780                tws_set_fot_data
                0x000000001000d784                tws_get_fot_data
                0x000000001000d788                tws_get_dueros_dma_data
                0x000000001000d78c                tws_set_dueros_dma_data
                0x000000001000d790                tws_send_dueros_dma_data_cfm
                0x000000001000d792                tws_set_switch_fix_acl
                0x000000001000d796                is_bt_nor_linkkey_prohibit_del
                0x000000001000d79a                bt_voice_callback
                0x000000001000d79c                spp_custom1_rx_callback
                0x000000001000d79e                spp_custom2_rx_callback
                0x000000001000d7a2                spp_client_cfg_callback
                0x000000001000d7a8                spp_custom1_connect_callback
                0x000000001000d7aa                spp_custom1_disconnect_callback
                0x000000001000d7ac                spp_custom2_connect_callback
                0x000000001000d7ae                spp_custom2_disconnect_callback
 .text          0x000000001000d7b0      0x398 ..\..\..\Libraries\libs\libbtstack_master.a(spp.o)
                0x000000001000d814                spp_disconnect
                0x000000001000d8cc                spp_service_flush
                0x000000001000d8d8                get_spp_connection_context_for_rfcomm_cid
                0x000000001000d908                get_spp_connection_context_for_bd_addr
                0x000000001000d9e4                provide_spp_connection_context_for_bd_addr
                0x000000001000da4c                spp_establish_service_level_connection
                0x000000001000dac6                spp_release_service_level_connection
                0x000000001000db10                spp_init
                0x000000001000db30                spp_init_var
                0x000000001000db40                spp_support_mul_server
 .text.stack.spp.handler
                0x000000001000db48      0x23c ..\..\..\Libraries\libs\libbtstack_master.a(spp.o)
                0x000000001000db48                spp_packet_handler
 .text.stack.sdp.util
                0x000000001000dd84      0x60e ..\..\..\Libraries\libs\libbtstack_master.a(sdp_util.o)
                0x000000001000de36                de_get_size_type
                0x000000001000de3e                de_get_element_type
                0x000000001000de46                de_get_header_size
                0x000000001000de64                de_get_data_size
                0x000000001000dea8                de_get_len
                0x000000001000df80                de_element_get_uint16
                0x000000001000dfac                de_get_normalized_uuid
                0x000000001000e006                de_get_uuid32
                0x000000001000e02e                de_store_descriptor_with_len
                0x000000001000e06c                des_iterator_init
                0x000000001000e09c                des_iterator_get_type
                0x000000001000e0ac                des_iterator_get_size
                0x000000001000e0d4                des_iterator_has_more
                0x000000001000e0e2                des_iterator_get_element
                0x000000001000e0f8                des_iterator_next
                0x000000001000e116                sdp_attribute_list_constains_id
                0x000000001000e242                sdp_filter_attributes_in_attributeIDList
                0x000000001000e27a                spd_get_filtered_size
                0x000000001000e29c                sdp_get_attribute_value_for_attribute_id
                0x000000001000e2bc                sdp_set_attribute_value_for_attribute_id
                0x000000001000e2e2                sdp_record_contains_UUID128
                0x000000001000e340                sdp_traversal_match_pattern
                0x000000001000e36c                sdp_record_matches_service_search_pattern
                0x000000001000e390                de_dump_data_element
 .text          0x000000001000e392       0x42 ..\..\..\Libraries\libs\libbtstack_master.a(sdp_server.o)
                0x000000001000e3ca                remove_sdp_server_context
 .text.stack.sdp.server
                0x000000001000e3d4      0x750 ..\..\..\Libraries\libs\libbtstack_master.a(sdp_server.o)
                0x000000001000e422                sdp_get_service_record_handle
                0x000000001000e456                sdp_get_record_for_handle
                0x000000001000e464                sdp_create_service_record_handle
                0x000000001000e484                sdp_handle_service_search_request
                0x000000001000e624                sdp_handle_service_attribute_request
                0x000000001000e7a0                sdp_handle_service_search_attribute_request
 .text.stack.setup
                0x000000001000eb24       0x3a ..\..\..\Libraries\libs\libbtstack_master.a(sdp_server.o)
                0x000000001000eb24                sdp_init
 .text.stack.sdp.server_add
                0x000000001000eb5e       0x46 ..\..\..\Libraries\libs\libbtstack_master.a(sdp_server.o)
                0x000000001000eb5e                sdp_add_service
 *fill*         0x000000001000eba4        0x0 
 .text          0x000000001000eba4      0x79c ..\..\..\Libraries\libs\libbtstack_master.a(sdp_client.o)
                0x000000001000eba4                remove_sdp_client_context
                0x000000001000ebae                de_state_init
                0x000000001000ebbe                de_state_size
                0x000000001000ec1c                sdp_parser_init
                0x000000001000ec42                sdp_parser_handle_chunk
                0x000000001000ee86                sdp_parser_handle_done
                0x000000001000eee2                sdp_client_packet_handler
                0x000000001000f226                sdp_client_init
                0x000000001000f242                sdp_client_free
                0x000000001000f256                sdp_client_query
 .text          0x000000001000f340     0x195a ..\..\..\Libraries\libs\libbtstack_master.a(rfcomm.o)
                0x000000001000f908                rfcomm_multiplexer_finalize
                0x000000001000f9a2                rfcomm_set_required_security_level
                0x000000001000f9aa                rfcomm_can_send_packet_now
                0x000000001000f9bc                rfcomm_request_can_send_now_event
                0x000000001000f9d8                rfcomm_reserve_packet_buffer
                0x000000001000f9dc                rfcomm_release_packet_buffer
                0x000000001000f9e0                rfcomm_get_outgoing_buffer
                0x000000001000f9ee                rfcomm_get_max_frame_size
                0x000000001000fa02                rfcomm_create_channel_with_initial_credits
                0x000000001000fa0a                rfcomm_create_channel
                0x000000001000fa12                rfcomm_disconnect
                0x000000001000fa42                rfcomm_register_service_with_initial_credits
                0x000000001000fa4a                rfcomm_unregister_service
                0x000000001000fa80                rfcomm_accept_connection
                0x000000001000fad0                crc8_calc
                0x000000001000fb06                rfcomm_send_prepared
                0x000000001000fbc2                rfcomm_send
                0x0000000010010bc6                provide_rfcomm_multiplexer
                0x0000000010010be2                provide_rfcomm_channel
                0x0000000010010c3a                rfcomm_set_packet_handler_for_channels
                0x0000000010010c4e                rfcomm_get_now_incoming_credit
                0x0000000010010c64                rfcomm_set_to_send_new_incoming_credit
 .text.stack.rfcomm
                0x0000000010010c9a       0x90 ..\..\..\Libraries\libs\libbtstack_master.a(rfcomm.o)
                0x0000000010010d24                rfcomm_register_service
 .text.stack.setup
                0x0000000010010d2a       0x22 ..\..\..\Libraries\libs\libbtstack_master.a(rfcomm.o)
                0x0000000010010d2a                rfcomm_init
 .text.stack.link_key
                0x0000000010010d4c      0x60c ..\..\..\Libraries\libs\libbtstack_master.a(btstack_link_key_db.o)
                0x0000000010010ebe                btstack_get_link_addr
                0x0000000010010f72                btstack_get_link_key
                0x0000000010011006                btstack_get_link_feature
                0x000000001001103a                btstack_delete_link_key
                0x00000000100110d4                btstack_delete_all_link_key
                0x0000000010011142                btstack_put_link_key
                0x0000000010011240                btstack_put_link_offset
                0x000000001001128c                btstack_delete_all_link_offset
                0x00000000100112f8                btstack_put_link_feature
 .text.stack.setup
                0x0000000010011358      0x184 ..\..\..\Libraries\libs\libbtstack_master.a(btstack_link_key_db.o)
                0x0000000010011358                btstack_open_link_info
 .text.stack.link_key.get.name
                0x00000000100114dc       0x62 ..\..\..\Libraries\libs\libbtstack_master.a(btstack_link_key_db.o)
                0x00000000100114dc                btstack_get_link_name
 .text.stack.link_key.put.name
                0x000000001001153e       0x94 ..\..\..\Libraries\libs\libbtstack_master.a(btstack_link_key_db.o)
                0x000000001001153e                btstack_put_link_name
 .text          0x00000000100115d2       0xac ..\..\..\Libraries\libs\libbtstack_master.a(btstack_util.o)
                0x00000000100115d2                log_info_hexdump
                0x00000000100115d4                log_info_key
                0x00000000100115d6                uuid_add_bluetooth_prefix
                0x00000000100115f8                uuid_has_bluetooth_prefix
                0x0000000010011614                sscanf_bd_addr
 .text.stack.util
                0x000000001001167e      0x126 ..\..\..\Libraries\libs\libbtstack_master.a(btstack_util.o)
                0x000000001001167e                bd_addr_cmp
                0x0000000010011684                bd_addr_copy
                0x000000001001168a                big_endian_read_16
                0x000000001001169a                big_endian_read_32
                0x00000000100116ba                big_endian_store_16
                0x00000000100116ce                big_endian_store_32
                0x0000000010011702                reverse_bytes
                0x000000001001171e                reverse_24
                0x0000000010011722                reverse_48
                0x0000000010011726                reverse_56
                0x000000001001172a                reverse_64
                0x000000001001172e                reverse_128
                0x0000000010011732                reverse_256
                0x0000000010011738                reverse_bd_addr
                0x000000001001173a                btstack_min
                0x0000000010011740                btstack_max
                0x0000000010011746                char_for_nibble
                0x000000001001176c                nibble_for_char
 .text.stack.hci_dump
                0x00000000100117a4       0x52 ..\..\..\Libraries\libs\libbtstack_master.a(btstack_util.o)
                0x00000000100117a4                bd_addr_to_str
 .text          0x00000000100117f6       0x7c ..\..\..\Libraries\libs\libbtstack_master.a(btstack_txpkt.o)
                0x00000000100117f6                txpkt_init
 *fill*         0x0000000010011872        0xe 
 .text.stk.txpkt.flush
                0x0000000010011880       0x82 ..\..\..\Libraries\libs\libbtstack_master.a(btstack_txpkt.o)
                0x0000000010011880                txpkt_flush
 *fill*         0x0000000010011902       0x7e 
 .text.stack.run_loop
                0x0000000010011980      0x174 ..\..\..\Libraries\libs\libbtstack_master.a(btstack_run_loop.o)
                0x0000000010011980                btstack_run_loop_set_timer_handler
                0x0000000010011984                btstack_run_loop_set_data_source_handler
                0x0000000010011988                btstack_run_loop_set_data_source_fd
                0x000000001001198c                btstack_run_loop_get_data_source_fd
                0x0000000010011990                btstack_run_loop_enable_data_source_callbacks
                0x000000001001199c                btstack_run_loop_disable_data_source_callbacks
                0x00000000100119ac                btstack_run_loop_add_data_source
                0x00000000100119b8                btstack_run_loop_remove_data_source
                0x00000000100119c4                btstack_run_loop_set_timer
                0x00000000100119e0                btstack_run_loop_set_timer_context
                0x00000000100119e4                btstack_run_loop_get_timer_context
                0x0000000010011a00                btstack_run_loop_set_trig_ticks
                0x0000000010011a3c                btstack_run_loop_add_timer
                0x0000000010011a6c                btstack_run_loop_remove_timer
                0x0000000010011a9a                btstack_run_loop_get_ticks
                0x0000000010011aa6                btstack_run_loop_ticks_for_ms
                0x0000000010011aac                btstack_run_loop_get_time_ms
                0x0000000010011aba                btstack_run_loop_timer_dump
 .text.stack.setup
                0x0000000010011af4       0x34 ..\..\..\Libraries\libs\libbtstack_master.a(btstack_run_loop.o)
                0x0000000010011af4                btstack_run_loop_init
 .text          0x0000000010011b28       0x16 ..\..\..\Libraries\libs\libbtstack_master.a(btstack_memory.o)
                0x0000000010011b28                btstack_memory_gatt_client_get
                0x0000000010011b32                btstack_memory_gatt_client_free
 .text.stack.memory
                0x0000000010011b3e       0x9a ..\..\..\Libraries\libs\libbtstack_master.a(btstack_memory.o)
                0x0000000010011b3e                btstack_memory_l2cap_service_get
                0x0000000010011b48                btstack_memory_l2cap_service_free
                0x0000000010011b54                btstack_memory_l2cap_channel_get
                0x0000000010011b5e                btstack_memory_l2cap_channel_free
                0x0000000010011b6a                btstack_memory_rfcomm_multiplexer_get
                0x0000000010011b74                btstack_memory_rfcomm_multiplexer_free
                0x0000000010011b80                btstack_memory_rfcomm_service_get
                0x0000000010011b8a                btstack_memory_rfcomm_service_free
                0x0000000010011b96                btstack_memory_rfcomm_channel_get
                0x0000000010011ba0                btstack_memory_rfcomm_channel_free
                0x0000000010011bac                btstack_memory_whitelist_entry_get
                0x0000000010011bb6                btstack_memory_whitelist_entry_free
                0x0000000010011bc2                btstack_memory_sm_lookup_entry_get
                0x0000000010011bcc                btstack_memory_sm_lookup_entry_free
 .text.stack.setup
                0x0000000010011bd8       0xa6 ..\..\..\Libraries\libs\libbtstack_master.a(btstack_memory.o)
                0x0000000010011bd8                btstack_memory_init
 .text.stack.linked_list
                0x0000000010011c7e       0x6c ..\..\..\Libraries\libs\libbtstack_master.a(btstack_linked_list.o)
                0x0000000010011c7e                btstack_linked_list_get_last_item
                0x0000000010011c8c                btstack_linked_list_add
                0x0000000010011ca0                btstack_linked_list_add_tail
                0x0000000010011cb4                btstack_linked_list_remove
                0x0000000010011ccc                btstack_linked_list_count
                0x0000000010011cda                btstack_linked_list_iterator_remove
 .text          0x0000000010011cea      0x270 ..\..\..\Libraries\libs\libbtstack_master.a(btstack_link_ctrl.o)
                0x0000000010011cea                alloc_link_ctrl_context_for_bd_addr
                0x0000000010011d6e                btstack_link_ctrl_stop_timer
                0x0000000010011d8a                btstack_link_ctrl_set_timer
                0x0000000010011dc0                link_ctrl_timer_handler
                0x0000000010011e4c                btstack_link_ctrl_get_num
                0x0000000010011e6a                btstack_link_ctrl_get_recon_sta
                0x0000000010011e94                btstack_link_ctrl_get_links
                0x0000000010011ea8                btstack_link_ctrl_is_exist
                0x0000000010011ee0                btstack_link_ctrl_abort_reconnect
 .text.stack.linkctrl
                0x0000000010011f5a      0x17a ..\..\..\Libraries\libs\libbtstack_master.a(btstack_link_ctrl.o)
                0x0000000010011f5a                chk_link_ctrl_context_use_up
                0x0000000010011f74                get_link_ctrl_context_for_bd_addr
                0x0000000010011fbe                provide_link_ctrl_context_for_bd_addr
                0x0000000010011fd6                remove_link_ctrl_context
                0x0000000010012040                remove_pending_link_ctrl_context
                0x0000000010012082                remove_waiting_link_ctrl_context_for_bd_addr
 .text.stack.setup
                0x00000000100120d4       0x16 ..\..\..\Libraries\libs\libbtstack_master.a(btstack_link_ctrl.o)
                0x00000000100120d4                btstack_link_ctrl_init
 *fill*         0x00000000100120ea        0x2 
 .text          0x00000000100120ec     0x2436 ..\..\..\Libraries\libs\libbtstack_master.a(sm.o)
                0x0000000010013f1e                sm_address_resolution_lookup
                0x0000000010013fa0                sm_cmac_ready
                0x0000000010013fae                sm_cmac_general_start
                0x0000000010014014                sm_cmac_signed_write_start
                0x0000000010014046                get_rand_addr
                0x0000000010014054                sm_register_oob_data_callback
                0x000000001001405c                sm_add_event_handler
                0x000000001001406a                sm_set_accepted_stk_generation_methods
                0x0000000010014074                sm_set_encryption_key_size_range
                0x0000000010014086                sm_set_authentication_requirements
                0x000000001001408e                sm_set_io_capabilities
                0x0000000010014096                sm_set_request_security
                0x00000000100140a0                sm_set_er
                0x00000000100140b0                sm_set_ir
                0x00000000100140c0                sm_test_set_irk
                0x00000000100140e0                sm_test_use_fixed_local_csrk
                0x00000000100140ec                sm_init
                0x00000000100141ce                sm_use_fixed_ec_keypair
                0x00000000100141d0                sm_test_use_fixed_ec_keypair
                0x00000000100141d2                sm_encryption_key_size
                0x00000000100141f2                sm_authenticated
                0x0000000010014212                sm_authorization_state
                0x0000000010014236                sm_send_security_request
                0x000000001001425a                sm_request_pairing
                0x00000000100142de                sm_authorization_decline
                0x0000000010014328                sm_authorization_grant
                0x0000000010014374                sm_bonding_decline
                0x00000000100143ce                sm_just_works_confirm
                0x0000000010014406                sm_numeric_comparison_confirm
                0x0000000010014408                sm_passkey_input
                0x0000000010014446                sm_keypress_notification
                0x0000000010014468                sm_le_device_index
                0x000000001001447c                gap_random_address_set_mode
                0x00000000100144b8                gap_random_address_get_mode
                0x00000000100144c0                gap_random_address_set_update_period
                0x00000000100144e6                gap_random_address_set
 .text          0x0000000010014522      0x3bc ..\..\..\Libraries\libs\libbtstack_master.a(le_device_db_memory.o)
                0x0000000010014522                le_device_db_init
                0x000000001001453c                le_device_db_set_local_bd_addr
                0x000000001001453e                le_device_db_count
                0x000000001001456a                le_device_db_remove
                0x0000000010014584                le_device_db_add
                0x00000000100145fa                le_device_db_info
                0x000000001001465a                le_device_db_encryption_set
                0x00000000100146c4                le_device_db_encryption_get
                0x0000000010014788                le_device_db_remote_csrk_get
                0x00000000100147b2                le_device_db_remote_csrk_set
                0x00000000100147d8                le_device_db_local_csrk_get
                0x0000000010014802                le_device_db_local_csrk_set
                0x0000000010014828                le_device_db_remote_counter_get
                0x000000001001483e                le_device_db_remote_counter_set
                0x0000000010014854                le_device_db_local_counter_get
                0x000000001001486a                le_device_db_local_counter_set
                0x0000000010014880                le_device_db_dump
 .text          0x00000000100148de      0x1ac ..\..\..\Libraries\libs\libbtstack_master.a(gatt_server.o)
                0x0000000010014902                ble_init_att_do
                0x0000000010014944                ble_init_att_for_handle
                0x0000000010014982                ble_register_att_buf_for_handle
                0x00000000100149cc                ble_tx_notify
                0x0000000010014a26                ble_tx_indication
                0x0000000010014a28                ble_update_conn_param
                0x0000000010014a4a                ble_set_adv_interval
                0x0000000010014a76                btstack_ble_disconnect
                0x0000000010014a82                btstack_ble_update_conn_param
                0x0000000010014a84                btstack_ble_set_adv_interval
                0x0000000010014a86                btstack_ble_set_adv_data
                0x0000000010014a88                btstack_ble_set_scan_rsp_data
 .text.att.r_cb
                0x0000000010014a8a       0xb4 ..\..\..\Libraries\libs\libbtstack_master.a(gatt_server.o)
                0x0000000010014a8a                att_read_callback
 .text.att.w_cb
                0x0000000010014b3e      0x1c6 ..\..\..\Libraries\libs\libbtstack_master.a(gatt_server.o)
                0x0000000010014b3e                att_write_callback
 .text.ble.att  0x0000000010014d04       0x76 ..\..\..\Libraries\libs\libbtstack_master.a(gatt_server.o)
                0x0000000010014d04                btstack_gatt_init
                0x0000000010014d6e                btstack_ble_send_req
 .text          0x0000000010014d7a      0x360 ..\..\..\Libraries\libs\libbtstack_master.a(gatt_profile.o)
                0x0000000010014d7a                ble_gatts_service_add
                0x0000000010014e38                ble_gatts_characteristic_add
                0x0000000010015028                ble_gatts_init
                0x0000000010015054                ble_att_write_callback
                0x0000000010015092                ble_att_read_callback
                0x00000000100150d0                ble_get_profile_data
 *fill*         0x00000000100150da        0x2 
 .text          0x00000000100150dc     0x1be4 ..\..\..\Libraries\libs\libbtstack_master.a(gatt_client.o)
                0x00000000100156a6                att_client_register_handler
                0x00000000100156b4                gatt_client_init
                0x0000000010015712                gatt_client_is_ready
                0x0000000010015728                gatt_client_get_mtu
                0x0000000010015750                att_exchange_mtu_request
                0x00000000100163e8                gatt_client_listen_for_characteristic_value_updates
                0x0000000010016408                gatt_client_signed_write_without_response
                0x0000000010016454                gatt_client_discover_primary_services
                0x0000000010016490                gatt_client_discover_primary_services_by_uuid16
                0x00000000100164da                gatt_client_discover_primary_services_by_uuid128
                0x0000000010016528                gatt_client_discover_characteristics_for_service
                0x0000000010016570                gatt_client_find_included_services_for_service
                0x00000000100165b0                gatt_client_discover_characteristics_for_handle_range_by_uuid16
                0x0000000010016606                gatt_client_discover_characteristics_for_handle_range_by_uuid128
                0x000000001001665e                gatt_client_discover_characteristics_for_service_by_uuid16
                0x000000001001666a                gatt_client_discover_characteristics_for_service_by_uuid128
                0x0000000010016676                gatt_client_discover_characteristic_descriptors
                0x00000000100166c2                gatt_client_read_value_of_characteristic_using_value_handle
                0x00000000100166fa                gatt_client_read_value_of_characteristics_by_uuid16
                0x000000001001674e                gatt_client_read_value_of_characteristics_by_uuid128
                0x00000000100167a4                gatt_client_read_value_of_characteristic
                0x00000000100167aa                gatt_client_read_long_value_of_characteristic_using_value_handle_with_offset
                0x00000000100167e6                gatt_client_read_long_value_of_characteristic_using_value_handle
                0x00000000100167ea                gatt_client_read_long_value_of_characteristic
                0x00000000100167f0                gatt_client_read_multiple_characteristic_values
                0x000000001001682a                gatt_client_write_value_of_characteristic_without_response
                0x000000001001687e                gatt_client_write_value_of_characteristic
                0x00000000100168be                gatt_client_write_long_value_of_characteristic_with_offset
                0x0000000010016904                gatt_client_write_long_value_of_characteristic
                0x000000001001690c                gatt_client_reliable_write_long_value_of_characteristic
                0x0000000010016950                gatt_client_write_client_characteristic_configuration
                0x00000000100169c0                gatt_client_read_characteristic_descriptor_using_descriptor_handle
                0x00000000100169f6                gatt_client_read_characteristic_descriptor
                0x00000000100169fc                gatt_client_read_long_characteristic_descriptor_using_descriptor_handle_with_offset
                0x0000000010016a3a                gatt_client_read_long_characteristic_descriptor_using_descriptor_handle
                0x0000000010016a3e                gatt_client_read_long_characteristic_descriptor
                0x0000000010016a44                gatt_client_write_characteristic_descriptor_using_descriptor_handle
                0x0000000010016a8a                gatt_client_write_characteristic_descriptor
                0x0000000010016a90                gatt_client_write_long_characteristic_descriptor_using_descriptor_handle_with_offset
                0x0000000010016ad8                gatt_client_write_long_characteristic_descriptor_using_descriptor_handle
                0x0000000010016ae0                gatt_client_write_long_characteristic_descriptor
                0x0000000010016ae6                gatt_client_prepare_write
                0x0000000010016b2e                gatt_client_execute_write
                0x0000000010016b5c                gatt_client_cancel_write
                0x0000000010016b8a                gatt_client_pts_suppress_mtu_exchange
                0x0000000010016b94                gatt_client_deserialize_service
                0x0000000010016bd6                gatt_client_deserialize_characteristic
                0x0000000010016c28                gatt_client_deserialize_characteristic_descriptor
                0x0000000010016c3c                ble_client_discover_primary_services
                0x0000000010016c48                ble_client_discover_primary_services_by_uuid16
                0x0000000010016c56                ble_client_discover_primary_services_by_uuid128
                0x0000000010016c64                ble_service_query_result_get_service
                0x0000000010016c6a                ble_client_discover_characteristics_for_service
                0x0000000010016c78                ble_characteristic_query_result_get_characteristic
                0x0000000010016c7e                ble_client_discover_characteristics_for_service_by_uuid16
                0x0000000010016c8e                ble_client_discover_characteristics_for_service_by_uuid128
                0x0000000010016c9e                ble_client_write_client_characteristic_configuration
                0x0000000010016cae                ble_gatt_client_write_value_of_characteristic
 .text          0x0000000010016cc0      0x7cc ..\..\..\Libraries\libs\libbtstack_master.a(att_server.o)
                0x0000000010016eee                ble_get_max_mtu
                0x0000000010016ef4                att_server_register_service_handler
                0x0000000010016f1c                att_server_init
                0x0000000010016f9a                att_server_register_packet_handler
                0x0000000010016fa2                att_server_can_send_packet_now
                0x0000000010016fb4                att_server_request_can_send_now_event
                0x00000000100173bc                att_server_notify
                0x0000000010017408                att_server_indicate
 .text          0x000000001001748c       0xe6 ..\..\..\Libraries\libs\libbtstack_master.a(att_dispatch.o)
                0x0000000010017526                att_dispatch_register_client
                0x000000001001753a                att_dispatch_register_server
                0x000000001001754e                att_dispatch_client_can_send_now
                0x0000000010017554                att_dispatch_server_can_send_now
                0x0000000010017556                att_dispatch_client_request_can_send_now_event
                0x0000000010017564                att_dispatch_server_request_can_send_now_event
 *fill*         0x0000000010017572        0x2 
 .text          0x0000000010017574      0xf8c ..\..\..\Libraries\libs\libbtstack_master.a(att_db.o)
                0x000000001001776e                att_uuid_for_handle
                0x0000000010017798                att_set_db
                0x00000000100177a0                att_set_read_callback
                0x00000000100177a8                att_set_write_callback
                0x00000000100177b0                att_dump_attributes
                0x00000000100177f4                att_clear_transaction_queue
                0x0000000010017810                att_prepare_handle_value_notification
                0x000000001001784e                att_prepare_handle_value_indication
                0x000000001001788c                att_handle_request
                0x00000000100182c6                gatt_server_get_get_handle_range_for_service_with_uuid16
                0x000000001001834c                gatt_server_get_value_handle_for_characteristic_with_uuid16
                0x000000001001838e                gatt_server_get_client_configuration_handle_for_characteristic_with_uuid16
                0x000000001001841a                gatt_server_get_value_handle_for_characteristic_with_uuid128
                0x0000000010018468                gatt_server_get_client_configuration_handle_for_characteristic_with_uuid128
 .text          0x0000000010018500       0x8c ..\..\..\Libraries\libs\libbtstack_master.a(btstack_main.o)
                0x0000000010018582                btstack_test_func
                0x0000000010018584                btstack_ble_set_init_callback
 .text.stack.handler
                0x000000001001858c      0x1b6 ..\..\..\Libraries\libs\libbtstack_master.a(btstack_main.o)
 .text.stack.ble.sm
                0x0000000010018742       0x20 ..\..\..\Libraries\libs\libbtstack_master.a(btstack_main.o)
                0x0000000010018742                le_sm_init
 .text.stack.ble.setup
                0x0000000010018762       0x18 ..\..\..\Libraries\libs\libbtstack_master.a(btstack_main.o)
                0x0000000010018762                btstack_ble_init
 .text.stack.setup
                0x000000001001877a       0x8c ..\..\..\Libraries\libs\libbtstack_master.a(btstack_main.o)
                0x000000001001877a                btstack_main
 .text          0x0000000010018806       0x18 ..\..\..\Libraries\libs\libbtstack_master.a(btstack_hal.o)
                0x0000000010018806                hal_tick_init
                0x000000001001880c                hal_tick_set_handler
 .text          0x000000001001881e      0x77a ..\..\..\Libraries\libs\libbtstack_master.a(btstack_api.o)
                0x000000001001881e                dma_start_speech_to_ai
                0x0000000010018820                btstack_ctl0_api
                0x0000000010018830                btstack_comm_api
                0x000000001001884a                btstack_hid_api
                0x0000000010018864                btstack_ble_disable_scan
                0x0000000010018868                btstack_ble_enable_scan
                0x000000001001886c                btstack_ble_set_scan_param
                0x0000000010018882                btstack_ble_conn_by_addr
                0x0000000010018886                btstack_fcc_test_func
                0x000000001001888a                btstack_spp_api
                0x0000000010018896                btstack_audio_bypass
                0x00000000100188e8                btstack_audio_enable
                0x0000000010018926                btstack_ctl_api
                0x00000000100189b2                btstack_tws_api
                0x00000000100189b4                btstack_a2dp_msg
                0x00000000100189b6                dma_stop_speech_to_ai
                0x00000000100189b8                btstack_reset_bt_name
                0x00000000100189ba                btstack_tws_switch_role
                0x00000000100189bc                btstack_tws_connect
                0x00000000100189be                btstack_low_latency_en
                0x00000000100189c0                btstack_low_latency_dis
                0x00000000100189c2                btstack_ble_set_adv_param
                0x00000000100189c4                btstack_nor_connect
                0x00000000100189c6                bt_decode_init
                0x00000000100189c8                btstack_var_init
                0x00000000100189f8                btstack_establish_service_connection_do
                0x0000000010018a18                btstack_establish_service_connection
                0x0000000010018a20                btstack_continue_establish_service_connection
                0x0000000010018a48                btstack_tws_search_slave
                0x0000000010018a4a                btstack_emit_notice_status
                0x0000000010018a82                btstack_connect_address
                0x0000000010018b12                btstack_emit_notice
                0x0000000010018b26                btstack_tws_disc_continue
                0x0000000010018b28                bt_emit_player_notice
                0x0000000010018b76                btstack_tws_set_status
                0x0000000010018b78                btstack_clr_dis_flag
                0x0000000010018b90                btstack_get_ext_feature
                0x0000000010018bba                btstack_set_hfp_status_ptr
                0x0000000010018bec                btstack_set_hsp_status_ptr
                0x0000000010018c02                btstack_clr_hfp_status_ptr
                0x0000000010018c48                btstack_clr_hsp_status_ptr
                0x0000000010018c64                bt_get_siri_status
                0x0000000010018c68                btstack_get_tws_key
                0x0000000010018c94                btstack_get_tws_msg
                0x0000000010018cc2                btstack_get_tws_hid_key
                0x0000000010018ce8                btstack_get_tws_hid_msg
                0x0000000010018d26                bt_tws_is_playing
                0x0000000010018d3c                bt_tws_is_calling
                0x0000000010018d40                btstack_clr_l2cap_status
                0x0000000010018e04                btstack_sco_setup
                0x0000000010018e52                btstack_sco_kill
                0x0000000010018eba                btstack_msg_is_busy
                0x0000000010018ece                btstack_msg_set_busy
                0x0000000010018ee4                btstack_audio_is_busy
                0x0000000010018ef8                btstack_audio_set_busy
                0x0000000010018f06                audio_bypass_get_cnt
                0x0000000010018f16                btstack_set_lmp_test
                0x0000000010018f2e                btstack_set_clk_offset
                0x0000000010018f46                tws_remote_is_busy
                0x0000000010018f4a                btstack_tws_is_nego_ring
                0x0000000010018f4e                btstack_tws_is_connected_for_handle
                0x0000000010018f52                btstack_tws_user_key
                0x0000000010018f54                btstack_sync_info
                0x0000000010018f56                btstack_tws_set_ring
                0x0000000010018f58                btstack_tws_remote_switch_role
                0x0000000010018f5a                btstack_get_connect_delay
 .text.stack.api
                0x0000000010018f98      0x5c8 ..\..\..\Libraries\libs\libbtstack_master.a(btstack_api.o)
                0x0000000010018f98                btstack_tws_disconnect
                0x0000000010018fb8                btstack_nor_disconnect
                0x0000000010018fba                btstack_dma_stat_change
                0x0000000010018fbc                btstack_off
                0x0000000010018fea                btstack_start_work
                0x0000000010019002                btstack_set_scan
                0x000000001001902a                btstack_set_scan_param
                0x0000000010019040                btstack_hid_connect
                0x0000000010019070                btstack_spp_disconnect
                0x00000000100190ac                btstack_hid_disconnect
                0x00000000100190e8                btstack_fot_resp
                0x00000000100190ea                bt_init
                0x0000000010019102                btstack_tws_set_scan
                0x0000000010019104                btstack_connect_for_bd_addr_do
                0x000000001001919a                btstack_tws_disconnect_do
                0x000000001001919c                btstack_connect_for_bd_addr
                0x00000000100191bc                btstack_connect
                0x0000000010019214                btstack_disconnect_do
                0x000000001001928e                btstack_disconnect
                0x00000000100192b6                bt_hid_is_ready_to_discon
                0x00000000100192f6                btstack_set_l2cap_status
                0x000000001001945a                bt_get_call_indicate
                0x00000000100194d6                bt_is_playing
                0x00000000100194f4                bt_is_ios_device
                0x00000000100194f8                bt_is_support_vol_ctrl
                0x00000000100194fc                bt_is_connected
                0x0000000010019514                dma_get_change_key
                0x0000000010019518                dma_get_change_value
                0x000000001001951c                btstack_message
 .text.stack.sleep
                0x0000000010019560       0x32 ..\..\..\Libraries\libs\libbtstack_master.a(btstack_api.o)
                0x0000000010019560                btstack_enter_sleep
                0x0000000010019578                btstack_exit_sleep
 .text.stack.setup
                0x0000000010019592       0xc4 ..\..\..\Libraries\libs\libbtstack_master.a(btstack_api.o)
                0x0000000010019592                btstack_setup
 *fill*         0x0000000010019656      0x1aa 
 .text.stack.status
                0x0000000010019800      0x1ec ..\..\..\Libraries\libs\libbtstack_master.a(btstack_api.o)
                0x0000000010019800                bt_get_status_do
 .text          0x00000000100199ec      0x158 ..\..\..\Libraries\libs\libbtstack_master.a(bt_api.o)
                0x0000000010019a0c                bt_wait_disconnect
                0x0000000010019a50                bt_sync_info
                0x0000000010019a5e                bt_start_work
                0x0000000010019a6c                bt_updata_local_name
                0x0000000010019a76                bt_nor_connect
                0x0000000010019a78                bt_nor_disconnect
                0x0000000010019a7a                bt_tws_get_scan
                0x0000000010019a7e                bt_tws_set_scan
                0x0000000010019a80                bt_tws_get_link_info
                0x0000000010019a84                bt_tws_delete_link_info
                0x0000000010019a86                bt_tws_user_key
                0x0000000010019a8a                bt_tws_switch
                0x0000000010019a8c                bt_sync_init
                0x0000000010019a8e                bt_tws_get_first_role
                0x0000000010019a92                bt_tws_is_en
                0x0000000010019a96                bt_nor_delete_link_info
                0x0000000010019a9c                bt_nor_get_link_info_addr
                0x0000000010019acc                bt_nor_get_link_info
                0x0000000010019ad0                bt_get_link_btname
                0x0000000010019b28                bt_is_low_latency
                0x0000000010019b36                bt_connect_address
                0x0000000010019b40                bt_map_start
                0x0000000010019b42                bt_map_abort
 .text.stack.api
                0x0000000010019b44      0x144 ..\..\..\Libraries\libs\libbtstack_master.a(bt_api.o)
                0x0000000010019b44                bt_off
                0x0000000010019b76                bt_setup
                0x0000000010019ba8                bt_connect
                0x0000000010019bd6                bt_disconnect
                0x0000000010019c08                bt_set_scan
                0x0000000010019c12                bt_audio_bypass
                0x0000000010019c3a                bt_audio_enable
                0x0000000010019c62                bt_get_stack_local_name
                0x0000000010019c78                bt_set_stack_local_name
 .text          0x0000000010019c88       0x5a ..\..\..\Libraries\libs\libbtstack_master.a(ble_api.o)
                0x0000000010019c88                ble_disconnect
                0x0000000010019c92                ble_set_adv_data
                0x0000000010019c96                ble_set_scan_rsp_data
                0x0000000010019c9a                ble_enable_adv
                0x0000000010019c9c                ble_disable_adv
                0x0000000010019c9e                ble_set_adv_params
                0x0000000010019ca2                ble_set_scan_param
                0x0000000010019cc6                ble_scan_en
                0x0000000010019cce                ble_scan_dis
                0x0000000010019cd6                ble_adv0_set_ctrl
                0x0000000010019cde                ble_init_callback_register
 .text.ble.api.conn
                0x0000000010019ce2       0x4a ..\..\..\Libraries\libs\libbtstack_master.a(ble_api.o)
                0x0000000010019ce2                ble_connect_by_addr
 .text          0x0000000010019d2c       0x44 ..\..\..\Libraries\libs\libbtstack_master.a(bb_sche.o)
                0x0000000010019d2c                bb_sche_frag_ble_dur_set
                0x0000000010019d3e                bb_sche_init
 .text          0x0000000010019d70       0x68 ..\..\..\Libraries\libs\libbtstack_master.a(bb_dbg.o)
                0x0000000010019d70                my_spi_init
                0x0000000010019dd6                bb_dbg_init
 .text          0x0000000010019dd8       0xf6 ..\..\..\Libraries\libs\libbtstack_master.a(bb_clk.o)
                0x0000000010019dd8                bb_clk_init
                0x0000000010019ecc                bb_clk_off
 .text.bb.aes   0x0000000010019ece      0x2a6 ..\..\..\Libraries\libs\libbtstack_master.a(aes.o)
                0x0000000010019ece                aes_init
                0x0000000010019f18                aes_alloc
                0x0000000010019f3a                aes_start
                0x0000000010019f78                aes_encrypt
                0x0000000010019fc4                aes_rand
                0x000000001001a000                aes_result_handler
                0x000000001001a068                aes_xor_128
                0x000000001001a08a                aes_shift_left_128
                0x000000001001a0b4                ble_ecpy
 .text          0x000000001001a174      0x102 ..\..\..\Libraries\libs\libbtstack_master.a(vs_proc.o)
                0x000000001001a266                bt_fcc_test_ctrl
 .text          0x000000001001a276       0xd4 ..\..\..\Libraries\libs\libbtstack_master.a(vs_fcc.o)
                0x000000001001a2c8                vs_con_start
                0x000000001001a2f4                vs_con_end
                0x000000001001a310                vs_fcc_3m_packet_filter
 .text.bb.vs.fcc
                0x000000001001a34a      0x1b8 ..\..\..\Libraries\libs\libbtstack_master.a(vs_fcc.o)
                0x000000001001a34e                vs_fcc_test_cmd_do
 .text          0x000000001001a502       0x9e ..\..\..\Libraries\libs\libbtstack_master.a(vs.o)
                0x000000001001a502                vs_init
                0x000000001001a540                vs_reset_complete_evt
 .text          0x000000001001a5a0      0xb48 ..\..\..\Libraries\libs\libbtstack_master.a(rf_smart.o)
                0x000000001001a77a                rfphy_pll_afc
                0x000000001001a7d6                rfphy_pll_idle
                0x000000001001a7ec                rfphy_rx_dcoc
                0x000000001001a800                rfphy_rx_rccal
                0x000000001001a88a                rfphy_t2r
                0x000000001001a91e                rfphy_tx_dcoc
                0x000000001001a97a                rfphy_rx
                0x000000001001aa24                rfphy_tx
                0x000000001001aaba                rfphy_tx_tone
                0x000000001001aafe                rfphy_sw_ctrl
                0x000000001001ab2c                rfphy_test
                0x000000001001ab2e                rfphy_txrx_init
                0x000000001001ab76                rfphy_init
 .text.bb.rf    0x000000001001b0e8       0x48 ..\..\..\Libraries\libs\libbtstack_master.a(rf_smart.o)
                0x000000001001b0e8                rfphy_tx_pwr
 .text          0x000000001001b130      0x3f6 ..\..\..\Libraries\libs\libbtstack_master.a(rf.o)
                0x000000001001b130                rf_txpwr_dec
                0x000000001001b16c                rf_txpwr_inc
                0x000000001001b1a8                rf_txpwr_max
                0x000000001001b1ce                rf_txpwr_epc_inc
                0x000000001001b20e                rf_txpwr_epc_dec
                0x000000001001b250                rf_off
                0x000000001001b260                rf_reset
                0x000000001001b262                rf_init
 *fill*         0x000000001001b526       0x5a 
 .text          0x000000001001b580       0x82 ..\..\..\Libraries\libs\libbtstack_master.a(bt_hook.o)
                0x000000001001b580                bt_scan_update_param
                0x000000001001b5d8                bt_inq_scan_hook
 .text          0x000000001001b602       0x1c ..\..\..\Libraries\libs\libbtstack_master.a(ble_hook.o)
                0x000000001001b602                ble_hal_init_hook
 *fill*         0x000000001001b61e      0x1e2 
 .text          0x000000001001b800      0xdcc ..\..\..\Libraries\libs\libbtstack_master.a(hct_tl.o)
                0x000000001001bc00                hct_flush_acl_rx_pend
                0x000000001001be00                hci_tx_done_do
                0x000000001001bef4                hci_tx_done
                0x000000001001c000                hci_tl_send
                0x000000001001c154                hci_tl_init
                0x000000001001c192                hci_cmd_get_max_param_size
                0x000000001001c1aa                hci_cmd_received
                0x000000001001c3fe                hci_acl_tx_data_alloc
                0x000000001001c4f4                hci_acl_tx_data_received
 .text          0x000000001001c5cc      0x6da ..\..\..\Libraries\libs\libbtstack_master.a(hct_msg.o)
                0x000000001001cb82                hci_check_desc_tabs_order
                0x000000001001cb84                hci_look_for_cmd_desc
                0x000000001001cc06                hci_look_for_evt_desc
                0x000000001001cc4a                hci_look_for_dbg_evt_desc
                0x000000001001cc64                hci_look_for_le_evt_desc
 .text          0x000000001001cca6       0xb8 ..\..\..\Libraries\libs\libbtstack_master.a(hct_fc.o)
                0x000000001001cca6                hci_fc_init
                0x000000001001ccb6                hci_fc_acl_buf_size_set
                0x000000001001cccc                hci_fc_acl_en
                0x000000001001cd12                hci_fc_host_nb_acl_pkts_complete
                0x000000001001cd34                hci_fc_check_host_available_nb_acl_packets
 .text          0x000000001001cd5e      0x710 ..\..\..\Libraries\libs\libbtstack_master.a(hct.o)
                0x000000001001cdd0                hci_send_2_host
                0x000000001001d18e                hci_ble_conhdl_register
                0x000000001001d1a0                hci_ble_conhdl_unregister
                0x000000001001d1b0                hci_bt_acl_bdaddr_register
                0x000000001001d1da                hci_bt_acl_conhdl_register
                0x000000001001d1f2                hci_bt_acl_bdaddr_unregister
                0x000000001001d208                hci_evt_mask_set
                0x000000001001d246                hct_init
                0x000000001001d290                hci_evt_filter_add
                0x000000001001d458                hci_voice_settings_get
                0x000000001001d462                hci_voice_settings_set
 .text          0x000000001001d46e      0x81a ..\..\..\Libraries\libs\libbtstack_master.a(lm.o)
                0x000000001001d4c2                lm_init
                0x000000001001d654                lm_set_scan_int
                0x000000001001d668                lm_new_link_alloc
                0x000000001001d682                lm_stop_link_alloc
                0x000000001001d6a8                lm_lt_addr_alloc
                0x000000001001d6e0                lm_lt_addr_free
                0x000000001001d70c                lm_get_nb_acl
                0x000000001001d770                lm_role_switch_start
                0x000000001001d7ba                lm_role_switch_finished
                0x000000001001d842                lm_get_features
                0x000000001001d8c4                lm_pscan_start
                0x000000001001d914                lm_pscan_restart
                0x000000001001d924                lm_acl_disc
                0x000000001001d958                lm_get_auth_en
                0x000000001001d968                lm_get_sp_en
                0x000000001001d978                lm_get_sec_con_host_supp
                0x000000001001d986                lm_get_pin_type
                0x000000001001d990                lm_get_con_accept_timeout
                0x000000001001d99a                lm_set_loc_name
                0x000000001001da04                lm_get_loc_name
                0x000000001001da0e                lm_get_loc_name_seg
                0x000000001001da68                lm_get_loopback_mode
                0x000000001001da72                lm_get_pub_key_192
                0x000000001001da94                lm_get_priv_key_192
                0x000000001001dab4                lm_get_oob_local_commit
                0x000000001001dade                lm_get_sp_debug_mode
                0x000000001001dae8                lm_debug_key_compare_192
                0x000000001001db1a                lm_get_dut_mode_en
                0x000000001001db24                lm_afh_get_ch_ass_en
                0x000000001001db2e                lm_afh_get_host_ch_class
                0x000000001001db38                lm_afh_set_peer_ch_class
                0x000000001001db52                lm_afh_get_master_ch_map
                0x000000001001db5c                lm_afh_init_timer
                0x000000001001db88                lm_is_acl_con
                0x000000001001dba4                lm_is_acl_con_role
                0x000000001001dbce                lm_page_scan_rep_mode_get
                0x000000001001dbd8                lm_sco_move_en
                0x000000001001dbe2                lm_extract_max_enc_key_size
                0x000000001001dbfc                lm_create_master_key
                0x000000001001dc48                lm_create_master_key_rand
                0x000000001001dc54                lm_get_master_key
                0x000000001001dc62                lm_get_master_key_rand
                0x000000001001dc70                lm_get_master_enc_rand
                0x000000001001dc7e                lm_get_master_enc_key_size
 .text          0x000000001001dc88      0x382 ..\..\..\Libraries\libs\libbtstack_master.a(bt_hal.o)
                0x000000001001dc88                bt_hal_init
                0x000000001001de0a                bt_hal_reset
                0x000000001001df8e                bt_bd_addr_get
                0x000000001001df9c                bt_bd_addr_set
                0x000000001001dfc8                bt_class_of_dev_get
                0x000000001001dfd6                bt_class_of_dev_set
                0x000000001001dfe6                bt_tim_acc_get
                0x000000001001e000                bt_afh_ch_assess_get
 .text          0x000000001001e00a      0x14e ..\..\..\Libraries\libs\libbtstack_master.a(bt21.o)
                0x000000001001e00a                bt_buf_init
                0x000000001001e0f4                bt21_init
                0x000000001001e12e                bt21_reset
 .text          0x000000001001e158       0x62 ..\..\..\Libraries\libs\libbtstack_master.a(bc.o)
                0x000000001001e158                bc_init
                0x000000001001e17a                bc_reset
                0x000000001001e1aa                bc_get_nb_broadcast
                0x000000001001e1b2                bc_set_nb_broadcast
 *fill*         0x000000001001e1ba        0x6 
 .text          0x000000001001e1c0      0x430 ..\..\..\Libraries\libs\libbtstack_master.a(ble_hal.o)
                0x000000001001e1e6                ble_ral_search
                0x000000001001e238                ble_hal_init
                0x000000001001e4a4                ble_ch_assess_data_get
                0x000000001001e4ae                ble_rpa_renew
                0x000000001001e52c                ble_aa_gen
 *fill*         0x000000001001e5f0       0x10 
 .text          0x000000001001e600      0xb76 ..\..\..\Libraries\libs\libbtstack_master.a(ble_adv.o)
                0x000000001001e600                ble_get_adv_var
                0x000000001001e60a                ble_adv_init
                0x000000001001e700                ble_adv_stop
                0x000000001001e780                ble_adv_adv_data_update
                0x000000001001e800                ble_adv_scan_rsp_data_update
                0x000000001001e900                ble_adv_start_do
                0x000000001001e9ac                ble_adv_start
                0x000000001001f080                ble_adv_rand_addr_update
                0x000000001001f100                ble_adv_restart
 .text          0x000000001001f176       0x48 ..\..\..\Libraries\libs\libbtstack_master.a(ble.o)
                0x000000001001f176                ble_init
 .text.ble.var.init
                0x000000001001f1be       0x38 ..\..\..\Libraries\libs\libbtstack_master.a(ble.o)
                0x000000001001f1be                ble_var_init
 .text          0x000000001001f1f6      0x30c ..\..\..\Libraries\libs\libbtstack_master.a(l2cap_test.o)
                0x000000001001f2f0                l2cap_end_of_test
                0x000000001001f306                l2cap_test_support_ext_feature
                0x000000001001f322                l2cap_test_cmd
                0x000000001001f42a                l2cap_test_rsp
                0x000000001001f42c                l2cap_vd_acl_init
                0x000000001001f44e                l2cap_vd_enter_updateota
                0x000000001001f45c                l2cap_vd_exit_updateota
                0x000000001001f468                l2cap_vd_acl_tx_request
 .text          0x000000001001f502      0x34e ..\..\..\Libraries\libs\libbtstack_master.a(l2cap.o)
                0x000000001001f552                l2cap_register_packet_handler
                0x000000001001f55a                l2cap_send_test_cmd
                0x000000001001f5ac                l2cap_send_test_key
                0x000000001001f5da                gap_request_connection_parameter_update
                0x000000001001f612                l2cap_get_outgoing_buffer
                0x000000001001f620                l2cap_reserve_packet_buffer
                0x000000001001f624                l2cap_release_packet_buffer
                0x000000001001f628                l2cap_send_prepared_connectionless
                0x000000001001f67a                l2cap_send_connectionless
                0x000000001001f6b0                l2cap_send_echo_request
                0x000000001001f6bc                l2cap_max_mtu
                0x000000001001f6c2                l2cap_max_le_mtu
                0x000000001001f6c8                l2cap_create_channel
                0x000000001001f7a8                l2cap_disconnect
                0x000000001001f7c4                provide_l2cap_channel
                0x000000001001f826                l2cap_unregister_service
 *fill*         0x000000001001f850        0x0 
 .text.stack.handler.l2cap
                0x000000001001f850      0x94c ..\..\..\Libraries\libs\libbtstack_master.a(l2cap.o)
                0x000000001001faec                l2cap_emit_channel_closed
                0x000000001002013a                l2cap_can_send_packet_now
                0x0000000010020158                l2cap_can_send_prepared_packet_now
                0x0000000010020176                l2cap_can_send_fixed_channel_packet_now
                0x000000001002017a                l2cap_get_remote_mtu_for_local_cid
                0x0000000010020194                l2cap_stop_rtx
 .text.stack.l2cap
                0x000000001002019c      0x860 ..\..\..\Libraries\libs\libbtstack_master.a(l2cap.o)
                0x00000000100201b4                l2cap_clear_pending_tx
                0x00000000100208c4                l2cap_send_prepared
                0x000000001002092c                l2cap_send
                0x000000001002097e                l2cap_accept_connection
                0x0000000010020998                l2cap_decline_connection
                0x00000000100209b8                l2cap_register_service
 .text.stack.setup
                0x00000000100209fc       0x72 ..\..\..\Libraries\libs\libbtstack_master.a(l2cap.o)
                0x00000000100209fc                l2cap_init
                0x0000000010020a4c                l2cap_register_fixed_channel
 .text.stack.setup
                0x0000000010020a6e        0x2 ..\..\..\Libraries\libs\libbtstack_master.a(hci_dump.o)
                0x0000000010020a6e                hci_dump_open
 .text.stack.hci_send
                0x0000000010020a70      0x24e ..\..\..\Libraries\libs\libbtstack_master.a(hci_cmd.o)
                0x0000000010020a70                hci_cmd_create_from_template
 .text          0x0000000010020cbe      0x5c8 ..\..\..\Libraries\libs\libbtstack_master.a(hci.o)
                0x0000000010020e6a                hci_alloc_num_packets_sent
                0x0000000010020eaa                hci_shutdown_connection
                0x0000000010020ee6                le_handle_advertisement_report
                0x0000000010020f50                hci_free_connect_waiting
                0x0000000010020fae                gap_local_bd_addr
                0x0000000010020fbe                hci_emit_start_action
                0x0000000010020ff4                hci_emit_service_establish
                0x0000000010021022                gap_set_connection_outgoing_addr
                0x0000000010021040                gap_get_connection_type
                0x0000000010021076                hci_set_sco_voice_setting_for_addr
                0x000000001002108e                hci_get_sco_voice_setting_for_addr
                0x00000000100210d4                gap_start_scan
                0x00000000100210f6                gap_stop_scan
                0x0000000010021114                gap_set_scan_parameters
                0x0000000010021136                gap_create_connect
                0x000000001002117c                gap_update_connection_parameters
                0x00000000100211b4                gap_inquiry
                0x00000000100211ca                gap_inquiry_cancel
                0x00000000100211e0                gap_disconnect
                0x0000000010021232                hci_set_sco_voice_setting
                0x000000001002123e                hci_setup_sync
                0x0000000010021282                hci_rx_flush
 .text.stack.hci
                0x0000000010021286      0x91e ..\..\..\Libraries\libs\libbtstack_master.a(hci.o)
                0x0000000010021376                hci_authentication_active_for_handle
                0x0000000010021396                gap_drop_link_key_for_bd_addr
                0x00000000100213b8                gap_store_link_key_for_bd_addr
                0x00000000100213dc                gap_get_link_feature_for_bd_addr
                0x00000000100213fa                gap_store_link_feature_for_bd_addr
                0x0000000010021418                gap_get_link_addr_by_order
                0x000000001002141c                hci_number_free_acl_slots_for_handle
                0x0000000010021436                hci_can_send_acl_classic_packet_now
                0x000000001002144c                hci_can_send_acl_le_packet_now
                0x000000001002145e                hci_can_send_prepared_acl_packet_now
                0x000000001002147e                hci_can_send_acl_packet_now
                0x0000000010021490                hci_is_packet_buffer_reserved
                0x000000001002149c                hci_reserve_packet_buffer
                0x00000000100214b4                hci_release_packet_buffer
                0x0000000010021584                hci_send_acl_packet_buffer
                0x00000000100215d4                hci_usable_acl_packet_types
                0x00000000100215e0                hci_get_outgoing_packet_buffer
                0x00000000100215ea                hci_max_acl_data_packet_length
                0x00000000100215f6                hci_non_flushable_packet_boundary_flag_supported
                0x0000000010021606                hci_disconnect_security_block
                0x0000000010021620                gap_ssp_set_enable
                0x000000001002162c                update_extend_inquiry_response
                0x0000000010021654                hci_run_le_connection
                0x00000000100216d6                hci_remote_esco_supported
                0x00000000100216f0                gap_ssp_supported_on_both_sides
                0x0000000010021722                hci_local_had_auth_request
                0x000000001002174c                gap_security_level_for_link_key_type
                0x000000001002177e                hci_run_pend_connection
                0x0000000010021a16                gap_mitm_protection_required_for_security_level
                0x0000000010021a20                gap_security_level
                0x0000000010021a38                hci_run_w2_connection
                0x0000000010021b44                gap_w_scan_control
                0x0000000010021b5e                gap_request_security_level
 *fill*         0x0000000010021ba4        0x0 
 .text.stack.hci_init
                0x0000000010021ba4      0x3c6 ..\..\..\Libraries\libs\libbtstack_master.a(hci.o)
                0x0000000010021bdc                gap_set_local_name
                0x0000000010021f38                hci_power_control
 .text.stack.handler.acl
                0x0000000010021f6a       0x16 ..\..\..\Libraries\libs\libbtstack_master.a(hci.o)
 .text.stack.setup
                0x0000000010021f80      0x17c ..\..\..\Libraries\libs\libbtstack_master.a(hci.o)
                0x0000000010021fe6                hci_add_event_handler
                0x0000000010021ff4                hci_register_acl_packet_handler
                0x0000000010021ffe                hci_init
                0x000000001002209a                hci_set_chipset
                0x00000000100220ae                gap_set_class_of_device
                0x00000000100220b8                hci_set_bd_addr
                0x00000000100220d8                gap_ssp_set_io_capability
                0x00000000100220e4                gap_ssp_set_authentication_requirement
                0x00000000100220f0                gap_ssp_set_auto_accept
 .text.stack.hci_emit
                0x00000000100220fc      0x148 ..\..\..\Libraries\libs\libbtstack_master.a(hci.o)
                0x00000000100221aa                hci_emit_state
                0x00000000100221d8                hci_emit_scan_ctrl
                0x00000000100221fe                hci_emit_inquiry_ctrl
                0x0000000010022224                hci_emit_test_active
 .text.stack.hci.conn
                0x0000000010022244      0x1e2 ..\..\..\Libraries\libs\libbtstack_master.a(hci.o)
                0x0000000010022244                create_connection_for_bd_addr_and_type
                0x000000001002234e                gap_get_connection_parameter_range
                0x000000001002235e                gap_set_connection_parameter_range
                0x0000000010022370                hci_get_connections
                0x000000001002237a                hci_connection_for_bd_addr_and_type
                0x00000000100223b8                hci_connection_get_other_for_bd_addr_and_type
                0x00000000100223f6                hci_connection_for_index
 .text.ble.hci  0x0000000010022426      0x122 ..\..\..\Libraries\libs\libbtstack_master.a(hci.o)
                0x0000000010022426                ble_event_cmd_complete
                0x000000001002249c                ble_event_meta
 .text.stack.hci_send
                0x0000000010022548      0x2a4 ..\..\..\Libraries\libs\libbtstack_master.a(hci.o)
                0x0000000010022548                hci_send_cmd_packet
                0x00000000100226f0                hci_send_cmd
                0x0000000010022746                hci_send_create_connection_cmd
 *fill*         0x00000000100227ec       0x14 
 .text.stack.hci.run
                0x0000000010022800      0x1c8 ..\..\..\Libraries\libs\libbtstack_master.a(hci.o)
 .text.stack.hci_rx
                0x00000000100229c8      0x106 ..\..\..\Libraries\libs\libbtstack_master.a(hci.o)
                0x00000000100229c8                acl_handler
 *fill*         0x0000000010022ace        0x2 
 .text.stack.handler.event
                0x0000000010022ad0      0xd24 ..\..\..\Libraries\libs\libbtstack_master.a(hci.o)
 .text          0x00000000100237f4      0x1d4 ..\..\..\Libraries\libs\libbtstack_master.a(hid_usage.o)
                0x00000000100237f4                hid_report_init
                0x0000000010023806                hid_report_set
                0x0000000010023826                hid_send_report_callback
                0x0000000010023874                btstack_hid_send
                0x000000001002389a                btstack_hid_key
                0x00000000100238f4                btstack_hid_consumer
                0x0000000010023928                btstack_hid_touch_screen
                0x00000000100239b6                bt_hid_is_send_complete
 .text          0x00000000100239c8      0x55e ..\..\..\Libraries\libs\libbtstack_master.a(hid_device.o)
                0x0000000010023de6                bt_hid_is_connected
                0x0000000010023e0e                hid_device_init
                0x0000000010023e4e                hid_device_request_can_send_now_event
                0x0000000010023e52                hid_device_send_interrupt_message
                0x0000000010023e56                hid_device_send_contro_message
                0x0000000010023e5a                hid_establish_service_level_connection
                0x0000000010023ed0                hid_release_service_level_connection
                0x0000000010023ef6                bt_hid_index_set
                0x0000000010023ef8                hid_get_interrupt_cid
 *fill*         0x0000000010023f26        0x2 
 .text          0x0000000010023f28      0xbd8 ..\..\..\Libraries\libs\libbtstack_master.a(hfp_hf.o)
                0x0000000010024950                hfp_hf_packet_handler
                0x00000000100249c2                hfp_hf_init_codecs
                0x00000000100249ec                hfp_hf_init_supported_features
                0x00000000100249f4                hfp_hf_init_hf_indicators
                0x00000000100249f6                hfp_hf_establish_service_level_connection
                0x0000000010024a00                hfp_hf_release_service_level_connection
                0x0000000010024a1a                hfp_hf_get_siri_status
                0x0000000010024a4e                hfp_hf_set_call_switch_flag
                0x0000000010024a62                hfp_hf_call_switch_for_index
                0x0000000010024ac0                hfp_hf_call_for_index
                0x0000000010024afe                hfp_hf_init
 .text.stack.api
                0x0000000010024b00      0x316 ..\..\..\Libraries\libs\libbtstack_master.a(hfp_hf.o)
                0x0000000010024b00                hfp_hf_switch_siri
                0x0000000010024b38                hfp_hf_is_calling
                0x0000000010024b54                hfp_hf_answer_incoming_call
                0x0000000010024bca                hfp_hf_terminate_call
                0x0000000010024c1e                hfp_hf_reject_incoming_call
                0x0000000010024c20                hfp_hf_swap_calls
                0x0000000010024c50                hfp_hf_dial_number
                0x0000000010024c8e                hfp_hf_at_cmd
                0x0000000010024cc4                hfp_hf_custom_at_cmd
                0x0000000010024cf2                hfp_hf_redial_last_number_do
                0x0000000010024d32                hfp_hf_redial_last_number
                0x0000000010024d46                hfp_hf_set_speaker_gain
                0x0000000010024d80                hfp_hf_set_microphone_gain
                0x0000000010024dba                hfp_hf_report_bat_state
                0x0000000010024df8                hfp_hf_start_codec
 .text.stack.hfp.api1
                0x0000000010024e16       0x28 ..\..\..\Libraries\libs\libbtstack_master.a(hfp_hf.o)
                0x0000000010024e16                hfp_is_connect
 *fill*         0x0000000010024e3e        0x2 
 .text          0x0000000010024e40      0xbcc ..\..\..\Libraries\libs\libbtstack_master.a(hfp.o)
                0x0000000010024e40                hfp_init
                0x0000000010024e52                hfp_var_init
                0x0000000010024e54                send_str_over_rfcomm
                0x0000000010024e7c                join
                0x0000000010024ef0                join_bitmap
                0x0000000010024f6e                hfp_emit_call_indicate
                0x0000000010024f70                hfp_get_connections
                0x0000000010024f7a                hfp_get_connection_for_index
                0x0000000010024f7e                get_hfp_connection_context_for_rfcomm_cid
                0x0000000010024f82                get_hfp_connection_context_for_bd_addr
                0x0000000010024f86                get_hfp_connection_context_for_sco_handle
                0x0000000010024f8a                hfp_reset_context_flags
                0x0000000010024fb2                hfp_reset_voice_recognition_flags
                0x0000000010024fcc                provide_hfp_connection_context_for_bd_addr
                0x0000000010024fe4                hfp_handle_hci_event
                0x0000000010025098                hfp_parse
                0x00000000100258fc                hfp_establish_service_level_connection
                0x000000001002593e                hfp_rfcomm_service_supported
                0x0000000010025942                hfp_release_audio_connection
                0x000000001002595a                hfp_release_service_level_connection
                0x00000000100259b4                hfp_setup_synchronous_connection
                0x0000000010025a0a                hfp_set_packet_handler_for_rfcomm_connections
 .text          0x0000000010025a0c        0x8 ..\..\..\Libraries\libs\libbtstack_master.a(a2dp.o)
                0x0000000010025a0c                a2dp_is_playing
                0x0000000010025a10                a2dp_is_playing_fast
 .text.stack.memory
                0x0000000010025a14       0x46 ..\..\..\Libraries\libs\libbtstack_master.a(btstack_memory_pool.o)
                0x0000000010025a14                btstack_memory_pool_get
                0x0000000010025a20                btstack_memory_pool_free
                0x0000000010025a34                btstack_memory_pool_create
 .text          0x0000000010025a5a       0x92 ..\..\..\Libraries\libs\libbtstack_master.a(btstack_adv0.o)
                0x0000000010025a5a                btstack_adv0_ctrl
                0x0000000010025abe                ble_adv0_set_intv
                0x0000000010025ada                ble_adv0_get_adv_en
                0x0000000010025aea                ble_adv0_idx_update
 .text          0x0000000010025aec       0x7c ..\..\..\Libraries\libs\libbtstack_master.a(hci_transport_hcic.o)
                0x0000000010025aec                hcic_recv_packet
                0x0000000010025b08                hcic_send_acl_segment
                0x0000000010025b3c                hcic_rx_flush
                0x0000000010025b5a                hci_init_var
 .text.stack.hcic
                0x0000000010025b68      0x128 ..\..\..\Libraries\libs\libbtstack_master.a(hci_transport_hcic.o)
                0x0000000010025b6a                hcic_register_packet_handler
                0x0000000010025bd2                hcic_close
                0x0000000010025be8                hcic_open
                0x0000000010025c2a                hcic_send_packet
 .text          0x0000000010025c90       0x24 ..\..\..\Libraries\libs\libbtstack_master.a(btstack_chipset_inner.o)
                0x0000000010025caa                btstack_chipset_inner_instance
 .text          0x0000000010025cb4       0x1e ..\..\..\Libraries\libs\libbtstack_master.a(lm_hook.o)
                0x0000000010025cb4                lm_init_hook
                0x0000000010025cce                lm_set_iac_en
                0x0000000010025cd0                lm_page_scan_end_hook
 .text          0x0000000010025cd2     0x1d9a ..\..\..\Libraries\libs\libbtstack_master.a(lm_sp.o)
                0x00000000100263ea                lm_n_is_zero
                0x0000000010026814                lm_sp_sha256_calculate
                0x000000001002689c                lm_sp_n_one
                0x0000000010026a58                lm_sp_n192_convert_wnaf
                0x0000000010026afc                lm_sp_p192_point_to_inf
                0x0000000010026b10                lm_sp_p192_point_jacobian_to_affine
                0x0000000010026b86                lm_sp_p192_points_jacobian_to_affine
                0x0000000010026c96                lm_sp_p192_dbl
                0x0000000010026e0e                lm_sp_p192_add
                0x00000000100270a6                lm_sp_pre_compute_points
                0x00000000100270ee                lm_sp_p192_invert
                0x0000000010027134                lm_f1
                0x00000000100272a6                lm_f2
                0x0000000010027424                lm_oob_f1
                0x0000000010027596                lm_g
                0x0000000010027658                lm_f3
                0x0000000010027802                lm_generate_rand_16bytes
                0x0000000010027860                lm_dhkey_calc_init
                0x0000000010027998                lm_dhkey_compare
 .text          0x0000000010027a6c     0x1cca ..\..\..\Libraries\libs\libbtstack_master.a(lm_proc.o)
                0x00000000100296f2                lm_inq_start
                0x000000001002970c                lm_inq_stop
 .text          0x0000000010029736      0xd3c ..\..\..\Libraries\libs\libbtstack_master.a(lm_key.o)
                0x0000000010029b88                lm_e1
                0x0000000010029be4                lm_e21
                0x0000000010029c20                lm_e22
                0x0000000010029ca0                lm_e3
                0x0000000010029cfe                lm_kc_key
                0x000000001002a44e                lm_xor_key
                0x000000001002a452                lm_get_rand_vec
 *fill*         0x000000001002a472        0x2 
 .text          0x000000001002a474     0x2e60 ..\..\..\Libraries\libs\libbtstack_master.a(lc.o)
                0x000000001002a4e6                lc_util_set_loc_trans_coll
                0x000000001002a502                lc_cmd_stat_send
                0x000000001002a52a                lc_mode_chg_evt_send
                0x000000001002a566                lc_init
                0x000000001002a5ac                lc_reset
                0x000000001002a5fc                lc_afh_set
                0x000000001002a6ca                lc_chg_pkt_type_cmp
                0x000000001002a730                lc_chg_pkt_type_cont
                0x000000001002a79e                lc_afh_start
                0x000000001002a808                lc_con_cmp_evt_send
                0x000000001002a870                lc_max_slot_mgt
                0x000000001002a922                lc_mst_qos_done
                0x000000001002a996                lc_ptt
                0x000000001002aa3c                lc_ptt_cmp
                0x000000001002aaa2                lc_resp_auth
                0x000000001002ab5c                lc_release
                0x000000001002ab7c                lc_restore_to
                0x000000001002abc8                lc_start_lmp_to
                0x000000001002ac32                lc_start
                0x000000001002ae56                lc_comb_key_svr
                0x000000001002af58                lc_locepr_rsw
                0x000000001002afac                lc_locepr_lkref
                0x000000001002b004                lc_enc_key_refresh
                0x000000001002b0e6                lc_initiator_epr
                0x000000001002b130                lc_init_calc_f3
                0x000000001002b1b2                lc_dhkey
                0x000000001002b1f8                lc_init_start_mutual_auth
                0x000000001002b246                lc_mst_send_mst_key
                0x000000001002b336                lc_init_passkey_loop
                0x000000001002b3a4                lc_pairing_cont
                0x000000001002b4d6                lc_legacy_pair
                0x000000001002b53a                lc_passkey_comm
                0x000000001002b5d2                lc_qos_setup
                0x000000001002b64a                lc_rd_rem_name
                0x000000001002b69a                lc_resp_oob_wait_nonce
                0x000000001002b6b8                lc_start_enc
                0x000000001002b7ba                lc_epr_rsw_cmp
                0x000000001002b822                lc_start_enc_key_size
                0x000000001002b88e                lc_start_key_exch
                0x000000001002b8fe                lc_resp_num_comp
                0x000000001002b962                lc_stop_enc
                0x000000001002b9ca                lc_epr_resp
                0x000000001002ba44                lc_rem_enc
                0x000000001002babe                lc_stop_afh_reporting
                0x000000001002baec                lc_local_switch
                0x000000001002bbc6                lc_restore_afh_reporting
                0x000000001002bc1a                lc_skip_hl_oob_req
                0x000000001002bc74                lc_start_oob
                0x000000001002bca0                lc_send_enc_mode
                0x000000001002bd0a                lc_restart_enc
                0x000000001002bd50                lc_restart_enc_cont
                0x000000001002be08                lc_detach
                0x000000001002beb8                lc_chg_pkt_type_retry
                0x000000001002bf9a                lc_rem_name_cont
                0x000000001002c010                lc_semi_key_cmp
                0x000000001002c0da                lc_mst_key
                0x000000001002c1c0                lc_feat
                0x000000001002c218                lc_hl_connect
                0x000000001002c264                lc_version
                0x000000001002c2a0                lc_ext_feat
                0x000000001002c2de                lc_loc_auth
                0x000000001002c38c                lc_packet_type
                0x000000001002c416                lc_conn_seq_done
                0x000000001002c438                lc_rsw_done
                0x000000001002c55e                lc_switch_cmp
                0x000000001002c57a                lc_rem_switch
                0x000000001002c666                lc_send_enc_chg_evt
                0x000000001002c6bc                lc_auth_cmp
                0x000000001002c79a                lc_con_cmp
                0x000000001002c872                lc_end_chk_colli
                0x000000001002c8c6                lc_enc_cmp
                0x000000001002c97c                lc_mutual_auth_end2
                0x000000001002cabc                lc_epr_change_lk
                0x000000001002cb12                lc_epr_cmp
                0x000000001002cb9e                lc_mutual_auth_end
                0x000000001002ccd0                lc_key_exch_end
                0x000000001002cd42                lc_sp_end
                0x000000001002cd98                lc_calc_link_key
                0x000000001002ce34                lc_sp_fail
                0x000000001002ce6c                lc_resp_oob_nonce
                0x000000001002cef2                lc_resp_calc_f3
                0x000000001002cfbe                lc_start_passkey_loop
                0x000000001002d02a                lc_start_passkey
                0x000000001002d0f8                lc_resp_pair
                0x000000001002d1b4                lc_pair
                0x000000001002d26a                lc_check_all_slaves_support_sec_con
                0x000000001002d2a0                lc_get_curr_mode
 .text          0x000000001002d2d4      0x52c ..\..\..\Libraries\libs\libbtstack_master.a(mgr.o)
                0x000000001002d2d4                mgr_cmd_cmp_send
                0x000000001002d2fc                mgr_cmd_stat_send
                0x000000001002d324                mgr_is_dev_connected
                0x000000001002d378                mgr_is_dev_synced
                0x000000001002d3e4                mgr_ral_search
                0x000000001002d42a                mgr_ral_is_empty
                0x000000001002d43c                mgr_ch_map_update
                0x000000001002d5aa                mgr_init
                0x000000001002d6ac                mgr_clk_acc_set
                0x000000001002d6ec                mgr_link_disc
                0x000000001002d724                mgr_master_ch_map_get
                0x000000001002d72e                mgr_le_evt_mask_check
                0x000000001002d74a                mgr_le_get_features
                0x000000001002d76e                mgr_ral_get
                0x000000001002d778                mgr_plan_elt_get
                0x000000001002d78a                mgr_act_get_free
                0x000000001002d7da                mgr_act_set_free
 .text.le.ll_cntl
                0x000000001002d800      0x2f4 ..\..\..\Libraries\libs\libbtstack_master.a(ll.o)
                0x000000001002d868                ll_cleanup
                0x000000001002d8f4                ll_init
                0x000000001002d960                ll_role_get
                0x000000001002d996                ll_proc_reg
                0x000000001002d9e2                ll_proc_id_get
                0x000000001002da02                ll_proc_state_get
                0x000000001002da08                ll_proc_state_set
                0x000000001002da0e                ll_proc_get
                0x000000001002da26                ll_proc_err_ind
                0x000000001002da4e                ll_proc_unreg
                0x000000001002dabe                ll_proc_collision_check
 .text.le.ll_cntl.start
                0x000000001002daf4      0x20e ..\..\..\Libraries\libs\libbtstack_master.a(ll.o)
                0x000000001002daf4                ll_start
 .text.le.ll_cntl.state
                0x000000001002dd02       0x60 ..\..\..\Libraries\libs\libbtstack_master.a(ll.o)
                0x000000001002dd02                ll_cntl_state_set
 .text.le.ll_cntl.stop
                0x000000001002dd62       0x48 ..\..\..\Libraries\libs\libbtstack_master.a(ll.o)
                0x000000001002dd62                ll_stop
 .text.le.ll_cntl.timer
                0x000000001002ddaa       0xd8 ..\..\..\Libraries\libs\libbtstack_master.a(ll.o)
                0x000000001002ddaa                ll_proc_timer_set
                0x000000001002de1a                ll_proc_timer_set_state
 .text          0x000000001002de82       0x20 ..\..\..\Libraries\libs\libbtstack_master.a(ble_test.o)
                0x000000001002de82                ble_test_init
 *fill*         0x000000001002dea2       0x5e 
 .text          0x000000001002df00      0x702 ..\..\..\Libraries\libs\libbtstack_master.a(ble_scan.o)
                0x000000001002df66                ble_get_scan_var
                0x000000001002df70                ble_get_sync_var
                0x000000001002df7a                ble_scan_init
                0x000000001002dff2                ble_scan_start
                0x000000001002e500                ble_scan_stop
                0x000000001002e538                ble_scan_params_update
 .text          0x000000001002e602        0x4 ..\..\..\Libraries\libs\libbtstack_master.a(ble_per_adv.o)
                0x000000001002e602                ble_get_per_adv_var
 *fill*         0x000000001002e606       0x3a 
 .text          0x000000001002e640      0x86e ..\..\..\Libraries\libs\libbtstack_master.a(ble_init.o)
                0x000000001002e640                ble_init_connect_req_pack
                0x000000001002e6ea                ble_init_init
                0x000000001002e758                ble_init_start
                0x000000001002ee40                ble_init_stop
 .text          0x000000001002eeae      0x158 ..\..\..\Libraries\libs\libbtstack_master.a(ble_buf.o)
                0x000000001002eeae                ble_buf_init_do
                0x000000001002efbc                ble_buf_init
 .text.bb.ble.adv0
                0x000000001002f006      0x208 ..\..\..\Libraries\libs\libbtstack_master.a(ble_adv0.o)
                0x000000001002f0bc                ble_adv0_init
                0x000000001002f10e                ble_adv0_end_ind
                0x000000001002f148                ble_adv0_set_en
                0x000000001002f1a0                ble_adv0_update_adv_data
                0x000000001002f204                ble_adv0_set_interval
                0x000000001002f20c                ble_adv0_copy
 .text          0x000000001002f20e       0x2a ..\..\..\Libraries\libs\libbtstack_master.a(extern_hfhs.o)
                0x000000001002f20e                hfp_notice_network_time
                0x000000001002f210                hfp_notice_ring_number
                0x000000001002f216                hfp_get_last_call_number
                0x000000001002f21a                msbc_exit
                0x000000001002f21c                bt_pbap_data_callback
                0x000000001002f21e                hfp_get_mic_gain
                0x000000001002f222                hfp_get_spk_gain
                0x000000001002f226                hfp_get_bat_level
                0x000000001002f22a                hfp_hf_established_hook
                0x000000001002f22e                hfp_hf_send_custom_at_cmd_hook
                0x000000001002f232                hfp_hf_recv_custom_at_cmd_hook
                0x000000001002f236                hfp_hf_release_hook
 .text.func.outgoing
                0x000000001002f238       0x14 ..\..\..\Libraries\libs\libbtstack_master.a(extern_hfhs.o)
                0x000000001002f238                hfp_get_outgoing_number
                0x000000001002f242                hfp_get_at_cmd
 .text.func.btring
                0x000000001002f24c        0x6 ..\..\..\Libraries\libs\libbtstack_master.a(extern_hfhs.o)
                0x000000001002f24c                hfp_is_list_curr_calls
                0x000000001002f250                hfp_hf_emit_curr_calls
 .text          0x000000001002f252       0x4c ..\..\..\Libraries\libs\libbtstack_master.a(extern_ble.o)
                0x000000001002f26c                ble_get_aap_addr
                0x000000001002f27a                ble_adv0_get_adv_data_cb
                0x000000001002f27e                ble_adv0_get_tws_role
                0x000000001002f292                ble_adv0_get_tws_loc_var
                0x000000001002f296                ble_adv0_set_tws_rem_var
                0x000000001002f29c                ble_tx_test
 .text.bb.ble.adv0
                0x000000001002f29e       0x28 ..\..\..\Libraries\libs\libbtstack_master.a(extern_ble.o)
                0x000000001002f29e                ble_adv0_get_addr_cb
 .text.stack.l2cap_sig
                0x000000001002f2c6      0x134 ..\..\..\Libraries\libs\libbtstack_master.a(l2cap_signaling.o)
                0x000000001002f3a6                l2cap_next_sig_id
                0x000000001002f3c2                l2cap_next_local_cid
                0x000000001002f3e6                l2cap_create_signaling_classic
                0x000000001002f3f0                l2cap_create_signaling_le
 .text          0x000000001002f3fa       0xdc ..\..\..\Libraries\libs\libbtstack_master.a(lc_hook.o)
                0x000000001002f3fa                lc_lmp_ver_req_hook
                0x000000001002f420                lc_lmp_ver_res_hook
                0x000000001002f422                lc_loc_sniff_req_hook
                0x000000001002f45e                lmp_sniff_req_hook
                0x000000001002f480                lc_auto_sniff_step_set
 *fill*         0x000000001002f4d6        0x2 
 .text          0x000000001002f4d8     0x17ca ..\..\..\Libraries\libs\libbtstack_master.a(lm_sco.o)
                0x000000001002ff5c                lm_get_sync_param
                0x00000000100308d6                lm_init_sync
                0x00000000100308f8                lm_reset_sync
                0x0000000010030928                lm_check_active_sync
                0x0000000010030936                lm_add_sync
                0x0000000010030ac0                lm_check_sync_hl_rsp
                0x0000000010030b94                lm_get_synchdl
                0x0000000010030bb2                lm_look_for_sync
                0x0000000010030bfc                lm_get_nb_sync_link
                0x0000000010030c06                lm_get_min_sync_intv
                0x0000000010030c2a                lm_remove_sync
                0x0000000010030c98                lm_sco_nego_end
 .text          0x0000000010030ca2      0x498 ..\..\..\Libraries\libs\libbtstack_master.a(lc_util.o)
                0x0000000010030ca2                lc_get_max_pkt_size
                0x0000000010030d0e                lc_compute_pkt_types
                0x0000000010030d34                lc_update_acl_pkt_types
                0x0000000010030d86                lc_update_acl_edr_pkt_types
                0x0000000010030dfe                lc_reduce_acl_pkt_types
                0x0000000010030e34                lc_pkt_types_to_max_slot
                0x0000000010030e7a                lc_get_qos_param
                0x0000000010030fa8                lc_gen_cof_for_addr
                0x0000000010030fce                lc_check_edr_feature_for_pkt_types
                0x0000000010030fde                lc_check_feature
                0x000000001003100c                lc_pref_rate_to_pkt_types
                0x000000001003109c                lc_max_slot_to_pkt_types
                0x00000000100310bc                lc_get_common_pkt_types
 .text          0x000000001003113a      0x9b2 ..\..\..\Libraries\libs\libbtstack_master.a(lc_sniff.o)
                0x0000000010031376                lc_sniff_init
                0x0000000010031388                lc_sniff_clear
                0x00000000100313be                lc_sniff_interval_get
                0x00000000100313de                lc_sniff_offset_update
                0x000000001003140e                lc_sniff_host_request
                0x00000000100315a4                lc_sniff_peer_request
                0x0000000010031874                lc_sniff_peer_accept
                0x0000000010031944                lc_sniff_peer_reject
                0x000000001003196e                lc_sniff_acc_tx_cfm
                0x0000000010031970                lc_sniff_timeout
                0x0000000010031976                lc_sniff_unsniff
                0x00000000100319da                lc_sniff_unsniff_peer_request
                0x0000000010031a86                lc_sniff_unsniff_peer_accept
                0x0000000010031aa6                lc_sniff_unsniff_peer_reject
 .text          0x0000000010031aec     0x164c ..\..\..\Libraries\libs\libbtstack_master.a(lc_sco.o)
                0x00000000100322ba                lc_sco_alloc_link
                0x0000000010032302                lc_sco_free_link
                0x000000001003233a                lc_sco_get_conhdl
                0x0000000010032376                lc_sco_get_snoop_service
                0x00000000100323ba                lc_sco_set_snoop_service
                0x00000000100323ea                lc_sco_start_snoop
                0x00000000100324dc                lc_sco_init
                0x000000001003250a                lc_sco_reset
                0x0000000010032556                lc_sco_detach
                0x00000000100325ee                lc_sco_release
                0x0000000010032668                lc_sco_host_request
                0x0000000010032766                lc_sco_host_accept
                0x00000000100328f4                lc_sco_host_reject
                0x000000001003298e                lc_sco_host_request_disc
                0x0000000010032a18                lc_sco_peer_request
                0x0000000010032c80                lc_sco_peer_accept
                0x0000000010032cf0                lc_sco_peer_reject
                0x0000000010032d72                lc_sco_peer_request_disc
                0x0000000010032e62                lc_sco_peer_accept_disc
                0x0000000010032f08                lc_sco_peer_reject_disc
                0x0000000010032f88                lc_sco_baseband_ack
                0x0000000010033058                lc_sco_timeout
                0x0000000010033104                lc_sco_offset_update
 *fill*         0x0000000010033138        0x0 
 .text          0x0000000010033138     0x9234 ..\..\..\Libraries\libs\libbtstack_master.a(lc_proc.o)
                0x0000000010033312                hci_acl_data_lc_func
                0x00000000100338c4                lmp_detach_func
                0x00000000100339ba                lc_acl_rx_ind_func
                0x000000001003c322                lc_flush_acl_tx_pend
 .text          0x000000001003c36c      0x6dc ..\..\..\Libraries\libs\libbtstack_master.a(lc_lmppdu.o)
                0x000000001003c36c                lmp_find_desc
                0x000000001003c3ba                lmp_estab_allowed
                0x000000001003c3f2                lmp_msg_pk
                0x000000001003c456                lmp_msg_unpk
                0x000000001003c4c8                lc_send_lmp
                0x000000001003c532                lc_send_pdu_acc
                0x000000001003c550                lc_send_pdu_acc_ext4
                0x000000001003c57a                lc_send_pdu_not_acc
                0x000000001003c59c                lc_send_pdu_not_acc_ext4
                0x000000001003c5ca                lc_send_pdu_set_afh
                0x000000001003c60c                lc_send_pdu_au_rand
                0x000000001003c636                lc_send_pdu_in_rand
                0x000000001003c660                lc_send_pdu_comb_key
                0x000000001003c68a                lc_send_pdu_max_slot
                0x000000001003c6a8                lc_send_pdu_max_slot_req
                0x000000001003c6c6                lc_send_pdu_encaps_payl
                0x000000001003c6f0                lc_send_pdu_encaps_head
                0x000000001003c716                lc_send_pdu_ptt_req
                0x000000001003c738                lc_send_pdu_sp_nb
                0x000000001003c762                lc_send_pdu_sp_cfm
                0x000000001003c78c                lc_send_pdu_sres
                0x000000001003c7b6                lc_send_pdu_sco_lk_rem_req
                0x000000001003c7d8                lc_send_pdu_esco_lk_rem_req
                0x000000001003c7fe                lc_send_pdu_auto_rate
                0x000000001003c818                lc_send_pdu_sup_to
                0x000000001003c836                lc_send_pdu_enc_key_sz_req
                0x000000001003c854                lc_send_pdu_feats_res
                0x000000001003c880                lc_send_pdu_tim_acc
                0x000000001003c89a                lc_send_pdu_feats_ext_req
                0x000000001003c8d0                lc_send_pdu_io_cap_res
                0x000000001003c91a                lc_send_pdu_num_comp_fail
                0x000000001003c938                lc_send_pdu_paus_enc_req
                0x000000001003c956                lc_send_pdu_resu_enc_req
                0x000000001003c974                lc_send_pdu_setup_cmp
                0x000000001003c98e                lc_send_pdu_qos_req
                0x000000001003c9b0                lc_send_pdu_slot_off
                0x000000001003c9f2                lc_send_pdu_vers_req
                0x000000001003ca20                lc_send_pdu_dhkey_chk
 .text          0x000000001003ca48      0x11a ..\..\..\Libraries\libs\libbtstack_master.a(mgr_proc.o)
 .text          0x000000001003cb62      0xa60 ..\..\..\Libraries\libs\libbtstack_master.a(mgr_init.o)
                0x000000001003cb62                hci_le_create_con_cmd_func
                0x000000001003ce7a                hci_le_ext_create_con_cmd_func
                0x000000001003d1d8                hci_le_create_con_cancel_cmd_func
                0x000000001003d24e                ble_init_end_ind_func
 .text          0x000000001003d5c2      0x6da ..\..\..\Libraries\libs\libbtstack_master.a(mgr_hci.o)
 .text.le.mgr   0x000000001003dc9c       0x38 ..\..\..\Libraries\libs\libbtstack_master.a(mgr_hci.o)
                0x000000001003dc9c                hci_command_mgr_func
 .text          0x000000001003dcd4      0x40a ..\..\..\Libraries\libs\libbtstack_master.a(ll_scan.o)
                0x000000001003dcd4                hci_le_set_scan_param_cmd_func
                0x000000001003de22                hci_le_set_scan_en_cmd_func
 .text.le.ll_scan
                0x000000001003e0de      0x628 ..\..\..\Libraries\libs\libbtstack_master.a(ll_scan.o)
                0x000000001003e0de                ble_adv_rep_ind_func
                0x000000001003e674                ble_scan_end_ind_func
 .text          0x000000001003e706      0x826 ..\..\..\Libraries\libs\libbtstack_master.a(ll_adv.o)
                0x000000001003e7be                ll_adv_hdl_to_idx
                0x000000001003e802                hci_le_rd_adv_ch_tx_pw_cmd_func
                0x000000001003e862                hci_le_set_adv_param_cmd_func
                0x000000001003ea0c                hci_le_set_adv_data_cmd_func
                0x000000001003eae0                hci_le_set_scan_rsp_data_cmd_func
                0x000000001003ebb4                hci_le_set_adv_en_cmd_func
                0x000000001003ee36                ll_adv_get_act_idx
                0x000000001003eea0                ll_adv_get_set_id
 .text.le.ll_adv
                0x000000001003ef2c      0x30a ..\..\..\Libraries\libs\libbtstack_master.a(ll_adv.o)
                0x000000001003ef2c                ble_scan_req_ind_func
                0x000000001003ef94                ble_adv_end_ind_func
 .text.le.ll_adv.con
                0x000000001003f236      0x250 ..\..\..\Libraries\libs\libbtstack_master.a(ll_adv.o)
                0x000000001003f236                ble_adv_end_con_ind
 .text          0x000000001003f486      0x3ae ..\..\..\Libraries\libs\libbtstack_master.a(ll_proc.o)
                0x000000001003f486                hci_command_ll_func
                0x000000001003f4d6                ble_acl_rx_ind_func
                0x000000001003f66c                ble_acl_tx_cfm_func
                0x000000001003f67c                hci_acl_data_func
                0x000000001003f74e                ll_cmd_cmp_send
                0x000000001003f77c                hci_vs_set_pref_slave_latency_cmd_func
                0x000000001003f7c0                hci_vs_set_pref_slave_evt_dur_cmd_func
                0x000000001003f80c                ll_cmd_stat_send
 .text          0x000000001003f834      0x32e ..\..\..\Libraries\libs\libbtstack_master.a(ll_ping.o)
                0x000000001003f8b4                hci_rd_auth_payl_to_cmd_func
                0x000000001003f918                ll_op_ping_ind_func
                0x000000001003f96e                ll_auth_payl_nearly_to_func
                0x000000001003f9dc                ll_ping_restart
                0x000000001003fa34                ll_auth_payl_real_to_func
                0x000000001003fa92                ll_ping_set
                0x000000001003fafa                hci_wr_auth_payl_to_cmd_func
 .text.le.ll_cntl.pdu
                0x000000001003fb62       0x3c ..\..\..\Libraries\libs\libbtstack_master.a(ll_ping.o)
                0x000000001003fb62                ll_ping_req_func
                0x000000001003fb7e                ll_ping_rsp_func
 *fill*         0x000000001003fb9e        0x2 
 .text          0x000000001003fba0      0xad0 ..\..\..\Libraries\libs\libbtstack_master.a(ll_phy_upd.o)
                0x0000000010040394                hci_le_rd_phy_cmd_func
                0x00000000100403fc                hci_le_set_phy_cmd_func
                0x000000001004053e                ll_op_phy_upd_ind_func
                0x00000000100405c8                ble_phy_upd_cfm_func
                0x0000000010040604                ll_phy_upd_proc_start
 .text.le.ll_cntl.pdu
                0x0000000010040670      0x212 ..\..\..\Libraries\libs\libbtstack_master.a(ll_phy_upd.o)
                0x0000000010040670                ll_phy_req_func
                0x0000000010040734                ll_phy_rsp_func
                0x00000000100407c8                ll_phy_update_ind_func
 .text          0x0000000010040882      0x136 ..\..\..\Libraries\libs\libbtstack_master.a(ll_past.o)
                0x0000000010040882                hci_le_per_adv_set_info_transf_cmd_func
                0x0000000010040936                hci_le_set_per_adv_sync_transf_param_cmd_func
 .text          0x00000000100409b8      0x57c ..\..\..\Libraries\libs\libbtstack_master.a(ll_length.o)
                0x0000000010040c20                hci_le_set_data_len_cmd_func
                0x0000000010040d2e                hci_vs_set_max_rx_size_and_time_cmd_func
                0x0000000010040e42                ll_op_length_upd_ind_func
                0x0000000010040ea8                ll_length_proc_start
 .text.le.ll_cntl.pdu
                0x0000000010040f34      0x204 ..\..\..\Libraries\libs\libbtstack_master.a(ll_length.o)
                0x0000000010040f34                ll_length_req_func
                0x000000001004109e                ll_length_rsp_func
 .text          0x0000000010041138      0x2d6 ..\..\..\Libraries\libs\libbtstack_master.a(ll_feature.o)
                0x00000000100412e8                hci_le_rd_rem_feats_cmd_func
                0x0000000010041398                ll_op_feats_exch_ind_func
 .text.le.ll_cntl.pdu
                0x000000001004140e      0x168 ..\..\..\Libraries\libs\libbtstack_master.a(ll_feature.o)
                0x000000001004140e                ll_feature_req_func
                0x0000000010041484                ll_slave_feature_req_func
                0x00000000100414fa                ll_feature_rsp_func
 *fill*         0x0000000010041576        0x2 
 .text          0x0000000010041578      0xaa0 ..\..\..\Libraries\libs\libbtstack_master.a(ll_encrypt.o)
                0x0000000010041cd0                hci_le_en_enc_cmd_func
                0x0000000010041da6                hci_le_ltk_req_reply_cmd_func
                0x0000000010041e1a                hci_le_ltk_req_neg_reply_cmd_func
                0x0000000010041ea6                ll_encrypt_ind_func
                0x0000000010041fb0                ll_op_encrypt_ind_func
 .text.le.ll_cntl.pdu
                0x0000000010042018      0x2fa ..\..\..\Libraries\libs\libbtstack_master.a(ll_encrypt.o)
                0x0000000010042018                ll_pause_enc_req_func
                0x0000000010042096                ll_pause_enc_rsp_func
                0x00000000100420f8                ll_enc_req_func
                0x00000000100421de                ll_enc_rsp_func
                0x0000000010042260                ll_start_enc_req_func
                0x00000000100422ba                ll_start_enc_rsp_func
 .text          0x0000000010042312      0x30a ..\..\..\Libraries\libs\libbtstack_master.a(ll_disconnect.o)
                0x0000000010042312                ble_disc_ind_func
                0x000000001004236a                ll_stopped_ind_func
                0x00000000100423c2                hci_disconnect_cmd_func
                0x0000000010042470                ll_disconnect
                0x0000000010042552                ll_op_disconnect_ind_func
                0x00000000100425cc                ll_init_term_proc
 .text.le.ll_cntl.pdu
                0x000000001004261c       0x44 ..\..\..\Libraries\libs\libbtstack_master.a(ll_disconnect.o)
                0x000000001004261c                ll_terminate_ind_func
 .text          0x0000000010042660      0xce4 ..\..\..\Libraries\libs\libbtstack_master.a(ll_con_upd.o)
                0x0000000010042ed6                hci_le_con_upd_cmd_func
                0x0000000010043002                hci_le_rem_con_param_req_reply_cmd_func
                0x000000001004309c                hci_le_rem_con_param_req_neg_reply_cmd_func
                0x00000000100430fe                ll_op_con_upd_ind_func
                0x0000000010043190                ble_con_param_upd_cfm_func
                0x00000000100431fc                ble_con_offset_upd_ind_func
                0x000000001004324e                ll_con_move_cb
 .text.le.ll_cntl.pdu
                0x0000000010043344      0x30c ..\..\..\Libraries\libs\libbtstack_master.a(ll_con_upd.o)
                0x0000000010043344                ll_con_update_ind_func
                0x00000000100434a4                ll_con_param_req_func
                0x00000000100435ba                ll_con_param_rsp_func
 .text          0x0000000010043650      0x2cc ..\..\..\Libraries\libs\libbtstack_master.a(ll_cntl.o)
                0x0000000010043650                ll_pdu_send_reject_ind
                0x00000000100436a4                ble_cntl_rx_ind_func
                0x000000001004380c                ble_cntl_tx_cfm_func
                0x0000000010043864                hci_vs_send_cntl_cmd_func
                0x00000000100438c8                hci_vs_cntl_discard_cmd_func
 .text.le.ll_cntl.pdu
                0x000000001004391c       0x64 ..\..\..\Libraries\libs\libbtstack_master.a(ll_cntl.o)
 .text.le.ll_cntl.send
                0x0000000010043980      0x18a ..\..\..\Libraries\libs\libbtstack_master.a(ll_cntl.o)
                0x0000000010043980                ll_cntl_tx_check
                0x0000000010043a70                ll_cntl_send
 .text          0x0000000010043b0a      0x2d6 ..\..\..\Libraries\libs\libbtstack_master.a(ll_clk_acc.o)
                0x0000000010043c6a                ll_op_clk_acc_ind_func
                0x0000000010043cc0                ll_clk_acc_modify
                0x0000000010043d3e                hci_le_req_peer_sca_cmd_func
 .text.le.ll_cntl.pdu
                0x0000000010043de0       0xb4 ..\..\..\Libraries\libs\libbtstack_master.a(ll_clk_acc.o)
                0x0000000010043de0                ll_clk_acc_req_func
                0x0000000010043e3e                ll_clk_acc_rsp_func
 .text          0x0000000010043e94      0x37a ..\..\..\Libraries\libs\libbtstack_master.a(ll_chmap_upd.o)
                0x0000000010044096                hci_le_rd_chnl_map_cmd_func
                0x0000000010044100                ll_op_ch_map_upd_ind_func
                0x0000000010044160                mgr_ch_map_update_ind_func
                0x00000000100441da                ble_ch_map_upd_cfm_func
 .text.le.ll_cntl.pdu
                0x000000001004420e      0x172 ..\..\..\Libraries\libs\libbtstack_master.a(ll_chmap_upd.o)
                0x000000001004420e                ll_channel_map_ind_func
                0x00000000100442d6                ll_min_used_channels_ind_func
 .text          0x0000000010044380      0x176 ..\..\..\Libraries\libs\libbtstack_master.a(aes_rpa.o)
                0x0000000010044442                aes_rpa_gen
                0x0000000010044494                aes_rpa_resolve
 .text          0x00000000100444f6        0x4 ..\..\..\Libraries\libs\libbtstack_master.a(scan_hook.o)
                0x00000000100444f6                ble_scan_end_ind_hook
 .text          0x00000000100444fa        0x8 ..\..\..\Libraries\libs\libbtstack_master.a(adv_hook.o)
                0x00000000100444fa                ble_adv_end_ind_hook
 .text          0x0000000010044502      0x21e ..\..\..\Libraries\libs\libbtstack_master.a(ll_version.o)
                0x0000000010044610                ll_op_ver_exch_ind_func
                0x0000000010044686                hci_rd_rem_ver_info_cmd_func
 .text.le.ll_cntl.pdu
                0x0000000010044720       0x6e ..\..\..\Libraries\libs\libbtstack_master.a(ll_version.o)
                0x0000000010044720                ll_version_ind_func
 .text          0x000000001004478e      0x11a ..\..\..\Libraries\libs\libbtstack_master.a(ll_pwr.o)
                0x000000001004478e                hci_rd_tx_pwr_lvl_cmd_func
                0x0000000010044824                hci_rd_rssi_cmd_func
 *(.rodata*)
 *fill*         0x00000000100448a8        0x0 
 .rodata.str1.4
                0x00000000100448a8       0x3e Output\obj\Libraries\bsp\bsp_bt.o
 *fill*         0x00000000100448e6        0x2 
 .rodata.str1.4
                0x00000000100448e8      0x11d Output\obj\Libraries\bsp\bsp_fot.o
 *fill*         0x0000000010044a05        0x3 
 .rodata.str1.4
                0x0000000010044a08       0x76 Output\obj\Libraries\bsp\bsp_sys.o
 *fill*         0x0000000010044a7e        0x2 
 .rodata.str1.4
                0x0000000010044a80       0x3d Output\obj\Libraries\BT\ble\ab_link\app.o
 *fill*         0x0000000010044abd        0x3 
 .rodata.str1.4
                0x0000000010044ac0       0x3a Output\obj\Libraries\BT\ble\ble.o
 *fill*         0x0000000010044afa        0x2 
 .rodata.str1.4
                0x0000000010044afc        0x5 Output\obj\Libraries\BT\spp\bt.o
 *fill*         0x0000000010044b01        0x3 
 .rodata.str1.4
                0x0000000010044b04       0x58 Output\obj\Libraries\BT\spp\spp.o
 .rodata.str1.4
                0x0000000010044b5c      0x229 Output\obj\Examples\BLE_Host\Source\ble_client.o
 *fill*         0x0000000010044d85        0x3 
 .rodata.str1.4
                0x0000000010044d88       0x1d Output\obj\Examples\BLE_Host\Project\main.o
 *fill*         0x0000000010044da5        0x3 
 .rodata.str1.4
                0x0000000010044da8       0xfc ..\..\..\Libraries\libs\libplatform.a(cm.o)
 .rodata.str1.4
                0x0000000010044ea4       0x10 ..\..\..\Libraries\libs\libplatform.a(main.o)
 .rodata.str1.4
                0x0000000010044eb4       0x57 ..\..\..\Libraries\libs\libplatform.a(startup.o)
 *fill*         0x0000000010044f0b        0x1 
 .rodata.str1.4
                0x0000000010044f0c      0x104 ..\..\..\Libraries\libs\libplatform.a(lock.o)
 .rodata.str1.4
                0x0000000010045010       0x1d ..\..\..\Libraries\libs\libplatform.a(sys.o)
 *fill*         0x000000001004502d        0x3 
 .rodata.volt_trim
                0x0000000010045030       0xbc ..\..\..\Libraries\libs\libplatform.a(voltage_trim.o)
                0x0000000010045030                charge_trim_step
                0x0000000010045044                vddcore_trim_step
                0x0000000010045064                vddio_trim_step
                0x0000000010045084                vddbko_trim_step
 .rodata.bb.tbl
                0x00000000100450ec        0x8 ..\..\..\Libraries\libs\libbtstack_master.a(ble_con.o)
                0x00000000100450ec                connect_req_dur_tab
 .rodata.bb.tbl
                0x00000000100450f4       0x16 ..\..\..\Libraries\libs\libbtstack_master.a(bb_utils.o)
                0x00000000100450f4                null_array
                0x0000000010045104                dft_addr
 *fill*         0x000000001004510a        0x2 
 .rodata        0x000000001004510c       0x20 ..\..\..\Libraries\libs\libbtstack_master.a(bb.o)
                0x000000001004510c                bb_hook
 .rodata.str1.4
                0x000000001004512c        0x5 ..\..\..\Libraries\libs\libbtstack_master.a(extern_bt.o)
                                          0xd (size before relaxing)
 *fill*         0x0000000010045131        0x3 
 .rodata        0x0000000010045134       0x18 ..\..\..\Libraries\libs\libbtstack_master.a(spp.o)
 .rodata.stack.spp
                0x000000001004514c        0x2 ..\..\..\Libraries\libs\libbtstack_master.a(spp.o)
 *fill*         0x000000001004514e        0x2 
 .rodata        0x0000000010045150       0x10 ..\..\..\Libraries\libs\libbtstack_master.a(sdp_util.o)
                0x0000000010045150                mfi_search_uuid128
 .rodata.sdp.tbl.spp
                0x0000000010045160      0x11f ..\..\..\Libraries\libs\libbtstack_master.a(sdp_tbl.o)
                0x0000000010045160                sdp_spp_dueros_ota_service_record
                0x00000000100451c4                sdp_spp_proc_test_service_record
                0x0000000010045228                sdp_spp_service_record
 *fill*         0x000000001004527f        0x1 
 .rodata.str1.4
                0x0000000010045280        0x8 ..\..\..\Libraries\libs\libbtstack_master.a(sdp_client.o)
 .rodata        0x0000000010045288       0x17 ..\..\..\Libraries\libs\libbtstack_master.a(sdp_client.o)
 *fill*         0x000000001004529f        0x1 
 .rodata        0x00000000100452a0      0x100 ..\..\..\Libraries\libs\libbtstack_master.a(rfcomm.o)
 .rodata        0x00000000100453a0       0x20 ..\..\..\Libraries\libs\libbtstack_master.a(btstack_util.o)
                0x00000000100453b0                bluetooth_base_uuid
 .rodata.str1.4
                0x00000000100453c0       0x1a ..\..\..\Libraries\libs\libbtstack_master.a(btstack_link_ctrl.o)
 *fill*         0x00000000100453da        0x2 
 .rodata.str1.4
                0x00000000100453dc       0x51 ..\..\..\Libraries\libs\libbtstack_master.a(sm.o)
                                         0x55 (size before relaxing)
 *fill*         0x000000001004542d        0x3 
 .rodata        0x0000000010045430       0x64 ..\..\..\Libraries\libs\libbtstack_master.a(sm.o)
 .rodata.str1.4
                0x0000000010045494       0x18 ..\..\..\Libraries\libs\libbtstack_master.a(le_device_db_memory.o)
                                         0x1c (size before relaxing)
 .rodata        0x00000000100454ac       0x11 ..\..\..\Libraries\libs\libbtstack_master.a(gatt_server.o)
 *fill*         0x00000000100454bd        0x3 
 .rodata        0x00000000100454c0       0x30 ..\..\..\Libraries\libs\libbtstack_master.a(gatt_profile.o)
 .rodata.str1.4
                0x00000000100454f0        0xc ..\..\..\Libraries\libs\libbtstack_master.a(att_server.o)
 .rodata        0x00000000100454fc       0x10 ..\..\..\Libraries\libs\libbtstack_master.a(att_db.o)
 .rodata.str1.4
                0x000000001004550c       0x2e ..\..\..\Libraries\libs\libbtstack_master.a(btstack_api.o)
 *fill*         0x000000001004553a        0x2 
 .rodata        0x000000001004553c       0xe0 ..\..\..\Libraries\libs\libbtstack_master.a(btstack_api.o)
                0x000000001004553c                tws_key_tbl
                0x0000000010045604                tws_hid_key_tbl
 .rodata.stack.api
                0x000000001004561c      0x184 ..\..\..\Libraries\libs\libbtstack_master.a(btstack_api.o)
                0x000000001004561c                btstack_ctl0_tbl
                0x0000000010045674                btstack_comm_tbl
                0x0000000010045694                btstack_hid_tbl
                0x00000000100456a0                btstack_ctl_tbl
                0x000000001004576c                btstack_api_tbl
                0x000000001004579c                btstack_spp_tbl
 .rodata.stack.setup
                0x00000000100457a0       0x14 ..\..\..\Libraries\libs\libbtstack_master.a(btstack_api.o)
 .rodata        0x00000000100457b4       0x2c ..\..\..\Libraries\libs\libbtstack_master.a(bb_sche.o)
 .rodata        0x00000000100457e0       0x18 ..\..\..\Libraries\libs\libbtstack_master.a(vs_proc.o)
 .rodata.bb.tbl
                0x00000000100457f8        0x6 ..\..\..\Libraries\libs\libbtstack_master.a(rf_smart.o)
 *fill*         0x00000000100457fe        0x2 
 .rodata.str1.4
                0x0000000010045800       0x20 ..\..\..\Libraries\libs\libbtstack_master.a(hct_tl.o)
 .rodata.str1.4
                0x0000000010045820      0x312 ..\..\..\Libraries\libs\libbtstack_master.a(hct_msg.o)
                                        0x362 (size before relaxing)
 *fill*         0x0000000010045b32        0x2 
 .rodata        0x0000000010045b34      0xc20 ..\..\..\Libraries\libs\libbtstack_master.a(hct_msg.o)
                0x0000000010045b34                hci_cmd_desc_root_tab
                0x0000000010045b74                hci_evt_desc_tab
                0x0000000010045cf4                hci_evt_le_desc_tab
                0x0000000010045d64                hci_cmd_desc_tab_vs
                0x0000000010045e30                hci_cmd_desc_tab_le
                0x0000000010046094                hci_cmd_desc_tab_testing
                0x00000000100460d0                hci_cmd_desc_tab_stat_par
                0x0000000010046124                hci_cmd_desc_tab_info_par
                0x00000000100461a8                hci_cmd_desc_tab_ctrl_bb
                0x0000000010046520                hci_cmd_desc_tab_lk_pol
                0x00000000100465a4                hci_cmd_desc_tab_lk_ctrl
 .rodata        0x0000000010046754       0x9c ..\..\..\Libraries\libs\libbtstack_master.a(lm.o)
 .rodata.bb.tbl
                0x00000000100467f0       0x14 ..\..\..\Libraries\libs\libbtstack_master.a(bt21.o)
                0x00000000100467f0                bt_ctl
 .rodata.bb.tbl
                0x0000000010046804        0x7 ..\..\..\Libraries\libs\libbtstack_master.a(ble_hal.o)
 *fill*         0x000000001004680b        0x1 
 .rodata.bb.tbl
                0x000000001004680c       0x14 ..\..\..\Libraries\libs\libbtstack_master.a(ble.o)
                0x000000001004680c                ble_ctl
 .rodata.l2cap  0x0000000010046820        0x9 ..\..\..\Libraries\libs\libbtstack_master.a(l2cap_test.o)
                0x0000000010046820                vs_test_actived_cmd
 *fill*         0x0000000010046829        0x3 
 .rodata.stack.l2cap
                0x000000001004682c        0x5 ..\..\..\Libraries\libs\libbtstack_master.a(l2cap.o)
 *fill*         0x0000000010046831        0x3 
 .rodata.str1.4
                0x0000000010046834       0xb8 ..\..\..\Libraries\libs\libbtstack_master.a(hci_cmd.o)
                                         0xd0 (size before relaxing)
 .rodata.stack.hci_send
                0x00000000100468ec      0x2a0 ..\..\..\Libraries\libs\libbtstack_master.a(hci_cmd.o)
                0x00000000100468ec                hci_le_set_default_phy
                0x00000000100468f4                hci_le_write_suggested_default_data_len
                0x00000000100468fc                hci_le_test_end
                0x0000000010046904                hci_le_transmitter_test
                0x000000001004690c                hci_le_receiver_test
                0x0000000010046914                hci_le_read_supported_states
                0x000000001004691c                hci_le_long_term_key_negative_reply
                0x0000000010046924                hci_le_long_term_key_request_reply
                0x000000001004692c                hci_le_start_encryption
                0x0000000010046934                hci_le_rand
                0x000000001004693c                hci_le_encrypt
                0x0000000010046944                hci_le_read_remote_used_features
                0x000000001004694c                hci_le_read_channel_map
                0x0000000010046954                hci_le_set_host_channel_classification
                0x000000001004695c                hci_le_connection_update
                0x0000000010046964                hci_le_remove_device_from_white_list
                0x000000001004696c                hci_le_add_device_to_white_list
                0x0000000010046974                hci_le_clear_white_list
                0x000000001004697c                hci_le_read_white_list_size
                0x0000000010046984                hci_le_create_connection_cancel
                0x000000001004698c                hci_le_create_connection
                0x0000000010046994                hci_le_set_scan_enable
                0x000000001004699c                hci_le_set_scan_parameters
                0x00000000100469a4                hci_le_set_advertise_enable
                0x00000000100469ac                hci_le_set_scan_response_data
                0x00000000100469b4                hci_le_set_advertising_data
                0x00000000100469bc                hci_le_read_advertising_channel_tx_power
                0x00000000100469c4                hci_le_set_advertising_parameters
                0x00000000100469cc                hci_le_set_random_address
                0x00000000100469d4                hci_le_read_supported_features
                0x00000000100469dc                hci_le_read_buffer_size
                0x00000000100469e4                hci_le_set_event_mask
                0x00000000100469ec                hci_test_mode_emul
                0x00000000100469f4                hci_read_rssi
                0x00000000100469fc                hci_read_bd_addr
                0x0000000010046a04                hci_read_buffer_size
                0x0000000010046a0c                hci_read_local_supported_features
                0x0000000010046a14                hci_read_local_supported_commands
                0x0000000010046a1c                hci_write_loopback_mode
                0x0000000010046a24                hci_read_loopback_mode
                0x0000000010046a2c                hci_write_le_host_supported
                0x0000000010046a34                hci_read_le_host_supported
                0x0000000010046a3c                hci_write_simple_pairing_mode
                0x0000000010046a44                hci_write_extended_inquiry_response
                0x0000000010046a4c                hci_write_inquiry_scan_type
                0x0000000010046a54                hci_write_inquiry_mode
                0x0000000010046a5c                hci_write_link_supervision_timeout
                0x0000000010046a64                hci_host_buffer_size
                0x0000000010046a6c                hci_write_class_of_device
                0x0000000010046a74                hci_write_scan_enable
                0x0000000010046a7c                hci_write_page_timeout
                0x0000000010046a84                hci_write_local_name
                0x0000000010046a8c                hci_reset
                0x0000000010046a94                hci_set_event_mask
                0x0000000010046a9c                hci_switch_role_command
                0x0000000010046aa4                hci_role_discovery
                0x0000000010046aac                hci_io_capability_request_negative_reply
                0x0000000010046ab4                hci_remote_oob_data_request_negative_reply
                0x0000000010046abc                hci_user_passkey_request_negative_reply
                0x0000000010046ac4                hci_user_passkey_request_reply
                0x0000000010046acc                hci_user_confirmation_request_negative_reply
                0x0000000010046ad4                hci_user_confirmation_request_reply
                0x0000000010046adc                hci_io_capability_request_reply
                0x0000000010046ae4                hci_accept_synchronous_connection
                0x0000000010046aec                hci_setup_synchronous_connection
                0x0000000010046af4                hci_read_clock_offset_command
                0x0000000010046afc                hci_read_remote_version_info_command
                0x0000000010046b04                hci_read_remote_supported_features_command
                0x0000000010046b0c                hci_remote_name_request_cancel
                0x0000000010046b14                hci_remote_name_request
                0x0000000010046b1c                hci_change_connection_link_key
                0x0000000010046b24                hci_set_connection_encryption
                0x0000000010046b2c                hci_authentication_requested
                0x0000000010046b34                hci_pin_code_request_negative_reply
                0x0000000010046b3c                hci_pin_code_request_reply
                0x0000000010046b44                hci_link_key_request_negative_reply
                0x0000000010046b4c                hci_link_key_request_reply
                0x0000000010046b54                hci_reject_connection_request
                0x0000000010046b5c                hci_accept_connection_request
                0x0000000010046b64                hci_create_connection_cancel
                0x0000000010046b6c                hci_disconnect
                0x0000000010046b74                hci_create_connection
                0x0000000010046b7c                hci_inquiry_cancel
                0x0000000010046b84                hci_inquiry
 .rodata.str1.4
                0x0000000010046b8c       0x21 ..\..\..\Libraries\libs\libbtstack_master.a(hci.o)
 *fill*         0x0000000010046bad        0x3 
 .rodata        0x0000000010046bb0        0xc ..\..\..\Libraries\libs\libbtstack_master.a(hci.o)
 .rodata        0x0000000010046bbc       0x2d ..\..\..\Libraries\libs\libbtstack_master.a(hid_usage.o)
                0x0000000010046bd4                ts_release
                0x0000000010046be0                ts_press
 *fill*         0x0000000010046be9        0x3 
 .rodata.str1.4
                0x0000000010046bec      0x116 ..\..\..\Libraries\libs\libbtstack_master.a(hfp_hf.o)
                                        0x11a (size before relaxing)
 *fill*         0x0000000010046d02        0x2 
 .rodata.str1.4
                0x0000000010046d04       0x6d ..\..\..\Libraries\libs\libbtstack_master.a(hfp.o)
                                         0xd5 (size before relaxing)
 *fill*         0x0000000010046d71        0x3 
 .rodata        0x0000000010046d74       0x12 ..\..\..\Libraries\libs\libbtstack_master.a(hfp.o)
 *fill*         0x0000000010046d86        0x2 
 .rodata.str1.4
                0x0000000010046d88        0x6 ..\..\..\Libraries\libs\libbtstack_master.a(btstack_chipset_inner.o)
 *fill*         0x0000000010046d8e        0x2 
 .rodata        0x0000000010046d90       0x14 ..\..\..\Libraries\libs\libbtstack_master.a(btstack_chipset_inner.o)
 .rodata        0x0000000010046da4      0x1c8 ..\..\..\Libraries\libs\libbtstack_master.a(lm_sp.o)
 .rodata        0x0000000010046f6c      0x2f4 ..\..\..\Libraries\libs\libbtstack_master.a(lm_proc.o)
 .rodata.bb.tbl
                0x0000000010047260       0x1e ..\..\..\Libraries\libs\libbtstack_master.a(lm_proc.o)
                0x0000000010047260                lm_local_supp_feats
 *fill*         0x000000001004727e        0x2 
 .rodata        0x0000000010047280      0x420 ..\..\..\Libraries\libs\libbtstack_master.a(lm_key.o)
 .rodata        0x00000000100476a0       0x10 ..\..\..\Libraries\libs\libbtstack_master.a(lc.o)
 .rodata.str1.4
                0x00000000100476b0        0x2 ..\..\..\Libraries\libs\libbtstack_master.a(extern_hfhs.o)
                                          0x6 (size before relaxing)
 *fill*         0x00000000100476b2        0x2 
 .rodata.str1.4
                0x00000000100476b4       0x16 ..\..\..\Libraries\libs\libbtstack_master.a(l2cap_signaling.o)
                                         0x2a (size before relaxing)
 *fill*         0x00000000100476ca        0x2 
 .rodata        0x00000000100476cc       0x58 ..\..\..\Libraries\libs\libbtstack_master.a(l2cap_signaling.o)
 .rodata        0x0000000010047724       0x7c ..\..\..\Libraries\libs\libbtstack_master.a(lm_sco.o)
 .rodata        0x00000000100477a0       0x40 ..\..\..\Libraries\libs\libbtstack_master.a(lc_util.o)
 .rodata        0x00000000100477e0      0x5dc ..\..\..\Libraries\libs\libbtstack_master.a(lc_proc.o)
 .rodata.str1.4
                0x0000000010047dbc       0x6b ..\..\..\Libraries\libs\libbtstack_master.a(lc_lmppdu.o)
                                         0x9b (size before relaxing)
 *fill*         0x0000000010047e27        0x1 
 .rodata        0x0000000010047e28      0x280 ..\..\..\Libraries\libs\libbtstack_master.a(lc_lmppdu.o)
 .rodata        0x00000000100480a8       0x60 ..\..\..\Libraries\libs\libbtstack_master.a(mgr_proc.o)
 .rodata.le.mgr_cntl.tbl
                0x0000000010048108       0xf0 ..\..\..\Libraries\libs\libbtstack_master.a(mgr_hci.o)
                0x0000000010048108                mgr_hci_cmd_tbl
 .rodata        0x00000000100481f8       0x1c ..\..\..\Libraries\libs\libbtstack_master.a(ll_scan.o)
 .rodata.le.ll_cntl.tbl
                0x0000000010048214      0x1a8 ..\..\..\Libraries\libs\libbtstack_master.a(ll_proc.o)
                0x0000000010048214                ll_msg_tbl
                0x00000000100482f4                ll_hci_cmd_tbl
 .rodata.str1.4
                0x00000000100483bc       0x3c ..\..\..\Libraries\libs\libbtstack_master.a(ll_cntl.o)
                                         0x59 (size before relaxing)
 .rodata.le.ll_cntl.tbl
                0x00000000100483f8      0x1c8 ..\..\..\Libraries\libs\libbtstack_master.a(ll_cntl.o)
                0x00000000100483f8                ll_cntl_pdu_tbl
 *(.srodata*)
 .srodata       0x00000000100485c0        0x4 ..\..\..\Libraries\libs\libbtstack_master.a(bt_acl.o)
 .srodata       0x00000000100485c4        0x3 ..\..\..\Libraries\libs\libbtstack_master.a(extern_bt.o)
                0x00000000100485c5                cfg_bb_rf_ctl
 *fill*         0x00000000100485c7        0x1 
 .srodata       0x00000000100485c8        0x2 ..\..\..\Libraries\libs\libbtstack_master.a(btstack_link_key_db.o)
                0x00000000100485c8                link_info_page_size
 *fill*         0x00000000100485ca        0x2 
 .srodata       0x00000000100485cc        0x8 ..\..\..\Libraries\libs\libbtstack_master.a(vs_proc.o)
 .srodata       0x00000000100485d4        0x8 ..\..\..\Libraries\libs\libbtstack_master.a(hct_msg.o)
                0x00000000100485d4                hci_evt_dbg_desc_tab
 .srodata       0x00000000100485dc       0x1c ..\..\..\Libraries\libs\libbtstack_master.a(hct.o)
 .srodata       0x00000000100485f8        0x6 ..\..\..\Libraries\libs\libbtstack_master.a(hci.o)
 *fill*         0x00000000100485fe        0x2 
 .srodata       0x0000000010048600       0x10 ..\..\..\Libraries\libs\libbtstack_master.a(mgr.o)
 .srodata       0x0000000010048610        0x3 ..\..\..\Libraries\libs\libbtstack_master.a(lc_proc.o)
 *fill*         0x0000000010048613        0x1 
 .srodata       0x0000000010048614        0x8 ..\..\..\Libraries\libs\libbtstack_master.a(mgr_hci.o)
 .srodata       0x000000001004861c        0x5 ..\..\..\Libraries\libs\libbtstack_master.a(ll_adv.o)
 *(.rela*)
 .rela.text.bsp_bt_init
                0x0000000010048621        0x0 Output\obj\Libraries\bsp\bsp_bt.o
 .rela.text.bsp_spp_disinit
                0x0000000010048621        0x0 Output\obj\Libraries\bsp\bsp_bt.o
 .rela.text.bt_emit_notice
                0x0000000010048621        0x0 Output\obj\Libraries\bsp\bsp_bt.o
 .rela.text.cm_factory
                0x0000000010048621        0x0 Output\obj\Libraries\bsp\bsp_bt.o
 .rela.text.fot.cache
                0x0000000010048621        0x0 Output\obj\Libraries\bsp\bsp_bt.o
 .rela.text.fot.update
                0x0000000010048621        0x0 Output\obj\Libraries\bsp\bsp_bt.o
 .rela.text.fot_ble_disconnect_callback
                0x0000000010048621        0x0 Output\obj\Libraries\bsp\bsp_bt.o
 .rela.text.fot_ble_connect_callback
                0x0000000010048621        0x0 Output\obj\Libraries\bsp\bsp_bt.o
 .rela.text.fot_spp_connect_callback
                0x0000000010048621        0x0 Output\obj\Libraries\bsp\bsp_bt.o
 .rela.text.fot_spp_disconnect_callback
                0x0000000010048621        0x0 Output\obj\Libraries\bsp\bsp_bt.o
 .rela.com_text.fot
                0x0000000010048621        0x0 Output\obj\Libraries\bsp\bsp_bt.o
 .rela.text.bsp.param
                0x0000000010048621        0x0 Output\obj\Libraries\bsp\bsp_bt.o
 .rela.text.bsp.sys.init
                0x0000000010048621        0x0 Output\obj\Libraries\bsp\bsp_bt.o
 .rela.com_text.timer
                0x0000000010048621        0x0 Output\obj\Libraries\bsp\bsp_bt.o
 .rela.text.bsp_get_xosc_xcfg
                0x0000000010048621        0x0 Output\obj\Libraries\bsp\bsp_bt.o
 .rela.text.gatt_callback_fota
                0x0000000010048621        0x0 Output\obj\Libraries\bsp\bsp_bt.o
 .rela.text.gatt_callback_app
                0x0000000010048621        0x0 Output\obj\Libraries\bsp\bsp_bt.o
 .rela.text.ble_get_scan_data
                0x0000000010048621        0x0 Output\obj\Libraries\bsp\bsp_bt.o
 .rela.text.ble_get_adv_data
                0x0000000010048621        0x0 Output\obj\Libraries\bsp\bsp_bt.o
 .rela.text.ble_txpkt_init
                0x0000000010048621        0x0 Output\obj\Libraries\bsp\bsp_bt.o
 .rela.text.ble_service_change_indicate
                0x0000000010048621        0x0 Output\obj\Libraries\bsp\bsp_bt.o
 .rela.text.ble_send_packet1
                0x0000000010048621        0x0 Output\obj\Libraries\bsp\bsp_bt.o
 .rela.text.ble_send_packet2
                0x0000000010048621        0x0 Output\obj\Libraries\bsp\bsp_bt.o
 .rela.text.ble_read_value
                0x0000000010048621        0x0 Output\obj\Libraries\bsp\bsp_bt.o
 .rela.text.ble_fot_send_packet
                0x0000000010048621        0x0 Output\obj\Libraries\bsp\bsp_bt.o
 .rela.text.ble_app_gatts_service_init
                0x0000000010048621        0x0 Output\obj\Libraries\bsp\bsp_bt.o
 .rela.text.ble_client_cfg_callback
                0x0000000010048621        0x0 Output\obj\Libraries\bsp\bsp_bt.o
 .rela.text.ble_slave_process
                0x0000000010048621        0x0 Output\obj\Libraries\bsp\bsp_bt.o
 .rela.text.ble_get_local_bd_addr
                0x0000000010048621        0x0 Output\obj\Libraries\bsp\bsp_bt.o
 .rela.text.ble_enter_transmit
                0x0000000010048621        0x0 Output\obj\Libraries\bsp\bsp_bt.o
 .rela.text.ble_exit_transmit
                0x0000000010048621        0x0 Output\obj\Libraries\bsp\bsp_bt.o
 .rela.text.ble_disconnect_callback
                0x0000000010048621        0x0 Output\obj\Libraries\bsp\bsp_bt.o
 .rela.text.ble_connect_callback
                0x0000000010048621        0x0 Output\obj\Libraries\bsp\bsp_bt.o
 .rela.text.bt_get_local_name
                0x0000000010048621        0x0 Output\obj\Libraries\bsp\bsp_bt.o
 .rela.text.bt_clr_all_link_info
                0x0000000010048621        0x0 Output\obj\Libraries\bsp\bsp_bt.o
 .rela.text.bt_get_local_bd_addr
                0x0000000010048621        0x0 Output\obj\Libraries\bsp\bsp_bt.o
 .rela.text.bt_get_link_info
                0x0000000010048621        0x0 Output\obj\Libraries\bsp\bsp_bt.o
 .rela.text.bt_put_link_info
                0x0000000010048621        0x0 Output\obj\Libraries\bsp\bsp_bt.o
 .rela.text.bt_get_ext_link_info
                0x0000000010048621        0x0 Output\obj\Libraries\bsp\bsp_bt.o
 .rela.text.bt_put_ext_link_info
                0x0000000010048621        0x0 Output\obj\Libraries\bsp\bsp_bt.o
 .rela.text.bt_sync_link_info
                0x0000000010048621        0x0 Output\obj\Libraries\bsp\bsp_bt.o
 .rela.text.bsp_bt_hid_screen_left
                0x0000000010048621        0x0 Output\obj\Libraries\bsp\bsp_bt.o
 .rela.text.bsp_bt_hid_screen_right
                0x0000000010048621        0x0 Output\obj\Libraries\bsp\bsp_bt.o
 .rela.data     0x0000000010048621        0x0 Output\obj\Libraries\bsp\bsp_bt.o
 .rela.text.bt_init_lib
                0x0000000010048621        0x0 Output\obj\Libraries\bsp\bsp_bt.o
 .rela.text.spp_txpkt_init
                0x0000000010048621        0x0 Output\obj\Libraries\bsp\bsp_bt.o
 .rela.text.spp_connect_callback
                0x0000000010048621        0x0 Output\obj\Libraries\bsp\bsp_bt.o
 .rela.text.spp_disconnect_callback
                0x0000000010048621        0x0 Output\obj\Libraries\bsp\bsp_bt.o
 .rela.text.spp_rx_callback
                0x0000000010048621        0x0 Output\obj\Libraries\bsp\bsp_bt.o
 .rela.text.gpio_pic_config
                0x0000000010048621        0x0 Output\obj\Libraries\bsp\bsp_bt.o
 .rela.com_text.hsuart
                0x0000000010048621        0x0 Output\obj\Libraries\bsp\bsp_bt.o
 .rela.text.hsuart_pic_config
                0x0000000010048621        0x0 Output\obj\Libraries\bsp\bsp_bt.o
 .rela.text.ble_att_read_callback
                0x0000000010048621        0x0 Output\obj\Libraries\bsp\bsp_bt.o
 .rela.text.ble_clent_event_packet_handle
                0x0000000010048621        0x0 Output\obj\Libraries\bsp\bsp_bt.o
 .rela.text.ble_client_notify_callback
                0x0000000010048621        0x0 Output\obj\Libraries\bsp\bsp_bt.o
 .rela.text.ble_client_init
                0x0000000010048621        0x0 Output\obj\Libraries\bsp\bsp_bt.o
 .rela.text.ble_client_user_process
                0x0000000010048621        0x0 Output\obj\Libraries\bsp\bsp_bt.o
 .rela.text.hsuart_transfer_example
                0x0000000010048621        0x0 Output\obj\Libraries\bsp\bsp_bt.o
 .rela.text.btstack_ble_init_callback
                0x0000000010048621        0x0 Output\obj\Libraries\bsp\bsp_bt.o
 .rela.text.ble_init_register
                0x0000000010048621        0x0 Output\obj\Libraries\bsp\bsp_bt.o
 .rela.text.gpio_input_init
                0x0000000010048621        0x0 Output\obj\Libraries\bsp\bsp_bt.o
 .rela.com_text.isr
                0x0000000010048621        0x0 Output\obj\Libraries\bsp\bsp_bt.o
 .rela.text.my_hsuart_init
                0x0000000010048621        0x0 Output\obj\Libraries\bsp\bsp_bt.o
 .rela.text.huart_SendByte
                0x0000000010048621        0x0 Output\obj\Libraries\bsp\bsp_bt.o
 .rela.text.huart_SendArray
                0x0000000010048621        0x0 Output\obj\Libraries\bsp\bsp_bt.o
 .rela.text.huart_SendString
                0x0000000010048621        0x0 Output\obj\Libraries\bsp\bsp_bt.o
 .rela.text.huart_SendNumber
                0x0000000010048621        0x0 Output\obj\Libraries\bsp\bsp_bt.o
 .rela.text.getcfg_vddbt_sel
                0x0000000010048621        0x0 Output\obj\Libraries\bsp\bsp_bt.o
 .rela.text.getcfg_vddio_sel
                0x0000000010048621        0x0 Output\obj\Libraries\bsp\bsp_bt.o
 .rela.text.getcfg_vddbt_capless_en
                0x0000000010048621        0x0 Output\obj\Libraries\bsp\bsp_bt.o
 .rela.text.startup.main
                0x0000000010048621        0x0 Output\obj\Libraries\bsp\bsp_bt.o
 .rela.text.pll_vco_band_trimming
                0x0000000010048621        0x0 Output\obj\Libraries\bsp\bsp_bt.o
 .rela.com_text.dac
                0x0000000010048621        0x0 Output\obj\Libraries\bsp\bsp_bt.o
 .rela.text.adpll_divider_update_do
                0x0000000010048621        0x0 Output\obj\Libraries\bsp\bsp_bt.o
 .rela.text.adpll_divider_update
                0x0000000010048621        0x0 Output\obj\Libraries\bsp\bsp_bt.o
 .rela.text.adpll_init
                0x0000000010048621        0x0 Output\obj\Libraries\bsp\bsp_bt.o
 .rela.text.spires
                0x0000000010048621        0x0 Output\obj\Libraries\bsp\bsp_bt.o
 .rela.text.cm_loadpage
                0x0000000010048621        0x0 Output\obj\Libraries\bsp\bsp_bt.o
 .rela.text.cm_next_freepage
                0x0000000010048621        0x0 Output\obj\Libraries\bsp\bsp_bt.o
 .rela.text.cm_movepage
                0x0000000010048621        0x0 Output\obj\Libraries\bsp\bsp_bt.o
 .rela.text.cm_move_allpages
                0x0000000010048621        0x0 Output\obj\Libraries\bsp\bsp_bt.o
 .rela.text.cm_release
                0x0000000010048621        0x0 Output\obj\Libraries\bsp\bsp_bt.o
 .rela.text.cm_savepage
                0x0000000010048621        0x0 Output\obj\Libraries\bsp\bsp_bt.o
 .rela.text.cm_check_loadpage
                0x0000000010048621        0x0 Output\obj\Libraries\bsp\bsp_bt.o
 .rela.text.cm_sync
                0x0000000010048621        0x0 Output\obj\Libraries\bsp\bsp_bt.o
 .rela.text.cm_release_all
                0x0000000010048621        0x0 Output\obj\Libraries\bsp\bsp_bt.o
 .rela.text.cm_read
                0x0000000010048621        0x0 Output\obj\Libraries\bsp\bsp_bt.o
 .rela.text.cm_read8
                0x0000000010048621        0x0 Output\obj\Libraries\bsp\bsp_bt.o
 .rela.text.cm_read16
                0x0000000010048621        0x0 Output\obj\Libraries\bsp\bsp_bt.o
 .rela.text.cm_read32
                0x0000000010048621        0x0 Output\obj\Libraries\bsp\bsp_bt.o
 .rela.text.cm_write
                0x0000000010048621        0x0 Output\obj\Libraries\bsp\bsp_bt.o
 .rela.text.cm_write8
                0x0000000010048621        0x0 Output\obj\Libraries\bsp\bsp_bt.o
 .rela.text.cm_write16
                0x0000000010048621        0x0 Output\obj\Libraries\bsp\bsp_bt.o
 .rela.text.cm_write32
                0x0000000010048621        0x0 Output\obj\Libraries\bsp\bsp_bt.o
 .rela.text.cm_clear
                0x0000000010048621        0x0 Output\obj\Libraries\bsp\bsp_bt.o
 .rela.text.cm_init
                0x0000000010048621        0x0 Output\obj\Libraries\bsp\bsp_bt.o
 .rela.com_text.spiflash
                0x0000000010048621        0x0 Output\obj\Libraries\bsp\bsp_bt.o
 .rela.text.xcfg_init
                0x0000000010048621        0x0 Output\obj\Libraries\bsp\bsp_bt.o
 .rela.text.sd_disable_user
                0x0000000010048621        0x0 Output\obj\Libraries\bsp\bsp_bt.o
 .rela.text.device.init
                0x0000000010048621        0x0 Output\obj\Libraries\bsp\bsp_bt.o
 .rela.text.device
                0x0000000010048621        0x0 Output\obj\Libraries\bsp\bsp_bt.o
 .rela.com_text.sd.isr
                0x0000000010048621        0x0 Output\obj\Libraries\bsp\bsp_bt.o
 .rela.com_text.sd.api
                0x0000000010048621        0x0 Output\obj\Libraries\bsp\bsp_bt.o
 .rela.text.fs_lock
                0x0000000010048621        0x0 Output\obj\Libraries\bsp\bsp_bt.o
 .rela.text.fs_unlock
                0x0000000010048621        0x0 Output\obj\Libraries\bsp\bsp_bt.o
 .rela.com_text.exception.hook
                0x0000000010048621        0x0 Output\obj\Libraries\bsp\bsp_bt.o
 .rela.com_text.exception
                0x0000000010048621        0x0 Output\obj\Libraries\bsp\bsp_bt.o
 .rela.com_text.delay
                0x0000000010048621        0x0 Output\obj\Libraries\bsp\bsp_bt.o
 .rela.com_text.exception.do
                0x0000000010048621        0x0 Output\obj\Libraries\bsp\bsp_bt.o
 .rela.com_text.ledseg
                0x0000000010048621        0x0 Output\obj\Libraries\bsp\bsp_bt.o
 .rela.text.platform_main
                0x0000000010048621        0x0 Output\obj\Libraries\bsp\bsp_bt.o
 .rela.text.main_startup
                0x0000000010048621        0x0 Output\obj\Libraries\bsp\bsp_bt.o
 .rela.text.compiler
                0x0000000010048621        0x0 Output\obj\Libraries\bsp\bsp_bt.o
 .rela.com_text.irq
                0x0000000010048621        0x0 Output\obj\Libraries\bsp\bsp_bt.o
 .rela.text.sys_irq_init
                0x0000000010048621        0x0 Output\obj\Libraries\bsp\bsp_bt.o
 .rela.text.timer0_init
                0x0000000010048621        0x0 Output\obj\Libraries\bsp\bsp_bt.o
 .rela.text.soft_irq_init
                0x0000000010048621        0x0 Output\obj\Libraries\bsp\bsp_bt.o
 .rela.text.bthw_irq_init
                0x0000000010048621        0x0 Output\obj\Libraries\bsp\bsp_bt.o
 .rela.text.sd0_irq_init
                0x0000000010048621        0x0 Output\obj\Libraries\bsp\bsp_bt.o
 .rela.text.usb_irq_init
                0x0000000010048621        0x0 Output\obj\Libraries\bsp\bsp_bt.o
 .rela.text.timer1_irq_init
                0x0000000010048621        0x0 Output\obj\Libraries\bsp\bsp_bt.o
 .rela.com_text.tws.isr
                0x0000000010048621        0x0 Output\obj\Libraries\bsp\bsp_bt.o
 .rela.text.aubuf_irq_init
                0x0000000010048621        0x0 Output\obj\Libraries\bsp\bsp_bt.o
 .rela.text.huart_irq_init
                0x0000000010048621        0x0 Output\obj\Libraries\bsp\bsp_bt.o
 .rela.text.watch_point_set
                0x0000000010048621        0x0 Output\obj\Libraries\bsp\bsp_bt.o
 .rela.text.thread_main_entry
                0x0000000010048621        0x0 Output\obj\Libraries\bsp\bsp_bt.o
 .rela.text.thread_idle_create
                0x0000000010048621        0x0 Output\obj\Libraries\bsp\bsp_bt.o
 .rela.text.startup.init
                0x0000000010048621        0x0 Output\obj\Libraries\bsp\bsp_bt.o
 .rela.reset    0x0000000010048621        0x0 Output\obj\Libraries\bsp\bsp_bt.o
 .rela.vector   0x0000000010048621        0x0 Output\obj\Libraries\bsp\bsp_bt.o
 .rela.com_text.debug
                0x0000000010048621        0x0 Output\obj\Libraries\bsp\bsp_bt.o
 .rela.text.fot_init
                0x0000000010048621        0x0 Output\obj\Libraries\bsp\bsp_bt.o
 .rela.text.lock_code_bt_sleep
                0x0000000010048621        0x0 Output\obj\Libraries\bsp\bsp_bt.o
 .rela.text.lock_code_pwrsave
                0x0000000010048621        0x0 Output\obj\Libraries\bsp\bsp_bt.o
 .rela.text.lock_code_charge
                0x0000000010048621        0x0 Output\obj\Libraries\bsp\bsp_bt.o
 .rela.text.lock_code_usbdev
                0x0000000010048621        0x0 Output\obj\Libraries\bsp\bsp_bt.o
 .rela.text.load_code_btdec
                0x0000000010048621        0x0 Output\obj\Libraries\bsp\bsp_bt.o
 .rela.text.load_code_bt_voice
                0x0000000010048621        0x0 Output\obj\Libraries\bsp\bsp_bt.o
 .rela.text.lock_code_sniff
                0x0000000010048621        0x0 Output\obj\Libraries\bsp\bsp_bt.o
 .rela.text.lock_code_huart
                0x0000000010048621        0x0 Output\obj\Libraries\bsp\bsp_bt.o
 .rela.text.lock_code_bb_test
                0x0000000010048621        0x0 Output\obj\Libraries\bsp\bsp_bt.o
 .rela.text.load_code_fota
                0x0000000010048621        0x0 Output\obj\Libraries\bsp\bsp_bt.o
 .rela.text.patch_init
                0x0000000010048621        0x0 Output\obj\Libraries\bsp\bsp_bt.o
 .rela.text.vddio_voltage_configure
                0x0000000010048621        0x0 Output\obj\Libraries\bsp\bsp_bt.o
 .rela.text.vddbt_voltage_configure
                0x0000000010048621        0x0 Output\obj\Libraries\bsp\bsp_bt.o
 .rela.text.pmu_voltage_configure
                0x0000000010048621        0x0 Output\obj\Libraries\bsp\bsp_bt.o
 .rela.text.pmu_init
                0x0000000010048621        0x0 Output\obj\Libraries\bsp\bsp_bt.o
 .rela.com_text.voltage.trim
                0x0000000010048621        0x0 Output\obj\Libraries\bsp\bsp_bt.o
 .rela.text.sys_clk
                0x0000000010048621        0x0 Output\obj\Libraries\bsp\bsp_bt.o
 .rela.text.set_peripherals_clkdiv
                0x0000000010048621        0x0 Output\obj\Libraries\bsp\bsp_bt.o
 .rela.com_huart.text
                0x0000000010048621        0x0 Output\obj\Libraries\bsp\bsp_bt.o
 .rela.com_text.thread.usb
                0x0000000010048621        0x0 Output\obj\Libraries\bsp\bsp_bt.o
 .rela.bt_voice.plc
                0x0000000010048621        0x0 Output\obj\Libraries\bsp\bsp_bt.o
 .rela.text.stack.api
                0x0000000010048621        0x0 Output\obj\Libraries\bsp\bsp_bt.o
 .rela.com_text.stack.run_loop
                0x0000000010048621        0x0 Output\obj\Libraries\bsp\bsp_bt.o
 .rela.com_text.bb.bthw
                0x0000000010048621        0x0 Output\obj\Libraries\bsp\bsp_bt.o
 .rela.com_text.usbdev
                0x0000000010048621        0x0 Output\obj\Libraries\bsp\bsp_bt.o
 .rela.usbdev.com
                0x0000000010048621        0x0 Output\obj\Libraries\bsp\bsp_bt.o
 .rela.com_text.bulkep
                0x0000000010048621        0x0 Output\obj\Libraries\bsp\bsp_bt.o
 .rela.text.udp_init
                0x0000000010048621        0x0 Output\obj\Libraries\bsp\bsp_bt.o
 .rela.text.usb_device_init
                0x0000000010048621        0x0 Output\obj\Libraries\bsp\bsp_bt.o
 .rela.text.usb_device_enter
                0x0000000010048621        0x0 Output\obj\Libraries\bsp\bsp_bt.o
 .rela.com_text.usb.device
                0x0000000010048621        0x0 Output\obj\Libraries\bsp\bsp_bt.o
 .rela.text.usb.host.init
                0x0000000010048621        0x0 Output\obj\Libraries\bsp\bsp_bt.o
 .rela.com_text.usb.host
                0x0000000010048621        0x0 Output\obj\Libraries\bsp\bsp_bt.o
 .rela.text.udisk_read
                0x0000000010048621        0x0 Output\obj\Libraries\bsp\bsp_bt.o
 .rela.text.udisk_write
                0x0000000010048621        0x0 Output\obj\Libraries\bsp\bsp_bt.o
 .rela.text.do_transfer
                0x0000000010048621        0x0 Output\obj\Libraries\bsp\bsp_bt.o
 .rela.text.do_receive
                0x0000000010048621        0x0 Output\obj\Libraries\bsp\bsp_bt.o
 .rela.text.uhs_start
                0x0000000010048621        0x0 Output\obj\Libraries\bsp\bsp_bt.o
 .rela.text.uhs_init
                0x0000000010048621        0x0 Output\obj\Libraries\bsp\bsp_bt.o
 .rela.text.usb_init
                0x0000000010048621        0x0 Output\obj\Libraries\bsp\bsp_bt.o
 .rela.text.usb_host_enter
                0x0000000010048621        0x0 Output\obj\Libraries\bsp\bsp_bt.o
 .rela.text.uhe_start
                0x0000000010048621        0x0 Output\obj\Libraries\bsp\bsp_bt.o
 .rela.text     0x0000000010048621        0x0 Output\obj\Libraries\bsp\bsp_bt.o
 .rela.com_text.bb.nanos
                0x0000000010048621        0x0 Output\obj\Libraries\bsp\bsp_bt.o
 .rela.com_text.bb.patch
                0x0000000010048621        0x0 Output\obj\Libraries\bsp\bsp_bt.o
 .rela.com_text.ble.isr.con
                0x0000000010048621        0x0 Output\obj\Libraries\bsp\bsp_bt.o
 .rela.com_text.bb.isr.timer
                0x0000000010048621        0x0 Output\obj\Libraries\bsp\bsp_bt.o
 .rela.com_text.bb.isr
                0x0000000010048621        0x0 Output\obj\Libraries\bsp\bsp_bt.o
 .rela.sleep_text.bb
                0x0000000010048621        0x0 Output\obj\Libraries\bsp\bsp_bt.o
 .rela.com_text.bb.sleep
                0x0000000010048621        0x0 Output\obj\Libraries\bsp\bsp_bt.o
 .rela.com_text.bb.btisr
                0x0000000010048621        0x0 Output\obj\Libraries\bsp\bsp_bt.o
 .rela.rodata   0x0000000010048621        0x0 Output\obj\Libraries\bsp\bsp_bt.o
 .rela.com_text.pp.send_pkt
                0x0000000010048621        0x0 Output\obj\Libraries\bsp\bsp_bt.o
 .rela.com_text.spp.tx
                0x0000000010048621        0x0 Output\obj\Libraries\bsp\bsp_bt.o
 .rela.com_text.spp.send_req
                0x0000000010048621        0x0 Output\obj\Libraries\bsp\bsp_bt.o
 .rela.com_text.spp.event_send
                0x0000000010048621        0x0 Output\obj\Libraries\bsp\bsp_bt.o
 .rela.com_text.spp.rx_set_new_credit
                0x0000000010048621        0x0 Output\obj\Libraries\bsp\bsp_bt.o
 .rela.text.stack.spp.handler
                0x0000000010048621        0x0 Output\obj\Libraries\bsp\bsp_bt.o
 .rela.text.stack.sdp.util
                0x0000000010048621        0x0 Output\obj\Libraries\bsp\bsp_bt.o
 .rela.text.stack.sdp.server
                0x0000000010048621        0x0 Output\obj\Libraries\bsp\bsp_bt.o
 .rela.text.stack.setup
                0x0000000010048621        0x0 Output\obj\Libraries\bsp\bsp_bt.o
 .rela.text.stack.sdp.server_add
                0x0000000010048621        0x0 Output\obj\Libraries\bsp\bsp_bt.o
 .rela.text.stack.sdp.server_rmv
                0x0000000010048621        0x0 Output\obj\Libraries\bsp\bsp_bt.o
 .rela.text.stack.rfcomm
                0x0000000010048621        0x0 Output\obj\Libraries\bsp\bsp_bt.o
 .rela.text.stack.link_key
                0x0000000010048621        0x0 Output\obj\Libraries\bsp\bsp_bt.o
 .rela.text.stack.run_loop
                0x0000000010048621        0x0 Output\obj\Libraries\bsp\bsp_bt.o
 .rela.com_text.stack.ticks
                0x0000000010048621        0x0 Output\obj\Libraries\bsp\bsp_bt.o
 .rela.text.stack.memory
                0x0000000010048621        0x0 Output\obj\Libraries\bsp\bsp_bt.o
 .rela.text.stack.linkctrl
                0x0000000010048621        0x0 Output\obj\Libraries\bsp\bsp_bt.o
 .rela.com_text.ble.send_pkt
                0x0000000010048621        0x0 Output\obj\Libraries\bsp\bsp_bt.o
 .rela.text.att.r_cb
                0x0000000010048621        0x0 Output\obj\Libraries\bsp\bsp_bt.o
 .rela.text.att.w_cb
                0x0000000010048621        0x0 Output\obj\Libraries\bsp\bsp_bt.o
 .rela.com_text.stack.ble.mtu
                0x0000000010048621        0x0 Output\obj\Libraries\bsp\bsp_bt.o
 .rela.text.ble.notify_handle
                0x0000000010048621        0x0 Output\obj\Libraries\bsp\bsp_bt.o
 .rela.text.ble.att
                0x0000000010048621        0x0 Output\obj\Libraries\bsp\bsp_bt.o
 .rela.text.stack.handler
                0x0000000010048621        0x0 Output\obj\Libraries\bsp\bsp_bt.o
 .rela.text.stack.status
                0x0000000010048621        0x0 Output\obj\Libraries\bsp\bsp_bt.o
 .rela.rodata.stack.api
                0x0000000010048621        0x0 Output\obj\Libraries\bsp\bsp_bt.o
 .rela.text.stack.api.hid_con
                0x0000000010048621        0x0 Output\obj\Libraries\bsp\bsp_bt.o
 .rela.text.stack.api.hid_disc
                0x0000000010048621        0x0 Output\obj\Libraries\bsp\bsp_bt.o
 .rela.text.stack.api.hid_send
                0x0000000010048621        0x0 Output\obj\Libraries\bsp\bsp_bt.o
 .rela.text.ble.api.conn
                0x0000000010048621        0x0 Output\obj\Libraries\bsp\bsp_bt.o
 .rela.text.bb.vs.fcc
                0x0000000010048621        0x0 Output\obj\Libraries\bsp\bsp_bt.o
 .rela.com_text.isr.txrx
                0x0000000010048621        0x0 Output\obj\Libraries\bsp\bsp_bt.o
 .rela.com_text.bt21.isr
                0x0000000010048621        0x0 Output\obj\Libraries\bsp\bsp_bt.o
 .rela.text.ble.var.init
                0x0000000010048621        0x0 Output\obj\Libraries\bsp\bsp_bt.o
 .rela.text.stk.l2cap.txreq
                0x0000000010048621        0x0 Output\obj\Libraries\bsp\bsp_bt.o
 .rela.text.stack.handler.l2cap
                0x0000000010048621        0x0 Output\obj\Libraries\bsp\bsp_bt.o
 .rela.text.stack.l2cap
                0x0000000010048621        0x0 Output\obj\Libraries\bsp\bsp_bt.o
 .rela.text.stack.hci
                0x0000000010048621        0x0 Output\obj\Libraries\bsp\bsp_bt.o
 .rela.text.stack.hci_init
                0x0000000010048621        0x0 Output\obj\Libraries\bsp\bsp_bt.o
 .rela.com_text.stack.hci
                0x0000000010048621        0x0 Output\obj\Libraries\bsp\bsp_bt.o
 .rela.text.stack.hci_send
                0x0000000010048621        0x0 Output\obj\Libraries\bsp\bsp_bt.o
 .rela.text.stack.hci.run
                0x0000000010048621        0x0 Output\obj\Libraries\bsp\bsp_bt.o
 .rela.text.stack.handler.event
                0x0000000010048621        0x0 Output\obj\Libraries\bsp\bsp_bt.o
 .rela.com_text.stack.hci_recv
                0x0000000010048621        0x0 Output\obj\Libraries\bsp\bsp_bt.o
 .rela.text.stack.hfp.api1
                0x0000000010048621        0x0 Output\obj\Libraries\bsp\bsp_bt.o
 .rela.text.bb.lm.inq.start
                0x0000000010048621        0x0 Output\obj\Libraries\bsp\bsp_bt.o
 .rela.text.le.ll_cntl
                0x0000000010048621        0x0 Output\obj\Libraries\bsp\bsp_bt.o
 .rela.text.le.ll_cntl.start
                0x0000000010048621        0x0 Output\obj\Libraries\bsp\bsp_bt.o
 .rela.text.le.ll_cntl.state
                0x0000000010048621        0x0 Output\obj\Libraries\bsp\bsp_bt.o
 .rela.text.le.ll_cntl.stop
                0x0000000010048621        0x0 Output\obj\Libraries\bsp\bsp_bt.o
 .rela.text.bb.ble.adv0
                0x0000000010048621        0x0 Output\obj\Libraries\bsp\bsp_bt.o
 .rela.text.le.mgr
                0x0000000010048621        0x0 Output\obj\Libraries\bsp\bsp_bt.o
 .rela.rodata.le.mgr_cntl.tbl
                0x0000000010048621        0x0 Output\obj\Libraries\bsp\bsp_bt.o
 .rela.text.le.ll_scan
                0x0000000010048621        0x0 Output\obj\Libraries\bsp\bsp_bt.o
 .rela.text.le.ll_adv
                0x0000000010048621        0x0 Output\obj\Libraries\bsp\bsp_bt.o
 .rela.text.le.ll_adv.con
                0x0000000010048621        0x0 Output\obj\Libraries\bsp\bsp_bt.o
 .rela.com_rodata.bb.tbl
                0x0000000010048621        0x0 Output\obj\Libraries\bsp\bsp_bt.o
 .rela.rodata.le.ll_cntl.tbl
                0x0000000010048621        0x0 Output\obj\Libraries\bsp\bsp_bt.o
 .rela.text.le.ll_cntl.pdu
                0x0000000010048621        0x0 Output\obj\Libraries\bsp\bsp_bt.o
 .rela.text.le.ll_cntl.send
                0x0000000010048621        0x0 Output\obj\Libraries\bsp\bsp_bt.o
                0x0000000010048621        0x4 LONG 0x0
                0x0000000010048800                . = ALIGN (0x200)
 *fill*         0x0000000010048625      0x1db 

.stack          0x0000000000010800      0x400
                0x0000000000010800                __irq_stack_start = .
                0x0000000000000400                . = 0x400
 *fill*         0x0000000000010800      0x400 
                0x0000000000010c00                __irq_stack = .
                0x0000000000000400                __irq_stack_size = (__irq_stack - __irq_stack_start)

.bss            0x0000000000013c00     0x1f44
                0x0000000000013c00                __bss_start = .
 *(COMMON)
 COMMON         0x0000000000013c00        0x7 Output\obj\Libraries\bsp\bsp_bt.o
                0x0000000000013c00                f_bt
 *fill*         0x0000000000013c07        0x1 
 COMMON         0x0000000000013c08       0x22 Output\obj\Libraries\bsp\bsp_fot.o
                0x0000000000013c08                fot_var
 *fill*         0x0000000000013c2a        0x2 
 COMMON         0x0000000000013c2c       0xb2 Output\obj\Libraries\bsp\bsp_sys.o
                0x0000000000013c2c                ticks_50ms
                0x0000000000013c30                xcfg_cb
 *fill*         0x0000000000013cde        0x2 
 COMMON         0x0000000000013ce0      0x604 Output\obj\Examples\BLE_Host\Source\hsuart_transfer.o
                0x0000000000013ce0                RECEIVE_BUF
                0x0000000000013ee0                TRANSMIT_BUF
                0x00000000000142e0                BtTxBuferCount
                0x00000000000142e2                RECEIVE_Len
 *(.bss*)
 .bss           0x00000000000142e4      0x188 Output\obj\Examples\BLE_Host\Source\ble_client.o
 .bss           0x000000000001446c      0x22c ..\..\..\Libraries\libs\libplatform.a(cm.o)
 .bss           0x0000000000014698       0xa0 ..\..\..\Libraries\libs\libplatform.a(main.o)
                0x0000000000014698                cpu_gprs
                0x0000000000014718                sys
 .bss.irq_tbl   0x0000000000014738       0x84 ..\..\..\Libraries\libs\libplatform.a(interrupt.o)
                0x0000000000014738                tbl_irq_vector
                0x00000000000147b8                irq_mask
 .bss           0x00000000000147bc       0x28 ..\..\..\Libraries\libs\libplatform.a(startup.o)
 .bss           0x00000000000147e4       0x20 ..\..\..\Libraries\libs\libplatform.a(fot_update.o)
 *fill*         0x0000000000014804        0x4 
 .bss           0x0000000000014808       0x78 ..\..\..\Libraries\libs\libplatform.a(lock.o)
 .bss           0x0000000000014880        0xc ..\..\..\Libraries\libs\libplatform.a(voltage_trim.o)
                0x0000000000014880                sys_trim
 .bss           0x000000000001488c       0x24 ..\..\..\Libraries\libs\libdrivers.a(usb_device_ep.o)
                0x000000000001488c                eps
 .bss           0x00000000000148b0        0x9 ..\..\..\Libraries\libs\libbtstack_master.a(bb.o)
                0x00000000000148b0                rf_api
 *fill*         0x00000000000148b9        0x3 
 .bss           0x00000000000148bc       0x3e ..\..\..\Libraries\libs\libbtstack_master.a(btstack_link_key_db.o)
 *fill*         0x00000000000148fa        0x2 
 .bss           0x00000000000148fc      0x4fc ..\..\..\Libraries\libs\libbtstack_master.a(btstack_memory.o)
 .bss           0x0000000000014df8       0x10 ..\..\..\Libraries\libs\libbtstack_master.a(sm.o)
 .bss           0x0000000000014e08       0x48 ..\..\..\Libraries\libs\libbtstack_master.a(btstack_api.o)
                0x0000000000014e08                btstack_cb
                0x0000000000014e14                btstack_st
 .bss           0x0000000000014e50      0x184 ..\..\..\Libraries\libs\libbtstack_master.a(bb_sche.o)
                0x0000000000014e50                ss_params
 .bss           0x0000000000014fd4        0xc ..\..\..\Libraries\libs\libbtstack_master.a(aes.o)
                0x0000000000014fd4                aes_env
 .bss           0x0000000000014fe0       0x24 ..\..\..\Libraries\libs\libbtstack_master.a(hct_tl.o)
 .bss           0x0000000000015004       0x26 ..\..\..\Libraries\libs\libbtstack_master.a(bc.o)
                0x0000000000015004                bc_env
 *fill*         0x000000000001502a        0x2 
 .bss           0x000000000001502c       0x40 ..\..\..\Libraries\libs\libbtstack_master.a(l2cap_test.o)
                0x000000000001502c                vd_tx
 .bss           0x000000000001506c       0xc0 ..\..\..\Libraries\libs\libbtstack_master.a(lm_sp.o)
 .bss           0x000000000001512c      0x100 ..\..\..\Libraries\libs\libbtstack_master.a(ble_buf.o)
 .bss           0x000000000001522c      0x21c ..\..\..\Libraries\libs\libbtstack_master.a(ll_proc.o)
 *(.sbss*)
 .sbss          0x0000000000015448        0x4 Output\obj\Libraries\bsp\bsp_fot.o
 .sbss          0x000000000001544c       0x23 Output\obj\Libraries\BT\ble\ab_link\app.o
                0x0000000000015450                str
                0x000000000001546e                battery_client_config
 .sbss          0x000000000001546f        0x1 Output\obj\Libraries\BT\ble\ble.o
 .sbss          0x0000000000015470        0xc Output\obj\Libraries\BT\spp\bt.o
                0x0000000000015470                cfg_bt_hid_type
                0x0000000000015472                cfg_bt_support_codec
                0x0000000000015474                cfg_bt_simple_pair_mode
                0x0000000000015475                cfg_bt_scan_ctrl_mode
                0x0000000000015476                cfg_bt_work_mode
                0x0000000000015477                cfg_ble_page_rssi_thr
                0x0000000000015478                cfg_ble_page_txpwr
                0x0000000000015479                cfg_bt_inq_txpwr
                0x000000000001547a                cfg_bt_page_txpwr
                0x000000000001547b                cfg_bt_rf_def_txpwr
 .sbss          0x000000000001547c        0x2 Output\obj\Libraries\BT\spp\spp.o
                0x000000000001547c                SPP_CreditCount
                0x000000000001547d                BtFlowControl_start
 *fill*         0x000000000001547e        0x2 
 .sbss          0x0000000000015480        0xc Output\obj\Examples\BLE_Host\Source\ble_client.o
                0x0000000000015484                write_handler
 .sbss          0x000000000001548c        0x8 ..\..\..\Libraries\libs\libplatform.a(audio.o)
                0x0000000000015490                aux_cur_gain
 .sbss          0x0000000000015494        0x8 ..\..\..\Libraries\libs\libplatform.a(os_flash.o)
                0x0000000000015494                spi_baud_w
                0x0000000000015498                spi_baud_r
 .sbss          0x000000000001549c        0xc ..\..\..\Libraries\libs\libplatform.a(interrupt.o)
                0x000000000001549c                tmr5ms_cnt
                0x00000000000154a0                ms_tick
                0x00000000000154a4                tmr0_counter
 .sbss          0x00000000000154a8       0x3c ..\..\..\Libraries\libs\libplatform.a(startup.o)
                0x00000000000154a8                user_timer_isr_en
                0x00000000000154ac                bt_timer_isr_en
                0x00000000000154b0                pmutex_pff
                0x00000000000154b4                pmutex_bt_sta
                0x00000000000154b8                pmutex_math
                0x00000000000154bc                pmutex_dac
                0x00000000000154c0                pmutex_uart
                0x00000000000154c4                pmutex_clk
                0x00000000000154c8                pmutex_cm
                0x00000000000154cc                pmq_usb
                0x00000000000154d0                pmq_btstack
                0x00000000000154d4                psem_sd
                0x00000000000154d8                psem_aubuf
                0x00000000000154dc                psem_btstack
                0x00000000000154e0                psem_bthw
 .sbss          0x00000000000154e4        0xc ..\..\..\Libraries\libs\libplatform.a(fot_update.o)
 .sbss          0x00000000000154f0        0x4 ..\..\..\Libraries\libs\libplatform.a(bt.o)
                0x00000000000154f0                bt_thread_res
 .sbss          0x00000000000154f4        0x1 ..\..\..\Libraries\libs\libbtstack_master.a(bb.o)
 .sbss          0x00000000000154f5        0x1 ..\..\..\Libraries\libs\libbtstack_master.a(platform.o)
                0x00000000000154f5                cfg_bt_spp_rx_flow_ctrl_en
 .sbss          0x00000000000154f6        0x6 ..\..\..\Libraries\libs\libbtstack_master.a(extern_tws.o)
                0x00000000000154f6                cfg_bt_tws_limit_pair_time
                0x00000000000154f8                cfg_bt_tws_feat
                0x00000000000154fa                cfg_bt_tws_pair_mode
 .sbss          0x00000000000154fc        0x9 ..\..\..\Libraries\libs\libbtstack_master.a(extern_bt.o)
                0x00000000000154fe                cfg_bt_tws_mode
 *fill*         0x0000000000015505        0x3 
 .sbss          0x0000000000015508        0x4 ..\..\..\Libraries\libs\libbtstack_master.a(sdp_server.o)
 .sbss          0x000000000001550c       0x13 ..\..\..\Libraries\libs\libbtstack_master.a(rfcomm.o)
                0x0000000000015514                rfcomm_channels
                0x0000000000015518                rfcomm_multiplexers
 *fill*         0x000000000001551f        0x1 
 .sbss          0x0000000000015520        0x5 ..\..\..\Libraries\libs\libbtstack_master.a(btstack_run_loop.o)
 *fill*         0x0000000000015525        0x3 
 .sbss          0x0000000000015528       0x20 ..\..\..\Libraries\libs\libbtstack_master.a(btstack_memory.o)
 .sbss          0x0000000000015548        0xf ..\..\..\Libraries\libs\libbtstack_master.a(sm.o)
 .sbss          0x0000000000015557        0x1 ..\..\..\Libraries\libs\libbtstack_master.a(gatt_client.o)
 .sbss          0x0000000000015558       0x20 ..\..\..\Libraries\libs\libbtstack_master.a(att_server.o)
 .sbss          0x0000000000015578        0xc ..\..\..\Libraries\libs\libbtstack_master.a(att_dispatch.o)
 .sbss          0x0000000000015584       0x10 ..\..\..\Libraries\libs\libbtstack_master.a(att_db.o)
 .sbss          0x0000000000015594        0xd ..\..\..\Libraries\libs\libbtstack_master.a(btstack_main.o)
 *fill*         0x00000000000155a1        0x3 
 .sbss          0x00000000000155a4        0x7 ..\..\..\Libraries\libs\libbtstack_master.a(btstack_api.o)
                0x00000000000155a4                scan_parameters
 *fill*         0x00000000000155ab        0x1 
 .sbss          0x00000000000155ac        0x8 ..\..\..\Libraries\libs\libbtstack_master.a(hct_fc.o)
 .sbss          0x00000000000155b4        0xd ..\..\..\Libraries\libs\libbtstack_master.a(l2cap_test.o)
                0x00000000000155b4                vd_tx_cnt
                0x00000000000155b8                vd_tx_w
                0x00000000000155bc                vd_tx_r
 *fill*         0x00000000000155c1        0x3 
 .sbss          0x00000000000155c4        0x5 ..\..\..\Libraries\libs\libbtstack_master.a(hci.o)
 *fill*         0x00000000000155c9        0x3 
 .sbss          0x00000000000155cc        0x5 ..\..\..\Libraries\libs\libbtstack_master.a(hid_usage.o)
                0x00000000000155cc                ts_ctl
 *fill*         0x00000000000155d1        0x3 
 .sbss          0x00000000000155d4        0x9 ..\..\..\Libraries\libs\libbtstack_master.a(hfp_hf.o)
 *fill*         0x00000000000155dd        0x3 
 .sbss          0x00000000000155e0        0x9 ..\..\..\Libraries\libs\libbtstack_master.a(hci_transport_hcic.o)
                0x00000000000155e4                p_hci_transport
 *fill*         0x00000000000155e9        0x3 
 .sbss          0x00000000000155ec        0x2 ..\..\..\Libraries\libs\libbtstack_master.a(lc_proc.o)
                0x00000000000155ec                lc_state
 *fill*         0x00000000000155ee        0x2 
 .sbss          0x00000000000155f0        0x1 ..\..\..\Libraries\libs\libbtstack_master.a(mgr_proc.o)
 *fill*         0x00000000000155f1        0x3 
 .sbss          0x00000000000155f4        0x4 ..\..\..\Libraries\libs\libbtstack_master.a(ll_proc.o)
 *(.buf*)
 .buf.bsp.sys_cb
                0x00000000000155f8       0x40 Output\obj\Libraries\bsp\bsp_sys.o
                0x00000000000155f8                sys_cb
 .buf.device.cb
                0x0000000000015638       0x1b ..\..\..\Libraries\libs\libplatform.a(device.o)
                0x0000000000015638                dev_cb
 *fill*         0x0000000000015653        0x1 
 .buf.usb       0x0000000000015654      0x15c ..\..\..\Libraries\libs\libdrivers.a(usb_device_run_loop.o)
                0x0000000000015654                ude_0
                0x000000000001567c                udp_0
                0x0000000000015688                epcb_printer_tx
                0x00000000000156a0                epcb_printer_rx
                0x00000000000156b8                udh_0
                0x00000000000156c0                epcb3_tx
                0x00000000000156d8                udu_0
                0x00000000000156dc                epcb_user
                0x00000000000156f4                uds_0
                0x0000000000015728                epcb2_rx
                0x0000000000015740                epcb2_tx
                0x0000000000015758                uda_0
                0x0000000000015768                epcb1_rx
                0x0000000000015780                epcb1_tx
                0x0000000000015798                lun_0
 *(.dac_obuf)
 *(.btmem.stack.sdp)
 .btmem.stack.sdp
                0x00000000000157b0      0x18c ..\..\..\Libraries\libs\libbtstack_master.a(sdp_server.o)
 .btmem.stack.sdp
                0x000000000001593c       0xba ..\..\..\Libraries\libs\libbtstack_master.a(sdp_client.o)
 *(.btmem.stack.spp)
 *fill*         0x00000000000159f6        0x2 
 .btmem.stack.spp
                0x00000000000159f8       0x58 ..\..\..\Libraries\libs\libbtstack_master.a(spp.o)
                0x00000000000159f8                spp_connections
 *(.btmem.stack.l2cap)
 .btmem.stack.l2cap
                0x0000000000015a50       0xbc ..\..\..\Libraries\libs\libbtstack_master.a(l2cap.o)
                0x0000000000015a78                l2cap_channels
 *(.btmem.stack.hid)
 .btmem.stack.hid
                0x0000000000015b0c       0x38 ..\..\..\Libraries\libs\libbtstack_master.a(hid_device.o)
 *(.qtest_buf)
                0x0000000000015b44                __bss_end = .
                0x0000000000001f44                __bss_size = (__bss_end - __bss_start)

.heap           0x0000000000010c00     0x3000
 *(.mem_heap)
 .mem_heap      0x0000000000010c00     0x3000 ..\..\..\Libraries\libs\libplatform.a(startup.o)
                0x0000000000010c00                mem_heap

.bram           0x0000000000020000     0xbba8
 *(.btmem.bthw)
 .btmem.bthw    0x0000000000020000     0x45f8 ..\..\..\Libraries\libs\libbtstack_master.a(bb.o)
                0x0000000000020000                bthw_mem
 *(.btmem*)
 .btmem.bb.buf  0x00000000000245f8       0x4c ..\..\..\Libraries\libs\libbtstack_master.a(nanos.o)
 .btmem.bt.sco  0x0000000000024644        0xa ..\..\..\Libraries\libs\libbtstack_master.a(bt_sco.o)
 *fill*         0x000000000002464e        0x2 
 .btmem.bt.acl  0x0000000000024650        0x8 ..\..\..\Libraries\libs\libbtstack_master.a(bt_acl.o)
                0x0000000000024650                bt_acl_env
 .btmem.bt.sco  0x0000000000024658        0x8 ..\..\..\Libraries\libs\libbtstack_master.a(bt_acl.o)
                0x0000000000024658                bt_sco_env
 .btmem.ble.con
                0x0000000000024660       0x14 ..\..\..\Libraries\libs\libbtstack_master.a(ble_con.o)
 .btmem.bb.env  0x0000000000024674       0x4c ..\..\..\Libraries\libs\libbtstack_master.a(bb_int.o)
                0x0000000000024674                bb_env
 .btmem.bb.buf  0x00000000000246c0     0x3278 ..\..\..\Libraries\libs\libbtstack_master.a(bb.o)
 .btmem.stack.util
                0x0000000000027938       0x12 ..\..\..\Libraries\libs\libbtstack_master.a(btstack_util.o)
 *fill*         0x000000000002794a        0x2 
 .btmem.stack   0x000000000002794c       0x14 ..\..\..\Libraries\libs\libbtstack_master.a(btstack_run_loop.o)
 .btmem.stack.linkctrl
                0x0000000000027960       0x58 ..\..\..\Libraries\libs\libbtstack_master.a(btstack_link_ctrl.o)
                0x0000000000027964                hci_link_max
 .btmem.bb.vs   0x00000000000279b8        0xd ..\..\..\Libraries\libs\libbtstack_master.a(vs_proc.o)
                0x00000000000279b8                vs_env
                0x00000000000279c4                vs_state
 *fill*         0x00000000000279c5        0x3 
 .btmem.bb.rf   0x00000000000279c8        0x4 ..\..\..\Libraries\libs\libbtstack_master.a(rf_smart.o)
 .btmem.bb.hci  0x00000000000279cc       0x62 ..\..\..\Libraries\libs\libbtstack_master.a(hct.o)
                0x00000000000279cc                hci_env
 *fill*         0x0000000000027a2e        0x2 
 .btmem.bt.lm   0x0000000000027a30      0x1ac ..\..\..\Libraries\libs\libbtstack_master.a(lm.o)
                0x0000000000027a34                lm_env
 .btmem.bt.env  0x0000000000027bdc      0x1cc ..\..\..\Libraries\libs\libbtstack_master.a(bt_hal.o)
                0x0000000000027bdc                bt_env
 .btmem.bt.buf  0x0000000000027da8       0xdc ..\..\..\Libraries\libs\libbtstack_master.a(bt21.o)
 .btmem.ble.hal
                0x0000000000027e84      0x130 ..\..\..\Libraries\libs\libbtstack_master.a(ble_hal.o)
                0x0000000000027e88                ble_env
                0x0000000000027fac                ble_exp_sync_pos_tab
 .btmem.ble.adv
                0x0000000000027fb4       0x10 ..\..\..\Libraries\libs\libbtstack_master.a(ble_adv.o)
 .btmem.stack.hci
                0x0000000000027fc4      0xad1 ..\..\..\Libraries\libs\libbtstack_master.a(hci.o)
 *fill*         0x0000000000028a95        0x3 
 .btmem.stack.hci_buf
                0x0000000000028a98      0x3ac ..\..\..\Libraries\libs\libbtstack_master.a(hci.o)
 .btmem.stack.hid.usage
                0x0000000000028e44       0x12 ..\..\..\Libraries\libs\libbtstack_master.a(hid_usage.o)
                0x0000000000028e44                hrpt_cb
                0x0000000000028e4c                hid_report_buf
 *fill*         0x0000000000028e56        0x2 
 .btmem.stack.hfp
                0x0000000000028e58        0x5 ..\..\..\Libraries\libs\libbtstack_master.a(hfp.o)
                0x0000000000028e58                hfp_connections
                0x0000000000028e5c                hfp_index
 *fill*         0x0000000000028e5d        0x3 
 .btmem.ble.adv
                0x0000000000028e60       0x1f ..\..\..\Libraries\libs\libbtstack_master.a(btstack_adv0.o)
 *fill*         0x0000000000028e7f        0x1 
 .btmem.hci.transport
                0x0000000000028e80       0x20 ..\..\..\Libraries\libs\libbtstack_master.a(hci_transport_hcic.o)
 .btmem.bt.lm   0x0000000000028ea0        0x1 ..\..\..\Libraries\libs\libbtstack_master.a(lm_proc.o)
                0x0000000000028ea0                lm_state
 *fill*         0x0000000000028ea1        0x3 
 .btmem.bt.lc   0x0000000000028ea4        0x8 ..\..\..\Libraries\libs\libbtstack_master.a(lc.o)
                0x0000000000028ea4                lc_env
 .btmem.ble.lm  0x0000000000028eac      0x24c ..\..\..\Libraries\libs\libbtstack_master.a(mgr.o)
                0x0000000000028eac                mgr_env
 .btmem.ble.lc  0x00000000000290f8       0x10 ..\..\..\Libraries\libs\libbtstack_master.a(ll.o)
                0x00000000000290f8                ll_env
 .btmem.ble.test
                0x0000000000029108        0x4 ..\..\..\Libraries\libs\libbtstack_master.a(ble_test.o)
 .btmem.ble.scan
                0x000000000002910c        0x8 ..\..\..\Libraries\libs\libbtstack_master.a(ble_scan.o)
 .btmem.ble.init
                0x0000000000029114        0x4 ..\..\..\Libraries\libs\libbtstack_master.a(ble_init.o)
 .btmem.ble.buf
                0x0000000000029118       0x30 ..\..\..\Libraries\libs\libbtstack_master.a(ble_buf.o)
 .btmem.bt.lm.sco
                0x0000000000029148        0xf ..\..\..\Libraries\libs\libbtstack_master.a(lm_sco.o)
 *fill*         0x0000000000029157        0x1 
 .btmem.bt.lc.sniff
                0x0000000000029158       0x68 ..\..\..\Libraries\libs\libbtstack_master.a(lc_sniff.o)
                0x0000000000029158                lc_sniff_env
 .btmem.bt.lc.sco
                0x00000000000291c0       0x12 ..\..\..\Libraries\libs\libbtstack_master.a(lc_sco.o)
 *(.ble_cache*)
 *fill*         0x00000000000291d2        0x2 
 .ble_cache.sm  0x00000000000291d4      0x214 ..\..\..\Libraries\libs\libbtstack_master.a(sm.o)
 .ble_cache.att
                0x00000000000293e8       0x10 ..\..\..\Libraries\libs\libbtstack_master.a(gatt_server.o)
                0x00000000000293e8                notify_tx
 .ble_cache.att
                0x00000000000293f8      0x458 ..\..\..\Libraries\libs\libbtstack_master.a(gatt_profile.o)
 .ble_cache.att
                0x0000000000029850       0x50 ..\..\..\Libraries\libs\libbtstack_master.a(ad_parser.o)
                0x0000000000029850                ad_param
 *(.ble_buf*)
 .ble_buf.stack.spp
                0x00000000000298a0       0x10 ..\..\..\Libraries\libs\libbtstack_master.a(spp.o)
                0x00000000000298a0                spp_tx
 .ble_buf.att   0x00000000000298b0      0x180 ..\..\..\Libraries\libs\libbtstack_master.a(le_device_db_memory.o)
 .ble_buf.att   0x0000000000029a30      0x138 ..\..\..\Libraries\libs\libbtstack_master.a(gatt_server.o)
                0x0000000000029a30                att_attributes
 .ble_buf.att.buf
                0x0000000000029b68      0x400 ..\..\..\Libraries\libs\libbtstack_master.a(gatt_server.o)
                0x0000000000029b68                attribute_buf
 .ble_buf.queue.buf
                0x0000000000029f68       0xc0 ..\..\..\Libraries\libs\libbtstack_master.a(gatt_server.o)
                0x0000000000029f68                att_queue_buf
 .ble_buf.att   0x000000000002a028       0x20 ..\..\..\Libraries\libs\libbtstack_master.a(gatt_client.o)
 .ble_buf.att   0x000000000002a048      0x2e0 ..\..\..\Libraries\libs\libbtstack_master.a(att_server.o)
                0x000000000002a048                att_connection
 *(.spp_tx_buff.*)
 .spp_tx_buff.spp_tx_pool
                0x000000000002a328     0x1040 Output\obj\Libraries\BT\spp\spp.o
                0x000000000002a328                spp_tx_pool
 *(.ble_tx_buff.*)
 .ble_tx_buff.att
                0x000000000002b368      0x840 Output\obj\Libraries\BT\ble\ab_link\app.o
                0x000000000002b368                notify_tx_pool

.aram           0x0000000000050000     0x1000
 *(.usb_buf*)
 .usb_buf.hid   0x0000000000050000        0x8 ..\..\..\Libraries\libs\libdrivers.a(usb_device_run_loop.o)
                0x0000000000050000                ep3_buf
 .usb_buf.user  0x0000000000050008      0x400 ..\..\..\Libraries\libs\libdrivers.a(usb_device_run_loop.o)
                0x0000000000050008                ep_user_buf
                0x0000000000001000                . = 0x1000
 *fill*         0x0000000000050408      0xbf8 

.fcc_buf        0x0000000000050000     0x1000
                0x0000000000001000                . = 0x1000
 *fill*         0x0000000000050000     0x1000 
 *(.fcc_buf.huart)

.aram_msc_stm   0x0000000000050000     0x1000
 *(.stm_buf)
                0x0000000000001000                . = 0x1000
 *fill*         0x0000000000050000     0x1000 

.cram_user
 *(.user.*)

.dram_upd       0x0000000000058000     0x4500
                0x0000000000003800                . = 0x3800
 *fill*         0x0000000000058000     0x3800 
 *(.upd_ota*)
 *(.upd_buf*)
                0x0000000000004500                . = 0x4500
 *fill*         0x000000000005b800      0xd00 

.eram_fot       0x0000000000054000      0xa00
 *(.fot_data.*)
 .fot_data.buf  0x0000000000054000      0x200 Output\obj\Libraries\bsp\bsp_fot.o
                0x0000000000054000                fot_data
 .fot_data.buf  0x0000000000054200      0x4e4 ..\..\..\Libraries\libs\libplatform.a(fot_update.o)
                0x0000000000054478                mac_ctl
                0x0000000000000a00                . = 0xa00
 *fill*         0x00000000000546e4      0x31c 
                0x0000000000044e00                __bank_size = SIZEOF (.flash)
                0x0000000010000200                __comm_lma = LOADADDR (.comm)
                0x0000000000003800                __comm_size = SIZEOF (.comm)
LOAD ..\..\..\Libraries\libs\libplatform.a
LOAD ..\..\..\Libraries\libs\libdrivers.a
LOAD ..\..\..\Libraries\libs\libbtstack_master.a
LOAD ..\..\..\Libraries\libs\libbtstack.a
LOAD ..\..\..\Libraries\libs\libc.a
LOAD ..\..\..\Libraries\libs\libgcc.a
LOAD ..\..\..\Libraries\libs\libm.a
OUTPUT(Output\bin\app.rv32 elf32-littleriscv)

.comment        0x0000000000000000       0x23
 .comment       0x0000000000000000       0x11 Output\obj\Libraries\bsp\bsp_bt.o
                                         0x12 (size before relaxing)
 .comment       0x0000000000000011       0x12 Output\obj\Libraries\bsp\bsp_cm.o
 .comment       0x0000000000000011       0x12 Output\obj\Libraries\bsp\bsp_fot.o
 .comment       0x0000000000000011       0x12 Output\obj\Libraries\bsp\bsp_param.o
 .comment       0x0000000000000011       0x12 Output\obj\Libraries\bsp\bsp_sys.o
 .comment       0x0000000000000011       0x12 Output\obj\Libraries\BT\ble\ab_link\app.o
 .comment       0x0000000000000011       0x12 Output\obj\Libraries\BT\ble\adv0.o
 .comment       0x0000000000000011       0x12 Output\obj\Libraries\BT\ble\ble.o
 .comment       0x0000000000000011       0x12 Output\obj\Libraries\BT\spp\bt.o
 .comment       0x0000000000000011       0x12 Output\obj\Libraries\BT\spp\profile.o
 .comment       0x0000000000000011       0x12 Output\obj\Libraries\BT\spp\spp.o
 .comment       0x0000000000000011       0x12 Output\obj\Libraries\Device\Source\gw3323_clk.o
 .comment       0x0000000000000011       0x12 Output\obj\Libraries\Device\Source\gw3323_gpio.o
 .comment       0x0000000000000011       0x12 Output\obj\Libraries\Device\Source\gw3323_hsuart.o
 .comment       0x0000000000000011       0x12 Output\obj\Libraries\libs\strong_symbol.o
 .comment       0x0000000000000011       0x12 Output\obj\Examples\BLE_Host\Source\ble_client.o
 .comment       0x0000000000000011       0x12 Output\obj\Examples\BLE_Host\Source\ble_init.o
 .comment       0x0000000000000011       0x12 Output\obj\Examples\BLE_Host\Source\hsuart_transfer.o
 .comment       0x0000000000000011       0x12 Output\obj\Examples\BLE_Host\Project\config.o
 .comment       0x0000000000000011       0x12 Output\obj\Examples\BLE_Host\Project\main.o
 .comment       0x0000000000000011       0x12 ..\..\..\Libraries\libs\libplatform.a(audio.o)
                                         0x13 (size before relaxing)
 .comment       0x0000000000000023       0x13 ..\..\..\Libraries\libs\libplatform.a(cm.o)
 .comment       0x0000000000000023       0x13 ..\..\..\Libraries\libs\libplatform.a(os_flash.o)
 .comment       0x0000000000000023       0x13 ..\..\..\Libraries\libs\libplatform.a(xcfg.o)
 .comment       0x0000000000000023       0x13 ..\..\..\Libraries\libs\libplatform.a(device.o)
 .comment       0x0000000000000023       0x13 ..\..\..\Libraries\libs\libplatform.a(main.o)
 .comment       0x0000000000000023       0x13 ..\..\..\Libraries\libs\libplatform.a(interrupt.o)
 .comment       0x0000000000000023       0x13 ..\..\..\Libraries\libs\libplatform.a(startup.o)
 .comment       0x0000000000000023       0x13 ..\..\..\Libraries\libs\libplatform.a(sys_hook.o)
 .comment       0x0000000000000023       0x13 ..\..\..\Libraries\libs\libplatform.a(spiflash.o)
 .comment       0x0000000000000023       0x13 ..\..\..\Libraries\libs\libplatform.a(debug.o)
 .comment       0x0000000000000023       0x13 ..\..\..\Libraries\libs\libplatform.a(fot_update.o)
 .comment       0x0000000000000023       0x13 ..\..\..\Libraries\libs\libplatform.a(lock.o)
 .comment       0x0000000000000023       0x13 ..\..\..\Libraries\libs\libplatform.a(patch.o)
 .comment       0x0000000000000023       0x13 ..\..\..\Libraries\libs\libplatform.a(power.o)
 .comment       0x0000000000000023       0x13 ..\..\..\Libraries\libs\libplatform.a(rc.o)
 .comment       0x0000000000000023       0x13 ..\..\..\Libraries\libs\libplatform.a(sys.o)
 .comment       0x0000000000000023       0x13 ..\..\..\Libraries\libs\libplatform.a(sys_clk.o)
 .comment       0x0000000000000023       0x13 ..\..\..\Libraries\libs\libplatform.a(voltage_trim.o)
 .comment       0x0000000000000023       0x13 ..\..\..\Libraries\libs\libplatform.a(weak_symbol.o)
 .comment       0x0000000000000023       0x13 ..\..\..\Libraries\libs\libplatform.a(usb.o)
 .comment       0x0000000000000023       0x13 ..\..\..\Libraries\libs\libplatform.a(bt.o)
 .comment       0x0000000000000023       0x13 ..\..\..\Libraries\libs\libdrivers.a(usb_device_hid.o)
 .comment       0x0000000000000023       0x13 ..\..\..\Libraries\libs\libdrivers.a(usb_device_printer.o)
 .comment       0x0000000000000023       0x13 ..\..\..\Libraries\libs\libdrivers.a(usb_device_run_loop.o)
 .comment       0x0000000000000023       0x13 ..\..\..\Libraries\libs\libdrivers.a(usb_comm.o)
 .comment       0x0000000000000023       0x13 ..\..\..\Libraries\libs\libdrivers.a(usb_device_ep.o)
 .comment       0x0000000000000023       0x13 ..\..\..\Libraries\libs\libbtstack_master.a(nanos.o)
 .comment       0x0000000000000023       0x13 ..\..\..\Libraries\libs\libbtstack_master.a(patch.o)
 .comment       0x0000000000000023       0x13 ..\..\..\Libraries\libs\libbtstack_master.a(platform.o)
 .comment       0x0000000000000023       0x13 ..\..\..\Libraries\libs\libbtstack_master.a(bt_sco.o)
 .comment       0x0000000000000023       0x13 ..\..\..\Libraries\libs\libbtstack_master.a(bt_acl.o)
 .comment       0x0000000000000023       0x13 ..\..\..\Libraries\libs\libbtstack_master.a(ble_con.o)
 .comment       0x0000000000000023       0x13 ..\..\..\Libraries\libs\libbtstack_master.a(bb_utils.o)
 .comment       0x0000000000000023       0x13 ..\..\..\Libraries\libs\libbtstack_master.a(bb_int.o)
 .comment       0x0000000000000023       0x13 ..\..\..\Libraries\libs\libbtstack_master.a(bb.o)
 .comment       0x0000000000000023       0x13 ..\..\..\Libraries\libs\libbtstack_master.a(platform.o)
 .comment       0x0000000000000023       0x13 ..\..\..\Libraries\libs\libbtstack_master.a(extern_tws.o)
 .comment       0x0000000000000023       0x13 ..\..\..\Libraries\libs\libbtstack_master.a(extern_bt.o)
 .comment       0x0000000000000023       0x13 ..\..\..\Libraries\libs\libbtstack_master.a(extern.o)
 .comment       0x0000000000000023       0x13 ..\..\..\Libraries\libs\libbtstack_master.a(spp.o)
 .comment       0x0000000000000023       0x13 ..\..\..\Libraries\libs\libbtstack_master.a(sdp_util.o)
 .comment       0x0000000000000023       0x13 ..\..\..\Libraries\libs\libbtstack_master.a(sdp_tbl.o)
 .comment       0x0000000000000023       0x13 ..\..\..\Libraries\libs\libbtstack_master.a(sdp_server.o)
 .comment       0x0000000000000023       0x13 ..\..\..\Libraries\libs\libbtstack_master.a(sdp_client.o)
 .comment       0x0000000000000023       0x13 ..\..\..\Libraries\libs\libbtstack_master.a(rfcomm.o)
 .comment       0x0000000000000023       0x13 ..\..\..\Libraries\libs\libbtstack_master.a(btstack_link_key_db.o)
 .comment       0x0000000000000023       0x13 ..\..\..\Libraries\libs\libbtstack_master.a(btstack_util.o)
 .comment       0x0000000000000023       0x13 ..\..\..\Libraries\libs\libbtstack_master.a(btstack_txpkt.o)
 .comment       0x0000000000000023       0x13 ..\..\..\Libraries\libs\libbtstack_master.a(btstack_run_loop.o)
 .comment       0x0000000000000023       0x13 ..\..\..\Libraries\libs\libbtstack_master.a(btstack_memory.o)
 .comment       0x0000000000000023       0x13 ..\..\..\Libraries\libs\libbtstack_master.a(btstack_linked_list.o)
 .comment       0x0000000000000023       0x13 ..\..\..\Libraries\libs\libbtstack_master.a(btstack_link_ctrl.o)
 .comment       0x0000000000000023       0x13 ..\..\..\Libraries\libs\libbtstack_master.a(sm.o)
 .comment       0x0000000000000023       0x13 ..\..\..\Libraries\libs\libbtstack_master.a(le_device_db_memory.o)
 .comment       0x0000000000000023       0x13 ..\..\..\Libraries\libs\libbtstack_master.a(gatt_server.o)
 .comment       0x0000000000000023       0x13 ..\..\..\Libraries\libs\libbtstack_master.a(gatt_profile.o)
 .comment       0x0000000000000023       0x13 ..\..\..\Libraries\libs\libbtstack_master.a(gatt_client.o)
 .comment       0x0000000000000023       0x13 ..\..\..\Libraries\libs\libbtstack_master.a(att_server.o)
 .comment       0x0000000000000023       0x13 ..\..\..\Libraries\libs\libbtstack_master.a(att_dispatch.o)
 .comment       0x0000000000000023       0x13 ..\..\..\Libraries\libs\libbtstack_master.a(att_db.o)
 .comment       0x0000000000000023       0x13 ..\..\..\Libraries\libs\libbtstack_master.a(ad_parser.o)
 .comment       0x0000000000000023       0x13 ..\..\..\Libraries\libs\libbtstack_master.a(btstack_main.o)
 .comment       0x0000000000000023       0x13 ..\..\..\Libraries\libs\libbtstack_master.a(btstack_hal.o)
 .comment       0x0000000000000023       0x13 ..\..\..\Libraries\libs\libbtstack_master.a(btstack_api.o)
 .comment       0x0000000000000023       0x13 ..\..\..\Libraries\libs\libbtstack_master.a(bt_api.o)
 .comment       0x0000000000000023       0x13 ..\..\..\Libraries\libs\libbtstack_master.a(ble_api.o)
 .comment       0x0000000000000023       0x13 ..\..\..\Libraries\libs\libbtstack_master.a(bb_sche.o)
 .comment       0x0000000000000023       0x13 ..\..\..\Libraries\libs\libbtstack_master.a(bb_dbg.o)
 .comment       0x0000000000000023       0x13 ..\..\..\Libraries\libs\libbtstack_master.a(bb_clk.o)
 .comment       0x0000000000000023       0x13 ..\..\..\Libraries\libs\libbtstack_master.a(aes.o)
 .comment       0x0000000000000023       0x13 ..\..\..\Libraries\libs\libbtstack_master.a(vs_proc.o)
 .comment       0x0000000000000023       0x13 ..\..\..\Libraries\libs\libbtstack_master.a(vs_fcc.o)
 .comment       0x0000000000000023       0x13 ..\..\..\Libraries\libs\libbtstack_master.a(vs.o)
 .comment       0x0000000000000023       0x13 ..\..\..\Libraries\libs\libbtstack_master.a(rf_smart.o)
 .comment       0x0000000000000023       0x13 ..\..\..\Libraries\libs\libbtstack_master.a(rf.o)
 .comment       0x0000000000000023       0x13 ..\..\..\Libraries\libs\libbtstack_master.a(bt_hook.o)
 .comment       0x0000000000000023       0x13 ..\..\..\Libraries\libs\libbtstack_master.a(ble_hook.o)
 .comment       0x0000000000000023       0x13 ..\..\..\Libraries\libs\libbtstack_master.a(hct_tl.o)
 .comment       0x0000000000000023       0x13 ..\..\..\Libraries\libs\libbtstack_master.a(hct_msg.o)
 .comment       0x0000000000000023       0x13 ..\..\..\Libraries\libs\libbtstack_master.a(hct_fc.o)
 .comment       0x0000000000000023       0x13 ..\..\..\Libraries\libs\libbtstack_master.a(hct.o)
 .comment       0x0000000000000023       0x13 ..\..\..\Libraries\libs\libbtstack_master.a(tws_sco.o)
 .comment       0x0000000000000023       0x13 ..\..\..\Libraries\libs\libbtstack_master.a(tws_acl.o)
 .comment       0x0000000000000023       0x13 ..\..\..\Libraries\libs\libbtstack_master.a(lm.o)
 .comment       0x0000000000000023       0x13 ..\..\..\Libraries\libs\libbtstack_master.a(bt_hal.o)
 .comment       0x0000000000000023       0x13 ..\..\..\Libraries\libs\libbtstack_master.a(bt21.o)
 .comment       0x0000000000000023       0x13 ..\..\..\Libraries\libs\libbtstack_master.a(bc.o)
 .comment       0x0000000000000023       0x13 ..\..\..\Libraries\libs\libbtstack_master.a(ble_hal.o)
 .comment       0x0000000000000023       0x13 ..\..\..\Libraries\libs\libbtstack_master.a(ble_adv.o)
 .comment       0x0000000000000023       0x13 ..\..\..\Libraries\libs\libbtstack_master.a(ble.o)
 .comment       0x0000000000000023       0x13 ..\..\..\Libraries\libs\libbtstack_master.a(l2cap_test.o)
 .comment       0x0000000000000023       0x13 ..\..\..\Libraries\libs\libbtstack_master.a(l2cap.o)
 .comment       0x0000000000000023       0x13 ..\..\..\Libraries\libs\libbtstack_master.a(hci_sco.o)
 .comment       0x0000000000000023       0x13 ..\..\..\Libraries\libs\libbtstack_master.a(hci_dump.o)
 .comment       0x0000000000000023       0x13 ..\..\..\Libraries\libs\libbtstack_master.a(hci_cmd.o)
 .comment       0x0000000000000023       0x13 ..\..\..\Libraries\libs\libbtstack_master.a(hci.o)
 .comment       0x0000000000000023       0x13 ..\..\..\Libraries\libs\libbtstack_master.a(hid_usage.o)
 .comment       0x0000000000000023       0x13 ..\..\..\Libraries\libs\libbtstack_master.a(hid_device.o)
 .comment       0x0000000000000023       0x13 ..\..\..\Libraries\libs\libbtstack_master.a(hfp_hf.o)
 .comment       0x0000000000000023       0x13 ..\..\..\Libraries\libs\libbtstack_master.a(hfp.o)
 .comment       0x0000000000000023       0x13 ..\..\..\Libraries\libs\libbtstack_master.a(avdtp.o)
 .comment       0x0000000000000023       0x13 ..\..\..\Libraries\libs\libbtstack_master.a(a2dp.o)
 .comment       0x0000000000000023       0x13 ..\..\..\Libraries\libs\libbtstack_master.a(btstack_memory_pool.o)
 .comment       0x0000000000000023       0x13 ..\..\..\Libraries\libs\libbtstack_master.a(btstack_adv0.o)
 .comment       0x0000000000000023       0x13 ..\..\..\Libraries\libs\libbtstack_master.a(hci_transport_hcic.o)
 .comment       0x0000000000000023       0x13 ..\..\..\Libraries\libs\libbtstack_master.a(btstack_chipset_inner.o)
 .comment       0x0000000000000023       0x13 ..\..\..\Libraries\libs\libbtstack_master.a(lm_hook.o)
 .comment       0x0000000000000023       0x13 ..\..\..\Libraries\libs\libbtstack_master.a(lm_sp.o)
 .comment       0x0000000000000023       0x13 ..\..\..\Libraries\libs\libbtstack_master.a(lm_proc.o)
 .comment       0x0000000000000023       0x13 ..\..\..\Libraries\libs\libbtstack_master.a(lm_key.o)
 .comment       0x0000000000000023       0x13 ..\..\..\Libraries\libs\libbtstack_master.a(lc.o)
 .comment       0x0000000000000023       0x13 ..\..\..\Libraries\libs\libbtstack_master.a(mgr.o)
 .comment       0x0000000000000023       0x13 ..\..\..\Libraries\libs\libbtstack_master.a(ll.o)
 .comment       0x0000000000000023       0x13 ..\..\..\Libraries\libs\libbtstack_master.a(ble_test.o)
 .comment       0x0000000000000023       0x13 ..\..\..\Libraries\libs\libbtstack_master.a(ble_scan.o)
 .comment       0x0000000000000023       0x13 ..\..\..\Libraries\libs\libbtstack_master.a(ble_per_adv.o)
 .comment       0x0000000000000023       0x13 ..\..\..\Libraries\libs\libbtstack_master.a(ble_init.o)
 .comment       0x0000000000000023       0x13 ..\..\..\Libraries\libs\libbtstack_master.a(ble_buf.o)
 .comment       0x0000000000000023       0x13 ..\..\..\Libraries\libs\libbtstack_master.a(ble_adv0.o)
 .comment       0x0000000000000023       0x13 ..\..\..\Libraries\libs\libbtstack_master.a(extern_hfhs.o)
 .comment       0x0000000000000023       0x13 ..\..\..\Libraries\libs\libbtstack_master.a(extern_ble.o)
 .comment       0x0000000000000023       0x13 ..\..\..\Libraries\libs\libbtstack_master.a(l2cap_signaling.o)
 .comment       0x0000000000000023       0x13 ..\..\..\Libraries\libs\libbtstack_master.a(lc_hook.o)
 .comment       0x0000000000000023       0x13 ..\..\..\Libraries\libs\libbtstack_master.a(lm_sco.o)
 .comment       0x0000000000000023       0x13 ..\..\..\Libraries\libs\libbtstack_master.a(lc_util.o)
 .comment       0x0000000000000023       0x13 ..\..\..\Libraries\libs\libbtstack_master.a(lc_sniff.o)
 .comment       0x0000000000000023       0x13 ..\..\..\Libraries\libs\libbtstack_master.a(lc_sco.o)
 .comment       0x0000000000000023       0x13 ..\..\..\Libraries\libs\libbtstack_master.a(lc_proc.o)
 .comment       0x0000000000000023       0x13 ..\..\..\Libraries\libs\libbtstack_master.a(lc_lmppdu.o)
 .comment       0x0000000000000023       0x13 ..\..\..\Libraries\libs\libbtstack_master.a(mgr_proc.o)
 .comment       0x0000000000000023       0x13 ..\..\..\Libraries\libs\libbtstack_master.a(mgr_init.o)
 .comment       0x0000000000000023       0x13 ..\..\..\Libraries\libs\libbtstack_master.a(mgr_hci.o)
 .comment       0x0000000000000023       0x13 ..\..\..\Libraries\libs\libbtstack_master.a(ll_scan.o)
 .comment       0x0000000000000023       0x13 ..\..\..\Libraries\libs\libbtstack_master.a(ll_adv.o)
 .comment       0x0000000000000023       0x13 ..\..\..\Libraries\libs\libbtstack_master.a(ll_proc.o)
 .comment       0x0000000000000023       0x13 ..\..\..\Libraries\libs\libbtstack_master.a(ll_ping.o)
 .comment       0x0000000000000023       0x13 ..\..\..\Libraries\libs\libbtstack_master.a(ll_phy_upd.o)
 .comment       0x0000000000000023       0x13 ..\..\..\Libraries\libs\libbtstack_master.a(ll_past.o)
 .comment       0x0000000000000023       0x13 ..\..\..\Libraries\libs\libbtstack_master.a(ll_length.o)
 .comment       0x0000000000000023       0x13 ..\..\..\Libraries\libs\libbtstack_master.a(ll_feature.o)
 .comment       0x0000000000000023       0x13 ..\..\..\Libraries\libs\libbtstack_master.a(ll_encrypt.o)
 .comment       0x0000000000000023       0x13 ..\..\..\Libraries\libs\libbtstack_master.a(ll_disconnect.o)
 .comment       0x0000000000000023       0x13 ..\..\..\Libraries\libs\libbtstack_master.a(ll_con_upd.o)
 .comment       0x0000000000000023       0x13 ..\..\..\Libraries\libs\libbtstack_master.a(ll_cntl.o)
 .comment       0x0000000000000023       0x13 ..\..\..\Libraries\libs\libbtstack_master.a(ll_clk_acc.o)
 .comment       0x0000000000000023       0x13 ..\..\..\Libraries\libs\libbtstack_master.a(ll_chmap_upd.o)
 .comment       0x0000000000000023       0x13 ..\..\..\Libraries\libs\libbtstack_master.a(aes_rpa.o)
 .comment       0x0000000000000023       0x13 ..\..\..\Libraries\libs\libbtstack_master.a(scan_hook.o)
 .comment       0x0000000000000023       0x13 ..\..\..\Libraries\libs\libbtstack_master.a(adv_hook.o)
 .comment       0x0000000000000023       0x13 ..\..\..\Libraries\libs\libbtstack_master.a(ll_version.o)
 .comment       0x0000000000000023       0x13 ..\..\..\Libraries\libs\libbtstack_master.a(ll_pwr.o)

.riscv.attributes
                0x0000000000000000     0x1e44
 .riscv.attributes
                0x0000000000000000       0x32 ..\..\..\Libraries\libs\libplatform.a(audio.o)
 .riscv.attributes
                0x0000000000000032       0x32 ..\..\..\Libraries\libs\libplatform.a(cm.o)
 .riscv.attributes
                0x0000000000000064       0x32 ..\..\..\Libraries\libs\libplatform.a(os_flash.o)
 .riscv.attributes
                0x0000000000000096       0x32 ..\..\..\Libraries\libs\libplatform.a(xcfg.o)
 .riscv.attributes
                0x00000000000000c8       0x32 ..\..\..\Libraries\libs\libplatform.a(device.o)
 .riscv.attributes
                0x00000000000000fa       0x32 ..\..\..\Libraries\libs\libplatform.a(main.o)
 .riscv.attributes
                0x000000000000012c       0x32 ..\..\..\Libraries\libs\libplatform.a(interrupt.o)
 .riscv.attributes
                0x000000000000015e       0x32 ..\..\..\Libraries\libs\libplatform.a(startup.o)
 .riscv.attributes
                0x0000000000000190       0x32 ..\..\..\Libraries\libs\libplatform.a(sys_hook.o)
 .riscv.attributes
                0x00000000000001c2       0x34 ..\..\..\Libraries\libs\libplatform.a(reset.o)
 .riscv.attributes
                0x00000000000001f6       0x32 ..\..\..\Libraries\libs\libplatform.a(spiflash.o)
 .riscv.attributes
                0x0000000000000228       0x32 ..\..\..\Libraries\libs\libplatform.a(debug.o)
 .riscv.attributes
                0x000000000000025a       0x32 ..\..\..\Libraries\libs\libplatform.a(fot_update.o)
 .riscv.attributes
                0x000000000000028c       0x32 ..\..\..\Libraries\libs\libplatform.a(lock.o)
 .riscv.attributes
                0x00000000000002be       0x32 ..\..\..\Libraries\libs\libplatform.a(patch.o)
 .riscv.attributes
                0x00000000000002f0       0x32 ..\..\..\Libraries\libs\libplatform.a(power.o)
 .riscv.attributes
                0x0000000000000322       0x32 ..\..\..\Libraries\libs\libplatform.a(rc.o)
 .riscv.attributes
                0x0000000000000354       0x30 ..\..\..\Libraries\libs\libplatform.a(s_sys.o)
 .riscv.attributes
                0x0000000000000384       0x32 ..\..\..\Libraries\libs\libplatform.a(sys.o)
 .riscv.attributes
                0x00000000000003b6       0x32 ..\..\..\Libraries\libs\libplatform.a(sys_clk.o)
 .riscv.attributes
                0x00000000000003e8       0x32 ..\..\..\Libraries\libs\libplatform.a(voltage_trim.o)
 .riscv.attributes
                0x000000000000041a       0x32 ..\..\..\Libraries\libs\libplatform.a(weak_symbol.o)
 .riscv.attributes
                0x000000000000044c       0x32 ..\..\..\Libraries\libs\libplatform.a(usb.o)
 .riscv.attributes
                0x000000000000047e       0x32 ..\..\..\Libraries\libs\libplatform.a(bt.o)
 .riscv.attributes
                0x00000000000004b0       0x32 ..\..\..\Libraries\libs\libdrivers.a(usb_device_hid.o)
 .riscv.attributes
                0x00000000000004e2       0x32 ..\..\..\Libraries\libs\libdrivers.a(usb_device_printer.o)
 .riscv.attributes
                0x0000000000000514       0x32 ..\..\..\Libraries\libs\libdrivers.a(usb_device_run_loop.o)
 .riscv.attributes
                0x0000000000000546       0x32 ..\..\..\Libraries\libs\libdrivers.a(usb_comm.o)
 .riscv.attributes
                0x0000000000000578       0x32 ..\..\..\Libraries\libs\libdrivers.a(usb_device_ep.o)
 .riscv.attributes
                0x00000000000005aa       0x32 ..\..\..\Libraries\libs\libbtstack_master.a(nanos.o)
 .riscv.attributes
                0x00000000000005dc       0x32 ..\..\..\Libraries\libs\libbtstack_master.a(patch.o)
 .riscv.attributes
                0x000000000000060e       0x32 ..\..\..\Libraries\libs\libbtstack_master.a(platform.o)
 .riscv.attributes
                0x0000000000000640       0x32 ..\..\..\Libraries\libs\libbtstack_master.a(bt_sco.o)
 .riscv.attributes
                0x0000000000000672       0x32 ..\..\..\Libraries\libs\libbtstack_master.a(bt_acl.o)
 .riscv.attributes
                0x00000000000006a4       0x32 ..\..\..\Libraries\libs\libbtstack_master.a(ble_con.o)
 .riscv.attributes
                0x00000000000006d6       0x32 ..\..\..\Libraries\libs\libbtstack_master.a(bb_utils.o)
 .riscv.attributes
                0x0000000000000708       0x32 ..\..\..\Libraries\libs\libbtstack_master.a(bb_int.o)
 .riscv.attributes
                0x000000000000073a       0x32 ..\..\..\Libraries\libs\libbtstack_master.a(bb.o)
 .riscv.attributes
                0x000000000000076c       0x32 ..\..\..\Libraries\libs\libbtstack_master.a(platform.o)
 .riscv.attributes
                0x000000000000079e       0x32 ..\..\..\Libraries\libs\libbtstack_master.a(extern_tws.o)
 .riscv.attributes
                0x00000000000007d0       0x32 ..\..\..\Libraries\libs\libbtstack_master.a(extern_bt.o)
 .riscv.attributes
                0x0000000000000802       0x32 ..\..\..\Libraries\libs\libbtstack_master.a(extern.o)
 .riscv.attributes
                0x0000000000000834       0x32 ..\..\..\Libraries\libs\libbtstack_master.a(spp.o)
 .riscv.attributes
                0x0000000000000866       0x32 ..\..\..\Libraries\libs\libbtstack_master.a(sdp_util.o)
 .riscv.attributes
                0x0000000000000898       0x32 ..\..\..\Libraries\libs\libbtstack_master.a(sdp_tbl.o)
 .riscv.attributes
                0x00000000000008ca       0x32 ..\..\..\Libraries\libs\libbtstack_master.a(sdp_server.o)
 .riscv.attributes
                0x00000000000008fc       0x32 ..\..\..\Libraries\libs\libbtstack_master.a(sdp_client.o)
 .riscv.attributes
                0x000000000000092e       0x32 ..\..\..\Libraries\libs\libbtstack_master.a(rfcomm.o)
 .riscv.attributes
                0x0000000000000960       0x32 ..\..\..\Libraries\libs\libbtstack_master.a(btstack_link_key_db.o)
 .riscv.attributes
                0x0000000000000992       0x32 ..\..\..\Libraries\libs\libbtstack_master.a(btstack_util.o)
 .riscv.attributes
                0x00000000000009c4       0x32 ..\..\..\Libraries\libs\libbtstack_master.a(btstack_txpkt.o)
 .riscv.attributes
                0x00000000000009f6       0x32 ..\..\..\Libraries\libs\libbtstack_master.a(btstack_run_loop.o)
 .riscv.attributes
                0x0000000000000a28       0x32 ..\..\..\Libraries\libs\libbtstack_master.a(btstack_memory.o)
 .riscv.attributes
                0x0000000000000a5a       0x32 ..\..\..\Libraries\libs\libbtstack_master.a(btstack_linked_list.o)
 .riscv.attributes
                0x0000000000000a8c       0x32 ..\..\..\Libraries\libs\libbtstack_master.a(btstack_link_ctrl.o)
 .riscv.attributes
                0x0000000000000abe       0x32 ..\..\..\Libraries\libs\libbtstack_master.a(sm.o)
 .riscv.attributes
                0x0000000000000af0       0x32 ..\..\..\Libraries\libs\libbtstack_master.a(le_device_db_memory.o)
 .riscv.attributes
                0x0000000000000b22       0x32 ..\..\..\Libraries\libs\libbtstack_master.a(gatt_server.o)
 .riscv.attributes
                0x0000000000000b54       0x32 ..\..\..\Libraries\libs\libbtstack_master.a(gatt_profile.o)
 .riscv.attributes
                0x0000000000000b86       0x32 ..\..\..\Libraries\libs\libbtstack_master.a(gatt_client.o)
 .riscv.attributes
                0x0000000000000bb8       0x32 ..\..\..\Libraries\libs\libbtstack_master.a(att_server.o)
 .riscv.attributes
                0x0000000000000bea       0x32 ..\..\..\Libraries\libs\libbtstack_master.a(att_dispatch.o)
 .riscv.attributes
                0x0000000000000c1c       0x32 ..\..\..\Libraries\libs\libbtstack_master.a(att_db.o)
 .riscv.attributes
                0x0000000000000c4e       0x32 ..\..\..\Libraries\libs\libbtstack_master.a(ad_parser.o)
 .riscv.attributes
                0x0000000000000c80       0x32 ..\..\..\Libraries\libs\libbtstack_master.a(btstack_main.o)
 .riscv.attributes
                0x0000000000000cb2       0x32 ..\..\..\Libraries\libs\libbtstack_master.a(btstack_hal.o)
 .riscv.attributes
                0x0000000000000ce4       0x32 ..\..\..\Libraries\libs\libbtstack_master.a(btstack_api.o)
 .riscv.attributes
                0x0000000000000d16       0x32 ..\..\..\Libraries\libs\libbtstack_master.a(bt_api.o)
 .riscv.attributes
                0x0000000000000d48       0x32 ..\..\..\Libraries\libs\libbtstack_master.a(ble_api.o)
 .riscv.attributes
                0x0000000000000d7a       0x32 ..\..\..\Libraries\libs\libbtstack_master.a(bb_sche.o)
 .riscv.attributes
                0x0000000000000dac       0x30 ..\..\..\Libraries\libs\libbtstack_master.a(patch_asm.o)
 .riscv.attributes
                0x0000000000000ddc       0x32 ..\..\..\Libraries\libs\libbtstack_master.a(bb_dbg.o)
 .riscv.attributes
                0x0000000000000e0e       0x32 ..\..\..\Libraries\libs\libbtstack_master.a(bb_clk.o)
 .riscv.attributes
                0x0000000000000e40       0x32 ..\..\..\Libraries\libs\libbtstack_master.a(aes.o)
 .riscv.attributes
                0x0000000000000e72       0x32 ..\..\..\Libraries\libs\libbtstack_master.a(vs_proc.o)
 .riscv.attributes
                0x0000000000000ea4       0x32 ..\..\..\Libraries\libs\libbtstack_master.a(vs_fcc.o)
 .riscv.attributes
                0x0000000000000ed6       0x32 ..\..\..\Libraries\libs\libbtstack_master.a(vs.o)
 .riscv.attributes
                0x0000000000000f08       0x32 ..\..\..\Libraries\libs\libbtstack_master.a(rf_smart.o)
 .riscv.attributes
                0x0000000000000f3a       0x32 ..\..\..\Libraries\libs\libbtstack_master.a(rf.o)
 .riscv.attributes
                0x0000000000000f6c       0x32 ..\..\..\Libraries\libs\libbtstack_master.a(bt_hook.o)
 .riscv.attributes
                0x0000000000000f9e       0x32 ..\..\..\Libraries\libs\libbtstack_master.a(ble_hook.o)
 .riscv.attributes
                0x0000000000000fd0       0x32 ..\..\..\Libraries\libs\libbtstack_master.a(hct_tl.o)
 .riscv.attributes
                0x0000000000001002       0x32 ..\..\..\Libraries\libs\libbtstack_master.a(hct_msg.o)
 .riscv.attributes
                0x0000000000001034       0x32 ..\..\..\Libraries\libs\libbtstack_master.a(hct_fc.o)
 .riscv.attributes
                0x0000000000001066       0x32 ..\..\..\Libraries\libs\libbtstack_master.a(hct.o)
 .riscv.attributes
                0x0000000000001098       0x32 ..\..\..\Libraries\libs\libbtstack_master.a(tws_sco.o)
 .riscv.attributes
                0x00000000000010ca       0x32 ..\..\..\Libraries\libs\libbtstack_master.a(tws_acl.o)
 .riscv.attributes
                0x00000000000010fc       0x32 ..\..\..\Libraries\libs\libbtstack_master.a(lm.o)
 .riscv.attributes
                0x000000000000112e       0x32 ..\..\..\Libraries\libs\libbtstack_master.a(bt_hal.o)
 .riscv.attributes
                0x0000000000001160       0x32 ..\..\..\Libraries\libs\libbtstack_master.a(bt21.o)
 .riscv.attributes
                0x0000000000001192       0x32 ..\..\..\Libraries\libs\libbtstack_master.a(bc.o)
 .riscv.attributes
                0x00000000000011c4       0x32 ..\..\..\Libraries\libs\libbtstack_master.a(ble_hal.o)
 .riscv.attributes
                0x00000000000011f6       0x32 ..\..\..\Libraries\libs\libbtstack_master.a(ble_adv.o)
 .riscv.attributes
                0x0000000000001228       0x32 ..\..\..\Libraries\libs\libbtstack_master.a(ble.o)
 .riscv.attributes
                0x000000000000125a       0x32 ..\..\..\Libraries\libs\libbtstack_master.a(l2cap_test.o)
 .riscv.attributes
                0x000000000000128c       0x32 ..\..\..\Libraries\libs\libbtstack_master.a(l2cap.o)
 .riscv.attributes
                0x00000000000012be       0x32 ..\..\..\Libraries\libs\libbtstack_master.a(hci_sco.o)
 .riscv.attributes
                0x00000000000012f0       0x32 ..\..\..\Libraries\libs\libbtstack_master.a(hci_dump.o)
 .riscv.attributes
                0x0000000000001322       0x32 ..\..\..\Libraries\libs\libbtstack_master.a(hci_cmd.o)
 .riscv.attributes
                0x0000000000001354       0x32 ..\..\..\Libraries\libs\libbtstack_master.a(hci.o)
 .riscv.attributes
                0x0000000000001386       0x32 ..\..\..\Libraries\libs\libbtstack_master.a(hid_usage.o)
 .riscv.attributes
                0x00000000000013b8       0x32 ..\..\..\Libraries\libs\libbtstack_master.a(hid_device.o)
 .riscv.attributes
                0x00000000000013ea       0x32 ..\..\..\Libraries\libs\libbtstack_master.a(hfp_hf.o)
 .riscv.attributes
                0x000000000000141c       0x32 ..\..\..\Libraries\libs\libbtstack_master.a(hfp.o)
 .riscv.attributes
                0x000000000000144e       0x32 ..\..\..\Libraries\libs\libbtstack_master.a(avdtp.o)
 .riscv.attributes
                0x0000000000001480       0x32 ..\..\..\Libraries\libs\libbtstack_master.a(a2dp.o)
 .riscv.attributes
                0x00000000000014b2       0x32 ..\..\..\Libraries\libs\libbtstack_master.a(btstack_memory_pool.o)
 .riscv.attributes
                0x00000000000014e4       0x32 ..\..\..\Libraries\libs\libbtstack_master.a(btstack_adv0.o)
 .riscv.attributes
                0x0000000000001516       0x32 ..\..\..\Libraries\libs\libbtstack_master.a(hci_transport_hcic.o)
 .riscv.attributes
                0x0000000000001548       0x32 ..\..\..\Libraries\libs\libbtstack_master.a(btstack_chipset_inner.o)
 .riscv.attributes
                0x000000000000157a       0x32 ..\..\..\Libraries\libs\libbtstack_master.a(lm_hook.o)
 .riscv.attributes
                0x00000000000015ac       0x32 ..\..\..\Libraries\libs\libbtstack_master.a(lm_sp.o)
 .riscv.attributes
                0x00000000000015de       0x32 ..\..\..\Libraries\libs\libbtstack_master.a(lm_proc.o)
 .riscv.attributes
                0x0000000000001610       0x32 ..\..\..\Libraries\libs\libbtstack_master.a(lm_key.o)
 .riscv.attributes
                0x0000000000001642       0x32 ..\..\..\Libraries\libs\libbtstack_master.a(lc.o)
 .riscv.attributes
                0x0000000000001674       0x32 ..\..\..\Libraries\libs\libbtstack_master.a(mgr.o)
 .riscv.attributes
                0x00000000000016a6       0x32 ..\..\..\Libraries\libs\libbtstack_master.a(ll.o)
 .riscv.attributes
                0x00000000000016d8       0x32 ..\..\..\Libraries\libs\libbtstack_master.a(ble_test.o)
 .riscv.attributes
                0x000000000000170a       0x32 ..\..\..\Libraries\libs\libbtstack_master.a(ble_scan.o)
 .riscv.attributes
                0x000000000000173c       0x32 ..\..\..\Libraries\libs\libbtstack_master.a(ble_per_adv.o)
 .riscv.attributes
                0x000000000000176e       0x32 ..\..\..\Libraries\libs\libbtstack_master.a(ble_init.o)
 .riscv.attributes
                0x00000000000017a0       0x32 ..\..\..\Libraries\libs\libbtstack_master.a(ble_buf.o)
 .riscv.attributes
                0x00000000000017d2       0x32 ..\..\..\Libraries\libs\libbtstack_master.a(ble_adv0.o)
 .riscv.attributes
                0x0000000000001804       0x32 ..\..\..\Libraries\libs\libbtstack_master.a(extern_hfhs.o)
 .riscv.attributes
                0x0000000000001836       0x32 ..\..\..\Libraries\libs\libbtstack_master.a(extern_ble.o)
 .riscv.attributes
                0x0000000000001868       0x32 ..\..\..\Libraries\libs\libbtstack_master.a(l2cap_signaling.o)
 .riscv.attributes
                0x000000000000189a       0x32 ..\..\..\Libraries\libs\libbtstack_master.a(lc_hook.o)
 .riscv.attributes
                0x00000000000018cc       0x32 ..\..\..\Libraries\libs\libbtstack_master.a(lm_sco.o)
 .riscv.attributes
                0x00000000000018fe       0x32 ..\..\..\Libraries\libs\libbtstack_master.a(lc_util.o)
 .riscv.attributes
                0x0000000000001930       0x32 ..\..\..\Libraries\libs\libbtstack_master.a(lc_sniff.o)
 .riscv.attributes
                0x0000000000001962       0x32 ..\..\..\Libraries\libs\libbtstack_master.a(lc_sco.o)
 .riscv.attributes
                0x0000000000001994       0x32 ..\..\..\Libraries\libs\libbtstack_master.a(lc_proc.o)
 .riscv.attributes
                0x00000000000019c6       0x32 ..\..\..\Libraries\libs\libbtstack_master.a(lc_lmppdu.o)
 .riscv.attributes
                0x00000000000019f8       0x32 ..\..\..\Libraries\libs\libbtstack_master.a(mgr_proc.o)
 .riscv.attributes
                0x0000000000001a2a       0x32 ..\..\..\Libraries\libs\libbtstack_master.a(mgr_init.o)
 .riscv.attributes
                0x0000000000001a5c       0x32 ..\..\..\Libraries\libs\libbtstack_master.a(mgr_hci.o)
 .riscv.attributes
                0x0000000000001a8e       0x32 ..\..\..\Libraries\libs\libbtstack_master.a(ll_scan.o)
 .riscv.attributes
                0x0000000000001ac0       0x32 ..\..\..\Libraries\libs\libbtstack_master.a(ll_adv.o)
 .riscv.attributes
                0x0000000000001af2       0x32 ..\..\..\Libraries\libs\libbtstack_master.a(ll_proc.o)
 .riscv.attributes
                0x0000000000001b24       0x32 ..\..\..\Libraries\libs\libbtstack_master.a(ll_ping.o)
 .riscv.attributes
                0x0000000000001b56       0x32 ..\..\..\Libraries\libs\libbtstack_master.a(ll_phy_upd.o)
 .riscv.attributes
                0x0000000000001b88       0x32 ..\..\..\Libraries\libs\libbtstack_master.a(ll_past.o)
 .riscv.attributes
                0x0000000000001bba       0x32 ..\..\..\Libraries\libs\libbtstack_master.a(ll_length.o)
 .riscv.attributes
                0x0000000000001bec       0x32 ..\..\..\Libraries\libs\libbtstack_master.a(ll_feature.o)
 .riscv.attributes
                0x0000000000001c1e       0x32 ..\..\..\Libraries\libs\libbtstack_master.a(ll_encrypt.o)
 .riscv.attributes
                0x0000000000001c50       0x32 ..\..\..\Libraries\libs\libbtstack_master.a(ll_disconnect.o)
 .riscv.attributes
                0x0000000000001c82       0x32 ..\..\..\Libraries\libs\libbtstack_master.a(ll_con_upd.o)
 .riscv.attributes
                0x0000000000001cb4       0x32 ..\..\..\Libraries\libs\libbtstack_master.a(ll_cntl.o)
 .riscv.attributes
                0x0000000000001ce6       0x32 ..\..\..\Libraries\libs\libbtstack_master.a(ll_clk_acc.o)
 .riscv.attributes
                0x0000000000001d18       0x32 ..\..\..\Libraries\libs\libbtstack_master.a(ll_chmap_upd.o)
 .riscv.attributes
                0x0000000000001d4a       0x32 ..\..\..\Libraries\libs\libbtstack_master.a(aes_rpa.o)
 .riscv.attributes
                0x0000000000001d7c       0x32 ..\..\..\Libraries\libs\libbtstack_master.a(scan_hook.o)
 .riscv.attributes
                0x0000000000001dae       0x32 ..\..\..\Libraries\libs\libbtstack_master.a(adv_hook.o)
 .riscv.attributes
                0x0000000000001de0       0x32 ..\..\..\Libraries\libs\libbtstack_master.a(ll_version.o)
 .riscv.attributes
                0x0000000000001e12       0x32 ..\..\..\Libraries\libs\libbtstack_master.a(ll_pwr.o)
